 RT2870

 Timestamp is 4b18d4b9 (Fri Dec 04 17:22:01 2009)

 Preferred load address is 10000000

 Start         Length     Name                   Class
 0001:00000000 0002f954H .rdata                  CODE
 0001:0002f954 00000023H .rdata$debug            CODE
 0001:0002f978 00143f6cH .text                   CODE
 0001:001738e4 000003c4H .xdata                  CODE
 0001:00173ca8 0000003cH .idata$2                CODE
 0001:00173ce4 00000014H .idata$3                CODE
 0001:00173cf8 00000160H .idata$4                CODE
 0001:00173e58 000004d0H .idata$6                CODE
 0001:00174330 0000009bH .edata                  CODE
 0002:00000000 00000160H .idata$5                DATA
 0002:00000160 0000a7e4H .data                   DATA
 0002:0000a960 00003ee5H .bss                    DATA
 0003:00000000 00001e90H .pdata                  DATA

  Address         Publics by Value              Rva+Base       Lib:Object

 0000:00000000       ___safe_se_handler_count   00000000     <absolute>
 0000:00000000       ___safe_se_handler_table   00000000     <absolute>
 0001:00000220       ??_C@_0EK@OMKDDAP@MlmeADDBAAction?5?9?5?9?9?9?9?$DOpInfo?9?$DOWc@ 10001220     action.obj
 0001:0000026c       ??_C@_0DA@GHFCJMIN@BA?5?9?5MlmeADDBAAction?$CI?$CJ?5allocate?5@ 1000126c     action.obj
 0001:000002a0       ??_C@_0EG@GNFIIOGI@BA?5?9?5MlmeDELBAAction?$CI?$CJ?5?4?5Send?5BA@ 100012a0     action.obj
 0001:000002e8       ??_C@_0DA@JJKAOPFN@BA?5?9?5MlmeDELBAAction?$CI?$CJ?5allocate?5@ 100012e8     action.obj
 0001:00000318       ??_C@_0DB@BKCAFACB@ACTION?5?9?5PeerBAAction?$CI?$CJ?5allocate@ 10001318     action.obj
 0001:0000034c       ??_C@_0CH@KACBODJH@ACTION?5?9?5PeerBAAction?$CI?$CJ?5BufSize?5@ 1000134c     action.obj
 0001:00000374       ??_C@_0BD@KLJMGMLG@STA?5is?5Intel?54965?6?$AA@ 10001374     action.obj
 0001:00000388       ??_C@_0DK@KOEFDOAO@PeerAddBAReqAction?3?5ACTION?5?9?5Del@ 10001388     action.obj
 0001:000003c4       ??_C@_0CJ@NFFKDHGI@ACTION?5?9?5PeerBAAction?$CI?$CJ?5Status?5?$DN@ 100013c4     action.obj
 0001:000003f0       ??_C@_0CP@DOPOGLMD@Chk9?3?3ACTION?5?9?5PeerBAAction?$CI?$CJ?5St@ 100013f0     action.obj
 0001:00000420       ??_C@_0CK@CAPLJKKN@Chk9?3?3?5?4?4?4?4?5no?5need?5Block?5Ack?5AT@ 10001420     action.obj
 0001:0000044c       ??_C@_0DD@ICNPAPOK@PeerAddBARspAction?5?9?5?9?9?9?9?$DO?5numAs@ 1000144c     action.obj
 0001:00000480       ??_C@_0DP@PMECOEGO@PeerAddBARsp?5?9?9?9?9?9?$DOWcid?5?$DN?5?$CFd?0?5TI@ 10001480     action.obj
 0001:000004c0       ??_C@_0EA@BFHPEHOB@PeerAddBARsp?9?9?9?9?$DOStatusCode?5?$DN?5?$CFd@ 100014c0     action.obj
 0001:00000500       ??_C@_0CF@KNNKHNDL@BA?5?9?5PeerDelBAAction?9?9?9?9?$DO?5RECIPI@ 10001500     action.obj
 0001:00000528       ??_C@_0CG@HDPGNLPP@BA?5?9?5PeerDelBAAction?9?9?9?9?$DO?5ORIGIN@ 10001528     action.obj
 0001:00000550       ??_C@_0FF@IJKMIGFF@Spectrum?5?9?5Action?5?$DN?5ChannelSwitc@ 10001550     action.obj
 0001:000005a8       ??_C@_0DI@PAANIPOM@Spectrum?5?9?5Action?5includes?5secon@ 100015a8     action.obj
 0001:000005e0       ??_C@_0CK@HIJHLCKJ@Spectrum?5?9?5Action?5?$DN?5SPEC_CHANNEL@ 100015e0     action.obj
 0001:0000060c       ??_C@_0DA@DFENBKKD@BA?5?9?5PeerBAAction?$CI?$CJ?5Action?5?$DN?5Pee@ 1000160c     action.obj
 0001:0000063c       ??_C@_0CK@PFBABAE@BA?5?9?5PeerBAAction?$CI?$CJ?5Action?5?$DN?5ADD@ 1000163c     action.obj
 0001:00000668       ??_C@_0CJ@CALOLFKE@BA?5?9?5PeerBAAction?$CI?$CJ?5Action?5?$DN?5ADD@ 10001668     action.obj
 0001:00000694       ??_C@_0CP@MOHCOGON@Spectrum?4?5New?5Channel?5?$DN?5?$CFd?0?5NewR@ 10001694     action.obj
 0001:000006c4       ??_C@_0DD@MLKNHKKD@ACTION?5?9?5StaPeerPublicAction?5?5Bs@ 100016c4     action.obj
 0001:000006f8       ??_C@_0CM@OAFILOJJ@ACTION?5?9?5HT?5Information?5Exchange@ 100016f8     action.obj
 0001:00000724       ??_C@_0BM@OFOPFKMG@ACTION?5?9?5SMPS?5action?9?9?9?9?$DO?5?6?$AA@ 10001724     action.obj
 0001:00000740       ??_C@_0EP@MGBLMLDA@ACTION?5?9?5HT?5Notify?5Channel?5bandw@ 10001740     action.obj
 0001:00000790       ??_C@_0FI@LAGFAOMB@ACTION?5?9?5Link?5Downd?5and?5Reassoci@ 10001790     action.obj
 0001:000007e8       ??_C@_0FI@DBJJANKN@ACTION?5?9?5HT?5Notify?5Channel?5bandw@ 100017e8     action.obj
 0001:00000840       ??_C@_0CL@CLIGAIEG@ACTION?5?9?5Set?5wicd?5?$DN?5?$CFd?5to?5use?5BW@ 10001840     action.obj
 0001:00000870       ??_C@_0EK@EMELHPFJ@ACTION?5?9?5HT?5Notify?5Channel?5bandw@ 10001870     action.obj
 0001:000008c0       ??_C@_0EM@JAJAOCPJ@ACTION?5?9Ignore?5HT?5Notify?5Channel@ 100018c0     action.obj
 0001:0000090c       ??_C@_0CJ@JMDDEDKF@666?4?5LastIndSeq?5?$DN?50x?$CFx?4?5NumOfRxP@ 1000190c     action.obj
 0001:00000938       ??_C@_0DL@KDMCMIHM@66?9?$CFd?4?5?5INDI?4?5?$CFdth?5buffer?4?5pBuff@ 10001938     action.obj
 0001:00000978       ??_C@_0EB@OGOEABPD@A?9MSDU?$CBNo?5SNAP?5LLC?5format?5Payloa@ 10001978     action.obj
 0001:000009c0       ??_C@_0EC@CBMKDLDG@A?9MSDU?$CBHas?5SNAP?5LLC?5format?5Paylo@ 100019c0     action.obj
 0001:00000a04       ??_C@_0DE@NHHOFEPI@A?9MSDU?$CBbreak?$DL?4Payload1Size?5?$DN?5?$CFd?4@ 10001a04     action.obj
 0001:00000a38       ??_C@_0EB@GLCBAGHN@6?9?$CFd?4?5ERR?5Timeout?5Refresh?4?5LastR@ 10001a38     action.obj
 0001:00000a7c       ??_C@_0DN@DHOCLFJM@6?9?$CFd?4?5Timeout?5Refresh?4?5LastIndSe@ 10001a7c     action.obj
 0001:00000abc       ??_C@_0BM@LAGMLFNE@BA?5?9?5Send?5BAR?0?5Seq?5?$DN?50x?$CFx?5?6?$AA@ 10001abc     action.obj
 0001:00000ad8       ??_C@_0CF@BPJHECBK@BA?5?9?9?$DO?5NoBADataCountDown?5?5?$FL?$DN?5?$CFd?$FN@ 10001ad8     action.obj
 0001:00000b00       ??_C@_0BF@EFOAPABH@BA?5?9?5bSendBAR?5?$DN?5?$CFd?5?6?$AA@ 10001b00     action.obj
 0001:00000b18       ??_C@_0EP@LAOCOGL@BA?5?9?53ADDBATimer?4?5?5BARecEntry?$FL0?$FN@ 10001b18     action.obj
 0001:00000b68       ??_C@_0CP@NAEFLINJ@BA?5?9?52ADDBATimer?4?5fCLIENT_STATUS@ 10001b68     action.obj
 0001:00000b98       ??_C@_0CP@KADCKODP@BA?5?9?54ADDBATimer?4?5fCLIENT_STATUS@ 10001b98     action.obj
 0001:00000bc8       ??_C@_0CO@NONNGEKC@BA?5?9?50ADDBATimer?4?5Send?5to?5wcid?5?$DN@ 10001bc8     action.obj
 0001:00000bf8       ??_C@_0CN@NIEACHNB@BA?5?9?5ADDBATimer?4?5Send?5to?5wcid?5?$DN?5@ 10001bf8     action.obj
 0001:00000c28       ??_C@_0CG@PHDGPKFF@77?9?$CFd?5?5INDI?4?5?5pHeader?9?$DOSequence?7@ 10001c28     action.obj
 0001:00000c50       ??_C@_0CJ@CLMEDJJE@777?9?$CFd?5refresh?5?4?5pHeader?9?$DOSequen@ 10001c50     action.obj
 0001:00000c7c       ??_C@_01EEMJAFIK@?6?$AA@   10001c7c     action.obj
 0001:00000c80       ??_C@_06COPILJFO@0x?$CFx?0?5?$AA@ 10001c80     action.obj
 0001:00000c88       ??_C@_0CC@CMFEGHEK@77?5Error?5Counting?5Reorder?5Buffer@ 10001c88     action.obj
 0001:00000cac       ??_C@_0BO@PIFCGII@77?9?$CFd?4?5INDI?5Sequences?5are?5?3?5?6?$AA@ 10001cac     action.obj
 0001:00000cd0       ??_C@_0FL@DCLKBOKL@7?9?$CFd?4?5Refresh?4?5pHeader?9?$DOSequence@ 10001cd0     action.obj
 0001:00000d2c       ??_C@_0DM@GBMLJELF@55?9?$CFd?4?5Duplicate?5?5Reorder?5Buffer@ 10001d2c     action.obj
 0001:00000d68       ??_C@_0IN@KDOJNJJI@5?9?$CFd?4?5Rx?5out?5of?5order?4?5Insert?$FL?$CFd@ 10001d68     action.obj
 0001:00000df8       ??_C@_0CC@ILFOEMA@55?5Error?5Counting?5Reorder?5Buffer@ 10001df8     action.obj
 0001:00000e1c       ??_C@_0BB@CIFHMFNA@RT2870?5ERROR?$CB?$CB?$CB?5?$AA@ 10001e1c     action.obj
 0001:00000e30       ??_C@_0EG@OHHEDAAD@5?9?$CFd?4?5Refresh?4?5ERROR?$CB?$CB?5shiftnumb@ 10001e30     action.obj
 0001:00000e78       ??_C@_0FL@GJHJMPNO@5?9?$CFd?4?5Refresh?4?5pHeader?9?$DOSequence@ 10001e78     action.obj
 0001:00000ed4       ??_C@_0DM@MCFEBPML@44?9?$CFd?4?5Duplicate?5?5Reorder?5Buffer@ 10001ed4     action.obj
 0001:00000f10       ??_C@_0IF@INPKOGLN@4?9?$CFd?4?5Rx?5out?5of?5order?4?5Insert?$FL?$CFd@ 10001f10     action.obj
 0001:00000f98       ??_C@_0EO@CJGACBDP@?$CB?$CBpHeader?9?$DOSequence?5?$DN?50x?$CFx?0pBAEn@ 10001f98     action.obj
 0001:00000fe8       ??_C@_0EM@JBJKFIBN@3?9?$CFd?4?5DUPLICATE?5receive?5pHeader?9@ 10001fe8     action.obj
 0001:00001038       ??_C@_0EN@JBJBLPNL@33?9?$CFd?4?5DUPLICATE?5receive?5pHeader@ 10002038     action.obj
 0001:00001088       ??_C@_0EF@DPHAOCGB@22?9?$CFd?4?5INDI?4?5?$CFdth?5buffer?4?5pBuffe@ 10002088     action.obj
 0001:000010d0       ??_C@_1FK@FNONLNGN@?$AA?$CF?$AAs?$AA?3?$AA?5?$AAD?$AAE?$AAB?$AAU?$AAG?$AAC?$AAH?$AAK?$AA?5?$AAf?$AAa?$AAi?$AAl?$AAe?$AAd?$AA?5?$AAi?$AAn?$AA?5?$AAf?$AAi?$AAl?$AAe?$AA?5?$AA?$CF?$AAs?$AA?5?$AAa@ 100020d0     action.obj
 0001:0000112c       ??_C@_1BA@LEPJIIOK@?$AAU?$AAn?$AAk?$AAn?$AAo?$AAw?$AAn?$AA?$AA@ 1000212c     action.obj
 0001:00001140       ??_C@_1FG@NIDPEPEC@?$AAC?$AA?3?$AA?2?$AAW?$AAi?$AAn?$AAC?$AAE?$AA6?$AA?4?$AA0?$AA?2?$AAN?$AAe?$AAw?$AA?2?$AAR?$AAT?$AA2?$AA8?$AA7?$AA0?$AA_?$AAv?$AA1?$AA?4?$AA4?$AA?4?$AA9?$AA?4?$AA0?$AA?2@ 10002140     action.obj
 0001:00001198       ??_C@_0EL@BOEAJILG@BAR?5?3?522?9?$CFd?4?5INDI?4?5?$CFdth?5buffer?4?5@ 10002198     action.obj
 0001:000011e8       ??_C@_0GA@FPDMNAIE@Receive?5BAR?5?3?5LastIndSeq?5?5?$DN?50x?$CFx@ 100021e8     action.obj
 0001:00001248       ??_C@_0EH@OPNCNPJG@MlmeEnqueueForRecv?3?5BlockAck?5Req@ 10002248     action.obj
 0001:00001290       ??_C@_0DB@BMOIKAPK@MlmeEnqueueForRecv?3?5frame?5too?5la@ 10002290     action.obj
 0001:000012c4       ??_C@_0L@ELOJIKMG@?5?3?5Manual?6?$AA@ 100022c4     action.obj
 0001:000012d0       ??_C@_08OILIPKPB@?5?3?5Auto?6?$AA@ 100022d0     action.obj
 0001:000012dc       ??_C@_0BF@FEPOGEAO@BaAutoManSwitch?$DN?$DN?$DN?$DN?$DO?$AA@ 100022dc     action.obj
 0001:000012f4       ??_C@_0BN@EBOHLKJD@HT?5?9?5SendPSMPAction?$CI?5?$CFd?5?$CJ?5?5?6?$AA@ 100022f4     action.obj
 0001:00001314       ??_C@_0CC@EIGLIAPM@?$CB?$CB?$CBChannelSwitchSanityCheck?5?$CB?$CB?$CB?5@ 10002314     action.obj
 0001:00001338       ??_C@_0EC@ODBFBCEF@?$CB?$CB?$CB40MHz?5Upper?5LINK?5UP?5?$CB?$CB?$CB?5Contr@ 10002338     action.obj
 0001:00001380       ??_C@_0EE@LIOJOJGF@?$CB?$CB?$CB40MHz?5Lower?5LINK?5UP?5?$CB?$CB?$CB?5Contr@ 10002380     action.obj
 0001:000013c4       ??_C@_0BB@CHNGKBMN@?$CB?$CB?$CB20MHz?5?5?5?$CB?$CB?$CB?5?6?$AA@ 100023c4     action.obj
 0001:000013d8       ??_C@_0BB@MFIFODHA@?$CB?$CB?$CBrt2860C?5?$CB?$CB?$CB?5?6?$AA@ 100023d8     action.obj
 0001:000013f0       ??_C@_0EE@IJPMLHLA@SPECTRUM?5?9?5ChannelSwitchAction?$CIN@ 100023f0     action.obj
 0001:00001434       ??_C@_0CK@KFGFKDE@?$CFx?5?$CFx?5?$CFx?5?$CFx?4?5?$CFx?5?$CFx?5?$CFx?5?$CFx?4?5?$CFx?5?$CFx?5@ 10002434     action.obj
 0001:00001460       ??_C@_0DG@CGFAIGAL@ACT?5?9?5BuildIntolerantChannelRep?5@ 10002460     action.obj
 0001:00001498       ??_C@_0DO@CDJIHGAN@ACT?5?9?5BuildIntolerantChannelRep?5@ 10002498     action.obj
 0001:000014d8       ??_C@_0EN@EEHALLBM@ACT?5?9?5Update2040CoexistFrameAndN@ 100024d8     action.obj
 0001:00001528       ??_C@_0DI@CBJPDEF@ACT?5?9?5Send2040CoexistAction?$CI?5BSS@ 10002528     action.obj
 0001:00001560       ??_C@_0DH@NOIPGNGO@ACT?5?9?5Send2040CoexistAction?$CI?$CJ?5al@ 10002560     action.obj
 0001:00001598       ??_C@_0DP@IKHLPMLA@ACT?5?9?5UpdateBssScanParm?$CI?5Dot11Bs@ 10002598     action.obj
 0001:000015d8       ??_C@_0EJ@MKGNGIMK@ACT?5?9?5UpdateBssScanParm?$CI?5Dot11OB@ 100025d8     action.obj
 0001:00001628       ??_C@_0FC@CAJOPBKO@ACT?5?9?5UpdateBssScanParm?$CI?5Dot11OB@ 10002628     action.obj
 0001:00001680       ??_C@_0FD@BNPADEDE@ACT?5?9?5UpdateBssScanParm?$CI?5Dot11OB@ 10002680     action.obj
 0001:000016d8       ??_C@_0EI@KKAFLGDI@ACT?5?9?5UpdateBssScanParm?$CI?5Dot11OB@ 100026d8     action.obj
 0001:00001720       ??_C@_0EJ@BAMGMGGK@ACT?5?9?5UpdateBssScanParm?$CI?5Dot11OB@ 10002720     action.obj
 0001:00001770       ??_C@_0EL@DOPDKEEP@ACT?5?9?5UpdateBssScanParm?$CI?5Dot11Bs@ 10002770     action.obj
 0001:000017c0       ??_C@_0FA@CHNEEBGI@ACT?5?9?5UpdateBssScanParm?$CI?5Dot11Bs@ 100027c0     action.obj
 0001:00001a10       ??_C@_0BL@IOLNFJGF@?$DM?9?9?9?9?9?9?9?9?9AcmReqCmdAction?6?$AA@ 10002a10     acm_action.obj
 0001:00001a2c       ??_C@_0CJ@HDAJBCEF@AcmReqCmdAction?5?9?5Unknow?5command@ 10002a2c     acm_action.obj
 0001:00001a58       ??_C@_0CB@FAHOFEN@ACM_DRIVER_AUTO_RESET_TCLAS?9?9?9?5?6@ 10002a58     acm_action.obj
 0001:00001a7c       ??_C@_0BL@HFACOPLJ@ACM_DRIVER_AUTO_DELTS?9?9?9?5?6?$AA@ 10002a7c     acm_action.obj
 0001:00001a98       ??_C@_0CG@DCNMFODN@ACM_DRIVER_AUTO_ADDTS_WITH_TCLAS@ 10002a98     acm_action.obj
 0001:00001ac0       ??_C@_0CF@HJOKDFFA@ACM_DRIVER_AUTO_ADDTS?5for?5Voice?9@ 10002ac0     acm_action.obj
 0001:00001ae8       ??_C@_0CG@MPKGKOLP@ACM_UI_CMD_RESET_TCLAS?5?9?5RESET?5T@ 10002ae8     acm_action.obj
 0001:00001b10       ??_C@_0CC@HAFOHEKD@ACM_UI_CMD_DELTX?5?9?5DELTS?0?5tid?$DN?$CFd@ 10002b10     acm_action.obj
 0001:00001b38       ??_C@_0EA@GCIHCGEF@ACM_UI_CMD_ADDTX_WITH_TCLAS?5?9?5AD@ 10002b38     acm_action.obj
 0001:00001b78       ??_C@_0BG@FPJMMHJN@ACM_UI_CMD_ADDTX?9?9?9?5?6?$AA@ 10002b78     acm_action.obj
 0001:00001b90       ??_C@_0BH@OJNABKJK@AcmReqCmdAction?5?9?9?9?$DO?5?6?$AA@ 10002b90     acm_action.obj
 0001:00001ba8       ??_C@_0DD@KMNMAJFK@?$DM?9?9?9?9?5AcmCmdAddTSRequest?0?5FrameL@ 10002ba8     acm_action.obj
 0001:00001bdc       ??_C@_0BK@JIBNCPMA@AcmCmdAddTSRequest?5?9?9?9?$DO?5?6?$AA@ 10002bdc     acm_action.obj
 0001:00001bf8       ??_C@_0BM@IAJAJCDL@?$DM?9?9?9?9?9?9?9?5AcmPeerRspHandle?5?6?$AA@ 10002bf8     acm_action.obj
 0001:00001c14       ??_C@_0CK@NBPGEJLL@non?9support?5ACM?5action?$CI?$CFd?$CJ?5for?5Q@ 10002c14     acm_action.obj
 0001:00001c40       ??_C@_0CJ@MABIOKNH@ACM_ACTION_WME_TEAR_DOWN?5from?5Pe@ 10002c40     acm_action.obj
 0001:00001c6c       ??_C@_0CK@FKLPNOAB@TSPEC?5embeds?5unsupported?5IE?$DN?50x?$CF@ 10002c6c     acm_action.obj
 0001:00001c98       ??_C@_0DN@CFCLHHLK@TSPEC?5embeds?5EDCA?5MSDU?5Lifetime?5@ 10002c98     acm_action.obj
 0001:00001cd8       ??_C@_0CA@HDBNMLDI@TSPEC?5embeds?5TS?5RATE?5IE?5?4?4?4?4?4?4?6?$AA@ 10002cd8     acm_action.obj
 0001:00001cf8       ??_C@_0DA@CCBABLEK@TSPEC?5embeds?5TS?5Metrics?5IE?0?5inte@ 10002cf8     acm_action.obj
 0001:00001d28       ??_C@_0DJ@KGCBFMAF@ACM_ACTION_WME_SETUP_RSP?5from?5Pe@ 10002d28     acm_action.obj
 0001:00001d64       ??_C@_0CP@OKDNDBDD@AcmPeerRspHandle?5status?$DN0x?$CFx?0?5ac@ 10002d64     acm_action.obj
 0001:00001d94       ??_C@_0CE@BILBPCCF@?$DM?9?9?9?5AcmCmdDelTSSend?0?5FrameLen?$DN?$CF@ 10002d94     acm_action.obj
 0001:00001db8       ??_C@_0BH@MKLGHLDO@AcmCmdDelTSSend?5?9?9?9?$DO?5?6?$AA@ 10002db8     acm_action.obj
 0001:00001fd0       ??_C@_0CD@GBBPODG@?$DM?9?9?9?9?9?5AironetMsgAction?0?5Index?$DN?$CF@ 10002fd0     aironet.obj
 0001:00001ff8       ??_C@_0EB@FJAMOJBF@?5AironetMsgAction?0?5ReqElem?4Lengt@ 10002ff8     aironet.obj
 0001:0000203c       ??_C@_0BP@NDLNJNFO@AironetMsgAction?0?5FR?5len?5?$DN?5?$CFd?6?$AA@ 1000303c     aironet.obj
 0001:0000205c       ??_C@_0DG@ONGIKHEI@Wrong?5IAPP?5subtype?$CI0x?$CFx?$CJ?5for?5Cis@ 1000305c     aironet.obj
 0001:00002094       ??_C@_0DE@MDEIDCJA@Wrong?5IAPP?5type?$CI0x?$CFx?$CJ?5for?5Cisco?5@ 10003094     aironet.obj
 0001:000020c8       ??_C@_0DE@HPJNPIMA@Unknown?5SubType?5?$CI?$CFx?$CJ?5for?5AIRONET@ 100030c8     aironet.obj
 0001:000020fc       ??_C@_0BO@DNNBHAKP@IAPP?5Measurement?5Offset?5?$DN?5?$CFx?6?$AA@ 100030fc     aironet.obj
 0001:0000211c       ??_C@_0BM@PFPNPAPH@IAPP?5Activation?5Delay?5?$DN?5?$CFx?6?$AA@ 1000311c     aironet.obj
 0001:00002138       ??_C@_0BK@GLNJKMCD@IAPP?5Dialog?5Token?5?$DN?50x?$CFx?6?$AA@ 10003138     aironet.obj
 0001:00002154       ??_C@_0BF@ONBCFILD@IAPP?5SubType?5?$DN?50x?$CFx?6?$AA@ 10003154     aironet.obj
 0001:0000216c       ??_C@_0BC@JLKPAGBN@IAPP?5Type?5?$DN?50x?$CFx?6?$AA@ 1000316c     aironet.obj
 0001:00002180       ??_C@_0BH@CHJKDAC@IAPP?5ID?5?$CG?5Length?5?$DN?5?$CFd?6?$AA@ 10003180     aironet.obj
 0001:00002198       ??_C@_0EA@PMGHDOEG@AironetMsgAction?3?5CCXEnable?$CI?$CFd?9?5@ 10003198     aironet.obj
 0001:000021d8       ??_C@_0BJ@MLDDEIEM@?9?9?9?9?9?$DO?5AironetMsgAction?6?$AA@ 100031d8     aironet.obj
 0001:000021f4       ??_C@_0CH@GLOKNDMN@AironetRequestAction?5Type?5?$DN?5?$CFd?5?9@ 100031f4     aironet.obj
 0001:0000221c       ??_C@_0CB@ELJJOMEK@ChannelLoadRequestAction?5?$DM?9?9?9?9?9?6@ 1000321c     aironet.obj
 0001:00002240       ??_C@_0BK@LAICFHGC@Duration?5?$CFd?0?5Channel?5?$CFd?$CB?6?$AA@ 10003240     aironet.obj
 0001:0000225c       ??_C@_0CB@OFOIMANG@ChannelLoadRequestAction?5?9?9?9?9?9?$DO?6@ 1000325c     aironet.obj
 0001:00002280       ??_C@_0BP@LMHEGMDC@NoiseHistRequestAction?5?$DM?9?9?9?9?9?6?$AA@ 10003280     aironet.obj
 0001:000022a0       ??_C@_0BP@BCAFEAKO@NoiseHistRequestAction?5?9?9?9?9?9?$DO?6?$AA@ 100032a0     aironet.obj
 0001:000022c0       ??_C@_0BM@JHFJHGOL@BeaconRequestAction?5?$DM?9?9?9?9?9?6?$AA@ 100032c0     aironet.obj
 0001:000022dc       ??_C@_0BC@LBJBAFBB@Wrong?5Scan?5Mode?$CB?6?$AA@ 100032dc     aironet.obj
 0001:000022f0       ??_C@_0BF@NEBMODEP@Beacon?5Report?5Mode?$CB?6?$AA@ 100032f0     aironet.obj
 0001:00002308       ??_C@_0DB@NDGFBOEC@MSRN_SCAN_MODE_ACTIVE?0?5Channel?$DN?$CF@ 10003308     aironet.obj
 0001:0000233c       ??_C@_0BD@HAAFBFOE@Active?5Scan?5Mode?$CB?6?$AA@ 1000333c     aironet.obj
 0001:00002350       ??_C@_0CG@NGGDOKOG@MSRN_SCAN_MODE_PASSIVE?0?5Duration@ 10003350     aironet.obj
 0001:00002378       ??_C@_0BE@FIFDBKHC@Passive?5Scan?5Mode?$CB?6?$AA@ 10003378     aironet.obj
 0001:0000238c       ??_C@_0BM@DJCIFKHH@BeaconRequestAction?5?9?9?9?9?9?$DO?6?$AA@ 1000338c     aironet.obj
 0001:000023a8       ??_C@_0BL@LDOLDGL@FrameRequestAction?5?$DM?9?9?9?9?9?6?$AA@ 100033a8     aironet.obj
 0001:000023c4       ??_C@_0CM@BFMFHNAK@FRAME_REQ_ACTION?0?5Duration?5?$CFd?0?5C@ 100033c4     aironet.obj
 0001:000023f0       ??_C@_0BL@KFEPJPPH@FrameRequestAction?5?9?9?9?9?9?$DO?6?$AA@ 100033f0     aironet.obj
 0001:0000240c       ??_C@_0BO@OMGJFAEC@PassLossRequestAction?5?$DM?9?9?9?9?9?6?$AA@ 1000340c     aironet.obj
 0001:00002430       ??_C@_0HP@HLCAADBM@MSRN_TYPE_PATH_LOSS_REQ?0?5BurstNu@ 10003430     aironet.obj
 0001:000024b0       ??_C@_0DJ@EJFOPBNC@PassLossRequestAction?3?5send?5back@ 100034b0     aironet.obj
 0001:000024ec       ??_C@_0DH@LADDGBBE@PassLossRequestAction?3?5send?5back@ 100034ec     aironet.obj
 0001:00002524       ??_C@_0DJ@FGGBDPIL@PassLossRequestAction?3?5Cancel?5Re@ 10003524     aironet.obj
 0001:00002560       ??_C@_0CO@GEOJFNHK@PassLossRequestAction?5OneSecTxCo@ 10003560     aironet.obj
 0001:00002590       ??_C@_0BJ@OENIMGHI@LogRequestAction?5?$DM?9?9?9?9?9?6?$AA@ 10003590     aironet.obj
 0001:000025b0       ??_C@_0GF@PBIHCEKM@AironetLogRequestAction?3?5CCX_EVE@ 100035b0     aironet.obj
 0001:00002618       ??_C@_0CL@JJNMBJLH@?$DM35?$DO?5Apr?516?503?305?302?5Authenticat@ 10003618     aironet.obj
 0001:00002644       ??_C@_0DP@NBBCPBLB@CCX_EVENT_RSNA_LOG?5?4?4?4?5FrameRepo@ 10003644     aironet.obj
 0001:00002688       ??_C@_0EB@BFGCCLBC@EVENT_RSNA_LOG?5?4?4?4?5pEntry?9?$DORSNIE@ 10003688     aironet.obj
 0001:000026d0       ??_C@_0FI@IODABBCE@AironetLogRequestAction?3?5CCX_EVE@ 100036d0     aironet.obj
 0001:00002728       ??_C@_0DH@BBGGFMLF@AironetLog?0?5IappLength?$DN?$CFd?0?5EVENT@ 10003728     aironet.obj
 0001:00002760       ??_C@_0DB@JEJJOJPP@AironetLogRequestAction?0?5Elem?9?$DOM@ 10003760     aironet.obj
 0001:00002794       ??_C@_0CA@OHEBGLEN@StatisticsRequestAction?5?$DM?9?9?9?9?9?6?$AA@ 10003794     aironet.obj
 0001:000027b4       ??_C@_0CL@EJHDNAOJ@Duration?5?$DN?5?$CFd?0?5ScanMode?$DN?5?$CFd?5Chan@ 100037b4     aironet.obj
 0001:000027e0       ??_C@_0CE@MBFJEADB@StatisticsRequestAction?$CI?$CFd?$CJ?5?9?9?9?9@ 100037e0     aironet.obj
 0001:00002804       ??_C@_0CA@POEPLGLK@AironetReportAction?5?$CI?$CFd?$CJ?$DM?9?9?9?9?9?6?$AA@ 10003804     aironet.obj
 0001:00002824       ??_C@_0BM@OEOKFHPK@RM?5?9?5ParallelReq?0?5Type?$DN?$CFd?5?6?$AA@ 10003824     aironet.obj
 0001:00002840       ??_C@_0CG@PKNOCNI@AironetReportAction?5?$CILen?5?$DN?5?$CFd?$CJ?9?9@ 10003840     aironet.obj
 0001:00002868       ??_C@_0EI@BDPHOGDF@AironetFinalReportAction?5?$CIFrameL@ 10003868     aironet.obj
 0001:000028b0       ??_C@_0EG@OHFEMDBK@AironetFinalReportAction?3?5pIAPP?9@ 100038b0     aironet.obj
 0001:000028f8       ??_C@_0DJ@OCFGCFPG@AironetFinalReportAction?$CILen?5?$DN?5?$CF@ 100038f8     aironet.obj
 0001:00002934       ??_C@_0CI@BILKEEKJ@ChannelLoadReportAction?5?$CILen?$DN?$CFd?$CJ@ 10003934     aironet.obj
 0001:0000295c       ??_C@_0BD@PGMLGBH@FrameReportLen?$DN?$CFd?6?$AA@ 1000395c     aironet.obj
 0001:00002970       ??_C@_0DA@IOHAAJGN@CLBusyByte?$DN?$CFd?0?5Duration?$DN?$CFd?0?5CCAB@ 10003970     aironet.obj
 0001:000029a0       ??_C@_0DN@OMDPJBGJ@ChannelLoadReportAction?5?$CICLFacto@ 100039a0     aironet.obj
 0001:000029e0       ??_C@_0CC@PFKKIMN@NoiseHistReportAction?$CI?$CFd?$CJ?5?$DM?9?9?9?9?9@ 100039e0     aironet.obj
 0001:00002a04       ??_C@_0BL@JFGNOGFD@Reported?5RPI?$FL0?$FN?5?5?$DN?50x?$CF02x?6?$AA@ 10003a04     aironet.obj
 0001:00002a20       ??_C@_0DA@CNBGKEGB@Overflow?0?5update?5?5RPI?$FL?$CFd?$FN?5?5?$DN?50x?$CF@ 10003a20     aironet.obj
 0001:00002a50       ??_C@_0CM@IEBMPIHH@Reported?5RPI?$FL?$CFd?$FN?5?5?$DN?50x?$CFx?5?$CI?$CFd?$CJ?0?5N@ 10003a50     aironet.obj
 0001:00002a7c       ??_C@_0CJ@NGFNNIAK@Total?5RPI?5Conuts?5?$DN?5?$CFd?0?5TotalRPIS@ 10003a7c     aironet.obj
 0001:00002aa8       ??_C@_0BC@MOKPKFAH@RPI?5?$CFd?5Conuts?5?$CFd?6?$AA@ 10003aa8     aironet.obj
 0001:00002ac0       ??_C@_0EJ@NJDHKAKL@RM?5?9?5for?5NH?5value?5optimization?4?4@ 10003ac0     aironet.obj
 0001:00002b10       ??_C@_0EC@GMIMBAOO@NoiseHistReportAction?5?$CILen?5?$DN?5?$CFd?0@ 10003b10     aironet.obj
 0001:00002b54       ??_C@_0CF@FMJIMMKJ@BeaconReportAction?5?$CILen?5?$DN?5?$CFd?$CJ?$DM?9?9@ 10003b54     aironet.obj
 0001:00002b7c       ??_C@_0BL@ENEDDFCJ@BeaconReportAction?5?9?9?9?9?9?$DO?6?$AA@ 10003b7c     aironet.obj
 0001:00002b98       ??_C@_0DN@BLMLMMK@AironetAddBeaconReport?0?5FR?5len?5?$DN@ 10003b98     aironet.obj
 0001:00002bd8       ??_C@_0EB@OBKMBNFK@?$CK?$CK?$CK?$CK?$CK?$CK?$CK?$CK?$CK?$CK?$CK?$CK?$CK?$CK?$CK?$CK?$CK?$CK?$CKMBSSID?5mask?0?5@ 10003bd8     aironet.obj
 0001:00002c1c       ??_C@_0CC@LJPKDEKK@after?5Mask?$DN?$CFd?4?4?4?4?5result?$DN?$CFd?4?4?4?$CB?$CB@ 10003c1c     aironet.obj
 0001:00002c40       ??_C@_0BF@COBOCKCM@FrameReportLen?5?$DN?5?$CFd?6?$AA@ 10003c40     aironet.obj
 0001:00002c58       ??_C@_0BI@HFDBADNK@RxPower?$FL?$CFd?$FN?0?5Rssi?5?$DN?5?$CFd?6?$AA@ 10003c58     aironet.obj
 0001:00002c70       ??_C@_0DP@HNICGIJE@AironetAddBeaconReport?3?5Bssid?5?$CF0@ 10003c70     aironet.obj
 0001:00002cb0       ??_C@_0CH@FDCOMDNO@?$CK?$CK?$CK?$CK?$CK?$CK?5FrameReportLen?5?$DN?5?$CFd?0?5retu@ 10003cb0     aironet.obj
 0001:00002cd8       ??_C@_0CJ@BHBGMGP@?$CK?$CK?$CK?$CK?$CK?$CK?5RxPower?$FL?$CFd?$FN?5Rssi?5?$CFd?0?5Avg?5@ 10003cd8     aironet.obj
 0001:00002d08       ??_C@_0GA@HOPJNKPL@?$CK?$CK?$CK?$CK?$CK?$CK?5AironetAddBeaconReport?0?5B@ 10003d08     aironet.obj
 0001:00002d68       ??_C@_0HD@MMDIDAHM@AironetAddFrameTestReport?5?4?4?4pFr@ 10003d68     aironet.obj
 0001:00002ddc       ??_C@_0CG@DAJCGIHC@FrameTestReportAction?5?$CILen?$DN?$CFd?$CJ?$DM?9@ 10003ddc     aironet.obj
 0001:00002e08       ??_C@_0FA@MDKCDDGP@FrameTestReportAction?5?$CIStaCfg?4Fr@ 10003e08     aironet.obj
 0001:00002e58       ??_C@_0DC@LNNPJEIP@PathLossReportAction?0?5FrameLen?$DN?$CF@ 10003e58     aironet.obj
 0001:00002e8c       ??_C@_0CO@DGLEEJKD@PathLossReportAction?0?5Token?$DN?$CFx?$DN?$DN@ 10003e8c     aironet.obj
 0001:00002ebc       ??_C@_0CG@CMGCADFP@PathlossMessageAction?5?$CILen?$DN?$CFd?$CJ?$DM?9@ 10003ebc     aironet.obj
 0001:00002ee4       ??_C@_0CL@CKOPNLHA@PathlossMessageAction?5?$CIFrameLen?$DN@ 10003ee4     aironet.obj
 0001:00002f10       ??_C@_0CN@EFMONDDE@Pathloss?5Message?5on?5?$CIChannel?$DN?$CFd?$CJ@ 10003f10     aironet.obj
 0001:00002f40       ??_C@_0DL@IONPCLCC@PathLossMessageAction?5sizeof?$CIPLM@ 10003f40     aironet.obj
 0001:00002f7c       ??_C@_0CD@FNIIPLPI@StatisticsReportAction?5?$CI?$CFd?$CJ?$DM?9?9?9?9@ 10003f7c     aironet.obj
 0001:00002fa0       ??_C@_04OKGDLNCL@NONE?$AA@ 10003fa0     aironet.obj
 0001:00002fa8       ??_C@_04GNNGJOGP@CCMP?$AA@ 10003fa8     aironet.obj
 0001:00002fb0       ??_C@_04HNKLFFMO@TKIP?$AA@ 10003fb0     aironet.obj
 0001:00002fb8       ??_C@_04OGBMLJCE@WEP?5?$AA@ 10003fb8     aironet.obj
 0001:00002fc0       ??_C@_0CM@BJINNCDM@StatisticsReportAction?5?$CIFrameLen@ 10003fc0     aironet.obj
 0001:00002fec       ??_C@_0DF@LOPBIBIG@CCXAironetTimeOutAction?3?5pAd?9?$DOSt@ 10003fec     aironet.obj
 0001:00003028       ??_C@_0HE@BPMJKKJG@L2Roaming?5IAPP?$CILen?$DN?$CFd?$CJ?5type?$DN0x?$CF0@ 10004028     aironet.obj
 0001:0000309c       ??_C@_0BM@CHINHJPL@?$DM?$DM?$DN?$DN?$DN?$DN?$DN?$DN?5AironetDirectRoam?6?$AA@ 1000409c     aironet.obj
 0001:000030b8       ??_C@_0DP@CJFINENN@Direct?5Roam?5to?5?$CF02x?3?$CF02x?3?$CF02x?3?$CF0@ 100040b8     aironet.obj
 0001:000030f8       ??_C@_0DO@JOBFJHKF@Aironet?5Direct?5Roam?5FAIL?9?5No?5eli@ 100040f8     aironet.obj
 0001:00003138       ??_C@_0DE@FPKCAMBK@Aironet?5Direct?5Roam?5?9?5Can?8t?5find@ 10004138     aironet.obj
 0001:0000316c       ??_C@_0CA@EIJLLNEB@LastRssi?5?$DN?5?$CFd?0?5pBss?9?$DORssi?5?$DN?5?$CFd?6?$AA@ 1000416c     aironet.obj
 0001:0000318c       ??_C@_0CO@NECLHMFE@AironetDirectRoam?0?5CCX_NBL?4NBENu@ 1000418c     aironet.obj
 0001:000031bc       ??_C@_0CK@GCJEBPNA@?4?4?4FrameReportLen?$DN?$CFd?0?5RealRssi?$DN?$CF@ 100041bc     aironet.obj
 0001:000031e8       ??_C@_0DI@PPELKPOC@AironetLinkTestAction?4?4?4?5Quality@ 100041e8     aironet.obj
 0001:00003220       ??_C@_0DK@NPNHOFML@LinkTest?5Request?5Signal?5?$DN?5?$CFx?0?5?$CFx@ 10004220     aironet.obj
 0001:0000325c       ??_C@_0P@ELMIHHGA@TimeStamp?$DN?5?$CFx?6?$AA@ 1000425c     aironet.obj
 0001:0000326c       ??_C@_0O@DGKPAAOD@FrameNum?5?$DN?$CFd?6?$AA@ 1000426c     aironet.obj
 0001:0000327c       ??_C@_0L@ODMDJMPC@Code?5?$DN?5?$CFx?6?$AA@ 1000427c     aironet.obj
 0001:00003288       ??_C@_0M@MJIJGMFK@Subtype?5?$CFx?6?$AA@ 10004288     aironet.obj
 0001:00003294       ??_C@_0CE@HCIKBDNP@IAPP?5LinkTest?5Length?5?$CFd?0?5MsgLen?$DN@ 10004294     aironet.obj
 0001:000032b8       ??_C@_0CJ@BJGFJHFK@AironetLinkTestAction?5?5?$DN?$DN?$DN?$DN?$DN?$DN?$DN?$DN?$DN@ 100042b8     aironet.obj
 0001:000032e4       ??_C@_0CP@IBKDKKJG@AironetLinkTestAction?0?5Elem?9?$DOMsg@ 100042e4     aironet.obj
 0001:00003314       ??_C@_0CH@DAFCLHAG@?$DM?$DN?$DN?$DN?$DN?$DN?$DN?$DNSendAironetReport?5?5Lengt@ 10004314     aironet.obj
 0001:0000333c       ??_C@_0BJ@NCJMDBGH@alloc?5ndis?5buffer?5?5fail?6?$AA@ 1000433c     aironet.obj
 0001:00003358       ??_C@_0BI@HDBLILBL@alloc?5ndis?5packet?5fail?6?$AA@ 10004358     aironet.obj
 0001:00003370       ??_C@_0CH@MNBGHNL@SendAironetReport?$DN?$DN?$DN?$DN?$DN?$DN?$DN?$DO?5?5Lengt@ 10004370     aironet.obj
 0001:00003398       ??_C@_0CG@NIAGEKCJ@SendAironetReport?5return?5?$CIflag?5?$DN@ 10004398     aironet.obj
 0001:000033c0       ??_C@_0CK@HHBIHOLK@TxAironetFromSupplicantAction?5?$CI?$CF@ 100043c0     aironet.obj
 0001:000033ec       ??_C@_0DF@FGJPOOHN@TxAironetFromSupplicantAction?5?$CIM@ 100043ec     aironet.obj
 0001:00003424       ??_C@_0BP@FMAGPLDE@InitCACTspec?5Size?$DN?$CFd?5?4?4?4?4?4?4?4?5?6?$AA@ 10004424     aironet.obj
 0001:00003448       ??_C@_0EH@PNJMNFJO@CacTsMetricsRptTimeoutAction?5pAd@ 10004448     aironet.obj
 0001:00003490       ??_C@_0DD@IPJMNGEC@CacTsMetricsRptTimeoutAction?0?5WM@ 10004490     aironet.obj
 0001:000034c8       ??_C@_0GF@PJHKPJPO@AironetApLogEntryUpdate?5?$FL?$CF02X?3?$CF0@ 100044c8     aironet.obj
 0001:00003530       ??_C@_0HE@LOAMFMI@ApLogTableSetEntry?5?$FL?$CF02X?3?$CF02X?3?$CF0@ 10004530     aironet.obj
 0001:000035a4       ??_C@_0CB@NGFMLKPK@?$DM?$DN?$DN?5SendEAPOLStart?0?5FrameLen?$DN?$CFd?6@ 100045a4     aironet.obj
 0001:000035c8       ??_C@_0BE@FLPELCNC@?$DM?$DN?$DN?5SendEAPOLStart?6?$AA@ 100045c8     aironet.obj
 0001:000035dc       ??_C@_0DL@PNLBLNDL@Send?5EAPOL?9Start?5Frame?5failed?0?5c@ 100045dc     aironet.obj
 0001:00003618       ??_C@_0BE@NEBFFEPG@?$DN?$DN?$DO?5SendEAPOLStart?6?$AA@ 10004618     aironet.obj
 0001:00003630       ??_C@_0GD@MDDFGDLD@AironetRFRoaming?5?9?9?5call?5MlmeChe@ 10004630     aironet.obj
 0001:00003694       ??_C@_0CJ@HDBMFCHO@AironetRFRoaming?5?9?9?9?$DO?5Drasticall@ 10004694     aironet.obj
 0001:000036c0       ??_C@_0DO@BJDGBEHI@LastBeaconRxTime?5?$DN?5?$CFd?0?5CCXPktLos@ 100046c0     aironet.obj
 0001:00003700       ??_C@_0DI@IFFCPMCJ@AironetRFRoaming?5?9?9?5MaxRSSI?$DN?$CFd?0?5@ 10004700     aironet.obj
 0001:00003738       ??_C@_0CA@HKCKPDOJ@?$DM?$DM?9?9?9?9?9?9?9?9?9?9?5AironetASTScanReq?6?$AA@ 10004738     aironet.obj
 0001:00003758       ??_C@_0BK@DAKNAHNJ@AironetASTScanReq?5?9?9?9?9?9?$DO?6?$AA@ 10004758     aironet.obj
 0001:00003774       ??_C@_0CB@OGOLGCPL@CCXDiagGetMemory?5?$DM?$DM?$DN?$DN?$DN?$DN?$DN?$DN?$DN?$DN?$DN?$DN?$DN?$DN?6@ 10004774     aironet.obj
 0001:00003798       ??_C@_0CF@GHMLKIBO@CCXDiagGetMemory?5return?5?$CIflag?5?$DN?5@ 10004798     aironet.obj
 0001:000037c0       ??_C@_0CH@GBCKEMOM@?$DN?$DN?$DO?5CCXDiagGetMemory?0?5CurrentInd@ 100047c0     aironet.obj
 0001:000037e8       ??_C@_0CH@IFLJOJFC@CCXDiagFreeMemoryHandler?5?5?$DM?$DM?$DN?$DN?$DN?$DN@ 100047e8     aironet.obj
 0001:00003810       ??_C@_0BO@LFEJJEPB@?$DN?$DN?$DO?5CCXDiagFreeMemoryHandler?6?$AA@ 10004810     aironet.obj
 0001:00003830       ??_C@_0CM@EHDMAPA@CCXDiagLogFrame?0?5Length?$DN?$CFd?5?$DM?$DM?$DN?$DN?$DN@ 10004830     aironet.obj
 0001:0000385c       ??_C@_0BF@EMCPLOHH@?$DN?$DN?$DO?5CCXDiagLogFrame?6?$AA@ 1000485c     aironet.obj
 0001:00003874       ??_C@_0DJ@LJDGENJN@?$DN?$DN?$DO?5TxCCXDiagLogFrames?0?5DiagMemo@ 10004874     aironet.obj
 0001:000038b0       ??_C@_0CH@DGBJJDNE@TxCCXDiagLogFrames?5return?5?$CIflag?5@ 100048b0     aironet.obj
 0001:000038d8       ??_C@_0CM@OBCIMEMP@has?5disassociated?5with?5invalid?5P@ 100048d8     ap.obj
 0001:00003904       ??_C@_0BH@IGJNPKB@active?5countermeasures?$AA@ 10004904     ap.obj
 0001:0000391c       ??_C@_0CE@JFLNOENI@has?5been?5aged?9out?5and?5disassocia@ 1000491c     ap.obj
 0001:00003940       ??_C@_0BC@HLHDIMIG@has?5disassociated?$AA@ 10004940     ap.obj
 0001:00003954       ??_C@_0BI@ICOOKKNB@successfully?5associated?$AA@ 10004954     ap.obj
 0001:0000396c       ??_C@_0BF@ILIMBFOC@restart?5access?5point?$AA@ 1000496c     ap.obj
 0001:00003b88       ??_C@_0BD@LHFBKBMP@?$DM?9?9?9?5APInitialize?6?$AA@ 10004b88     ap.obj
 0001:00003b9c       ??_C@_0BD@LMBOJAPB@?9?9?9?$DO?5APInitialize?6?$AA@ 10004b9c     ap.obj
 0001:00003bb0       ??_C@_0BA@MJDMODHK@?$DM?$DN?$DN?$DN?5APStartUp?6?$AA@ 10004bb0     ap.obj
 0001:00003bc0       ??_C@_0DI@NOJOFEJG@?5APStartUp?5?3?5?5Group?5rekey?5method@ 10004bc0     ap.obj
 0001:00003bf8       ??_C@_0CM@LMPNMIBE@AP?5AuthMode?$DN?$CFd?0?5disable?5Pairwise@ 10004bf8     ap.obj
 0001:00003c24       ??_C@_0CM@HHJMCJBG@AP?5AuthMode?$DN?$CFd?0?5Pairwise?5Key?5Tab@ 10004c24     ap.obj
 0001:00003c50       ??_C@_0EL@JJKOIOIM@ApStartUp?5?3?520MHz?0?5ChannelWidth?$DN@ 10004c50     ap.obj
 0001:00003ca0       ??_C@_0EF@HEPOMKKO@ApStartUp?5?3?5ExtBlow?0?5ChannelWidt@ 10004ca0     ap.obj
 0001:00003ce8       ??_C@_0EG@LKDFIHBC@ApStartUp?5?3?5ExtAbove?0?5ChannelWid@ 10004ce8     ap.obj
 0001:00003d30       ??_C@_09CEMLLPEP@?5rt2860C?6?$AA@ 10004d30     ap.obj
 0001:00003d3c       ??_C@_0CG@KLPPAIJF@11n?5check?5?$CFs?$CI?$CJ?5Line?$FL?$CFd?$FN?0?5PhyMode@ 10004d3c     ap.obj
 0001:00003d64       ??_C@_09DNHOHHEK@APStartUp?$AA@ 10004d64     ap.obj
 0001:00003d70       ??_C@_05GCOINAMN@My?5AP?$AA@ 10004d70     ap.obj
 0001:00003d78       ??_C@_0BA@NKJOBOCF@?$DN?$DN?$DN?$DO?5APStartUp?6?$AA@ 10004d78     ap.obj
 0001:00003d88       ??_C@_0BB@BEAHICHI@?$DM?$DN?$DN?$DN?5APStop?5?$CB?$CB?$CB?6?$AA@ 10004d88     ap.obj
 0001:00003d9c       ??_C@_0BE@GLBCENCC@After?5cancel?5timer?6?$AA@ 10004d9c     ap.obj
 0001:00003db0       ??_C@_0BB@OPMAGMOA@?$DN?$DN?$DN?$DO?5APStop?5?$CB?$CB?$CB?6?$AA@ 10004db0     ap.obj
 0001:00003dc4       ??_C@_0BB@GFJKJDIB@?$DM?9?9?9?5APShutdown?6?$AA@ 10004dc4     ap.obj
 0001:00003dd8       ??_C@_0BB@OPLONIAI@?9?9?9?$DO?5APShutdown?6?$AA@ 10004dd8     ap.obj
 0001:00003dec       ??_C@_0CJ@IDLCMGON@LOG?$CD?$CFd?5?$CF02x?3?$CF02x?3?$CF02x?3?$CF02x?3?$CF02x?3@ 10004dec     ap.obj
 0001:00003e18       ??_C@_0EA@CBKAIAPC@APUpdateCapabilityAndErpIe?5?9?5Cap@ 10004e18     ap.obj
 0001:00003e58       ??_C@_0DL@OOPKDIMB@APUpdateCapabilityAndErpIe?5?9?5Leg@ 10004e58     ap.obj
 0001:00003e94       ??_C@_0DD@DFAJOIFG@?$CF02x?3?$CF02x?3?$CF02x?3?$CF02x?3?$CF02x?3?$CF02x?5fa@ 10004e94     ap.obj
 0001:00003ec8       ??_C@_0DP@BFGIIGEB@APPsIndicate?5?9?$FL?$CFdth?$FN?5not?5match?5?$CF@ 10004ec8     ap.obj
 0001:00003f08       ??_C@_0DF@ICIKJFHP@APPsIndicate?5?9?5?$CF02x?3?$CF02x?3?$CF02x?3?$CF0@ 10004f08     ap.obj
 0001:00003f40       ??_C@_0EM@BIFGPPLM@APPsIndicate?5?9?5?$CF02x?3?$CF02x?3?$CF02x?3?$CF0@ 10004f40     ap.obj
 0001:00003f8c       ??_C@_0BH@DEDAPBGC@APPsIndicate?5wcid?$DN?$CFx?5?6?$AA@ 10004f8c     ap.obj
 0001:00003fa8       ??_C@_0EB@BLIEMIEF@ASSOC?5?9?5Send?5DISASSOC?5?5Reason?5?$DN?5@ 10004fa8     ap.obj
 0001:00003fec       ??_C@_0BM@DDKHEINB@?5?$CFdth?5PsQueue?4Number?5?$CFd?4?4?4?6?$AA@ 10004fec     ap.obj
 0001:00004008       ??_C@_0BL@GMKELHOH@McastPsQueue?4Number?5?$CFd?4?4?4?6?$AA@ 10005008     ap.obj
 0001:00004024       ??_C@_0DI@DCEFAMEE@MacTableInsertWDSEntry?5?9?5allocat@ 10005024     ap.obj
 0001:00004060       ??_C@_0EI@NBMKCPFJ@?$CFs?3?5Zero?5pEntry?0?5MacTab?4Size?5?$CFd?5@ 10005060     ap.obj
 0001:000040a8       ??_C@_0CN@FHELNLPJ@?$CFs?3?5The?5size?5of?5MacTable?5is?5alre@ 100050a8     ap.obj
 0001:000040d8       ??_C@_0BE@DJMFPIIF@MacTableDeleteEntry?$AA@ 100050d8     ap.obj
 0001:000040ec       ??_C@_0BK@NBFEDHKJ@Aid?$DN?50x?$CFx?4SetTid?$DN?50x?$CFx?4?5?6?$AA@ 100050ec     ap.obj
 0001:00004108       ??_C@_0CC@NHCAEDDI@MacTableDeleteEntry2?5?9?5Total?$DN?5?$CFd@ 10005108     ap.obj
 0001:0000412c       ??_C@_0CC@MGFNCJEB@MacTableDeleteEntry1?5?9?5Total?$DN?5?$CFd@ 1000512c     ap.obj
 0001:00004150       ??_C@_0CB@NELAKFLO@MacTableDeleteEntry?5?9?5Total?$DN?5?$CFd?6@ 10005150     ap.obj
 0001:00004174       ??_C@_0DH@FAAAAHPA@Write?50x?$CFx?5to?5MAC?5register?5MAX_L@ 10005174     ap.obj
 0001:000041ac       ??_C@_0DL@DJEJHCDC@ageout?5?$CF02x?3?$CF02x?3?$CF02x?3?$CF02x?3?$CF02x?3@ 100051ac     ap.obj
 0001:000041e8       ??_C@_0EA@CIPOOPMN@?$CF02x?3?$CF02x?3?$CF02x?3?$CF02x?3?$CF02x?3?$CF02x?5fa@ 100051e8     ap.obj
 0001:00004228       ??_C@_0DF@CHNGGFCO@WdsTableInsertEntry?5?9?5allocate?5e@ 10005228     ap.obj
 0001:00004260       ??_C@_0CB@GCFFJEKD@WdsTableDeleteEntry?5?9?5Total?$DN?5?$CFd?6@ 10005260     ap.obj
 0001:00004288       ??_C@_0EI@MFLIHAIM@ageout?5?$CF02x?3?$CF02x?3?$CF02x?3?$CF02x?3?$CF02x?3@ 10005288     ap.obj
 0001:000042d0       ??_C@_0CD@BPJOBPLO@STA?5on?5negative?5ACL?4?5remove?5it?4?4@ 100052d0     ap.obj
 0001:000042f8       ??_C@_0EE@ENBLOLKH@?$CFs?3?5ASSOC?5?9?5Send?5DISASSOC?$DL?5Reaso@ 100052f8     ap.obj
 0001:0000433c       ??_C@_0BK@OIMHNMKO@ApUpdateAccessControlList?$AA@ 1000533c     ap.obj
 0001:00004358       ??_C@_0CH@HKMFPMCF@STA?5not?5on?5positive?5ACL?4?5remove?5@ 10005358     ap.obj
 0001:00004580       ??_C@_0CM@MPNGPEKG@ASSOC?5?9?5Send?5ASSOC?5response?5?$CISta@ 10005580     ap_assoc.obj
 0001:000045b0       ??_C@_0EC@NCFIEELM@ASSOC?5?9?5receive?5ASSOC?5request?5fr@ 100055b0     ap_assoc.obj
 0001:000045f4       ??_C@_0DB@BIIEOGKJ@ASSOC?5?9?5Send?5RE?9ASSOC?5response?5?$CI@ 100055f4     ap_assoc.obj
 0001:00004628       ??_C@_0EF@ILBDJMFH@ASSOC?5?9?5receive?5RE?9ASSOC?5request@ 10005628     ap_assoc.obj
 0001:00004670       ??_C@_0FB@BKDILDDB@ASSOC?5?9?5receive?5DIS?9ASSOC?5reques@ 10005670     ap_assoc.obj
 0001:000046c4       ??_C@_0CG@BICMPCMA@ASSOC?5?9?51?5receive?5DIS?9ASSOC?5requ@ 100056c4     ap_assoc.obj
 0001:000046f0       ??_C@_0FB@GEHPAGBA@ASSOC?5?9?5MLME?5disassociates?5?$CF02x?3@ 100056f0     ap_assoc.obj
 0001:00004748       ??_C@_0EN@KFHOGFDG@ASSOC?5?9?5Class?53?5Error?0?5Send?5DISA@ 10005748     ap_assoc.obj
 0001:00004798       ??_C@_0GA@MCONOJPG@ASSOC?5?9?5MaxRAmpduFactor?$DN?$CFd?0?5Mmps@ 10005798     ap_assoc.obj
 0001:000047f8       ??_C@_0FL@HEADMCJA@ASSOC?5?9?5CurrTxRate?$DN?$CFd?0?5MODE?$DN?$CFd?0?5@ 100057f8     ap_assoc.obj
 0001:00004858       ??_C@_0GE@HCNHAGLL@ASSOC?5?9?5Assign?5AID?$DN?$CFd?5to?5STA?5?$CF02@ 10005858     ap_assoc.obj
 0001:000048c0       ??_C@_0FJ@OFJJEOOJ@ASSOC?5?9?5WMM?$DN?$CFd?0?5AuthMode?$DN?$CFd?0?5Wep@ 100058c0     ap_assoc.obj
 0001:00004920       ??_C@_0GI@EELCAMKH@ASSOC?5?9?5Update?5AP?5OperaionMode?$DN?$CF@ 10005920     ap_assoc.obj
 0001:00004988       ??_C@_0CP@LFAJJEMI@ASSOC?5?9?5TXBAbitmap?5?$DN?50x?$CFx?0?5RXBAb@ 10005988     ap_assoc.obj
 0001:000049b8       ??_C@_0BF@KKIOCLFG@ASSOC?0?5RDG?5enabled?5?6?$AA@ 100059b8     ap_assoc.obj
 0001:000049d0       ??_C@_0DG@IDFJJHIE@ASSOC?$DM?$DN?$DN?$DN?5pAd?9?$DOCommonCfg?4Desired@ 100059d0     ap_assoc.obj
 0001:00004a08       ??_C@_0BO@MDFDFDAE@ASSOC?$DM?$DN?$DN?$DN?5Use?5Fixed?5MCS?5?$DN?5?$CFd?6?$AA@ 10005a08     ap_assoc.obj
 0001:00004a28       ??_C@_0BG@DFLEAADG@ASSOC?5?9PiggyBack2?$DN?51?6?$AA@ 10005a28     ap_assoc.obj
 0001:00004a40       ??_C@_0BF@OAAIBLNK@ASSOC?5?9PiggyBack?$DN?51?6?$AA@ 10005a40     ap_assoc.obj
 0001:00004a58       ??_C@_0GF@GNEFIFAI@APBuildAssociation?3?3MAC?$FL?$CF02x?3?$CF02@ 10005a58     ap_assoc.obj
 0001:00004ac0       ??_C@_0IH@LPOHNHNJ@ASSOC?5?9?5The?5authentication?5mode?5@ 10005ac0     ap_assoc.obj
 0001:00004b48       ??_C@_0DN@DFBMMJOO@ASSOC?5?9?5MaxSupportedRate?5?$DN?5?$CFx?3pA@ 10005b48     ap_assoc.obj
 0001:00004b88       ??_C@_0DB@HHMDCEDH@ASSOC?5?9?5RSNIE_Len?5?$DN?50x?$CFx?0?5RSNIE?5@ 10005b88     ap_assoc.obj
 0001:00004bc0       ??_C@_0EA@IMGBINOC@?$CFs?3?5Invalid?5authentication?5mode?5@ 10005bc0     ap_assoc.obj
 0001:00004c00       ??_C@_0BD@HIJBOIEE@APBuildAssociation?$AA@ 10005c00     ap_assoc.obj
 0001:00004e18       ??_C@_0DK@KHNICBPP@AUTH?5?9?5Send?5DE?9AUTH?5req?5to?5?$CF02x?3@ 10005e18     ap_auth.obj
 0001:00004e58       ??_C@_0EK@KPHNFFAC@AUTH?5?9?5Class?52?5error?0?5Send?5DEAUT@ 10005e58     ap_auth.obj
 0001:000050a8       ??_C@_0BE@CPPNNHBP@Rcv?5Challenge?5?$DN?5?$CFs?6?$AA@ 100060a8     ap_authrsp.obj
 0001:000050bc       ??_C@_0BF@IMLGPCOG@Sent?5Challenge?5?$DN?5?$CFs?6?$AA@ 100060bc     ap_authrsp.obj
 0001:000050d4       ??_C@_0BC@INMJHEOG@pRcvHdr?9?$DOWep?$DN?5?$CFd?6?$AA@ 100060d4     ap_authrsp.obj
 0001:000050e8       ??_C@_0CI@BOFALBKA@AUTH_RSP?5?9?5Alg?$DN?$CFd?0?5Seq?$DN?$CFd?0?5AuthM@ 100060e8     ap_authrsp.obj
 0001:00005110       ??_C@_0CI@JDBPJGCF@AUTH_RSP?5?9?5Send?5AUTH?5seq?$CD2?5?$CIChal@ 10006110     ap_authrsp.obj
 0001:00005138       ??_C@_0FL@MKCGHLDA@AUTH_RSP?5?9?5Rcv?5AUTH?5seq?$CD?$CFd?0?5Alg?$DN@ 10006138     ap_authrsp.obj
 0001:00005198       ??_C@_0FM@DJNJEFNI@APPeerAuthAtAuthRspIdleAction?3?5F@ 10006198     ap_authrsp.obj
 0001:000051f4       ??_C@_0CF@HHNJFDNO@Atheros?5Problem?4?5Turn?5on?5RTS?1CTS@ 100061f4     ap_authrsp.obj
 0001:0000521c       ??_C@_0CK@CDMCPDEG@AUTH_RSP?5?9?5APPeerAuthAtAuthRspId@ 1000621c     ap_authrsp.obj
 0001:00005248       ??_C@_0EM@JHGIFBIF@AUTH_RSP?5?9?5receive?5DE?9AUTH?4?5dele@ 10006248     ap_authrsp.obj
 0001:00005294       ??_C@_0CC@GDOMGIMA@AUTH_RSP?5?9?5APPeerDeauthReqAction@ 10006294     ap_authrsp.obj
 0001:000052b8       ??_C@_0CM@KNJOJIGB@AUTH_RSP?5?9?5Peer?5AUTH?5fail?5?$CIStatu@ 100062b8     ap_authrsp.obj
 0001:000052e4       ??_C@_0CM@PJMHKBJK@AUTH_RSP?5?9?5Send?5AUTH?5response?5?$CIS@ 100062e4     ap_authrsp.obj
 0001:00005710       ??_C@_0CJ@CJAKMIMF@APSendPackets?5?9?9?$DO?5carrier?5assert@ 10006710     ap_data.obj
 0001:00005740       ??_C@_0EG@EBFMEOBJ@Drop?5send?5request?5since?5hardware@ 10006740     ap_data.obj
 0001:00005788       ??_C@_0DI@FCMNBHBG@?$CFs?3?5Drop?5those?5packets?5due?5to?5th@ 10006788     ap_data.obj
 0001:000057c0       ??_C@_0O@BMMIJDJE@APSendPackets?$AA@ 100067c0     ap_data.obj
 0001:000057d0       ??_C@_0BF@EOJKCLEC@?$DN?$DN?$DN?$DN?$DO?5APSendPackets?6?$AA@ 100067d0     ap_data.obj
 0001:000057e8       ??_C@_0DO@PLMHBEPD@STA?5?$CIAID?$DN?$CFd?$CJ?5in?5PSM?0?5move?5to?5PSQ@ 100067e8     ap_data.obj
 0001:00005828       ??_C@_0FP@COIHJKAJ@HardTx?5Header?$DN?5?$CF08x?3?5?$CF08x?3?5?$CF08x?3@ 10006828     ap_data.obj
 0001:00005888       ??_C@_0DN@ILLEELCD@Last?3?5HardTx?5TxWI?$DN?5?$CF08x?3?5?$CF08x?3?5?$CF@ 10006888     ap_data.obj
 0001:000058c8       ??_C@_0DN@JIMFDIFF@Multicast?5rate?5is?5the?5same?5with?5@ 100068c8     ap_data.obj
 0001:00005908       ??_C@_0DO@MNMFKEMJ@Auto?3?5MODE?$DNHTMIX?5or?5HTGF?0?5MCS?$DN?$CFd@ 10006908     ap_data.obj
 0001:00005948       ??_C@_0CO@OHEJAMDO@Auto?3?5MODE?$DNOFDM?0?5MCS?$DN?$CFd?0?5Force?5M@ 10006948     ap_data.obj
 0001:00005978       ??_C@_0GH@PDBNOBMB@User?5define?3?5SoftAPForceMulticas@ 10006978     ap_data.obj
 0001:000059e0       ??_C@_0IA@KIJMAOEG@Error?3?5Force?5multicast?5rate?5to?51@ 100069e0     ap_data.obj
 0001:00005a60       ??_C@_0IB@IPDLDOHH@Error?3?5Force?5multicast?5rate?5to?52@ 10006a60     ap_data.obj
 0001:00005ae4       ??_C@_0DH@EIHLCIFM@bHasValidCLI?$DN?$CFd?0?5LowestRateRAWci@ 10006ae4     ap_data.obj
 0001:00005b20       ??_C@_0EC@PKJMDEJI@More?5Frag?3?5HardTx?5TxWI?$DN?5?$CF08x?3?5?$CF0@ 10006b20     ap_data.obj
 0001:00005b64       ??_C@_05JNBEKFOE@?$CF02x?3?$AA@ 10006b64     ap_data.obj
 0001:00005b6c       ??_C@_0CM@BHAOKIBH@Calculated?5TX?5MIC?5value?5?$DN?5?5Bytes@ 10006b6c     ap_data.obj
 0001:00005b98       ??_C@_0DI@BKLBNBLI@?52pSrcBufVA?5IS?5NULL?5?$CB?$CB?$CB?$CB?$CB?$CB?$CB?$CB?$CB?$CB?$CB?$CB@ 10006b98     ap_data.obj
 0001:00005bd0       ??_C@_1FI@KJECFLHJ@?$AAC?$AA?3?$AA?2?$AAW?$AAi?$AAn?$AAC?$AAE?$AA6?$AA?4?$AA0?$AA?2?$AAN?$AAe?$AAw?$AA?2?$AAR?$AAT?$AA2?$AA8?$AA7?$AA0?$AA_?$AAv?$AA1?$AA?4?$AA4?$AA?4?$AA9?$AA?4?$AA0?$AA?2@ 10006bd0     ap_data.obj
 0001:00005c28       ??_C@_0BK@IGCCDMEB@?52RTMPCalculateMICValue?5?6?$AA@ 10006c28     ap_data.obj
 0001:00005c44       ??_C@_0BK@DBMMAJN@1?5RTMPCalculateMICValue?5?6?$AA@ 10006c44     ap_data.obj
 0001:00005c60       ??_C@_0EM@GDLKNPGO@RTUSBHardTransmit?5c3?5?9?9?$DO?5CurWrit@ 10006c60     ap_data.obj
 0001:00005cb0       ??_C@_0EM@HLBAANAK@RTUSBHardTransmit?5c2?5?9?9?$DO?5CurWrit@ 10006cb0     ap_data.obj
 0001:00005d00       ??_C@_0EM@FCOPHLKG@RTUSBHardTransmit?5c1?5?9?9?$DO?5CurWrit@ 10006d00     ap_data.obj
 0001:00005d4c       ??_C@_0DP@PJJMBJHH@APHardTransmit?$CIEAPOL?$DN?$CFd?0?5Mcast?$DN?$CF@ 10006d4c     ap_data.obj
 0001:00005d8c       ??_C@_0CN@FMACOKEJ@USE_LEGACY_MCAST_RATE?3?5Set?5bHTRa@ 10006d8c     ap_data.obj
 0001:00005dbc       ??_C@_0DA@KJOABIEL@USER_DEFINE_MCAST_RATE?3?5MODE?$DN?$CFd?0@ 10006dbc     ap_data.obj
 0001:00005dec       ??_C@_0DL@JFCHOLE@SoftAPForceMulticastRate?$DN0x?$CFx?0?5u@ 10006dec     ap_data.obj
 0001:00005e28       ??_C@_0EO@NGFBCNAK@bAllowChangeMcastRate?$DN?$CFd?0?5bMcast@ 10006e28     ap_data.obj
 0001:00005e78       ??_C@_0DB@GNGOGLOD@RTMPHardTransmit?5?9?9?$DO?5?$FL?$CFd?$FN?5Origin@ 10006e78     ap_data.obj
 0001:00005eac       ??_C@_0DE@HLLDDOPB@RTUSBHardTransmit?5?9?9?$DO?5Ndis?5Packe@ 10006eac     ap_data.obj
 0001:00005ee0       ??_C@_0BJ@GJFMDJBG@pVirtualAddress?5?$DN?$DN?5NULL?6?$AA@ 10006ee0     ap_data.obj
 0001:00005efc       ??_C@_0P@NEJNAILE@packetsize?3?$CFd?6?$AA@ 10006efc     ap_data.obj
 0001:00005f0c       ??_C@_0CH@DMPNFINM@APHardTransmit?$CI?$FL?$CFd?$FN?4bWDSEntry?5?$DN?5@ 10006f0c     ap_data.obj
 0001:00005f34       ??_C@_0CM@HMEBOIHH@RTMPHardTransmit?5?9?9?$DO?5carrier?5ass@ 10006f34     ap_data.obj
 0001:00005f60       ??_C@_0DL@ONHKKFCJ@RTUSBHardTransmit?5?9?9?$DO?5radar?5dete@ 10006f60     ap_data.obj
 0001:00005f9c       ??_C@_0BK@LAEKJJAJ@ignore?5CNTL?5?$CIsubtype?$DN?$CFd?$CJ?6?$AA@ 10006f9c     ap_data.obj
 0001:00005fb8       ??_C@_0CF@IBCMFFID@in?5ACK?5?3?5MFB?5?$DN0x?$CFx?5?3?5ID?$DN?$CFx?5?3?5MFS@ 10006fb8     ap_data.obj
 0001:00005fe0       ??_C@_0CH@CPIDLNNO@in?5B?9ACK?5?3?5MFB?5?$DN0x?$CFx?5?3?5ID?$DN?$CFx?5?3?5M@ 10006fe0     ap_data.obj
 0001:00006008       ??_C@_0ED@BPDGINKD@rcv?5PS?9POLL?5?$CIAID?$DN?$CFd?$CJ?5?$CIWCID?$DN?$CFd?$CJ?5f@ 10007008     ap_data.obj
 0001:0000604c       ??_C@_0BP@KDMEHEI@?5?5?5Disallow?5new?5Association?5?6?5?$AA@ 1000704c     ap_data.obj
 0001:0000606c       ??_C@_0BG@FDIJIFCM@Rx?5MIC?5Value?5error?52?6?$AA@ 1000706c     ap_data.obj
 0001:00006088       ??_C@_0GE@LNANMIMO@?$CB?$CB?$CB?5report?5DATA?5?$CIno?5frag?$CJ?5to?5LLC@ 10007088     ap_data.obj
 0001:000060f0       ??_C@_0GG@NMMPCKNB@?$CB?$CB?$CB?5report?5segregated?5MSDU2?5to?5L@ 100070f0     ap_data.obj
 0001:00006158       ??_C@_0GG@JFHJPPNC@?$CB?$CB?$CB?5report?5segregated?5MSDU1?5to?5L@ 10007158     ap_data.obj
 0001:000061c0       ??_C@_0BC@EKIDIFCL@report?5?5to?5mlme?5?6?$AA@ 100071c0     ap_data.obj
 0001:000061d4       ??_C@_0L@EAMNDNCL@bridge?5to?6?$AA@ 100071d4     ap_data.obj
 0001:000061e0       ??_C@_0CD@DOBPJO@WDS?5Packet?5not?5from?5our?5WDS?5AP?$CB?$CB@ 100071e0     ap_data.obj
 0001:00006204       ??_C@_0BJ@FJGMDLGD@WDS?5topology?5changed?$CB?$CB?$CB?6?$AA@ 10007204     ap_data.obj
 0001:00006220       ??_C@_0CE@JKIFFAJK@?5Drop?5Plain?5text?5packet?$CB?$CBseq?5?$DN?5?$CF@ 10007220     ap_data.obj
 0001:00006244       ??_C@_0BF@KGPCIHEL@get?5WPA?5frame?5?$DN?$DN?$DN?$DO?5?6?$AA@ 10007244     ap_data.obj
 0001:0000625c       ??_C@_0BA@MOKJNLI@A?9MSDU?5data?5?$DN?$CFx?$AA@ 1000725c     ap_data.obj
 0001:0000626c       ??_C@_0CI@NPLFDFC@?5Give?5up?5non?9U2M?5?$CIType?$DN?$CFd?0?5SubTy@ 1000726c     ap_data.obj
 0001:00006294       ??_C@_0DF@HCECPOCO@?$CFs?3?5Drop?5this?5frame?5due?5to?5the?5S@ 10007294     ap_data.obj
 0001:000062cc       ??_C@_0BG@ELPMMPOE@RTUSBAPHandleRxPacket?$AA@ 100072cc     ap_data.obj
 0001:000062e4       ??_C@_0DM@FFNJGKHH@RX?5err?5filtered2?5?$FLMPDUtotalByteC@ 100072e4     ap_data.obj
 0001:00006320       ??_C@_0CG@DPOFOOBO@pRxWI?$DNNULL?5Error?$CB?$CB?5ThisFrameLen?5@ 10007320     ap_data.obj
 0001:00006348       ??_C@_0CH@LDHKCKOD@RxInfo?$DNNULL?5Error?$CB?$CB?5ThisFrameLen@ 10007348     ap_data.obj
 0001:00006370       ??_C@_0GA@ODIGAJGI@bIsBulkINFail?5?$CFd?5ThisFrameLen?5?$CFd@ 10007370     ap_data.obj
 0001:000063d0       ??_C@_0FI@GLLKIJLD@?$CB?$CB?$CB?$CB?5?$CF02x?3?$CF02x?3?$CF02x?3?$CF02x?9?$CF02x?3?$CF0@ 100073d0     ap_data.obj
 0001:00006428       ??_C@_0FI@GADLFFDC@?$CB?$CB?$CB?5?5?$CF02x?3?$CF02x?3?$CF02x?3?$CF02x?9?$CF02x?3?$CF0@ 10007428     ap_data.obj
 0001:00006480       ??_C@_0FI@PKIPGHFI@?$CB?$CB?5?5?5?$CF02x?3?$CF02x?3?$CF02x?3?$CF02x?9?$CF02x?3?$CF0@ 10007480     ap_data.obj
 0001:000064d8       ??_C@_0HH@IKLHIH@5555?90?5ThisFrameLen?5?$DN?5?$CFd?0?5Transf@ 100074d8     ap_data.obj
 0001:00006550       ??_C@_0EO@FBGJJEJH@Total?5BulkIn?5length?$DN?$CFx?0?5Now?5left@ 10007550     ap_data.obj
 0001:000065a0       ??_C@_0CC@LHCLEIFC@This?5Frame?5Len?$CI0x?$CFx?$CJ?5outranges?4?5@ 100075a0     ap_data.obj
 0001:000065c8       ??_C@_0EF@CNBNBMAC@RXDMALen?5not?5multiple?5of?54?4?5?$FL?$CFd?$FN@ 100075c8     ap_data.obj
 0001:00006610       ??_C@_0CL@OCJALGHA@RTUSBRxPacket?5TransferBufferLeng@ 10007610     ap_data.obj
 0001:0000663c       ??_C@_0DB@IJHDEIAP@APCheckClass2Class3Error?0?5invali@ 1000763c     ap_data.obj
 0001:00006670       ??_C@_0ED@CLJOEGPD@rcv?5PS?9POLL?5?$CIAID?$DN?$CFd?5not?5match?$CJ?5f@ 10007670     ap_data.obj
 0001:000066b4       ??_C@_0L@EJFJHCIL@clear?5TIM?6?$AA@ 100076b4     ap_data.obj
 0001:000066c0       ??_C@_0DJ@IJEKGEPO@rcv?5PS?9POLL?5?$CIAID?$DN?$CFd?$CJ?5from?5?$CF02x?3?$CF@ 100076c0     ap_data.obj
 0001:00006700       ??_C@_0EL@FEEIGLJJ@WBRG?5?9?5len?$DN?$CFd?0?5from?5WDS?5?$CD?$CFd?0?5to?5@ 10007700     ap_data.obj
 0001:00006750       ??_C@_0HE@JPAMEPLN@APCheckNDSClient?3?3MAC?$FL?$CF02x?3?$CF02x?3@ 10007750     ap_data.obj
 0001:000069c8       ??_C@_0BM@NMDBEABN@Query?3?3unknown?5OID?50x?$CF08x?5?6?$AA@ 100079c8     ap_info.obj
 0001:000069e4       ??_C@_0CJ@IGGABC@Query?3?3RT_OID_802_11_QUERY_OP_MO@ 100079e4     ap_info.obj
 0001:00006a10       ??_C@_0CO@GJLJAFFP@?5Query?5?3?3?5RT_OID_802_11_QUERY_WP@ 10007a10     ap_info.obj
 0001:00006a40       ??_C@_0DG@IHDKJIIE@Query?3?3RT_OID_802_11_QUERY_ACL?5?$CI@ 10007a40     ap_info.obj
 0001:00006a78       ??_C@_0CG@IFFGHEJP@Query?3?3RT_OID_802_11_QUERY_AP_CO@ 10007a78     ap_info.obj
 0001:00006aa0       ??_C@_0CI@EPCFLDIM@Query?3?3RT_OID_802_11_QUERY_EVENT@ 10007aa0     ap_info.obj
 0001:00006ac8       ??_C@_0BO@CEGFCGIP@Query?3?3OID_802_11_BSSID_LIST?6?$AA@ 10007ac8     ap_info.obj
 0001:00006ae8       ??_C@_0CM@HFEMKMIN@Query?3?3OID_802_11_INFRASTRUCTURE@ 10007ae8     ap_info.obj
 0001:00006b14       ??_C@_0CD@DHAEIFI@Query?3?3RT_OID_802_11_SNR_1?$CI0x?$DN?$CFx@ 10007b14     ap_info.obj
 0001:00006b38       ??_C@_0CD@OMLCCDGG@Query?3?3RT_OID_802_11_SNR_0?$CI0x?$DN?$CFx@ 10007b38     ap_info.obj
 0001:00006b5c       ??_C@_0BN@MAOKAFBN@Query?3?3RT_OID_802_11_RSSI_2?6?$AA@ 10007b5c     ap_info.obj
 0001:00006b7c       ??_C@_0BN@MCKMLLEE@Query?3?3RT_OID_802_11_RSSI_1?6?$AA@ 10007b7c     ap_info.obj
 0001:00006b9c       ??_C@_0BN@CNKIHDGF@Query?3?3OID_802_11_RSSI?$CI?$DN?$CFd?$CJ?6?$AA@ 10007b9c     ap_info.obj
 0001:00006bbc       ??_C@_0DD@HCMDIGNL@Query?3?3OID_802_11_SSID?5?$CILen?$DN?$CFd?0?5@ 10007bbc     ap_info.obj
 0001:00006bf0       ??_C@_0DJ@IDKNAJBP@Query?3?3OID_802_11_BSSID?$CI?$DN?$CF02x?3?$CF0@ 10007bf0     ap_info.obj
 0001:00006c2c       ??_C@_0CA@KHEAIIHN@Query?3?3OID_GEN_SUPPORTED_LIST?5?6?$AA@ 10007c2c     ap_info.obj
 0001:00006c4c       ??_C@_0BN@CNMNLKDJ@Set?3?3?$CB?$CB?$CB?5unknown?5OID?50x?$CF08x?6?$AA@ 10007c4c     ap_info.obj
 0001:00006c6c       ??_C@_0CG@EDILLKLA@Set?3?3RT_OID_802_11_SET_OP_MODE?5?$CI@ 10007c6c     ap_info.obj
 0001:00006c94       ??_C@_0CP@MDABCIBC@Set?3?3RT_OID_802_11_SET_TX_POWER_@ 10007c94     ap_info.obj
 0001:00006cc4       ??_C@_0DD@IDGGBEPF@Set?3?3RT_OID_802_11_SET_ACL?5?$CIPoli@ 10007cc4     ap_info.obj
 0001:00006cf8       ??_C@_0BM@KGHOHKLC@Set?3?3RT_OID_802_11_SET_ACL?6?$AA@ 10007cf8     ap_info.obj
 0001:00006d14       ??_C@_0CC@OEPHIGOJ@Set?3?3RT_OID_802_11_SET_AP_CONFIG@ 10007d14     ap_info.obj
 0001:00006d38       ??_C@_0CD@LPKILJFO@Set?3?3RT_OID_802_11_SET_HT_PHYMOD@ 10007d38     ap_info.obj
 0001:00006d5c       ??_C@_0CO@MGMKFFHD@Set?3?3RT_OID_802_11_SET_PHY_MODE?5@ 10007d5c     ap_info.obj
 0001:00006d8c       ??_C@_0CH@PHDOBFHD@Set?3?3RT_OID_802_11_SET_PHY_MODE?5@ 10007d8c     ap_info.obj
 0001:00006db4       ??_C@_0DP@EOKAOKDM@Set?3?3OID_802_11_CONFIGURATION?5?$CIB@ 10007db4     ap_info.obj
 0001:00006df8       ??_C@_0EJ@JFEAGLFK@Set?3?3OID_802_11_DESIRED_RATES?5?$CI?$CF@ 10007df8     ap_info.obj
 0001:00006e44       ??_C@_0BP@PKDDENNG@Set?3?3OID_802_11_DESIRED_RATES?6?$AA@ 10007e44     ap_info.obj
 0001:00006e64       ??_C@_0CL@FMJJGPLE@Set?3?3OID_802_11_NETWORK_TYPE_IN_@ 10007e64     ap_info.obj
 0001:00006e90       ??_C@_0CF@NPOBMCFM@Set?3?3OID_802_11_NETWORK_TYPE_IN_@ 10007e90     ap_info.obj
 0001:00006eb8       ??_C@_0DE@DFNNFCDB@Set?3?3OID_802_11_RELOAD_DEFAULTS?5@ 10007eb8     ap_info.obj
 0001:00006eec       ??_C@_0CC@BNKDOJOB@Set?3?3OID_802_11_WEP_STATUS?5?$CI?$DN?$CFd?$CJ@ 10007eec     ap_info.obj
 0001:00006f10       ??_C@_0CC@FIBAHHID@Set?3?3OID_802_11_BSSID_LIST_SCAN?5@ 10007f10     ap_info.obj
 0001:00006f34       ??_C@_0CH@CICLDDKH@Set?3?3OID_802_11_PRIVACY_FILTER?5?$CI@ 10007f34     ap_info.obj
 0001:00006f5c       ??_C@_0CM@JKBNFDAO@Set?3?3OID_802_11_AUTHENTICATION_M@ 10007f5c     ap_info.obj
 0001:00006f88       ??_C@_0BP@KHNLCAOO@Set?3?3OID_802_11_DISASSOCIATE?5?6?$AA@ 10007f88     ap_info.obj
 0001:00006fa8       ??_C@_0CD@MCEDEGKD@EnqueueCmd?3?3OID_802_11_REMOVE_WE@ 10007fa8     ap_info.obj
 0001:00006fcc       ??_C@_0DA@DILJNKCA@Set?3?3OID_802_11_ADD_WEP?5failed?0?5@ 10007fcc     ap_info.obj
 0001:00006ffc       ??_C@_0BM@LAOPJNO@Set?3?3OID_802_11_REMOVE_WEP?6?$AA@ 10007ffc     ap_info.obj
 0001:00007018       ??_C@_0DF@MNANLIML@Set?3?3OID_802_11_ADD_WEP?0?5queue?5c@ 10008018     ap_info.obj
 0001:00007050       ??_C@_0CJ@JBPBNDAG@Set?3?3OID_802_11_ADD_WEP?0?5INVALID@ 10008050     ap_info.obj
 0001:0000707c       ??_C@_0DN@LPIFDIJ@APSetInformation?3?3OID_802_11_ADD@ 1000807c     ap_info.obj
 0001:000070bc       ??_C@_0BJ@CHKDJABG@Set?3?3OID_802_11_ADD_WEP?6?$AA@ 100080bc     ap_info.obj
 0001:000070d8       ??_C@_0DD@JIGMCONL@Set?3?3OID_802_11_REMOVE_KEY?5?$CIid?$DN0@ 100080d8     ap_info.obj
 0001:0000710c       ??_C@_0CN@IPAADAFF@Set?3?3OID_802_11_REMOVE_KEY?0?5?5INV@ 1000810c     ap_info.obj
 0001:0000713c       ??_C@_0DN@IMLIDPIH@Set?3?3OID_802_11_ADD_KEY?5?$CIinfo?9le@ 1000813c     ap_info.obj
 0001:0000717c       ??_C@_0CA@BMKGHFMM@Set?3?3OID_802_11_ADD_KEY?5ERROR?5?6?$AA@ 1000817c     ap_info.obj
 0001:0000719c       ??_C@_0DE@DJJIADNI@OID_802_11_ADD_KEY?3?3PMK?5?$DN?5?$CFx?3?$CFx?3@ 1000819c     ap_info.obj
 0001:000071d0       ??_C@_0BJ@INGCNBBK@Set?3?3OID_802_11_ADD_KEY?6?$AA@ 100081d0     ap_info.obj
 0001:000071f0       ??_C@_0EJ@ONKJNMHE@?5Set?3?3RT_OID_802_11_SET_WPA_REKE@ 100081f0     ap_info.obj
 0001:0000723c       ??_C@_0BL@DEKBNAKA@?5?5DISABLE?5WPA_REKEY?5?5?5?5?5?5?6?$AA@ 1000823c     ap_info.obj
 0001:00007258       ??_C@_0CC@CFJCMNFI@Set?3?3RT_OID_802_11_SET_WPA_REKEY@ 10008258     ap_info.obj
 0001:0000727c       ??_C@_0CF@CNCDMOGL@Set?3?3OID_802_11_INFRASTRUCTURE_M@ 1000827c     ap_info.obj
 0001:000072a4       ??_C@_0CF@HDAKPEGL@Set?3?3?5EnqueueCmd?5RT_OID_802_11_S@ 100082a4     ap_info.obj
 0001:000072cc       ??_C@_0BJ@IEMHPCEH@Set?3?3RT_OID_802_11_SSID?6?$AA@ 100082cc     ap_info.obj
 0001:000072e8       ??_C@_0BK@HBEEJLAF@Set?3?3RT_OID_802_11_BSSID?6?$AA@ 100082e8     ap_info.obj
 0001:00007508       ??_C@_0CJ@MLHDPCEP@Warning?0?5MAC?5specific?5condition?5@ 10008508     ap_mlme.obj
 0001:00007538       ??_C@_0FJ@COPNBINA@DRS?3?5unkown?5mode?5?$CIRateLen?$DN?$CFd?0?5MC@ 10008538     ap_mlme.obj
 0001:00007594       ??_C@_0CJ@KPFGDNOC@DRS?3?5unkown?5mode?0default?5use?511N@ 10008594     ap_mlme.obj
 0001:000075c0       ??_C@_0CJ@CBNJDKAB@DRS?3?5unkown?5mode?0default?5use?511N@ 100085c0     ap_mlme.obj
 0001:000075ec       ??_C@_0P@EFKLGNP@DRS?3?5A?1G?5STA?5?6?$AA@ 100085ec     ap_mlme.obj
 0001:000075fc       ??_C@_0BF@EEMEKFGI@DRS?3?5B?1G?5mixed?5STA?5?6?$AA@ 100085fc     ap_mlme.obj
 0001:00007614       ??_C@_0BC@JJCDMJMB@DRS?3?5B?5only?5STA?5?6?$AA@ 10008614     ap_mlme.obj
 0001:00007628       ??_C@_0BC@BMOHPLGG@DRS?3?511N?52S?5STA?5?6?$AA@ 10008628     ap_mlme.obj
 0001:0000763c       ??_C@_0BC@CFGKMHKD@DRS?3?511N?51S?5STA?5?6?$AA@ 1000863c     ap_mlme.obj
 0001:00007650       ??_C@_0BE@GABEDDIH@DRS?3?511BGN?52S?5STA?5?6?$AA@ 10008650     ap_mlme.obj
 0001:00007664       ??_C@_0BE@FJJJAPEC@DRS?3?511BGN?51S?5STA?5?6?$AA@ 10008664     ap_mlme.obj
 0001:00007678       ??_C@_0CH@ELCBMFII@DRS?3?5B?1G?5mixed?5AP?5?$CIMaxTx?$DN?$CFd?0MinT@ 10008678     ap_mlme.obj
 0001:000076a0       ??_C@_0CB@GDOJFBAA@DRS?3?5A?1G?5AP?5?$CIMaxTx?$DN?$CFd?0MinTx?$DN?$CFd?$CJ?6@ 100086a0     ap_mlme.obj
 0001:000076c4       ??_C@_0CE@CKHECAI@DRS?3?5B?5only?5AP?5?$CIMaxTx?$DN?$CFd?0MinTx?$DN?$CF@ 100086c4     ap_mlme.obj
 0001:000076e8       ??_C@_0FH@GDBEPKJK@DRS?3?5APMlmeSetTxRate?5?9?5CurrTxRat@ 100086e8     ap_mlme.obj
 0001:00007740       ??_C@_0BP@OECCEKLF@DRS?3?5?9?9TX?5rate?5from?5?$CFd?5to?5?$CFd?5?6?$AA@ 10008740     ap_mlme.obj
 0001:00007760       ??_C@_0BP@LACHPLKC@DRS?3?5?$CL?$CLTX?5rate?5from?5?$CFd?5to?5?$CFd?5?6?$AA@ 10008760     ap_mlme.obj
 0001:00007780       ??_C@_0DM@HLMMNGCN@DRS?3?5MCS?5is?5according?5to?5RSSI?0?5a@ 10008780     ap_mlme.obj
 0001:000077c0       ??_C@_0EN@MJACCFMJ@DRS?3?5AccuTxTotalCnt?5?$DM?$DN?515?0?5switc@ 100087c0     ap_mlme.obj
 0001:00007810       ??_C@_0IN@KDPGDCNK@DRS?3?5Before?9?5CurrTxRateIdx?$DN?$CFd?0?5M@ 10008810     ap_mlme.obj
 0001:000078a0       ??_C@_0FI@PPCOHFKP@DRS?3?5Fixed?5?9?5CurrTxRateIdx?$DN?$CFd?0?5M@ 100088a0     ap_mlme.obj
 0001:000078f8       ??_C@_0DM@CGMKIGLM@DRS?3Aid?$DN?$CFd?0?5TxRetransmit?$DN?$CFd?0?5TxF@ 100088f8     ap_mlme.obj
 0001:00007934       ??_C@_0CO@NDIFJMMJ@DRS?3?5CurrRateIdx?5?$DN?5?$CFd?0?5InitTxRat@ 10008934     ap_mlme.obj
 0001:00007964       ??_C@_0CE@FCGOJLNL@QuickDRS?3?5?9?9TX?5rate?5from?5?$CFd?5to?5?$CF@ 10008964     ap_mlme.obj
 0001:00007988       ??_C@_0CE@GGLCKMM@QuickDRS?3?5?$CL?$CLTX?5rate?5from?5?$CFd?5to?5?$CF@ 10008988     ap_mlme.obj
 0001:000079ac       ??_C@_0CO@NLDABNAN@QuickDRS?3?5?$CIDown?$CJ?5keep?5rate?9down?5@ 100089ac     ap_mlme.obj
 0001:000079dc       ??_C@_0CP@DIKKOFGF@QuickDRS?3?5?$CIDown?$CJ?5bad?5tx?5ok?5count@ 100089dc     ap_mlme.obj
 0001:00007a10       ??_C@_0EA@GDKIAGNL@QuickDRS?3?5?$CIDown?$CJ?5direct?5train?5do@ 10008a10     ap_mlme.obj
 0001:00007a50       ??_C@_0CK@MCHEPPNP@QuickDRS?3?5?$CIUp?$CJ?5keep?5rate?9up?5?$CIL?3?$CF@ 10008a50     ap_mlme.obj
 0001:00007a7c       ??_C@_0CN@PLAOPBCO@QuickDRS?3?5?$CIUp?$CJ?5bad?5tx?5ok?5count?5?$CI@ 10008a7c     ap_mlme.obj
 0001:00007aac       ??_C@_0DO@MAFJBEKB@QuickDRS?3?5AccuTxTotalCnt?5?$DM?$DN?515?0?5@ 10008aac     ap_mlme.obj
 0001:00007af0       ??_C@_0JC@GNNCCCPM@QuickDRS?3?5Before?9?5CurrTxRateIdx?$DN@ 10008af0     ap_mlme.obj
 0001:00007b88       ??_C@_0FN@HFOOIOC@QuickDRS?3?5Fixed?5?9?5CurrTxRateIdx?$DN@ 10008b88     ap_mlme.obj
 0001:00007be8       ??_C@_0EB@FNLBLMLD@QuickDRS?3Aid?$DN?$CFd?0?5TxRetransmit?$DN?$CFd@ 10008be8     ap_mlme.obj
 0001:00007c30       ??_C@_0EB@BGGEJPNF@wrong?5AUTH?5seq?$DN?$CFd?5Octet?$DN?$CF02x?5?$CF02@ 10008c30     ap_mlme.obj
 0001:00007c74       ??_C@_0DL@ODAJNJL@AUTH?5seq?$DN?$CFd?5Octet?$DN?$CF02x?5?$CF02x?5?$CF02x@ 10008c74     ap_mlme.obj
 0001:00007cb0       ??_C@_0BD@DLEJPKI@SUBTYPE_ASSOC_REQ?6?$AA@ 10008cb0     ap_mlme.obj
 0001:00007cc4       ??_C@_0CE@OBLEGPDG@AsicEvaluateRxAnt?5?3?5RealRxPath?$DN?$CF@ 10008cc4     ap_mlme.obj
 0001:00007ce8       ??_C@_0FA@GIHDOBOA@APAsicRxAntEvalTimeout?5?3?5RealRxP@ 10008ce8     ap_mlme.obj
 0001:00007f38       ??_C@_0BO@GMMMFDAO@PeerAssocReqSanity?5?9?5success?6?$AA@ 10008f38     ap_sanity.obj
 0001:00007f58       ??_C@_0CO@JKEIIAAH@PeerAssocReqSanity?5?9?5missing?5man@ 10008f58     ap_sanity.obj
 0001:00007f88       ??_C@_0CJ@HLJOGLKD@PeerAssocReqSanity?5?9?5missing?5IE_@ 10008f88     ap_sanity.obj
 0001:00007fb4       ??_C@_0CJ@JNPPFIF@PeerAssocReqSanity?$CIAID?$CD?$CFd?5WepSta@ 10008fb4     ap_sanity.obj
 0001:00007fe0       ??_C@_0BK@IGGJAIGM@RTMPCheckAUTH?5FAILED?5?$CB?$CB?$CB?6?$AA@ 10008fe0     ap_sanity.obj
 0001:00007ffc       ??_C@_0BL@MEMFICKG@RTMPCheckUcast?5FAILED?5?$CB?$CB?$CB?6?$AA@ 10008ffc     ap_sanity.obj
 0001:00008018       ??_C@_0BL@PNDHHALC@RTMPCheckMcast?5FAILED?5?$CB?$CB?$CB?6?$AA@ 10009018     ap_sanity.obj
 0001:00008034       ??_C@_0DK@HPNNMCHO@Receive?5IE_WPA?5?3?5?$CF02x?3?$CF02x?3?$CF02x?3@ 10009034     ap_sanity.obj
 0001:00008070       ??_C@_0BA@FPJDMBAK@null?5pEntry?$CB?$CB?$CB?6?$AA@ 10009070     ap_sanity.obj
 0001:00008080       ??_C@_0BN@DNCJLJGI@Not?5RSN?5IE?0?5maybe?5WMM?5IE?$CB?$CB?$CB?6?$AA@ 10009080     ap_sanity.obj
 0001:000080a0       ??_C@_0CD@LLDIGCHB@PeerAssocReqSanity?5?9?5PRE_N_HT_OU@ 100090a0     ap_sanity.obj
 0001:000080c4       ??_C@_0CG@IDBLAIBL@PeerAssocReqSanity?5?9?5wrong?5IE_WP@ 100090c4     ap_sanity.obj
 0001:000080ec       ??_C@_0DI@HEPGGCGI@PeerAssocReqSanity?5?9?5wrong?5IE_HT@ 100090ec     ap_sanity.obj
 0001:00008124       ??_C@_0CA@KHNDFHEB@PeerAssocReqSanity?5?9?5IE_HT_CAP?6?$AA@ 10009124     ap_sanity.obj
 0001:00008144       ??_C@_0DD@FNIEEFIP@PeerAssocReqSanity?5?9?5wrong?5IE_SU@ 10009144     ap_sanity.obj
 0001:00008178       ??_C@_0BP@MGLFMKDA@Rates?$FL1?$FN?$DN?$CFx?5?$CFx?5?$CFx?5?$CFx?5?$CFx?5?$CFx?5?$CFx?6?$AA@ 10009178     ap_sanity.obj
 0001:00008198       ??_C@_0DK@BIJAKHMD@PeerAssocReqSanity?5?9?5IE_SUPP_RAT@ 10009198     ap_sanity.obj
 0001:000081d4       ??_C@_0CE@NJPCFCJN@PeerAssocReqSanity?5?9?5wrong?5IE_SS@ 100091d4     ap_sanity.obj
 0001:000081f8       ??_C@_0CF@JDNDOJMB@PeerAssocReqSanity?5?9?5SsidLen?5?$DN?5?$CF@ 100091f8     ap_sanity.obj
 0001:00008220       ??_C@_0DA@LDNCBIBH@PeerReassocReqSanity?5?9?5missing?5m@ 10009220     ap_sanity.obj
 0001:00008250       ??_C@_0CH@MMEBLLOO@PeerReassocReqSanity?5?9?5missing?5I@ 10009250     ap_sanity.obj
 0001:00008278       ??_C@_0CI@OCAIHIBP@PeerAssocReqSanity?5?9?5wrong?5IE_HT@ 10009278     ap_sanity.obj
 0001:000082a0       ??_C@_0CC@PBJPILMD@PeerAssocReqSanity?5?9?5IE_HT_CAP?4?5@ 100092a0     ap_sanity.obj
 0001:000082c4       ??_C@_0DF@PHDHGILC@PeerReassocReqSanity?5?9?5wrong?5IE_@ 100092c4     ap_sanity.obj
 0001:000082fc       ??_C@_0CP@KAMGIBKK@PeerReassocReqSanity?5?9?5wrong?5IE_@ 100092fc     ap_sanity.obj
 0001:0000832c       ??_C@_0CP@DHPMGPOK@APPeerAuthSanity?5fail?5?9?5wrong?5al@ 1000932c     ap_sanity.obj
 0001:0000835c       ??_C@_0CK@FOAOBHBF@APPeerAuthSanity?5fail?5?9?5wrong?5Se@ 1000935c     ap_sanity.obj
 0001:00008388       ??_C@_0CL@NJFBBNHP@APPeerProbeReqSanity?5fail?5?9?5wron@ 10009388     ap_sanity.obj
 0001:000083b4       ??_C@_0DK@POIFGAJH@APPeerBeaconAndProbeRspSanity?5?9?5@ 100093b4     ap_sanity.obj
 0001:000083f0       ??_C@_0DH@PJMOBECP@APPeerBeaconAndProbeRspSanity?5?9?5@ 100093f0     ap_sanity.obj
 0001:00008428       ??_C@_0EB@FODGMFNA@APPeerBeaconAndProbeRspSanity?5?9?5@ 10009428     ap_sanity.obj
 0001:0000846c       ??_C@_0DL@JLEMKAHP@APPeerBeaconAndProbeRspSanity?5?9?5@ 1000946c     ap_sanity.obj
 0001:000084a8       ??_C@_0DO@NKMAOBDK@APPeerBeaconAndProbeRspSanity?5?9?5@ 100094a8     ap_sanity.obj
 0001:000084e8       ??_C@_0DI@BDCCGLBL@APPeerBeaconAndProbeRspSanity?5?9?5@ 100094e8     ap_sanity.obj
 0001:00008720       ??_C@_0DL@KHEEAHKC@SYNC?5?9?5Send?5PROBE_RSP?5to?5?$CF02x?3?$CF0@ 10009720     ap_sync.obj
 0001:00008760       ??_C@_0FL@NEIGCKPG@?$CF02x?3?$CF02x?3?$CF02x?3?$CF02x?3?$CF02x?3?$CF02x?5is@ 10009760     ap_sync.obj
 0001:000089c0       ISbox                      100099c0     Ap_wapi.obj
 0001:00008ac0       ??_C@_0CD@PALLGJDP@APWapiWAI_UnicastReq_Action?5?$DM?$DN?$DN?$DN@ 10009ac0     Ap_wapi.obj
 0001:00008ae4       ??_C@_0DL@OBAOBJOE@APWapiWAI_UnicastReq_Action?3?5Por@ 10009ae4     Ap_wapi.obj
 0001:00008b20       ??_C@_0CD@EEHJMNGF@APWapiWAI_UnicastReq_Action?5?$DN?$DN?$DN?$DO@ 10009b20     Ap_wapi.obj
 0001:00008b44       ??_C@_0CC@KAHOHHJG@APWapiWAI_MBcastReq_Action?5?$DM?$DN?$DN?$DN?5@ 10009b44     Ap_wapi.obj
 0001:00008b68       ??_C@_0EM@MGIFPNMJ@APWapiWAI_MBcastReq_Action?3?5Can?8@ 10009b68     Ap_wapi.obj
 0001:00008bb4       ??_C@_0CC@BELMNDMM@APWapiWAI_MBcastReq_Action?5?$DN?$DN?$DN?$DO?5@ 10009bb4     Ap_wapi.obj
 0001:00008bd8       ??_C@_0BN@CBOLAAEP@APWapiWAIPacketAction?5?$DM?$DN?$DN?$DN?5?6?$AA@ 10009bd8     Ap_wapi.obj
 0001:00008bf8       ??_C@_0DL@LEHMHOCK@APWapiWAIPacketAction?3?5AP?5don?8t?5@ 10009bf8     Ap_wapi.obj
 0001:00008c34       ??_C@_0DG@HOJHDADB@APWapiWAIPacketAction?3?5AP?5get?5WA@ 10009c34     Ap_wapi.obj
 0001:00008c6c       ??_C@_0DE@PBFAGCBC@APWapiWAIPacketAction?3?5AP?5get?5WA@ 10009c6c     Ap_wapi.obj
 0001:00008ca0       ??_C@_0DI@LJFANFL@APWapiWAIPacketAction?3uSubType?5?$DN@ 10009ca0     Ap_wapi.obj
 0001:00008cd8       ??_C@_0EJ@PFCOKIHF@APWapiWAIPacketAction?3?5OPMODE_ST@ 10009cd8     Ap_wapi.obj
 0001:00008d28       ??_C@_0GE@BLFNGNNM@APWapiWAIPacketAction?3?5Can?8t?5fin@ 10009d28     Ap_wapi.obj
 0001:00008d8c       ??_C@_0BM@BJFALCPO@APWapiWAIPacketAction?5?$DN?$DN?$DN?$DO?6?$AA@ 10009d8c     Ap_wapi.obj
 0001:00008da8       ??_C@_0CD@PGOBNCKL@indicate?5PORT_SECURED_EVENT_ID?4?4@ 10009da8     Ap_wapi.obj
 0001:00008dcc       ??_C@_0BO@KPFCJPNE@?$EA?$EA_?$EA?$EAWPA_802_1X_PORT_SECURED?6?$AA@ 10009dcc     Ap_wapi.obj
 0001:00008dec       ??_C@_0CH@PNLGCLIN@APWapiWAIPacket_HandleMBcastRsp?5@ 10009dec     Ap_wapi.obj
 0001:00008e18       ??_C@_0HM@FEHNIJHG@APWapiWAIPacket_HandleMBcastRsp?3@ 10009e18     Ap_wapi.obj
 0001:00008e94       ??_C@_0DL@MENOLLB@APWapiWAIPacket_HandleMBcastRsp?3@ 10009e94     Ap_wapi.obj
 0001:00008ed0       ??_C@_0DL@JBHJENK@APWapiWAIPacket_HandleMBcastRsp?3@ 10009ed0     Ap_wapi.obj
 0001:00008f0c       ??_C@_0DL@GKMLHJCI@APWapiWAIPacket_HandleMBcastRsp?3@ 10009f0c     Ap_wapi.obj
 0001:00008f48       ??_C@_0EC@LHOMMKEL@APWapiWAIPacket_HandleMBcastRsp?3@ 10009f48     Ap_wapi.obj
 0001:00008f8c       ??_C@_0DK@FBCAPFLD@APWapiWAIPacket_HandleMBcastRsp?3@ 10009f8c     Ap_wapi.obj
 0001:00008fc8       ??_C@_0EH@GLEKIOIO@APWapiWAIPacket_HandleMBcastRsp?3@ 10009fc8     Ap_wapi.obj
 0001:00009010       ??_C@_0CH@EJHEIPNH@APWapiWAIPacket_HandleMBcastRsp?5@ 1000a010     Ap_wapi.obj
 0001:00009038       ??_C@_0CI@HOHJELHJ@APWapiWAIPacket_HandleUnicastRsp@ 1000a038     Ap_wapi.obj
 0001:00009060       ??_C@_0EJ@NBBIKGPN@APWapiWAIPacket_HandleUnicastRsp@ 1000a060     Ap_wapi.obj
 0001:000090ac       ??_C@_0DK@IOHALMJP@0x?$CF02X?90x?$CF02X?90x?$CF02X?90x?$CF02X?90x?$CF0@ 1000a0ac     Ap_wapi.obj
 0001:000090e8       ??_C@_0CN@EHLFNAIE@RT2870Dump?5APWapiWAIPacket_Handl@ 1000a0e8     Ap_wapi.obj
 0001:00009118       ??_C@_0HB@IIPBPCOG@APWapiWAIPacket_HandleUnicastRsp@ 1000a118     Ap_wapi.obj
 0001:0000918c       ??_C@_0DC@DCPFDDHO@APWapiWAIPacket_HandleUnicastRsp@ 1000a18c     Ap_wapi.obj
 0001:000091c0       ??_C@_0DB@JPFFCFID@APWapiWAIPacket_HandleUnicastRsp@ 1000a1c0     Ap_wapi.obj
 0001:000091f8       ??_C@_0ED@GBDPEFHF@APWapiWAIPacket_HandleUnicastRsp@ 1000a1f8     Ap_wapi.obj
 0001:00009240       ??_C@_0ED@KLFODJG@APWapiWAIPacket_HandleUnicastRsp@ 1000a240     Ap_wapi.obj
 0001:00009288       ??_C@_0EC@IKMFCLOP@APWapiWAIPacket_HandleUnicastRsp@ 1000a288     Ap_wapi.obj
 0001:000092cc       ??_C@_0CI@MKLLOPCD@APWapiWAIPacket_HandleUnicastRsp@ 1000a2cc     Ap_wapi.obj
 0001:000092f4       ??_C@_0CI@EOOHPPCO@?$DM?$DN?$DN?$DN?5APWapiSend_MBcastKeyNegotia@ 1000a2f4     Ap_wapi.obj
 0001:0000931c       ??_C@_0BI@JPELCOND@Below?5are?5GROUP?5KEY?$CB?$CB?$CB?6?$AA@ 1000a31c     Ap_wapi.obj
 0001:00009334       ??_C@_08LPELDKHF@NMK?5key?6?$AA@ 1000a334     Ap_wapi.obj
 0001:00009340       ??_C@_0CE@KIKJDHLA@Below?5are?5GROUP?5KEY?$CB?$CB?$CB?$CIAdhoc?5Sen@ 1000a340     Ap_wapi.obj
 0001:00009364       ??_C@_0CO@BLBACCKG@RT2870Dump?5APWapiSend_MBcastKeyN@ 1000a364     Ap_wapi.obj
 0001:00009394       ??_C@_0BO@DEMNDGMC@NMK?5key?5?$CIWapi_NMK_AdhocSend?$CJ?6?$AA@ 1000a394     Ap_wapi.obj
 0001:000093b8       ??_C@_0EP@IFGBIBAC@APWapiSend_MBcastKeyNegotiate_Re@ 1000a3b8     Ap_wapi.obj
 0001:00009408       ??_C@_0CI@LLMCFCAJ@?$DN?$DN?$DN?$DO?5APWapiSend_MBcastKeyNegotia@ 1000a408     Ap_wapi.obj
 0001:00009430       ??_C@_0DJ@ODNNKOPI@?$DM?$DN?$DN?$DN?5APWapiSend_UnicastKeyNegoti@ 1000a430     Ap_wapi.obj
 0001:0000946c       ??_C@_0O@PPEBJIMM@Wapi_UserKey?6?$AA@ 1000a46c     Ap_wapi.obj
 0001:0000947c       ??_C@_0L@PNLLBLCL@1234567890?$AA@ 1000a47c     Ap_wapi.obj
 0001:00009488       ??_C@_0CP@FBHHDEGF@RT2870Dump?5APWapiSend_UnicastKey@ 1000a488     Ap_wapi.obj
 0001:000094b8       ??_C@_0M@GHLKICPJ@Wapi_ADDID?6?$AA@ 1000a4b8     Ap_wapi.obj
 0001:000094c4       ??_C@_0BJ@PNGPEMEH@WpaState?5not?5correct?$CB?$CB?5?6?$AA@ 1000a4c4     Ap_wapi.obj
 0001:000094e0       ??_C@_0CJ@BHLOFIGM@?$DN?$DN?$DN?$DO?5APWapiSend_UnicastKeyNegoti@ 1000a4e0     Ap_wapi.obj
 0001:0000950c       ??_C@_0CK@HNDFPKG@?$DM?$DN?$DN?$DN?5APWapiSend_UnicastKeyNegoti@ 1000a50c     Ap_wapi.obj
 0001:00009538       ??_C@_0EJ@EHFKFHC@APWapiSend_UnicastKeyNegotiate_C@ 1000a538     Ap_wapi.obj
 0001:00009588       ??_C@_0FB@HPJOOGCH@APWapiSend_UnicastKeyNegotiate_C@ 1000a588     Ap_wapi.obj
 0001:000095dc       ??_C@_0DO@EEBMFMDN@?$DN?$DN?$DN?$DO?5APWapiSend_UnicastKeyNegoti@ 1000a5dc     Ap_wapi.obj
 0001:00009620       ??_C@_0FD@HHMGDLDH@multicast?5or?5station?5key?5expansi@ 1000a620     Ap_wapi.obj
 0001:00009674       ??_C@_0DG@INKCAGAC@BK?50?8?$FL0x?$CF02X?$FN?51?8?$FL0x?$CF02X?$FN?5?4?4?4?514?8@ 1000a674     Ap_wapi.obj
 0001:000096b0       ??_C@_0FF@FPINOPLF@Ndis802_11AuthModeWAI_PSK?3?5KD_HM@ 1000a6b0     Ap_wapi.obj
 0001:00009708       ??_C@_0DP@OEHPIDIO@preshared?5key?5expansion?5for?5auth@ 1000a708     Ap_wapi.obj
 0001:00009748       ??_C@_0BI@NJMGBHKF@?$DM?$DN?$DN?$DN?5APSTAWapiGen_BKID?6?$AA@ 1000a748     Ap_wapi.obj
 0001:00009760       ??_C@_0DI@PEEEIJAG@BKID?50?8?$FL0x?$CF02X?$FN?51?8?$FL0x?$CF02X?$FN?5?4?4?4?51@ 1000a760     Ap_wapi.obj
 0001:00009798       ??_C@_0DA@PMPJACJC@KD_HMAC_SHA256?3?5Input?5BK?50?8?$FL0x?$CF0@ 1000a798     Ap_wapi.obj
 0001:000097c8       ??_C@_0BI@CDPNPAGB@?$DN?$DN?$DN?$DO?5APSTAWapiGen_BKID?6?$AA@ 1000a7c8     Ap_wapi.obj
 0001:000097e0       ??_C@_0BP@DKIAGGFD@?$DM?$DN?$DN?$DN?5APSTAWapiGen_PairwiseKey?6?$AA@ 1000a7e0     Ap_wapi.obj
 0001:00009800       ??_C@_0BP@DGLJIJKF@?$DN?$DN?$DN?$DO?5APSTAWapiGen_PairwiseKey?6?$AA@ 1000a800     Ap_wapi.obj
 0001:00009820       ??_C@_0EB@FIKGLGCJ@pairwise?5key?5expansion?5for?5unica@ 1000a820     Ap_wapi.obj
 0001:00009a68       ??_C@_0CC@DNLFCFG@WPAMsgTypeSubst?5?3?5return?5FALSE?$DL?5@ 1000aa68     ap_wpa.obj
 0001:00009a8c       ??_C@_0CI@EBAINOGL@Receive?5EAPOLASFAlert?5frame?0?5TYP@ 1000aa8c     ap_wpa.obj
 0001:00009ab4       ??_C@_0CP@LOIMBPDC@Receive?5EAPOL?9Key?5frame?0?5TYPE?5?$DN?5@ 1000aab4     ap_wpa.obj
 0001:00009ae4       ??_C@_0CG@FMONIBHH@Receive?5EAPOLLogoff?5frame?0?5TYPE?5@ 1000aae4     ap_wpa.obj
 0001:00009b0c       ??_C@_0CG@BFFGEABL@Receive?5EAPOL?9Start?5frame?0?5TYPE?5@ 1000ab0c     ap_wpa.obj
 0001:00009b34       ??_C@_0CF@NOKNNDIJ@Receive?5EAP?9Packet?5frame?0?5TYPE?5?$DN@ 1000ab34     ap_wpa.obj
 0001:00009b5c       ??_C@_0DA@BHFKCLIM@data?5?$DN?5?$CF02x?3?$CF02x?3?$CF02x?3?$CF02x?9?$CF02x?3@ 1000ab5c     ap_wpa.obj
 0001:00009b8c       ??_C@_0BJ@KKKCJFEA@RTMPCheckWPAframe?5?$DN?$DN?$DN?$DO?5?6?$AA@ 1000ab8c     ap_wpa.obj
 0001:00009ba8       ??_C@_0BP@ECFJLAFO@RTMPCheckMcast?5?$DN?$DN?$DO?5WPAIE?5?$DN?5?$CFd?6?$AA@ 1000aba8     ap_wpa.obj
 0001:00009bc8       ??_C@_0BP@FCONNMBP@RTMPCheckUcast?5?$DN?$DN?$DO?5WPAIE?5?$DN?5?$CFd?6?$AA@ 1000abc8     ap_wpa.obj
 0001:00009be8       ??_C@_0CK@MPMCANPJ@RTMPCheckAUTH?5?$DN?$DN?$DO?5WPAIE?$DN?$CFd?0?5WepS@ 1000abe8     ap_wpa.obj
 0001:00009c14       ??_C@_0BN@FAIAPPJP@APWpaEAPOLStartAction?5?$DN?$DN?$DN?$DO?5?6?$AA@ 1000ac14     ap_wpa.obj
 0001:00009c34       ??_C@_0CB@DDEILOPF@pAd?9?$DOApCfg?4GKeyDoneStations?$DN?$CFd?5?6@ 1000ac34     ap_wpa.obj
 0001:00009c58       ??_C@_0DE@ENNDGMPB@Receive?5CM?5Attack?5Twice?5within?56@ 1000ac58     ap_wpa.obj
 0001:00009c8c       ??_C@_0CK@PDBNJKPC@REQUEST?$DN1?0?5ERROR?$DN?50?0?5update?5pair@ 1000ac8c     ap_wpa.obj
 0001:00009cb8       ??_C@_0CG@EAKGPPKB@REQUEST?$DN1?0?5ERROR?$DN0?0?5update?5group@ 1000acb8     ap_wpa.obj
 0001:00009ce0       ??_C@_0DI@FCIKOLED@MIC?0?5REQUEST?0?5ERROR?5?5are?5all?51?0?5@ 1000ace0     ap_wpa.obj
 0001:00009d18       ??_C@_0CI@NCPNLMFN@Key?5descripter?5version?5not?5match@ 1000ad18     ap_wpa.obj
 0001:00009d40       ??_C@_0CJ@JFNOFDJC@Key?5descripter?5version?5not?5match@ 1000ad40     ap_wpa.obj
 0001:00009d6c       ??_C@_0CN@LJBKOPML@Key?5descripter?5does?5not?5match?5wi@ 1000ad6c     ap_wpa.obj
 0001:00009d9c       ??_C@_0BK@PLKNKIEF@APWpaEAPOLKeyAction?5?$DN?$DN?$DN?$DO?6?$AA@ 1000ad9c     ap_wpa.obj
 0001:00009db8       ??_C@_0CE@NOGIPACA@?$DM?$DN?$DN?$DN?5WPAStart4WayHS?0?5WpaState?$DN?5?$CF@ 1000adb8     ap_wpa.obj
 0001:00009ddc       ??_C@_0BH@IHIIMJNM@pEntry?9?$DOAuthMode?5?$DN?5?$CFx?6?$AA@ 1000addc     ap_wpa.obj
 0001:00009df4       ??_C@_0CF@HKDIBHJ@Not?5expect?5calling?5?5WPAStart4Way@ 1000adf4     ap_wpa.obj
 0001:00009e1c       ??_C@_0BF@OAOLBGLA@?$DN?$DN?$DN?$DO?5WPAStart4WayHS?6?$AA@ 1000ae1c     ap_wpa.obj
 0001:00009e34       ??_C@_0BK@OFJGJCNH@?$DM?$DN?$DN?$DN?5PeerPairMsg2Action?5?6?$AA@ 1000ae34     ap_wpa.obj
 0001:00009e50       ??_C@_0BM@KOPLBEIK@pEntry?9?$DOR_Counter?$FL?$CFd?$FN?$CL?$CL?$DN?$CFd?6?$AA@ 1000ae50     ap_wpa.obj
 0001:00009e6c       ??_C@_0CK@PMEJOPCH@RSN_IE?5VALID?5in?5msg?52?5of?54?9way?5h@ 1000ae6c     ap_wpa.obj
 0001:00009e98       ??_C@_0DA@NLOEEOLO@PeerPairMsg2Action?3?3Current?$CI?$CFd?$CJ?5@ 1000ae98     ap_wpa.obj
 0001:00009ec8       ??_C@_0DA@BCHGIGEL@PeerPairMsg2Action?3?3Receive?5?5?5?5?5@ 1000aec8     ap_wpa.obj
 0001:00009ef8       ??_C@_0ED@KIAHGNCA@PeerPairMsg2Action?3?3RSN_IE?5Diffe@ 1000aef8     ap_wpa.obj
 0001:00009f3c       ??_C@_0CH@HCGLMDN@MIC?5VALID?5in?5msg?52?5of?54?9way?5hand@ 1000af3c     ap_wpa.obj
 0001:00009f64       ??_C@_0BD@BJEHFPPJ@Receive?5?3?5?$CFx?5?$CFx?5?6?5?$AA@ 1000af64     ap_wpa.obj
 0001:00009f78       ??_C@_0CL@NMKMIBIK@MIC?5Different?5in?5msg?52?5of?54?9way?5@ 1000af78     ap_wpa.obj
 0001:00009fa4       ??_C@_0DI@DMFONDLM@Replay?5Counter?5Different?5in?5msg?5@ 1000afa4     ap_wpa.obj
 0001:00009fdc       ??_C@_0BJ@JLMKEEAA@?$DN?$DN?$DN?$DOPeerPairMsg2Action?5?6?$AA@ 1000afdc     ap_wpa.obj
 0001:00009ff8       ??_C@_0DI@LFEJBMJG@Find?5more?5than?5one?5entry?5which?5g@ 1000aff8     ap_wpa.obj
 0001:0000a030       ??_C@_0CN@PADJDHCK@WPARetryExec?3?3ReTry?5MSG1?5of?54?9wa@ 1000b030     ap_wpa.obj
 0001:0000a060       ??_C@_0CI@FMKLCCEO@WPARetryExec?3?3Retry?5MSG1?0?5the?5la@ 1000b060     ap_wpa.obj
 0001:0000a088       ??_C@_0DH@DJMCAHKM@WPARetryExec?3?3MSG3?5timeout?0?5pEnt@ 1000b088     ap_wpa.obj
 0001:0000a0c0       ??_C@_0DA@GFDLLHCG@WPARetryExec?3?3ReTry?52?9way?5group?9@ 1000b0c0     ap_wpa.obj
 0001:0000a0f0       ??_C@_0FN@FCPEPIDG@WPARetryExec?3?3Group?5Key?5HS?5excee@ 1000b0f0     ap_wpa.obj
 0001:0000a150       ??_C@_0EJ@PEEDMLIK@WPARetryExec?3?3?$FLOPMODE_STA?$FN?5Can?8t@ 1000b150     ap_wpa.obj
 0001:0000a19c       ??_C@_0DM@GLGLAPCF@WPARetryExec?5?9?5Send?5AP_WAPI_MT2_@ 1000b19c     ap_wpa.obj
 0001:0000a1d8       ??_C@_0EP@JAHDPDDC@WPARetryExec?3?3?5REASON_WAPI_UNICA@ 1000b1d8     ap_wpa.obj
 0001:0000a228       ??_C@_0GD@OAKJJNAL@WPARetryExec?3?3REASON_WAPI_UNICAS@ 1000b228     ap_wpa.obj
 0001:0000a28c       ??_C@_0BE@NCOGBGM@WPARetryExec?$CIWAPI?$CJ?6?$AA@ 1000b28c     ap_wpa.obj
 0001:0000a2a0       ??_C@_0DA@FNCCOHAI@WPARetryExec?9?9?9?$DO?5ReTryCounter?$DN?$CFd@ 1000b2a0     ap_wpa.obj
 0001:0000a2d0       ??_C@_0BN@NBPFBDKA@?$DM?$DN?$DN?$DN?5Wpa1PeerPairMsg4Action?6?$AA@ 1000b2d0     ap_wpa.obj
 0001:0000a2f0       ??_C@_0CI@OEEEGJPA@MAC?5Valid?5in?5msg?54?5of?54?9way?5hand@ 1000b2f0     ap_wpa.obj
 0001:0000a318       ??_C@_0CM@HLIAEIFF@MAC?5Different?5in?5msg?54?5of?54?9way?5@ 1000b318     ap_wpa.obj
 0001:0000a344       ??_C@_0BH@OFJNKAJL@Current?5?3?5?$CFd?5?$CFd?5?$CFd?5?$CFd?6?$AA@ 1000b344     ap_wpa.obj
 0001:0000a35c       ??_C@_0BH@EKBLKKML@Receive?5?3?5?$CFd?5?$CFd?5?$CFd?5?$CFd?6?$AA@ 1000b35c     ap_wpa.obj
 0001:0000a378       ??_C@_0EB@CNNJCJGE@Replay?5Counter?5Different?5in?5msg?5@ 1000b378     ap_wpa.obj
 0001:0000a3bc       ??_C@_0BN@EAKFCHHM@?$DN?$DN?$DN?$DO?5Wpa1PeerPairMsg4Action?6?$AA@ 1000b3bc     ap_wpa.obj
 0001:0000a3dc       ??_C@_0DE@CEOJACB@AP?5SETKEYS?5DONE?5?9?5WPA2?0?5AuthMode@ 1000b3dc     ap_wpa.obj
 0001:0000a410       ??_C@_0CH@DAKKFGD@MIC?5VALID?5in?5msg4?5of?54?9way?5hands@ 1000b410     ap_wpa.obj
 0001:0000a438       ??_C@_0CL@NIIAJINE@MIC?5Different?5in?5msg4?5of?54?9way?5h@ 1000b438     ap_wpa.obj
 0001:0000a464       ??_C@_0DC@JLODKOKL@Replay?5Counter?5VALID?5in?5msg4?5of?5@ 1000b464     ap_wpa.obj
 0001:0000a498       ??_C@_0BO@NIFHHDOI@Current?5?3?5?$CFd?5?5?5?$CFd?5?5?$CFd?5?5?5?$CFd?5?5?6?$AA@ 1000b498     ap_wpa.obj
 0001:0000a4b8       ??_C@_0BI@MDMJCLCO@Receive?5?3?5?$CFd?5?$CFd?5?$CFd?5?$CFd?5?6?$AA@ 1000b4b8     ap_wpa.obj
 0001:0000a4d0       ??_C@_0DG@BGEEOCAP@Replay?5Counter?5Different?5in?5msg4@ 1000b4d0     ap_wpa.obj
 0001:0000a508       ??_C@_0BM@JHJCMNMO@?$DN?$DN?$DN?$DOWpa2PeerPairMsg4Action?6?$AA@ 1000b508     ap_wpa.obj
 0001:0000a524       ??_C@_0DE@BBGGKJFC@AP?5SETKEYS?5DONE?5?9?5WPA1?0?5AuthMode@ 1000b524     ap_wpa.obj
 0001:0000a558       ??_C@_0CI@JIOEJHKD@MIC?5VALID?5in?5msg?52?5of?52?9way?5hand@ 1000b558     ap_wpa.obj
 0001:0000a580       ??_C@_0CM@MNDKDLLB@MIC?5Different?5in?5msg?52?5of?52?9way?5@ 1000b580     ap_wpa.obj
 0001:0000a5ac       ??_C@_0DK@IDMAMMEM@Replay?5Counter?5VALID?5in?5msg?52?5of@ 1000b5ac     ap_wpa.obj
 0001:0000a5e8       ??_C@_0CF@OCNEHABJ@Current?3?5?$CFd?5?$CFd?5?$CFd?5?$CFd?5?9?5?$CFd?5?$CFd?5?$CFd?5@ 1000b5e8     ap_wpa.obj
 0001:0000a610       ??_C@_0CF@BCPPFJCM@Receive?3?5?$CFd?5?$CFd?5?$CFd?5?$CFd?5?9?5?$CFd?5?$CFd?5?$CFd?5@ 1000b610     ap_wpa.obj
 0001:0000a638       ??_C@_0EA@LAODBLKG@Replay?5Counter?5?5Different?5?5in?5ms@ 1000b638     ap_wpa.obj
 0001:0000a678       ??_C@_0CO@FDDLLALA@PeerGroupMsg2Action?5?$DN?$DN?$DN?$DN?$DO?5?$CFx?5?$CFx?5@ 1000b678     ap_wpa.obj
 0001:0000a6a8       ??_C@_0CC@POKOGMGM@WPAHardTransmit?5?3?5FrameLen?5?$DN?5?$CFd?5@ 1000b6a8     ap_wpa.obj
 0001:0000a6cc       ??_C@_0DD@FPIGKEPE@APToWirelessSta?5?3?5ETHTYPE?5?$DN?5?$CFx?5?$CF@ 1000b6cc     ap_wpa.obj
 0001:0000a700       ??_C@_0DP@NOHEGHIP@ASSOC?5?9?5Send?5DISASSOC?5Reason?5?$DN?5?$CF@ 1000b700     ap_wpa.obj
 0001:0000a740       ??_C@_0FF@LMNJNCFP@Rekey?5interval?5excess?0?5Update?5Gr@ 1000b740     ap_wpa.obj
 0001:0000a798       ??_C@_0CM@FGOJBOK@Rekey?5Interval?5Excess?0?5GKeyDoneS@ 1000b798     ap_wpa.obj
 0001:0000a7c4       ??_C@_0CC@JPFMNAON@?$CFs?3?5pAd?9?$DOApCfg?4REKEYCOUNTER?5?$DN?5?$CFd@ 1000b7c4     ap_wpa.obj
 0001:0000a7e8       ??_C@_0BD@FFPBKBOO@GREKEYPeriodicExec?$AA@ 1000b7e8     ap_wpa.obj
 0001:0000a7fc       ??_C@_0CA@PAOFEDEO@GROUP?5REKEY?5PeriodicExec?5?$DN?$DN?$DO?$DO?5?6?$AA@ 1000b7fc     ap_wpa.obj
 0001:0000a81c       ??_C@_0CA@PFMOJOGO@RTMPMakeRSNIE?5?3?5RSNIE_Len?5?$DN?5?$CFd?6?$AA@ 1000b81c     ap_wpa.obj
 0001:0000a840       ??_C@_0EE@OMKJDAKP@APToWirelessSta?5?9?5len?$DN?$CFd?0?5AID?$DN?$CFd@ 1000b840     ap_wpa.obj
 0001:0000aa88       ??_C@_0CE@NPBEAIGG@ASSOC?5?9?5enqueue?5MT2_ASSOC_TIMEOU@ 1000ba88     assoc.obj
 0001:0000aaac       ??_C@_0CG@GMHNAAIK@ASSOC?5?9?5enqueue?5MT2_REASSOC_TIME@ 1000baac     assoc.obj
 0001:0000aad4       ??_C@_0CH@INCOHEHM@ASSOC?5?9?5enqueue?5MT2_DISASSOC_TIM@ 1000bad4     assoc.obj
 0001:0000aafc       ??_C@_0DO@GIHLKBMM@ASSOC?5?9?5MlmeAssocReqAction?$CI?$CJ?5san@ 1000bafc     assoc.obj
 0001:0000ab3c       ??_C@_0BL@HBJOKBKC@ASSOC?5?9?5STA_CAC_Active?$CB?$CB?5?6?$AA@ 1000bb3c     assoc.obj
 0001:0000ab58       ??_C@_0CG@BHHHDFKP@ASSOC?5?9?5pAd?9?$DOCommonCfg?4AuthMode?5@ 1000bb58     assoc.obj
 0001:0000ab80       ??_C@_0BD@KCBPEOEK@MlmeAssocReqAction?$AA@ 1000bb80     assoc.obj
 0001:0000ab94       ??_C@_0CO@DEBNKHNL@ASSOC?5?9?5Send?5ASSOC?5request?0?5CCX_@ 1000bb94     assoc.obj
 0001:0000abc4       ??_C@_0DG@DLEENDGL@ASSOC?5?9?5MlmeAssocReqAction?$CI?$CJ?5all@ 1000bbc4     assoc.obj
 0001:0000abfc       ??_C@_0DH@GNPKKAFJ@ASSOC?5?9?5Block?5Assoc?5request?5durn@ 1000bbfc     assoc.obj
 0001:0000ac34       ??_C@_0DO@JIHAFOIG@ASSOC?5?9?5MlmeReassocReqAction?$CI?$CJ?5s@ 1000bc34     assoc.obj
 0001:0000ac74       ??_C@_0CA@OEJDNFAK@AssocInfo?4RequestIELength?5?$DN?5?$CFx?6?$AA@ 1000bc74     assoc.obj
 0001:0000ac94       ??_C@_0CM@DBBFAIDC@CCKM?5ReassocReq?3?5tmp1Len?5?$DN?5?$CFd?5tm@ 1000bc94     assoc.obj
 0001:0000acc0       ??_C@_0BO@NDEGBKLH@Re?9ASSOC?5?9?5STA_CAC_Active?$CB?$CB?5?6?$AA@ 1000bcc0     assoc.obj
 0001:0000ace0       ??_C@_0CC@NIANDMMK@ASSOC?5?9?5Send?5RE?9ASSOC?5request?4?4?4@ 1000bce0     assoc.obj
 0001:0000ad04       ??_C@_0DI@OLCLJDEK@ASSOC?5?9?5MlmeReassocReqAction?$CI?$CJ?5a@ 1000bd04     assoc.obj
 0001:0000ad3c       ??_C@_0DJ@IKPPOPCA@ASSOC?5?9?5Block?5ReAssoc?5request?5du@ 1000bd3c     assoc.obj
 0001:0000ad78       ??_C@_0EE@DGPNBCDD@ASSOC?5?9?5Send?5DISASSOC?5request?$FLBS@ 1000bd78     assoc.obj
 0001:0000adbc       ??_C@_0DI@CDNFMMAA@ASSOC?5?9?5MlmeDisassocReqAction?$CI?$CJ?5@ 1000bdbc     assoc.obj
 0001:0000adf4       ??_C@_0DA@NLMEEBCP@ASSOC?5?9?5PeerAssocRspAction?$CI?$CJ?5san@ 1000bdf4     assoc.obj
 0001:0000ae24       ??_C@_0CF@JPFOGFGD@ASSOC?5Rsp?5?9?9?9?5TSPEC?5Rejected?5?$CI0x@ 1000be24     assoc.obj
 0001:0000ae4c       ??_C@_0CN@FKLFDBPN@?$DMS71?$DO?5PeerAssocRspAction?3?5Status@ 1000be4c     assoc.obj
 0001:0000ae7c       ??_C@_0CF@GPOCPJOK@?$DMCCX?$DO?5pAd?9?$DOStaCfg?4CkipFlag?5?$DN?50x?$CF@ 1000be7c     assoc.obj
 0001:0000aea4       ??_C@_0DJ@KJOBJJLB@MacTable?5?$FL?$CFd?$FN?4AMsduSize?5?$DN?5?$CFd?4?5Cl@ 1000bea4     assoc.obj
 0001:0000aee0       ??_C@_0CN@JCABFGDO@ASSOC?5?9?5receive?5ASSOC_RSP?5to?5me?5@ 1000bee0     assoc.obj
 0001:0000af10       ??_C@_0DC@INILAGHG@ASSOC?5?9?5PeerReassocRspAction?$CI?$CJ?5s@ 1000bf10     assoc.obj
 0001:0000af44       ??_C@_0CP@HPKKPNJH@?$DMS71?$DO?5PeerReassocRspAction?3?5Stat@ 1000bf44     assoc.obj
 0001:0000af78       ??_C@_0FC@LMPDMMBO@CCKM?5fast?9roaming?3?5indicate?5NDIS@ 1000bf78     assoc.obj
 0001:0000afcc       ??_C@_0DG@GECOPMDG@PeerReassocRspAction?0?5?$DMCCX?$DO?5StaC@ 1000bfcc     assoc.obj
 0001:0000b004       ??_C@_0CP@PMPOKCNK@ASSOC?5?9?5receive?5REASSOC_RSP?5to?5m@ 1000c004     assoc.obj
 0001:0000b034       ??_C@_0DH@MOGOHJDP@ASSOC?5?9?5Can?8t?5find?5BSS?5after?5rec@ 1000c034     assoc.obj
 0001:0000b06c       ??_C@_0DA@NKMGEKKC@AssocPostProc?$DN?$DN?$DN?$DO?5?5?5?5?$CIMmps?$DN?$CFd?0?5A@ 1000c06c     assoc.obj
 0001:0000b0a0       ??_C@_0EB@BBMCAIPG@AssocPostProc?$DN?$DN?$DN?$DO?5?5AP?4AMsduSize?5@ 1000c0a0     assoc.obj
 0001:0000b0e4       ??_C@_0O@JNDAGLNJ@AssocPostProc?$AA@ 1000c0e4     assoc.obj
 0001:0000b0f4       ??_C@_0DA@ODDHDAFC@ASSOC?5?9?5PeerDisassocAction?$CI?$CJ?5san@ 1000c0f4     assoc.obj
 0001:0000b124       ??_C@_0BI@JALLMALL@Clean?5MAC?5Entry?5in?5TAB?6?$AA@ 1000c124     assoc.obj
 0001:0000b140       ??_C@_0GI@BJLGKEFF@?$CFs?3?5ASSOC?5?9?5?$CICarrier?5detection?5i@ 1000c140     assoc.obj
 0001:0000b1a8       ??_C@_0BD@EIFBOPGI@PeerDisassocAction?$AA@ 1000c1a8     assoc.obj
 0001:0000b1bc       ??_C@_0CN@GIMJLEOF@?$DMS71?$DO?5PeerDisassocAction?3?5Reason@ 1000c1bc     assoc.obj
 0001:0000b1ec       ??_C@_0BO@HEPCBPIC@ASSOC?5?9?5PeerDisassocAction?$CI?$CJ?6?$AA@ 1000c1ec     assoc.obj
 0001:0000b20c       ??_C@_0BM@CEEKGCPG@ASSOC?5?9?5AssocTimeoutAction?6?$AA@ 1000c20c     assoc.obj
 0001:0000b228       ??_C@_0BO@JNNPCJJM@ASSOC?5?9?5ReassocTimeoutAction?6?$AA@ 1000c228     assoc.obj
 0001:0000b248       ??_C@_0BP@KEFGKFCG@ASSOC?5?9?5DisassocTimeoutAction?6?$AA@ 1000c248     assoc.obj
 0001:0000b268       ??_C@_0EE@MIINLNBE@ASSOC?5?9?5InvalidStateWhenAssoc?$CIst@ 1000c268     assoc.obj
 0001:0000b2b0       ??_C@_0EG@MMEHINEH@ASSOC?5?9?5InvalidStateWhenReassoc?$CI@ 1000c2b0     assoc.obj
 0001:0000b2f8       ??_C@_0EH@OEFLDGLE@ASSOC?5?9?5InvalidStateWhenDisassoc@ 1000c2f8     assoc.obj
 0001:0000b340       ??_C@_0CM@EJEDBDPE@ASSOC?5?9?5Class?53?5Error?0?5Send?5DISA@ 1000c340     assoc.obj
 0001:0000b36c       ??_C@_0DD@OPEAGCBM@SwitchBetweenWepAndCkip?3?5modify?5@ 1000c36c     assoc.obj
 0001:0000b5a0       ??_C@_0BE@KGNKGALE@AUTH?5?9?5AuthTimeout?6?$AA@ 1000c5a0     auth.obj
 0001:0000b5b4       ??_C@_0DA@FNHIJCI@AUTH?5?9?5MlmeAuthReqAction?$CI?$CJ?5sanit@ 1000c5b4     auth.obj
 0001:0000b5e8       ??_C@_0ED@LHJAJDKM@MlmeAuthReqAction?3?5AUTH?5?9?5Send?5A@ 1000c5e8     auth.obj
 0001:0000b62c       ??_C@_0DD@KECJJMAM@AUTH?5?9?5MlmeAuthReqAction?$CI?$CJ?5alloc@ 1000c62c     auth.obj
 0001:0000b660       ??_C@_0CG@PALPKFOK@MlmeAuthReqAction?$DN?$DN?$DN?$DO?5?5Is?5Athero@ 1000c660     auth.obj
 0001:0000b688       ??_C@_0DF@GEFOMOIC@AUTH?5?9?5Block?5Auth?5request?5durnin@ 1000c688     auth.obj
 0001:0000b6c0       ??_C@_0CL@EGHBHPJ@AUTH?5?9?5PeerAuthSanity?$CI?$CJ?5sanity?5c@ 1000c6c0     auth.obj
 0001:0000b6ec       ??_C@_0DC@GMGNGLMC@?$DMS71?$DO?5PeerAuthRspAtSeq2Action?3?5S@ 1000c6ec     auth.obj
 0001:0000b720       ??_C@_0CD@MHBJFLCM@AUTH?5?9?5Send?5AUTH?5request?5seq?$CD3?4?4@ 1000c720     auth.obj
 0001:0000b744       ??_C@_0DH@POGCGJBJ@AUTH?5?9?5PeerAuthRspAtSeq2Action?$CI?$CJ@ 1000c744     auth.obj
 0001:0000b77c       ??_C@_0DJ@HMHGLDLL@AUTH?5?9?5Receive?5AUTH_RSP?5seq?$CD2?5to@ 1000c77c     auth.obj
 0001:0000b7b8       ??_C@_0DE@IELPEDCO@AUTH?5?9?5PeerAuthRspAtSeq4Action?$CI?$CJ@ 1000c7b8     auth.obj
 0001:0000b7ec       ??_C@_0CF@KBAGKPNP@AUTH?5?9?5Receive?5AUTH_RSP?5seq?$CD4?5to@ 1000c7ec     auth.obj
 0001:0000b814       ??_C@_0CM@IGJEBLAE@AUTH?5?9?5Send?5DE?9AUTH?5request?5?$CIRea@ 1000c814     auth.obj
 0001:0000b840       ??_C@_0DD@PCPDANEG@AUTH?5?9?5MlmeDeauthReqAction?$CI?$CJ?5all@ 1000c840     auth.obj
 0001:0000b874       ??_C@_0BK@JNKOGFNM@AUTH?5?9?5AuthTimeoutAction?6?$AA@ 1000c874     auth.obj
 0001:0000b890       ??_C@_0EC@JIGOAOAF@AUTH?5?9?5InvalidStateWhenAuth?5?$CIsta@ 1000c890     auth.obj
 0001:0000b8d4       ??_C@_0CM@MJJCHKFC@AUTH?5?9?5Class?52?5error?0?5Send?5DEAUT@ 1000c8d4     auth.obj
 0001:0000bb00       ??_C@_0BP@OAFJBIFG@Send?5AUTH?5response?5?$CIseq?$CD2?$CJ?4?4?4?6?$AA@ 1000cb00     auth_rsp.obj
 0001:0000bb20       ??_C@_0BD@FPHMAHJL@Peer?5AUTH?5fail?4?4?4?6?$AA@ 1000cb20     auth_rsp.obj
 0001:0000bb34       ??_C@_0DB@IHPPNNAH@AUTH_RSP?5?9?5PeerDeauthAction?$CI?$CJ?5sa@ 1000cb34     auth_rsp.obj
 0001:0000bb68       ??_C@_0DE@KHKHNOPK@AUTH_RSP?5?9?5receive?5DE?9AUTH?5from?5@ 1000cb68     auth_rsp.obj
 0001:0000bb9c       ??_C@_0CL@CCLCENDG@?$DMS71?$DO?5PeerDeauthAction?3?5Reason?5C@ 1000cb9c     auth_rsp.obj
 0001:0000bbc8       ??_C@_0GL@DAKBBJKI@?$CFs?3?5AUTH_RSP?5?9?5?$CICarrier?5detectio@ 1000cbc8     auth_rsp.obj
 0001:0000bc34       ??_C@_0BB@DJIMNHIH@PeerDeauthAction?$AA@ 1000cc34     auth_rsp.obj
 0001:0000be48       ??_C@_0CJ@HJHHJFCL@?$CBERROR?$CB?5CNTL?5?9?5Illegal?5message?5t@ 1000ce48     connect.obj
 0001:0000be78       ??_C@_0EL@JIBOPDLD@?$CFs?5?$CICNTL_WAIT_SCAN_FOR_CONNECT?$CJ?3@ 1000ce78     connect.obj
 0001:0000bec4       ??_C@_0CG@PPGHGKC@Scan?5Complete?5?9?9?9?$DO?5Drastically?5R@ 1000cec4     connect.obj
 0001:0000bef0       ??_C@_0EP@GEEFBIAF@Because?5the?5current?5AP?5rejected?5@ 1000cef0     connect.obj
 0001:0000bf40       ??_C@_0HI@NPMIIMDN@?$CFs?5?$CICNTL_WAIT_OID_LIST_SCAN?$CJ?3?5pA@ 1000cf40     connect.obj
 0001:0000bfb8       ??_C@_0BN@LDGDLJBP@MlmeCntlMachinePerformAction?$AA@ 1000cfb8     connect.obj
 0001:0000bfd8       ??_C@_0DE@OGKJMNPD@CNTL?5?9?5Illegal?5message?5in?5CntlId@ 1000cfd8     connect.obj
 0001:0000c00c       ??_C@_0CH@KKBIOPMM@NDIS_STATUS_MEDIA_DISCONNECT?5Eve@ 1000d00c     connect.obj
 0001:0000c034       ??_C@_0BL@PPKLHBBN@CNTL?5?9?5drop?5current?5ADHOC?6?$AA@ 1000d034     connect.obj
 0001:0000c04f       ??_C@_00CNPNBAHC@?$AA@     1000d04f     connect.obj
 0001:0000c050       ??_C@_0BE@JOPIIDIP@CNTL?5?9?5SCAN?5starts?6?$AA@ 1000d050     connect.obj
 0001:0000c068       ??_C@_0EB@FAMJMDC@CNTL?5?9?5matching?5BSS?0?5IterateOnBs@ 1000d068     connect.obj
 0001:0000c0b0       ??_C@_0GL@PONBNEBD@?$CFs?3?5CNTL?5?9?5No?5matching?5BSS?5?$DMBSS_@ 1000d0b0     connect.obj
 0001:0000c120       ??_C@_0GL@DJILCAHI@?$CFs?3?5CNTL?5?9?5No?5matching?5BSS?5?$DMBSS_@ 1000d120     connect.obj
 0001:0000c18c       ??_C@_0CK@PCPNCK@CNTL?5?9?5No?5matching?5BSS?0?5start?5a?5@ 1000d18c     connect.obj
 0001:0000c1b8       ??_C@_0DO@POLPKGPG@CNTL?5?9?5already?5with?5this?5BSSID?4?5@ 1000d1b8     connect.obj
 0001:0000c1f8       ??_C@_0DP@IAJGDLGN@CNTL?5?9?5disassociate?5with?5current@ 1000d1f8     connect.obj
 0001:0000c238       ??_C@_0CI@GKCIGOMK@CNTL?5?9?5disassociate?5with?5current@ 1000d238     connect.obj
 0001:0000c260       ??_C@_0DE@GLCCLOHP@CNTL?5?9?5?$CFd?5BSS?5of?5?$CFd?5BSS?5match?5th@ 1000d260     connect.obj
 0001:0000c294       ??_C@_0CI@BGJFPECJ@?$CFs?3?5Update?5last?5valid?5SSID?5?$DN?5?$CFc?$CF@ 1000d294     connect.obj
 0001:0000c2bc       ??_C@_0BA@HNGCGMOG@CntlOidSsidProc?$AA@ 1000d2bc     connect.obj
 0001:0000c2cc       ??_C@_0DC@IICPANIA@CNTL?5?9?5joining?5?$CF02x?3?$CF02x?3?$CF02x?3?$CF0@ 1000d2cc     connect.obj
 0001:0000c300       ??_C@_0CJ@IEHKGEAG@CNTL?5?9?5disassociate?5with?5current@ 1000d300     connect.obj
 0001:0000c32c       ??_C@_0DN@NAOPGFPP@CNTL?5?9?5already?5in?5this?5BSSID?4?5ig@ 1000d32c     connect.obj
 0001:0000c36c       ??_C@_0DI@KNCMOGFJ@CNTL?5?9?5BSSID?5not?5found?4?5reply?5ND@ 1000d36c     connect.obj
 0001:0000c3a4       ??_C@_0DB@FPJDLMBE@CNTL?5?9?5We?5can?8t?5join?5ad?5hoc?5on?5J@ 1000d3a4     connect.obj
 0001:0000c3d8       ??_C@_0BP@JPMBCMNP@CNTL?5?9?5CntlOidRTBssidProc?5?4?4?4?6?$AA@ 1000d3d8     connect.obj
 0001:0000c3f8       ??_C@_0DP@BDNIGPEF@CCKM?5fast?9roaming?5start?3?5set?5pAd@ 1000d3f8     connect.obj
 0001:0000c438       ??_C@_0CG@DPLPNMHD@CNTL?5?9?5Roaming?5in?5MlmeAux?4RoamTa@ 1000d438     connect.obj
 0001:0000c460       ??_C@_0EI@NHFCLGFF@CNTL?5?9?5DLS?5not?5changed?5in?5entry?5@ 1000d460     connect.obj
 0001:0000c4a8       ??_C@_0CC@BCCPFDHN@CNTL?5?9?5DLS?5retry?5setup?5procedure@ 1000d4a8     connect.obj
 0001:0000c4cc       ??_C@_0CA@LGMDFFBA@CNTL?5?9?5DLS?5update?5timeout?5case?6?$AA@ 1000d4cc     connect.obj
 0001:0000c4ec       ??_C@_0CH@CNGBLNHB@CNTL?5?9?5DLS?5tear?5down?5and?5restart@ 1000d4ec     connect.obj
 0001:0000c514       ??_C@_0BH@DMEGDDPI@CNTL?5?9?5DLS?5setup?5case?6?$AA@ 1000d514     connect.obj
 0001:0000c52c       ??_C@_0CC@MOHAIDEM@CNTL?5?9?5start?5tear?5down?5procedure@ 1000d52c     connect.obj
 0001:0000c550       ??_C@_0BK@HFCBPDEC@CNTL?5?9?5setting?5unchanged?6?$AA@ 1000d550     connect.obj
 0001:0000c570       ??_C@_0GI@BDNNBLIH@CNTL?5?9?5?$CIOID?5set?5?$CF02x?3?$CF02x?3?$CF02x?3?$CF@ 1000d570     connect.obj
 0001:0000c5d8       ??_C@_0DI@EOEOHJBD@CNTL?5?9?5No?5matching?5BSS?0?5start?5a?5@ 1000d5d8     connect.obj
 0001:0000c610       ??_C@_0CB@MMEFCBNJ@CNTL?5?9?5Dis?9associate?5successful?6@ 1000d610     connect.obj
 0001:0000c638       ??_C@_0EE@JODJEKHN@Delete?5bssid?0?5?$CF02x?3?$CF02x?3?$CF02x?3?$CF02@ 1000d638     connect.obj
 0001:0000c67c       ??_C@_0DK@GNDGOIM@CNTL?5?9?5join?5the?5IBSS?5?$DN?5?$CF02x?3?$CF02x@ 1000d67c     connect.obj
 0001:0000c6b8       ??_C@_0CA@FLBFBMJE@Indicate?5connection?5in?5IBSS?4?4?4?6?$AA@ 1000d6b8     connect.obj
 0001:0000c6d8       ??_C@_0CC@BKCKLCJK@CNTL?5?9?5Start?5IBSS?5fail?4?5BUG?$CB?$CB?$CB?$CB?$CB@ 1000d6d8     connect.obj
 0001:0000c6fc       ??_C@_0DN@JKJJHMJO@CNTL?5?9?5start?5a?5new?5IBSS?5?$DN?5?$CF02x?3?$CF@ 1000d6fc     connect.obj
 0001:0000c73c       ??_C@_0DN@CIIECJPE@CntlWaitAuthProc?0?5CNTL?5?9?5AUTH?5FA@ 1000d73c     connect.obj
 0001:0000c77c       ??_C@_0CC@PCDLLDHO@CntlWaitAuthProc?3?5CNTL?5?9?5AUTH?5OK@ 1000d77c     connect.obj
 0001:0000c7a0       ??_C@_0DM@ONNKPCJM@CntlWaitAuthProc2?3?5CNTL?5?9?5AUTH?5F@ 1000d7a0     connect.obj
 0001:0000c7e0       ??_C@_0EH@BPFFNJNO@CntlWaitAuthProc2?3?5CNTL?5?9?5AUTH?5F@ 1000d7e0     connect.obj
 0001:0000c828       ??_C@_0DJ@JINOIAOC@CntlWaitAuthProc2?3?5CNTL?5?9?5AUTH?5F@ 1000d828     connect.obj
 0001:0000c864       ??_C@_0CD@EEMEDNJA@CntlWaitAuthProc2?3?5CNTL?5?9?5AUTH?5O@ 1000d864     connect.obj
 0001:0000c888       ??_C@_0CF@LMFEBJPF@CNTL?5?9?5Association?5fails?5on?5BSS?5@ 1000d888     connect.obj
 0001:0000c8b0       ??_C@_0CG@ONDODCOH@Indicate?5previous?5queued?5EAPOL?5f@ 1000d8b0     connect.obj
 0001:0000c8d8       ??_C@_0CK@DNGMGINB@CNTL?5?9?5Association?5successful?5on@ 1000d8d8     connect.obj
 0001:0000c904       ??_C@_0CH@NPFFEDFO@CNTL?5?9?5Re?9assocition?5fails?5on?5BS@ 1000d904     connect.obj
 0001:0000c92c       ??_C@_0CM@NBDJHLMD@CNTL?5?9?5Re?9assocition?5successful?5@ 1000d92c     connect.obj
 0001:0000c958       ??_C@_0DN@PLAJGFBI@CNTL?5?9?5TDLS?5not?5changed?5in?5entry@ 1000d958     connect.obj
 0001:0000c998       ??_C@_0CD@DHNPCNGO@CNTL?5?9?5TDLS?5retry?5setup?5procedur@ 1000d998     connect.obj
 0001:0000c9c0       ??_C@_0ED@GHAMIJOG@CNTL?5?9?5TDLS?5not?5changed?5in?5Idx?5?$DN@ 1000d9c0     connect.obj
 0001:0000ca04       ??_C@_0DA@PMJCPJFN@CNTL?5?9?5TDLS?5not?5changed?5in?5Idx?5?$DN@ 1000da04     connect.obj
 0001:0000ca34       ??_C@_0BI@HHIPEDKF@CNTL?5?9?5TDLS?5setup?5case?6?$AA@ 1000da34     connect.obj
 0001:0000ca50       ??_C@_0GF@NKFLGMMK@CNTL?5?9?5CntlOidTDLSRequestProc?5se@ 1000da50     connect.obj
 0001:0000cab8       ??_C@_0BL@MPFJGAFC@?$CFs?3?5?$CB?$CB?$CB20MHz?5LINK?5UP?5?$CB?$CB?$CB?5?6?$AA@ 1000dab8     connect.obj
 0001:0000cad4       ??_C@_0DN@MIMNAALC@?$CFs?3?$CB?$CB?$CB40MHz?5Upper?5?$CB?$CB?$CB?5Control?5Ch@ 1000dad4     connect.obj
 0001:0000cb18       ??_C@_0EA@HJMOBKAB@?$CFs?3?5?$CB?$CB?$CB40MHz?5Lower?5?$CB?$CB?$CB?5Control?5C@ 1000db18     connect.obj
 0001:0000cb58       ??_C@_0BB@GDDJODMP@?$CFs?3?$CB?$CB?$CB20MHz?$CB?$CB?$CB?5?6?$AA@ 1000db58     connect.obj
 0001:0000cb6c       ??_C@_0CC@DOFGAMMH@?$CFs?3?5SecondaryChannelOffset?7?$FL?$CFd?$FN?5@ 1000db6c     connect.obj
 0001:0000cb90       ??_C@_0BL@KCFIGCHA@?$CFs?3?5ChannelWidth?7?7?7?7?$FL?$CFd?$FN?5?6?$AA@ 1000db90     connect.obj
 0001:0000cbac       ??_C@_0BM@DDONAEML@?$CFs?3?5CentralChannel?7?7?7?$FL?$CFd?$FN?5?6?$AA@ 1000dbac     connect.obj
 0001:0000cbc8       ??_C@_0BM@MCGEAMML@?$CFs?3?5PrimaryChannel?7?7?7?$FL?$CFd?$FN?5?6?$AA@ 1000dbc8     connect.obj
 0001:0000cbe4       ??_C@_0BB@PEOHMOAB@CntlChannelWidth?$AA@ 1000dbe4     connect.obj
 0001:0000cbf8       ??_C@_0CL@EAIMAIGO@?$CFs?3?5pAd?9?$DOTxPowerCtrl?4idxTxPowerT@ 1000dbf8     connect.obj
 0001:0000cc28       ??_C@_0EH@BJKECOGJ@LinkUP?5AP?5supports?520?140?5BSS?5COE@ 1000dc28     connect.obj
 0001:0000cc70       ??_C@_0BP@HLFBLLCO@?$CB?$CB?$CBpAd?9?$DObNextDisableRxBA?$DN?5?$CFd?5?6?$AA@ 1000dc70     connect.obj
 0001:0000cc90       ??_C@_0CO@PEBCGNLF@AP?5set?5OperaionMode?5?$DN?5?$CFd?0?5?5NonGf@ 1000dc90     connect.obj
 0001:0000ccc0       ??_C@_0BE@NNKBFON@?9?9?9?$DOAsicEnableRDG?5?6?$AA@ 1000dcc0     connect.obj
 0001:0000ccd4       ??_C@_0BM@CFLPKPI@?$CB?$CB?$CBAP?5MaxRAmpduFactor?$DN?5?$CFd?5?6?$AA@ 1000dcd4     connect.obj
 0001:0000ccf0       ??_C@_0L@KJEHPHBA@Txburst?53?6?$AA@ 1000dcf0     connect.obj
 0001:0000ccfc       ??_C@_0L@KIIFJNCH@Txburst?52?6?$AA@ 1000dcfc     connect.obj
 0001:0000cd08       ??_C@_0L@KKMDCDHO@Txburst?51?6?$AA@ 1000dd08     connect.obj
 0001:0000cd18       ??_C@_0EO@NBOGBIAG@NDIS_STATUS_MEDIA_CONNECT?5Event?5@ 1000dd18     connect.obj
 0001:0000cd68       ??_C@_0BJ@DEEDFOIL@ClientStatusFlags?5?$DN?5?$CFx?$CB?6?$AA@ 1000dd68     connect.obj
 0001:0000cd84       ??_C@_0CJ@NMGIHBAM@?$CFs?3?5LED_NORMAL_CONNECTION_WITH_S@ 1000dd84     connect.obj
 0001:0000cdb0       ??_C@_0CM@NDCALDNC@?$CFs?3?5LED_NORMAL_CONNECTION_WITHOU@ 1000ddb0     connect.obj
 0001:0000cddc       ??_C@_0CP@MDHCHLMH@Link?5UP?$CB?$CB?5Resume?5the?5data?5transm@ 1000dddc     connect.obj
 0001:0000ce0c       ??_C@_0CE@KMIEAHPI@NDIS_STATUS_MEDIA_CONNECT?5Event?5@ 1000de0c     connect.obj
 0001:0000ce30       ??_C@_0GD@EOLKDFFM@CCKM?5fast?9roaming?3?5indicated?5NDI@ 1000de30     connect.obj
 0001:0000ce94       ??_C@_0CA@MDADEECB@?9?9?9?$DOAssoc?5with?5Ralink?5Chipset?5?6?$AA@ 1000de94     connect.obj
 0001:0000ceb4       ??_C@_0BF@HHBJOIFD@Turn?5on?5Aggregation?6?$AA@ 1000deb4     connect.obj
 0001:0000cecc       ??_C@_0BE@FGODCGJG@Turn?5on?5Piggy?9Back?6?$AA@ 1000decc     connect.obj
 0001:0000cee0       ??_C@_0CI@BNGJHDJM@NDIS_STATUS_MEDIA_DISCONNECT?5Eve@ 1000dee0     connect.obj
 0001:0000cf08       ??_C@_0CF@DEEKMBCH@CNTL?5?9?5?$CB?$CB?$CB?5Set?5to?5short?5preamble@ 1000df08     connect.obj
 0001:0000cf30       ??_C@_0FO@FELPKMJB@?$CB?$CB?$CB?5LINK?5UP?5?$CB?$CB?$CB?5?$CIInfra?$DN?$CFd?0?5AID?$DN?$CF@ 1000df30     connect.obj
 0001:0000cf90       ??_C@_0BH@KNCPHDDL@?$CB?$CB?$CB20MHz?5LINK?5UP?5?$CB?$CB?$CB?5?6?$AA@ 1000df90     connect.obj
 0001:0000cfa8       ??_C@_06EBKOENJN@LinkUp?$AA@ 1000dfa8     connect.obj
 0001:0000cfb0       ??_C@_0BN@PLHAAGBB@?$CB?$CB?$CB20MHz?5Adhoc?5LINK?5UP?5?$CB?$CB?$CB?5?6?$AA@ 1000dfb0     connect.obj
 0001:0000cfd0       ??_C@_0EM@MGBPMMJC@The?5same?5control?5channel?5and?5cen@ 1000dfd0     connect.obj
 0001:0000d020       ??_C@_0EK@PFNGJCOM@?$CB?$CB?$CB40MHz?5Upper?5Adhoc?5LINK?5UP?5?$CB?$CB?$CB@ 1000e020     connect.obj
 0001:0000d070       ??_C@_0EK@CFMGBPAL@?$CB?$CB?$CB40MHz?5Lower?5Adhoc?5LINK?5UP?5?$CB?$CB?$CB@ 1000e070     connect.obj
 0001:0000d0c0       ??_C@_0JK@KPPPOHAA@Adhoc?5LinkUp?5?9?5bAdhocNMode?$DN?$CFd?0?5A@ 1000e0c0     connect.obj
 0001:0000d160       ??_C@_0EP@HFHPOINJ@?$CB?$CB?$CB?5LINK?5UP?5?$CB?$CB?$CIMaxRAmpduFactor?$DN?$CF@ 1000e160     connect.obj
 0001:0000d1b0       ??_C@_0BG@DMMGHMIA@?$CB?$CB?$CB?5LINK?5DOWN?5?$DM?$DN?$DN?$CB?$CB?$CB?6?$AA@ 1000e1b0     connect.obj
 0001:0000d1c8       ??_C@_0CF@PGHCFCIL@?$CB?$CB?$CBLINK?5DOWN?5set?5back?5to?520MHz?5?$CB@ 1000e1c8     connect.obj
 0001:0000d1f0       ??_C@_0BF@PPKCCBOB@Double?5link?5down?5?$DP?$DP?6?$AA@ 1000e1f0     connect.obj
 0001:0000d208       ??_C@_0CH@DAOLMICM@?$FL070727?$FN?$CF02x?5?$CF02x?5?$CF02x?5?$CF02x?5?$CF02x@ 1000e208     connect.obj
 0001:0000d230       ??_C@_0DF@DKAOILPK@?$FL070727?$FNDelete?5bssid?0?5?$CF02x?5?$CF02x?5@ 1000e230     connect.obj
 0001:0000d268       ??_C@_0CH@BBCHEH@NDIS_STATUS_MEDIA_DISCONNECT?5Eve@ 1000e268     connect.obj
 0001:0000d290       ??_C@_0ED@MOFHDEPM@Delete?5adhoc?5bssid?5from?5scan?5tab@ 1000e290     connect.obj
 0001:0000d2d4       ??_C@_0BD@MFBGAHKA@?$CB?$CB?$CB?5LINK?5DOWN?5?$CB?$CB?$CB?6?$AA@ 1000e2d4     connect.obj
 0001:0000d2e8       ??_C@_0EA@PGOPIOEA@?$CFs?3?5CNTL?5?9?5Implicit?5scan?0?5pAd?9?$DOM@ 1000e2e8     connect.obj
 0001:0000d328       ??_C@_0BA@KNONKFA@IterateOnBssTab?$AA@ 1000e328     connect.obj
 0001:0000d338       ??_C@_0CK@DLNELIG@CNTL?5?9?5All?5roaming?5failed?0?5stay?5@ 1000e338     connect.obj
 0001:0000d364       ??_C@_0DF@FJJFLKBJ@CNTL?5?9?5All?5BSS?5fail?$DL?5start?5a?5new@ 1000e364     connect.obj
 0001:0000d3a0       ??_C@_0EL@OKNLKCPD@CNTL?5?9?5All?5BSS?5failed?$DL?5But?5we?5ca@ 1000e3a0     connect.obj
 0001:0000d3ec       ??_C@_0BO@NDPDGCCE@CNTL?5?9?5iterate?5BSS?$FL?$CFd?$FN?5of?5?$CFd?6?$AA@ 1000e3ec     connect.obj
 0001:0000d40c       ??_C@_0CC@OIJDKIID@IterateOnBssTab?3?5CCKMEnable?5?$DN?5?$CFd@ 1000e40c     connect.obj
 0001:0000d430       ??_C@_0EC@OGPHDHJB@CNTL?5?9?5IterateOnBssTab2?0?5All?5fas@ 1000e430     connect.obj
 0001:0000d474       ??_C@_0CC@HIKJNDPD@CNTL?5?9?5IterateOnBssTab2?5?$CFd?5of?5?$CFd@ 1000e474     connect.obj
 0001:0000d498       ??_C@_0P@NJEIDGPH@ComposePsPoll?6?$AA@ 1000e498     connect.obj
 0001:0000d4a8       ??_C@_0GN@GCPBELG@MakeIbssBeacon?5?$CIlen?$DN?$CFd?$CJ?0?5SupRate@ 1000e4a8     connect.obj
 0001:0000d718       ??_C@_0DC@JOCHAODH@DLS?5?9?5MlmeDlsReqAction?$CI?$CJ?5allocat@ 1000e718     dls.obj
 0001:0000d74c       ??_C@_0BL@HIPHFBFG@DLS?5?9?5MlmeDlsReqAction?$CI?$CJ?5?6?$AA@ 1000e74c     dls.obj
 0001:0000d768       ??_C@_0CE@JAKKNIAP@DLS?5?9?5PeerDlsReqAction?$CI?$CJ?5SEND?5OU@ 1000e768     dls.obj
 0001:0000d78c       ??_C@_0BD@CAEMGPKJ@DLS?5?9?5init?5MCS?5?$CFd?6?$AA@ 1000e78c     dls.obj
 0001:0000d7a0       ??_C@_0DM@KDEBEJEB@DLS?5?9?5HT?5cap?5found?0?5ch?5width?$CI?$CFd?$CJ@ 1000e7a0     dls.obj
 0001:0000d7dc       ??_C@_0DE@BELDOCHA@BA?5BaSizeInUse?5?$DN?5?$CFd?0?5TXBAbitmap?$DN@ 1000e7dc     dls.obj
 0001:0000d810       ??_C@_0EG@GAAOEKAN@DLS?5?9?5PeerDlsReqAction?$CI?$CJ?5use?5ent@ 1000e810     dls.obj
 0001:0000d858       ??_C@_0FA@PAMPCDCD@DLS?5?9?5PeerDlsReqAction?$CI?$CJ?5DLSEntr@ 1000e858     dls.obj
 0001:0000d8a8       ??_C@_0DD@PPOOAKFI@DLS?5?9?5PeerDlsReqAction?$CI?$CJ?5can?5not@ 1000e8a8     dls.obj
 0001:0000d8dc       ??_C@_0CG@PNLJCFHC@DLS?5?9?5PeerDlsReqAction?$CI?$CJ?5find?5en@ 1000e8dc     dls.obj
 0001:0000d904       ??_C@_0DA@OPOHDFDG@DLS?5?9?5PeerDlsReqAction?$CI?$CJ?5MLME_RE@ 1000e904     dls.obj
 0001:0000d934       ??_C@_0DG@NOMEMEHH@DLS?5?9?5PeerDlsReqAction?$CI?$CJ?5MLME_DE@ 1000e934     dls.obj
 0001:0000d96c       ??_C@_0DC@ONAPCAIE@DLS?5?9?5PeerDlsReqAction?$CI?$CJ?5allocat@ 1000e96c     dls.obj
 0001:0000d9a0       ??_C@_0DN@CAPFEHOK@DLS?5?9?5PeerDlsReqAction?$CI?$CJ?5from?5?$CF0@ 1000e9a0     dls.obj
 0001:0000d9e0       ??_C@_0DA@MPCJHPGL@DLS?5?9?5PeerDlsRspAction?$CI?$CJ?5update?5@ 1000e9e0     dls.obj
 0001:0000da10       ??_C@_0DD@MPKKIKFA@DLS?5?9?5PeerDlsRspAction?5failed?5wi@ 1000ea10     dls.obj
 0001:0000da48       ??_C@_0FN@ODBCHMFN@DLS?5?9?5PeerDlsRspAction?$CI?$CJ?5from?5?$CF0@ 1000ea48     dls.obj
 0001:0000daa8       ??_C@_0CO@NHLMCKGB@DLS?5?9?5waiting?5for?5STAKey?5handsha@ 1000eaa8     dls.obj
 0001:0000dad8       ??_C@_0EA@LLLJOGLO@DLS?5?9?5PeerDlsRspAction?5failed?5wh@ 1000ead8     dls.obj
 0001:0000db18       ??_C@_0GF@JBIFNCGL@DLS?5?9?5PeerDlsRspAction?$CI?$CJ?5from?5?$CF0@ 1000eb18     dls.obj
 0001:0000db80       ??_C@_0DH@GCECJFKB@DLS?5?9?5MlmeDlsTearDownAction?$CI?$CJ?5al@ 1000eb80     dls.obj
 0001:0000dbb8       ??_C@_0DD@PJBGNLAI@DLS?5?9?5MlmeDlsTearDownAction?$CI?$CJ?5wi@ 1000ebb8     dls.obj
 0001:0000dbf0       ??_C@_0FF@ICFDABNB@DLS?5?9?5PeerDlsTearDownAction?$CI?$CJ?5fr@ 1000ebf0     dls.obj
 0001:0000dc48       ??_C@_0CM@NBGKBBOH@DLS?5timeout?5?$CF02x?5?$CF02x?5?$CF02x?5?$CF02x?5@ 1000ec48     dls.obj
 0001:0000dc74       ??_C@_0DF@IBIKFPCF@DLS?5?9?5Finish?5STAKey?5handshake?5pr@ 1000ec74     dls.obj
 0001:0000dcb0       ??_C@_0ED@FIHDFLIM@DLS?5?9?5Receive?5STAKey?5Message?91?5?$CI@ 1000ecb0     dls.obj
 0001:0000dcf4       ??_C@_0DK@KOBLHKCI@DLS?5?9?5Finish?5STAKey?5handshake?5pr@ 1000ecf4     dls.obj
 0001:0000dd30       ??_C@_0DP@OPFEHIBH@DLS?5?9?5Receive?5STAKey?5Message?91?5?$CI@ 1000ed30     dls.obj
 0001:0000dd70       ??_C@_0FP@HKBEFJGE@DLS?5?9?52?5Sniff?5replay?5counter?52?$CI?$CF@ 1000ed70     dls.obj
 0001:0000ddd0       ??_C@_0FJ@PHAMBNJM@DLS?5?9?5Receive?5STAKey?5Message?91?5f@ 1000edd0     dls.obj
 0001:0000de2c       ??_C@_0CJ@CHKOOLBC@MIC?5VALID?5in?5Msg1?5of?5STAKey?5hand@ 1000ee2c     dls.obj
 0001:0000de58       ??_C@_0CN@NEECEEPG@MIC?5Different?5in?5Msg1?5of?5STAKey?5@ 1000ee58     dls.obj
 0001:0000de88       ??_C@_0CB@BBPBGEJA@IEEE802?411?5WIRELESS?5ACCESS?5POINT@ 1000ee88     dls.obj
 0001:0000deb0       ??_C@_0FO@EJFILBAA@DLS?5?9?51?5Sniff?5replay?5counter?5?$CI?$CF0@ 1000eeb0     dls.obj
 0001:0000df10       ??_C@_0DM@KBAENAOB@ASSOC?5?9?5RTMPSendDLSTearDownFrame@ 1000ef10     dls.obj
 0001:0000df4c       ??_C@_0BK@MDABLJDL@Send?5DLS?5TearDown?5Frame?5?6?$AA@ 1000ef4c     dls.obj
 0001:0000df68       ??_C@_0EG@BFBNCFIE@RTMPSendSTAKeyRequest?9?5Send?5STAK@ 1000ef68     dls.obj
 0001:0000dfb0       ??_C@_0EA@JHEFCJCH@DLS?5?9?5RTMPSendSTAKeyRequest?$CI?$CJ?5to@ 1000efb0     dls.obj
 0001:0000dff0       ??_C@_0EK@IOMEFILK@RTMPSendSTAKeyHandShake?9?5Send?5ST@ 1000eff0     dls.obj
 0001:0000e040       ??_C@_0EC@FCDKBFAE@DLS?5?9?5RTMPSendSTAKeyHandShake?$CI?$CJ?5@ 1000f040     dls.obj
 0001:0000e088       ??_C@_0EC@ECHAOJPL@DlsTimeout?5?9?5Tear?5down?5DLS?5links@ 1000f088     dls.obj
 0001:0000e2d0       ??_C@_0DF@NAHJKOKC@Add?3Rogue?5AP?$FL?$CF02X?3?$CF02X?3?$CF02X?3?$CF02X@ 1000f2d0     leap.obj
 0001:0000e308       ??_C@_0BL@MEIODHBJ@?$DM?$DN?$DN?5LeapSendRogueAPReport?6?$AA@ 1000f308     leap.obj
 0001:0000e324       ??_C@_0BL@JPOPJKAL@?$DN?$DN?$DO?5LeapSendRogueAPReport?6?$AA@ 1000f324     leap.obj
 0001:0000e340       ??_C@_0FM@OKKLKPEC@Report?5Adjacent?5Previous?5AP?$FL?$CF02X@ 1000f340     leap.obj
 0001:0000e39c       ??_C@_0DB@BAGFCAKC@Sending?5CCXAdjacentAPReport?4?4?4?4?4@ 1000f39c     leap.obj
 0001:0000e3d0       ??_C@_0DO@DHIPBOBC@Report?5CCXAAPReasonCodeReport?5?9R@ 1000f3d0     leap.obj
 0001:0000e410       ??_C@_0CH@PIDJAPFN@Sending?5CCXAAPReasonCodeReport?4?4@ 1000f410     leap.obj
 0001:0000e958       ??_C@_0N@BOOJCAPA@HW?5Diversity?$AA@ 1000f958     mlme.obj
 0001:0000e968       ??_C@_05LKLMIBEG@Ant?9B?$AA@ 1000f968     mlme.obj
 0001:0000e970       ??_C@_05JBJBNCIF@Ant?9A?$AA@ 1000f970     mlme.obj
 0001:0000e978       ??_C@_0N@ENCHDJIJ@SW?5Diversity?$AA@ 1000f978     mlme.obj
 0001:0000e988       ??_C@_0DC@DNIOBKKO@4?9way?5handshake?5IE?5diff?5among?5As@ 1000f988     mlme.obj
 0001:0000e9bc       ??_C@_0CE@ODBDOOLB@2?9way?5?$CIgroup?5key?$CJ?5handshake?5time@ 1000f9bc     mlme.obj
 0001:0000e9e0       ??_C@_0BI@IFDLABDB@4?9way?5handshake?5timeout?$AA@ 1000f9e0     mlme.obj
 0001:0000e9f8       ??_C@_09CJDAIAGP@MIC?5error?$AA@ 1000f9f8     mlme.obj
 0001:0000ea04       ??_C@_0L@LCBPMDKI@invalid?5IE?$AA@ 1000fa04     mlme.obj
 0001:0000ea10       ??_C@_0CD@EMJAOFKL@require?5auth?5before?5assoc?1re?9ass@ 1000fa10     mlme.obj
 0001:0000ea34       ??_C@_0O@IBGJFIPI@class?53?5error?$AA@ 1000fa34     mlme.obj
 0001:0000ea44       ??_C@_0O@ENMDFIGG@class?52?5error?$AA@ 1000fa44     mlme.obj
 0001:0000ea54       ??_C@_0CE@IOCPNGNK@AP?5unable?5to?5hanle?5all?5associati@ 1000fa54     mlme.obj
 0001:0000ea78       ??_C@_0BM@OBHJDPBG@DIS?9ASSOC?5due?5to?5inactivity?$AA@ 1000fa78     mlme.obj
 0001:0000ea94       ??_C@_0BK@BAGFOGKD@STA?5is?5leaving?5?1?5has?5left?$AA@ 1000fa94     mlme.obj
 0001:0000eab0       ??_C@_0BO@PEBKGJDA@Previous?5Auth?5no?5longer?5valid?$AA@ 1000fab0     mlme.obj
 0001:0000ead0       ??_C@_0BD@PBGFPAEA@Unspecified?5Reason?$AA@ 1000fad0     mlme.obj
 0001:0000eae4       ??_C@_08NKCLJDKG@Reserved?$AA@ 1000fae4     mlme.obj
 0001:0000ecf0       ??_C@_0BF@KFHIDKKF@?$DM?9?9?5MLME?5Initialize?6?$AA@ 1000fcf0     mlme.obj
 0001:0000ed08       ??_C@_0BF@MBFCBGHE@?9?9?$DO?5MLME?5Initialize?6?$AA@ 1000fd08     mlme.obj
 0001:0000ed20       ??_C@_0BO@NALBCFMJ@MlmeHandler?3?5MlmeQueue?5empty?6?$AA@ 1000fd20     mlme.obj
 0001:0000ed40       ??_C@_0CJ@GLPMGFH@ERROR?3?5Illegal?5machine?5in?5MlmeHa@ 1000fd40     mlme.obj
 0001:0000ed6c       ??_C@_0CC@CLKIEPMO@?$CB?$CB?$CB?5reset?5MLME?5state?5machine?5?$CB?$CB?$CB@ 1000fd6c     mlme.obj
 0001:0000ed90       ??_C@_0EK@EGLGGJEG@Device?5Halted?5or?5Removed?5or?5Mlme@ 1000fd90     mlme.obj
 0001:0000eddc       ??_C@_0O@DPOFPIAE@?$DM?$DN?$DN?5MlmeHalt?6?$AA@ 1000fddc     mlme.obj
 0001:0000edec       ??_C@_0O@NFHEMLIC@?$DN?$DN?$DO?5MlmeHalt?6?$AA@ 1000fdec     mlme.obj
 0001:0000edfc       ??_C@_0BA@FEFLNHKP@?$DM?$DN?$DNMlmeSuspend?6?$AA@ 1000fdfc     mlme.obj
 0001:0000ee0c       ??_C@_0CA@KBPCGKML@ERROR?3?5empty?5Elem?5in?5MlmeQueue?6?$AA@ 1000fe0c     mlme.obj
 0001:0000ee2c       ??_C@_0BA@IGFCGDOF@?$DN?$DN?$DOMlmeSuspend?6?$AA@ 1000fe2c     mlme.obj
 0001:0000ee3c       ??_C@_0P@DEFOPNOP@?$DM?$DN?$DNMlmeResume?6?$AA@ 1000fe3c     mlme.obj
 0001:0000ee4c       ??_C@_0P@DAGPEKMJ@?$DN?$DN?$DOMlmeResume?6?$AA@ 1000fe4c     mlme.obj
 0001:0000ee5c       ??_C@_0BH@EGNKNBGF@indicate?5ICV?5Event?4?4?4?6?$AA@ 1000fe5c     mlme.obj
 0001:0000ee74       ??_C@_0CD@HEDBGBO@OneSecAggCnt?$DN?$CFd?0OneSecNoAggCnt?$DN?$CF@ 1000fe74     mlme.obj
 0001:0000ee98       ??_C@_0CH@BCKEIIKJ@NDIS_STATUS_MEDIA_DISCONNECT?5Eve@ 1000fe98     mlme.obj
 0001:0000eec0       ??_C@_0FO@CNAEOJJ@?$FLPending?$FN?5Rx?$FL?$CFd?$FN?5Tx?$FL?$CFd?$FN?5SendTxWa@ 1000fec0     mlme.obj
 0001:0000ef20       ??_C@_0FG@NEIKENHP@hog?5the?5TCPwindowsize?3?5Update?5pA@ 1000ff20     mlme.obj
 0001:0000ef78       ??_C@_0GH@IFKAMFAF@SessionTimeout?5reset?5to?5default?$CB@ 1000ff78     mlme.obj
 0001:0000efe0       ??_C@_0CJ@HHINICLJ@MMCHK?5?9?5pAd?9?$DOBulkLastOneSecCount@ 1000ffe0     mlme.obj
 0001:0000f00c       ??_C@_0CE@ELOODNLJ@pAd?9?$DOStaCfg?4bAutoReconnect?5is?5TR@ 1001000c     mlme.obj
 0001:0000f030       ??_C@_0DK@KINFKHLB@CNTL?5?9?5No?5matching?5BSS?0?5start?5a?5@ 10010030     mlme.obj
 0001:0000f06c       ??_C@_0CL@CGKOOPBI@MLME?5periodic?5exec?0?5no?5associati@ 1001006c     mlme.obj
 0001:0000f098       ??_C@_0CJ@ICGACAGI@CLEAR?5S71?5BSSID?$CK?$CK?$CK?$CK?$CK?$CK?$CK?$CK?$CK?$CK?$CK?$CK?$CK?$CK?$CK?$CK?$CK@ 10010098     mlme.obj
 0001:0000f0c8       ??_C@_0EP@LAOHBGHC@MMCHK?5?9?5excessive?5BEACON?5lost?0?5l@ 100100c8     mlme.obj
 0001:0000f118       ??_C@_0CL@KJDFOMDE@Not?5found?5radar?5signal?0?5start?5se@ 10010118     mlme.obj
 0001:0000f144       ??_C@_0BI@CKMGBLNE@Found?5radar?5signal?$CB?$CB?$CB?6?6?$AA@ 10010144     mlme.obj
 0001:0000f15c       ??_C@_0CF@GCMBILBC@?5scanning?5for?5AST?5?0?5Rssi?$DN?$CFd?0?5AST@ 1001015c     mlme.obj
 0001:0000f184       ??_C@_0CI@BALPGCOP@STAMlmePeriodicExec?3?5Drastically@ 10010184     mlme.obj
 0001:0000f1b0       ??_C@_0ED@LHDBCMDB@MaxRssi?$DN?$CFd?0?5dBmToRoam?$DN?$CFd?0?5LastRs@ 100101b0     mlme.obj
 0001:0000f1f8       ??_C@_0GN@MAGDHIBI@?$CFs?3?5?$CICarrier?5detection?5is?5enable@ 100101f8     mlme.obj
 0001:0000f268       ??_C@_0CM@GJLCIBAC@MMCHK?5?9?5Bad?5CQI?4?5Auto?5Recovery?5a@ 10010268     mlme.obj
 0001:0000f298       ??_C@_0GO@DPJBGPCC@?$CFs?3?5?$CICarrier?5detection?5is?5enable@ 10010298     mlme.obj
 0001:0000f308       ??_C@_0DI@IJMMIEOH@MMCHK?5?9?5No?5BEACON?4?5Dead?5CQI?4?5Aut@ 10010308     mlme.obj
 0001:0000f340       ??_C@_0DG@ONANNFBI@MMCHK?5?9?5No?5BEACON?4?5restore?5R66?5t@ 10010340     mlme.obj
 0001:0000f378       ??_C@_0FK@PJBIOBIB@bFastRoamingScan?5?4?4?4?4?4?4?4?4?4?4?4?4?4?5R@ 10010378     mlme.obj
 0001:0000f3d4       ??_C@_0BH@GLGJLBNL@?$CFs?3?5recover?5TX_RTY_CFG?$AA@ 100103d4     mlme.obj
 0001:0000f3ec       ??_C@_0BE@EEDDGCDK@STAMlmePeriodicExec?$AA@ 100103ec     mlme.obj
 0001:0000f400       ??_C@_0BD@GDAANNNG@channel?5stay?$CI?$CFd?$CJ?5?6?$AA@ 10010400     mlme.obj
 0001:0000f418       ??_C@_0EG@HMPHDLDM@MlmePeriodicExec?3?5no?5connect?0?5sw@ 10010418     mlme.obj
 0001:0000f460       ??_C@_0CC@GDODIMJD@Ant?9realrssi0?$CI?$CFd?$CJ?0?5Lastrssi0?$CI?$CFd?$CJ@ 10010460     mlme.obj
 0001:0000f484       ??_C@_0DB@NLDAOOAH@MlmePeriodicExec?3?5no?5traffic?1bea@ 10010484     mlme.obj
 0001:0000f4b8       ??_C@_0EF@HBMLNPIK@MMCHK?5?9?5CommonCfg?4Ssid?$FL?$CFd?$FN?$DN?$CFc?$CFc?$CF@ 100104b8     mlme.obj
 0001:0000f500       ??_C@_0BM@ILNIJFKJ@PSM?5?9?5Issue?5Sleep?5command?$CJ?6?$AA@ 10010500     mlme.obj
 0001:0000f51c       ??_C@_0CJ@EBMBDAJM@pAd?9?$DOCommonCfg?4APEdcaParm?4Aifsn?$FL@ 1001051c     mlme.obj
 0001:0000f548       ??_C@_0BM@NHHFLMOE@EDCA_AC0_CFG?4Aifsn?$FL0?$FN?5?$DN?5?$CFd?6?$AA@ 10010548     mlme.obj
 0001:0000f564       ??_C@_0CD@PKEFFJMF@Clear?5up?5?$CB?$CB?$CB?$CB?$CB?$CB?$CB?$CB?$CB?$CB?$CB?$CB?$CB?$CB?$CBIndex?$FL?$CFd@ 10010564     mlme.obj
 0001:0000f588       ??_C@_0DP@MGAAPABM@Temporarily?5skipping?5write?5back?5@ 10010588     mlme.obj
 0001:0000f5c8       ??_C@_0DO@CFAMCNIE@TX?5QUEUE?50?5or?51?5Not?5EMPTY?4?5?$CB?$CB?$CB?$CB?$CB@ 100105c8     mlme.obj
 0001:0000f608       ??_C@_0BK@GAJBDICC@MMCHK?5?9?5Driver?5auto?5scan?6?$AA@ 10010608     mlme.obj
 0001:0000f628       ??_C@_0EG@NHNNNGNH@Driver?5auto?5reconnect?5to?5last?5OI@ 10010628     mlme.obj
 0001:0000f670       ??_C@_0CI@PEGBGEDL@?$DM?$DN?$DN?5MlmeCheckForFastRoaming?5?$CIBss@ 10010670     mlme.obj
 0001:0000f698       ??_C@_0DD@LEDDAC@MMCHK?5?9?5Roaming?0?5No?5eligable?5ent@ 10010698     mlme.obj
 0001:0000f6cc       ??_C@_0CC@GLDIDDHH@MMCHK?5?9?5Fast?5Roaming?5attempt?5?$CD?$CFd@ 100106cc     mlme.obj
 0001:0000f6f0       ??_C@_0FD@EHOOAHJH@Not?5Roam?0?5skip?5RH?0?5?$CIMaxRSSI?$DN?$CFd?$CJ?0@ 100106f0     mlme.obj
 0001:0000f748       ??_C@_0EM@JGPBEIN@RSSI?5is?5lower?5than?5MRSP?0?5don?8t?5R@ 10010748     mlme.obj
 0001:0000f798       ??_C@_0EA@KDJFJCHG@CheckForFastRoaming?5?9?9?5IGNORE?5th@ 10010798     mlme.obj
 0001:0000f7d8       ??_C@_0CP@BIJFOKCM@Drastically?5Roam?4?4?4?5CCXPktLossLi@ 100107d8     mlme.obj
 0001:0000f808       ??_C@_0DB@MLAKGEAA@?$DM?$DN?$DN?5Quit?5MlmeCheckForFastRoaming@ 10010808     mlme.obj
 0001:0000f840       ??_C@_0EB@NHEAGKCJ@?$DM?$DN?$DN?5Quit?5MlmeCheckForFastRoaming@ 10010840     mlme.obj
 0001:0000f884       ??_C@_0DE@LBNEJMLI@?$DM?$DN?$DN?5Quit?5MlmeCheckForFastRoaming@ 10010884     mlme.obj
 0001:0000f8b8       ??_C@_0GE@DLNFEIIA@?$DN?$DN?$DO?5MlmeCheckForFastRoaming?0?5Sca@ 100108b8     mlme.obj
 0001:0000f920       ??_C@_0FC@FNIFIADK@MMCHK?5?9?5CQI?$DN?5?$CFd?5?$CITx?5Fail?$DN?$CFd?1Retr@ 10010920     mlme.obj
 0001:0000f974       ??_C@_0DA@CIDAAHMM@BEACON?5lost?5?$DO?5?$CFd?5msec?5with?5TxOkC@ 10010974     mlme.obj
 0001:0000f9a8       ??_C@_0FF@PCOHFJHK@DRS?3?5MlmeSetTxRate?5?9?5CurrTxRateI@ 100109a8     mlme.obj
 0001:0000fa00       ??_C@_0CC@PJEGFOGN@?$DN?$DN?$DN?$DN?$DN?$DO?5MlmeUpdateLimitTxRateTabl@ 10010a00     mlme.obj
 0001:0000fa28       ??_C@_0FH@NFAMFKDN@?$CFs?3?5TableRowSize?$FL0x?$CF02x?$FN?0?5Init?5R@ 10010a28     mlme.obj
 0001:0000fa80       ??_C@_0BL@GHBPJGAG@MlmeUpdateLimitTxRateTable?$AA@ 10010a80     mlme.obj
 0001:0000fa9c       ??_C@_0CF@HKGEEBJF@0x?$CF02x?9?$DO0x?$CF02x?0?50x?$CF02x?0?5?$CFd?0?5?$CFd?0?5@ 10010a9c     mlme.obj
 0001:0000fac4       ??_C@_0CA@PMFGOAAG@0x?$CF02x?3pCurrTxRate?9?$DOCurrMCS?$DN?$CFd?6?$AA@ 10010ac4     mlme.obj
 0001:0000fae4       ??_C@_0CC@HIMMGEDH@?$DM?$DN?$DN?$DN?$DN?$DN?5MlmeUpdateLimitTxRateTabl@ 10010ae4     mlme.obj
 0001:0000fb08       ??_C@_0GM@PKJJDPMD@DRS?3?5unknown?5mode?5?$CISupRateLen?$DN?$CFd@ 10010b08     mlme.obj
 0001:0000fb78       ??_C@_0GJ@LEDMHBI@DRS?3?5unknown?5mode?0LimitTxRateTab@ 10010b78     mlme.obj
 0001:0000fbe8       ??_C@_0GA@FKPGLFJI@DRS?3?5unknown?5mode?0default?5use?5Li@ 10010be8     mlme.obj
 0001:0000fc48       ??_C@_0CK@IPIIDAKC@DRS?3?5unknown?5mode?0default?5use?511@ 10010c48     mlme.obj
 0001:0000fc74       ??_C@_0CK@BAHDHEB@DRS?3?5unknown?5mode?0default?5use?511@ 10010c74     mlme.obj
 0001:0000fca0       ??_C@_0O@NCHJBNBC@DRS?3?5A?1G?5AP?5?6?$AA@ 10010ca0     mlme.obj
 0001:0000fcb0       ??_C@_0BE@JDGBMMPI@DRS?3?5B?1G?5mixed?5AP?5?6?$AA@ 10010cb0     mlme.obj
 0001:0000fcc4       ??_C@_0BB@HJHBKMJH@DRS?3?5B?5only?5AP?5?6?$AA@ 10010cc4     mlme.obj
 0001:0000fcd8       ??_C@_0BB@NIHDNDMF@DRS?3?511N?52S?5AP?5?6?$AA@ 10010cd8     mlme.obj
 0001:0000fcec       ??_C@_0BB@FGPMNECG@DRS?3?511N?51S?5AP?5?6?$AA@ 10010cec     mlme.obj
 0001:0000fd00       ??_C@_0BD@PHFEIFAL@DRS?3?511BGN?52S?5AP?5?6?$AA@ 10010d00     mlme.obj
 0001:0000fd14       ??_C@_0BD@HJNLICOI@DRS?3?511BGN?51S?5AP?5?6?$AA@ 10010d14     mlme.obj
 0001:0000fd28       ??_C@_0CK@NDCIFABG@DRS?3?5unknown?5mode?0default?5use?511@ 10010d28     mlme.obj
 0001:0000fd54       ??_C@_0BB@KFMLEJC@DRS?3?511N?52S?5DL?5?6?$AA@ 10010d54     mlme.obj
 0001:0000fd68       ??_C@_0BB@IENDLDHB@DRS?3?511N?51S?5DL?5?6?$AA@ 10010d68     mlme.obj
 0001:0000fd7c       ??_C@_0BD@CFHLOCFM@DRS?3?511BGN?52S?5DL?5?6?$AA@ 10010d7c     mlme.obj
 0001:0000fd90       ??_C@_0BD@KLPEOFLP@DRS?3?511BGN?51S?5DL?5?6?$AA@ 10010d90     mlme.obj
 0001:0000fda4       ??_C@_0O@FGHKEF@DRS?3?5A?1G?5DL?5?6?$AA@ 10010da4     mlme.obj
 0001:0000fdb4       ??_C@_0BE@EBEOKLKP@DRS?3?5B?1G?5mixed?5DL?5?6?$AA@ 10010db4     mlme.obj
 0001:0000fdc8       ??_C@_0BB@KLFOMLMA@DRS?3?5B?5only?5DL?5?6?$AA@ 10010dc8     mlme.obj
 0001:0000fddc       ??_C@_0BH@ODOJOMIN@DRS?3?5B?1G?5mixed?5Adhoc?5?6?$AA@ 10010ddc     mlme.obj
 0001:0000fdf4       ??_C@_0BB@MMNDNFLC@DRS?3?5A?1G?5Adhoc?5?6?$AA@ 10010df4     mlme.obj
 0001:0000fe08       ??_C@_0BE@NICIBLLJ@DRS?3?5B?5only?5Adhoc?5?6?$AA@ 10010e08     mlme.obj
 0001:0000fe1c       ??_C@_0CM@NOKANJOF@DRS?3?5unkown?5mode?0default?5use?511N@ 10010e1c     mlme.obj
 0001:0000fe48       ??_C@_0BE@PBLJOFND@DRS?3?511N?52S?5Adhoc?5?6?$AA@ 10010e48     mlme.obj
 0001:0000fe5c       ??_C@_0BE@GIFLIDNC@DRS?3?511N?51S?5Adhoc?5?6?$AA@ 10010e5c     mlme.obj
 0001:0000fe70       ??_C@_0BM@MGDDMOFJ@DRS?3?5CH14?5only?5suports?511B?6?$AA@ 10010e70     mlme.obj
 0001:0000fe8c       ??_C@_0CD@GHIOAGOF@DRS?3?5rate?5table?5is?5from?5rate?4bin@ 10010e8c     mlme.obj
 0001:0000feb0       ??_C@_0EL@GLOIOACI@DRS?3?5Rx?$CI?$CFd?$CJ?5is?55?5times?5larger?5th@ 10010eb0     mlme.obj
 0001:0000fefc       ??_C@_0DL@PCEDKGPM@DRS?3?5MCS?5is?5according?5to?5RSSI?0?5a@ 10010efc     mlme.obj
 0001:0000ff38       ??_C@_0EH@JPELGHGJ@DRS?$CIAid?3?$CFd?$CJ?3?3?5AccuTxTotalCnt?5?$DM?$DN?5@ 10010f38     mlme.obj
 0001:0000ff80       ??_C@_0FK@CABLPJNP@DRS?3?5?$CD?$CD?$CD?$CD?5leave?5Noisy?5environmen@ 10010f80     mlme.obj
 0001:0000ffdc       ??_C@_0DE@MMBODGPB@DRS?3?5?$CD?$CD?$CD?$CD?5enter?5Noisy?5environmen@ 10010fdc     mlme.obj
 0001:00010010       ??_C@_0KD@IAOPDJML@DRS?3?5Before?9?5CurrTxRateIdx?$DN?$CFd?0?5M@ 10011010     mlme.obj
 0001:000100b8       ??_C@_0GN@ONPMBOAO@DRS?3?5Fixed?5?9?5CurrTxRateIdx?$DN?$CFd?0?5M@ 100110b8     mlme.obj
 0001:00010128       ??_C@_0BF@IDBJKKIN@DRS?3?5use?5lower?5rate?6?$AA@ 10011128     mlme.obj
 0001:00010140       ??_C@_0DE@KGCMELOD@Chk5?3?3?5CurrRateIdx?$DN?$CFd?0?5UpRateIdx@ 10011140     mlme.obj
 0001:00010174       ??_C@_0DD@BDPGIMLA@?$CFs?3?5CurrRateIdx?$FL?$CFd?$FN?5UpRateIdx?$FL?$CFd@ 10011174     mlme.obj
 0001:000101a8       ??_C@_0FA@KGPBFBB@DRS?3TxErrorRatio?5?$DN?5?$CFd?0?5TxNoRetry@ 100111a8     mlme.obj
 0001:000101f8       ??_C@_0BF@IDMHPDJL@?$CFs?3?5reset?5TX_RTY_CFG?$AA@ 100111f8     mlme.obj
 0001:00010210       ??_C@_0BL@PAGLPHLB@MlmeDynamicTxRateSwitching?$AA@ 10011210     mlme.obj
 0001:0001022c       ??_C@_0CA@NNFOKHOI@QuickDRS?3?5rate?5is?5not?5changed?5?6?$AA@ 1001122c     mlme.obj
 0001:00010250       ??_C@_0EI@OBJFDDLP@QuickDRS?3?5?$CIDown?$CJ?5direct?5train?5do@ 10011250     mlme.obj
 0001:00010298       ??_C@_0DO@EAIEOGHI@QuickDRS?3?5AccuTxTotalCnt?5?$DM?$DN?512?0?5@ 10011298     mlme.obj
 0001:000102d8       ??_C@_0EL@LCKHHBPJ@QuickDRS?3?5TxSuccess?$DN?$CFd?0?5TxRetran@ 100112d8     mlme.obj
 0001:00010324       ??_C@_0BE@BPMIFJNI@MlmeSetPsmBit?5?$DN?5?$CFd?6?$AA@ 10011324     mlme.obj
 0001:00010338       ??_C@_0CG@EENPFOPN@MlmeSetTxPreamble?5?$CI?$DN?5SHORT?5PREAM@ 10011338     mlme.obj
 0001:00010360       ??_C@_0CF@GGJHLABL@MlmeSetTxPreamble?5?$CI?$DN?5LONG?5PREAMB@ 10011360     mlme.obj
 0001:00010388       ??_C@_0FL@CBGHPJH@MlmeUpdateTxRates?5?$CIMlmeTransmit?$DN@ 10011388     mlme.obj
 0001:000103e8       ??_C@_0EE@BANLCMAO@?5MlmeUpdateTxRates?5?$CITxRate?$DN?$CFd?0?5R@ 100113e8     mlme.obj
 0001:00010430       ??_C@_0GA@HCCINNO@?5MlmeUpdateTxRates?5?$CIMaxDesire?$DN?$CFd@ 10011430     mlme.obj
 0001:00010490       ??_C@_0DG@DBIFONLM@?5MlmeUpdateTxRates?5?$CIRssi?$DN?$CFd?0?5ini@ 10011490     mlme.obj
 0001:000104c8       ??_C@_0DI@HHKKDIOC@MlmeUpdateTxRates?$FLMaxSupport?5?$DN?5?$CF@ 100114c8     mlme.obj
 0001:00010500       ??_C@_0CC@NNNGGMIO@Exptected?5ACK?5rate?$FL?$CFd?$FN?5?$DN?5?$CFd?5Mbps@ 10011500     mlme.obj
 0001:00010524       ??_C@_0DA@EJHIJFEM@MlmeUpdateTxRates?4?52?5MaxDesire?5?$DN@ 10011524     mlme.obj
 0001:00010554       ??_C@_0BG@MFOGFPNA@E?5ACK?5?5?$FL?$CFd?$FN?5?$DN?5?$CFd?5Mbps?$AA@ 10011554     mlme.obj
 0001:0001056c       ??_C@_0BK@PNPCFJIL@MlmeUpdateHtTxRates?$DM?$DN?$DN?$DN?5?6?$AA@ 1001156c     mlme.obj
 0001:00010588       ??_C@_0BN@ICPCPNFG@TX?3?5HTPhyMode?4word?5?$DN?5?$CFx?5?5?5?5?6?$AA@ 10011588     mlme.obj
 0001:000105a8       ??_C@_0CM@HKGOEJIE@MlmeUpdateHtTxRates?$DM?$DN?$DN?$DN?5Use?5Fixe@ 100115a8     mlme.obj
 0001:000105d4       ??_C@_0BE@PKOEONKE@MlmeUpdateHtTxRates?$AA@ 100115d4     mlme.obj
 0001:000105e8       ??_C@_0BK@EJDAPNNB@MlmeUpdateHtTxRates?$DN?$DN?$DN?$DO?5?6?$AA@ 100115e8     mlme.obj
 0001:00010608       ??_C@_0FC@PIFADGGK@AsicUpdateAutoFallBackTable?3?5HtC@ 10011608     mlme.obj
 0001:0001065c       ??_C@_0CJ@BCMJBJMF@AsicUpdateAutoFallBackTable?3?5not@ 1001165c     mlme.obj
 0001:00010688       ??_C@_0CJ@CKMFLHAG@AsicUpdateProtect?3?5OperaionMode?5@ 10011688     mlme.obj
 0001:000106b4       ??_C@_0BO@ICCGLDIP@AsicUpdateProtect?3?524M?5rate?5?6?$AA@ 100116b4     mlme.obj
 0001:000106d4       ??_C@_0BN@LIAAOEHG@AsicUpdateProtect?3?56M?5rate?5?6?$AA@ 100116d4     mlme.obj
 0001:000106f4       ??_C@_0BO@NKAFNJNH@AsicUpdateProtect?3?5CCK?5rate?5?6?$AA@ 100116f4     mlme.obj
 0001:00010714       ??_C@_0CD@JKJMDGED@AsicUpdateProtect?3?5Legacy?5?$CFd?5?0?$CFd@ 10011714     mlme.obj
 0001:00010738       ??_C@_0BO@GEKAED@Reserve?5Entry?$CD0?5to?5Ssid?5?$DN?$CFs?5?6?$AA@ 10011738     mlme.obj
 0001:00010758       ??_C@_0BA@KJDEKPLG@MlmeRadioOff?$CI?$CJ?6?$AA@ 10011758     mlme.obj
 0001:00010768       ??_C@_0EF@IMDEKBAH@NextRxBulkInReadIndex?5?$DN?5?$CFd?0?5Next@ 10011768     mlme.obj
 0001:000107b0       ??_C@_0P@JMAEHFGL@MlmeRadioOn?$CI?$CJ?6?$AA@ 100117b0     mlme.obj
 0001:000107c0       ??_C@_0BN@DADDKGLO@?$CFs?3?5scanningTableIndex?5?$DN?5?$CFd?6?$AA@ 100117c0     mlme.obj
 0001:000107e0       ??_C@_0P@EKNNFPHG@BssTableSearch?$AA@ 100117e0     mlme.obj
 0001:000107f0       ??_C@_0FN@BFMLFMDM@?$CFs?3?5Remove?5BSS?5entry?0?5BSSID?5?$DN?5?$CF0@ 100117f0     mlme.obj
 0001:00010850       ??_C@_0GK@GPOIJODF@?$CFs?3?5Skip?5the?5associated?5BSS?5entr@ 10011850     mlme.obj
 0001:000108bc       ??_C@_0BN@MHOFDNAK@BssTableDeleteEntryByChannel?$AA@ 100118bc     mlme.obj
 0001:000108dc       ??_C@_0CL@HHAADFEO@BATableDeleteORIEntry?5numAsOrigi@ 100118dc     mlme.obj
 0001:00010908       ??_C@_0EC@NCGJNKI@BATableDeleteRECEntry?5pBARECEntr@ 10011908     mlme.obj
 0001:00010950       ??_C@_0EO@BEBALCCH@RTUSBEnqueueInternalCmd?3?5RT_OID_@ 10011950     mlme.obj
 0001:000109a0       ??_C@_0CJ@HACPPOEF@BATableTearRECEntry?$DN?$DN?$DN?$DO?5Wcid?$DN?$CFd?4@ 100119a0     mlme.obj
 0001:000109cc       ??_C@_0DO@BCFKIFPF@BATableTearORIEntry?$DN?$DN?$DN?$DO?5Wcid?$DN?$CFd?4@ 100119cc     mlme.obj
 0001:00010a10       ??_C@_0ED@PBGAFDAJ@?9?9?$DO?5ControlChannel?5?$DN?5?$CFd?0?5ExtChan@ 10011a10     mlme.obj
 0001:00010a58       ??_C@_0HG@FLDKELEB@?$CFs?3?5Reserve?5the?5WPS?5IE?5in?5the?5pr@ 10011a58     mlme.obj
 0001:00010ad0       ??_C@_0GO@BNFEAGKI@?$CFs?3?5Reserve?5the?5WPS?5IE?5in?5the?5be@ 10011ad0     mlme.obj
 0001:00010b40       ??_C@_0M@FFACBGO@BssEntrySet?$AA@ 10011b40     mlme.obj
 0001:00010b4c       ??_C@_0BJ@CFBDKLND@?$DM?$DN?$DN?$DNBATableInsertEntry?5?6?$AA@ 10011b4c     mlme.obj
 0001:00010b68       ??_C@_0DC@BHBGADNE@MACEntry?$FL?$CFd?$FNTXBAbitmap?5?$DN?50x?$CFx?4?5B@ 10011b68     mlme.obj
 0001:00010b9c       ??_C@_0DD@ODDLHLLO@BATableInsert?5?9?5already?5exists?4?5@ 10011b9c     mlme.obj
 0001:00010bd0       ??_C@_0CF@IIEJKBKI@BATableInsert?5handshake?5in?5progr@ 10011bd0     mlme.obj
 0001:00010bf8       ??_C@_0CH@CMIOBEAB@BATableInsertEntry?$FL?$CFd?$FN?4?5BAWinSiz@ 10011bf8     mlme.obj
 0001:00010c20       ??_C@_0DO@JCLKKOEF@BATableInsert?5?$DN?$DN?$DN?$DOAid?$DN?$CFd?0?5BAIdx?5@ 10011c20     mlme.obj
 0001:00010c60       ??_C@_0DN@FNPNGMDG@MACEntry?$FL?$CFd?$FN?5Seq?5?$DN?5?$CFx?0?5RXBAbitma@ 10011c60     mlme.obj
 0001:00010ca0       ??_C@_0EF@FJLCMPIC@Recipient?5?3?5pAddr?5?$DN?$CFx?0?5?$CFx?0?5?5?$CFx?0?5@ 10011ca0     mlme.obj
 0001:00010ce8       ??_C@_0CL@CCPPLGGJ@BATableInsert?$FL?$CFd?$FN?5?$DN?$DN?$DN?$DOWcid?5?$DN?5?$CFd?0@ 10011ce8     mlme.obj
 0001:00010d18       ??_C@_0EH@OKLFKMHJ@BATableInsert?5Recipient?5Entry?5?$DN?$DN@ 10011d18     mlme.obj
 0001:00010d60       ??_C@_0JM@IFKHJOHI@?$CFs?3?5The?5NIC?5cannot?5connect?5a?5hid@ 10011d60     mlme.obj
 0001:00010dfc       ??_C@_0BB@PONFMPHG@BssTableSsidSort?$AA@ 10011dfc     mlme.obj
 0001:00010e10       ??_C@_0DG@BALAFOO@Let?5WEPEnabled?5STA?5try?5to?5connec@ 10011e10     mlme.obj
 0001:00010e48       ??_C@_0DE@KFDCONOO@CommonCfg?4WepStatus?$DN?$CFd?0?5while?5pI@ 10011e48     mlme.obj
 0001:00010e80       ??_C@_0FM@DCPGBCEB@Skip?5this?5BSS?5since?5it?8s?5on?5Japp@ 10011e80     mlme.obj
 0001:00010edc       ??_C@_0CD@NCHLFCOA@L2Roaming?5?9?5NBL?5?$CIswap?5BSS?5entry?$CJ@ 10011edc     mlme.obj
 0001:00010f00       ??_C@_0BO@JHNBDDPA@QbssLoad?5?9?5?$CIswap?5BSS?5entry?$CJ?5?6?$AA@ 10011f00     mlme.obj
 0001:00010f20       ??_C@_0CK@CFGONPAM@Check?5AuthMode?$FL0x?$CF08X?$FN?5WepStatus@ 10011f20     mlme.obj
 0001:00010f4c       ??_C@_0BN@KIPHBEBM@Check?5Multicast?5cipher?5Fail?6?$AA@ 10011f4c     mlme.obj
 0001:00010f6c       ??_C@_0BL@LEBLOLPM@Check?5Unicast?5cipher?5Fail?6?$AA@ 10011f6c     mlme.obj
 0001:00010f88       ??_C@_0CM@FKAGMGAF@Check?5AKM?5Fail?50x?$CF02X?30x?$CF02X?30x?$CF@ 10011f88     mlme.obj
 0001:00010fb4       ??_C@_0BJ@KIHADAFK@Check?5WAPI?5version?5Fail?6?$AA@ 10011fb4     mlme.obj
 0001:00010fd0       ??_C@_0BF@MNDOIEEO@MlmeEnqueue?0?5num?$DN?$CFd?6?$AA@ 10011fd0     mlme.obj
 0001:00010fe8       ??_C@_0EM@DCOKADDF@MlmeEnqueue?3?5full?0?5msg?5dropped?5a@ 10011fe8     mlme.obj
 0001:00011034       ??_C@_0CI@ODKFEBBA@MlmeEnqueue?3?5msg?5too?5large?0?5size@ 10012034     mlme.obj
 0001:0001105c       ??_C@_0BM@DNAMCAN@MlmeEnqueueForRecv?0?5num?$DN?$CFd?6?$AA@ 1001205c     mlme.obj
 0001:00011078       ??_C@_0DF@OGAGJABB@MlmeEnqueueForRecv?3?5un?9recongniz@ 10012078     mlme.obj
 0001:000110b0       ??_C@_0CG@HKDBINCL@MlmeEnqueueForRecv?3?5full?5and?5dro@ 100120b0     mlme.obj
 0001:000110d8       ??_C@_0BF@BAEDGELA@MlmeDequeue?0?5num?$DN?$CFd?6?$AA@ 100120d8     mlme.obj
 0001:000110f0       ??_C@_0BN@POPBCJAH@?$DM?$DN?$DN?5MlmeRestartStateMachine?6?$AA@ 100120f0     mlme.obj
 0001:00011110       ??_C@_0KO@BEJOIIEK@?$CFs?3?5pAd?9?$DOMlmeAux?4LastScanChannel@ 10012110     mlme.obj
 0001:000111c0       ??_C@_0BI@OCBFKIDC@MlmeRestartStateMachine?$AA@ 100121c0     mlme.obj
 0001:000111d8       ??_C@_0BN@COGCNNOA@?$DN?$DN?$DO?5MlmeRestartStateMachine?6?$AA@ 100121d8     mlme.obj
 0001:000111f8       ??_C@_0CK@CJDPKHKC@MlmeRestartStateMachine?3?5MlmeQue@ 100121f8     mlme.obj
 0001:00011224       ??_C@_0CO@FLLGKMIB@DROP?5ELEMENT?5MACHINE?5?$DN?5?$CFd?5MESSAG@ 10012224     mlme.obj
 0001:00011254       ??_C@_0CF@HOBJDIJC@CATEGORY_DLS?5not?5support?$CIaction?$DN@ 10012254     mlme.obj
 0001:0001127c       ??_C@_0DB@BAJOCNJI@IBSS?5STA?5get?5correct?5WAI?5packet?5@ 1001227c     mlme.obj
 0001:000112b0       ??_C@_0CM@KDFOHIFK@STA?5get?5correct?5WAI?5packet?5subTy@ 100122b0     mlme.obj
 0001:000112dc       ??_C@_0BO@INIPMPCA@STA?5get?5incorrect?5WAI?5packet?6?$AA@ 100122dc     mlme.obj
 0001:00011300       ??_C@_0GA@LGEHEGEC@SwitchChannel?$CD?$CFd?$CIRF?$DN?$CFd?0?5Pwr0?$DN?$CFd?0@ 10012300     mlme.obj
 0001:00011360       ??_C@_0CA@FJKGGGNN@AsicSwitchChannel?3?5TxPwer2?$DN?$CFd?5?6?$AA@ 10012360     mlme.obj
 0001:00011380       ??_C@_0BP@GPBIJLJI@AsicSwitchChannel?3?5TxPwer?$DN?$CFd?5?6?$AA@ 10012380     mlme.obj
 0001:000113a0       ??_C@_0FG@NPJLNEPF@RT35xx?3?5SwitchChannel?$CD?$CFd?$CIRF?$DN?$CFd?0?5@ 100123a0     mlme.obj
 0001:000113f8       ??_C@_0EO@CJIJMNGK@SwitchChannel?$CD?$CFd?$CIRF?$DN?$CFd?0?5Pwr0?$DN?$CFd?0@ 100123f8     mlme.obj
 0001:00011448       ??_C@_0BC@FBKGMPLF@AsicSwitchChannel?$AA@ 10012448     mlme.obj
 0001:0001145c       ??_C@_0CP@IEHFKKKI@AsicSwitchChannel?3?5Can?8t?5find?5th@ 1001245c     mlme.obj
 0001:0001148c       ??_C@_0CE@GCEMBPIF@?$DM?9?9?5AsicAdjustTxPower?0?5DeltaPwr?$DN@ 1001248c     mlme.obj
 0001:000114b0       ??_C@_0GN@MDMFOBLF@AsicAdjustTxPower?5?9?5DeltaPwr?$DN?$CFd?0@ 100124b0     mlme.obj
 0001:00011520       ??_C@_0EB@OLPFIMEE@TPC?3?5?$DMafter?$DO?5?$CIindex?5?$DN?5?$CFd?$CJ?5Value?5@ 10012520     mlme.obj
 0001:00011564       ??_C@_0BN@KACNKELN@?$CFs?3?5unknown?5register?5?$DN?50x?$CFX?6?$AA@ 10012564     mlme.obj
 0001:00011588       ??_C@_0EC@KCJKBIOI@TPC?3?5?$DMbefore?$DO?5?$CIindex?5?$DN?5?$CFd?$CJ?5Value@ 10012588     mlme.obj
 0001:000115cc       ??_C@_0DC@HNCPDKIM@TPC?3?5?$DMAfter?5BBP?5R1?$DO?5?$CFs?3?5TotalDel@ 100125cc     mlme.obj
 0001:00011600       ??_C@_0DE@MEPJABDI@TPC?3?5?$CFs?3?5Drop?5the?5transmit?5power@ 10012600     mlme.obj
 0001:00011634       ??_C@_0DF@EFPBHOBC@TPC?3?5?$CFs?3?5Drop?5the?5transmit?5power@ 10012634     mlme.obj
 0001:0001166c       ??_C@_0DD@IDGAKBJ@TPC?3?5?$CFs?3?5?$DMBefore?5BBP?5R1?$DO?5TotalDe@ 1001266c     mlme.obj
 0001:000116a0       ??_C@_0FC@CIBONPNG@TPC?3?5?$CFs?3?5The?5associated?5AP?5does?5@ 100126a0     mlme.obj
 0001:000116f8       ??_C@_0FO@NCPAHFOH@TPC?3?5?$CFs?3?5Not?5exceed?5the?5tranmsit@ 100126f8     mlme.obj
 0001:00011758       ??_C@_0FL@HFMCMGEM@TPC?3?5?$CFs?3?5Exceed?5the?5transmit?5pow@ 10012758     mlme.obj
 0001:000117b8       ??_C@_0MA@DLICCPKN@TPC?3?5?$CFs?3?5Exceed?5the?5transmit?5pow@ 100127b8     mlme.obj
 0001:00011878       ??_C@_0GE@HGFFBGDI@TPC?3?5?$CFs?3?5RealTxPower?5?$DN?5?$CFd?0?5pAd?9?$DO@ 10012878     mlme.obj
 0001:000118e0       ??_C@_0FB@HFLBGGPJ@TPC?3?5?$CFs?3?5Rssi?5?$DN?5?$CFd?0?5TotalDeltaPo@ 100128e0     mlme.obj
 0001:00011934       ??_C@_0DJ@PIPANKNN@Chk9?3?3?5?$CK?$CK?5DeltaPwr?5?$DN?$CFd?0?5DeltaPow@ 10012934     mlme.obj
 0001:00011970       ??_C@_0DM@KHGLHPIJ@Chk9?3?3?5?$DO?$DO?5?9?9?5DeltaPwr?5?$DN?$CFd?0?5Delta@ 10012970     mlme.obj
 0001:000119ac       ??_C@_0BF@FKICOALC@Chk9?3?3?5?$DO?$DO?5?93?550?$CF?5dbm?$AA@ 100129ac     mlme.obj
 0001:000119c4       ??_C@_0BL@BIIGAFOI@Chk9?3?3?5?$DO?$DO?5?96?525?$CF?5power?5dbm?$AA@ 100129c4     mlme.obj
 0001:000119e0       ??_C@_0BL@INKDNBNM@Chk9?3?3?5?$DO?$DO?5?97?518?$CF?5power?5dbm?$AA@ 100129e0     mlme.obj
 0001:000119fc       ??_C@_0BL@GBNMJDPA@Chk9?3?3?5?$DO?$DO?5?91?575?$CF?5power?5dbm?$AA@ 100129fc     mlme.obj
 0001:00011a18       ??_C@_0DM@JMBNMJMF@Chk9?3?3?5?$DO?$DO?5?$CL?$CL?5DeltaPwr?5?$DN?$CFd?0?5Delta@ 10012a18     mlme.obj
 0001:00011a54       ??_C@_0DI@DOFLACFB@AsicAdjustTxPower?5?$CIi?1j?$DN?$CFd?1?$CFd?0?5Va@ 10012a54     mlme.obj
 0001:00011a8c       ??_C@_0CN@DHCAHLA@AsicAdjustTxPower?5?$CIi?1j?$DN?$CFd?1?$CFd?0?5Va@ 10012a8c     mlme.obj
 0001:00011ac0       ??_C@_0EI@HHEGMKNF@AsicAdjustTxPower?5?$CIcriterion?$DN?$CFd?0@ 10012ac0     mlme.obj
 0001:00011b08       ??_C@_0EF@BHEFGBBN@AsicAdjustTxPower?5?9?5Invalid?5max?5@ 10012b08     mlme.obj
 0001:00011b50       ??_C@_0DP@BHAAHKPE@?5?5?5Tx?5Power?0?5BBP?5R49?$DN?$CFx?0?5TssiRef@ 10012b50     mlme.obj
 0001:00011b90       ??_C@_0DP@LPAIKPCF@?$CL?$CL?5Tx?5Power?0?5BBP?5R49?$DN?$CFx?0?5TssiRef@ 10012b90     mlme.obj
 0001:00011bd0       ??_C@_0DP@KCIGPKO@?9?9?5Tx?5Power?0?5BBP?5R49?$DN?$CFx?0?5TssiRef@ 10012bd0     mlme.obj
 0001:00011c10       ??_C@_0GI@NOKFBCDC@?$CFs?3?5desiredTSSI?5?$DN?5?$CFd?0?5currentTSS@ 10012c10     mlme.obj
 0001:00011c78       ??_C@_0BK@LMPHGMGD@?$CFs?3?5ChannelQuality?$DN?5?$CFd?5?5?6?$AA@ 10012c78     mlme.obj
 0001:00011c94       ??_C@_0CG@BMMCHLK@?$CFs?3?5OneSecTransmittedByteCount?$DN?5@ 10012c94     mlme.obj
 0001:00011cbc       ??_C@_0CE@NAGOIGFJ@?$CFs?3?5OneSecReceivedByteCount?5?$DN?5?$CFd@ 10012cbc     mlme.obj
 0001:00011ce0       ??_C@_0FM@NKMEBFMI@?$CFs?3?5?$FLFiveSec?$FN?5TxNoRetryOkCount?$DN?$CF@ 10012ce0     mlme.obj
 0001:00011d3c       ??_C@_0BC@BOELLOFD@AsicAdjustTxPower?$AA@ 10012d3c     mlme.obj
 0001:00011d50       ??_C@_0DG@EHOHOFFP@?$DM?9?9?5AsicSleepThenAutoWakeup?0?5Tbt@ 10012d50     mlme.obj
 0001:00011d88       ??_C@_0CD@LGPHKOHB@MlmeSet?5Sleep?5Mailbox?5?5value?$DN0x?$CF@ 10012d88     mlme.obj
 0001:00011dac       ??_C@_0BG@BGMAKPHO@?$DM?9?9?5AsicForceWakeup?5?6?$AA@ 10012dac     mlme.obj
 0001:00011dc4       ??_C@_0CO@BHFLCBMB@?$DN?$DN?$DN?$DN?$DN?$DN?$DN?$DN?$DN?$DN?$DN?$DN?$DN?$DNAsicSetBssid?5?$CFx?3?$CFx@ 10012dc4     mlme.obj
 0001:00011df4       ??_C@_0BO@KDMHBFE@AsicDelWcidTab?$DN?$DN?$DOWcid?5?$DN?50x?$CFx?6?$AA@ 10012df4     mlme.obj
 0001:00011e14       ??_C@_0DJ@FPGGPEFE@?9?9?9?$DOAsicSetCarrierDetectAction?5?$CI@ 10012e14     mlme.obj
 0001:00011e50       ??_C@_0CB@KJJMMDE@?9?9?9?$DODisable?5TSF?5synchronization?6@ 10012e50     mlme.obj
 0001:00011e74       ??_C@_0BF@CLLHJGOG@?9?9?9?$DOAsicDisableRDG?5?6?$AA@ 10012e74     mlme.obj
 0001:00011e8c       ??_C@_0CD@NNMMNNEG@?9?9?9?$DOAsicEnableBssSync?$CIINFRA?5mode@ 10012e8c     mlme.obj
 0001:00011eb0       ??_C@_0DN@KJJPPLJH@?9?9?9?$DOAsicEnableIbssSync?$CIADHOC?5mod@ 10012eb0     mlme.obj
 0001:00011ef0       ??_C@_0CC@PHJDCGPK@?7?5?5AC_VO?5?7?$CFd?7?5?5?5?$CFd?7?5?5?$CFd?7?5?$CF4d?7?5?$CFd@ 10012ef0     mlme.obj
 0001:00011f14       ??_C@_0CC@ELMKHLDN@?7?5?5AC_VI?5?7?$CFd?7?5?5?5?$CFd?7?5?5?$CFd?7?5?$CF4d?7?5?$CFd@ 10012f14     mlme.obj
 0001:00011f38       ??_C@_0CC@ILFKGIBL@?7?5?5AC_BK?5?7?$CFd?7?5?5?5?$CFd?7?5?5?$CFd?7?5?$CF4d?7?5?$CFd@ 10012f38     mlme.obj
 0001:00011f5c       ??_C@_0CC@PFIBODFG@?7?5?5AC_BE?5?7?$CFd?7?5?5?5?$CFd?7?5?5?$CFd?7?5?$CF4d?7?5?$CFd@ 10012f5c     mlme.obj
 0001:00011f80       ??_C@_0CO@EONIKGDE@EDCA?5?$FL?$CD?$CFd?$FN?3?5AIFSN?5CWmin?5CWmax?5?5T@ 10012f80     mlme.obj
 0001:00011fb0       ??_C@_0BE@HFPABFBM@AsicSetEdcaParm?$DN?$DN?$DO?6?$AA@ 10012fb0     mlme.obj
 0001:00011fc4       ??_C@_0BJ@NALBBIL@AsicSetSlotTime?$CI?$DN?$CFd?5us?$CJ?6?$AA@ 10012fc4     mlme.obj
 0001:00011fe0       ??_C@_0DK@DCDNMCAD@RSSI?$DN?$CFd?0?5CCA?$DN?$CFd?0?5BW?$DN?$CFd?0?5LNA_GAIN@ 10012fe0     mlme.obj
 0001:0001201c       ??_C@_0BF@IODHCAGA@?$DM?$DN?$DN?5AsicAddKeyEntry?6?$AA@ 1001301c     mlme.obj
 0001:00012038       ??_C@_0EP@PCLGELNE@?$DN?$DN?$DO?5AsicAddKeyEntry?5?$CIWCID?$DN?$CFd?0?5Ke@ 10013038     mlme.obj
 0001:00012088       ??_C@_0DH@MHJBMMBD@AsicAddWcidCipherEntry?$DN?$DN?$DN?$DOKeyTab@ 10013088     mlme.obj
 0001:000120c0       ??_C@_0CK@MEGJLHBC@MCAST_WCID?5?3?5offset?5?$DN?5?$CFx?0?5WCIDAt@ 100130c0     mlme.obj
 0001:000120ec       ??_C@_0BD@LLOFFKKH@?5?5?5?5?5Tx?5MIC?5Key?5?$DN?5?$AA@ 100130ec     mlme.obj
 0001:00012100       ??_C@_0BD@EDCHBBBB@?5?5?5?5?5Rx?5MIC?5Key?5?$DN?5?$AA@ 10013100     mlme.obj
 0001:00012114       ??_C@_0L@JJFMPIKH@?5?5?5?5?5Key?5?$DN?$AA@ 10013114     mlme.obj
 0001:00012120       ??_C@_0CD@PMFJLLCD@AsicAddSharedKeyEntry?3?5?$CFs?5key?5?$CD?$CF@ 10013120     mlme.obj
 0001:00012144       ??_C@_0CM@LPOGKFOO@AsicRemoveSharedKeyMode?3?5BssInde@ 10013144     mlme.obj
 0001:00012170       ??_C@_1FC@PDKEJDKG@?$AAC?$AA?3?$AA?2?$AAW?$AAi?$AAn?$AAC?$AAE?$AA6?$AA?4?$AA0?$AA?2?$AAN?$AAe?$AAw?$AA?2?$AAR?$AAT?$AA2?$AA8?$AA7?$AA0?$AA_?$AAv?$AA1?$AA?4?$AA4?$AA?4?$AA9?$AA?4?$AA0?$AA?2@ 10013170     mlme.obj
 0001:000121c4       ??_C@_0BK@FINDAKIA@AsicRemoveKeyEntry?3?5?$CD?$CFd?5?6?$AA@ 100131c4     mlme.obj
 0001:000121e0       ??_C@_0DF@CIDFLIFM@Write?3?5SHARED_KEY_MODE_BASE?5at?5t@ 100131e0     mlme.obj
 0001:00012218       ??_C@_0CA@GIKNBHP@AsicRemoveSharedKeyEntry?3?5?$CD?$CFd?5?6?$AA@ 10013218     mlme.obj
 0001:00012238       ??_C@_0EG@JGHJLIKD@SW?5interrupt?5MCU?5?$CIcmd?$DN0x?$CF02x?0?5to@ 10013238     mlme.obj
 0001:00012280       ??_C@_0CN@JOECDODM@H2M_MAILBOX?5still?5hold?5by?5MCU?4?5c@ 10013280     mlme.obj
 0001:000122b0       ??_C@_0CH@FGDLMDDA@AsicSendCommanToMcu?3?3Mail?5box?5is@ 100132b0     mlme.obj
 0001:000122d8       ??_C@_0CG@LMMALOMF@Total?5Channel?5in?5Channel?5List?5?$DN?5@ 100132d8     mlme.obj
 0001:00012300       ??_C@_0CJ@LAEJPBL@LowerChannel?$DN?$CFd?5?5is?5in?5Channel?5L@ 10013300     mlme.obj
 0001:0001232c       ??_C@_0CJ@NCPNOOOG@UpperChannel?$DN?$CFd?5?5is?5in?5Channel?5L@ 1001332c     mlme.obj
 0001:00012358       ??_C@_0CF@NODEDMEB@LinkUP?520MHz?5?4?5No?5Effected?5Chann@ 10013358     mlme.obj
 0001:00012380       ??_C@_0HL@BJECDBFJ@RTMPCheckHt?3?3?5HtCapInfo?4ChannelW@ 10013380     mlme.obj
 0001:000123fc       ??_C@_0BK@HNNLIIPA@RTMPCheckHt?7?3?5bIsAtheros?6?$AA@ 100133fc     mlme.obj
 0001:00012418       ??_C@_0CF@GKKCFEND@AsicSetRxAnt?0?5switch?5to?5aux?5ante@ 10013418     mlme.obj
 0001:00012440       ??_C@_0CG@FMKCNKCJ@AsicSetRxAnt?0?5switch?5to?5main?5ant@ 10013440     mlme.obj
 0001:00012468       ??_C@_0CM@NFDOCGJC@AntDiv?5?9?5before?5evaluate?5Pair1?9A@ 10013468     mlme.obj
 0001:00012498       ??_C@_0EN@IMJIFCDI@AsicRxAntEvalTimeout?5?3?5RealRxPat@ 10013498     mlme.obj
 0001:000124e8       ??_C@_0FB@GJEFGENF@AsicRxAntEvalAction?3?3After?5Eval?$CI@ 100134e8     mlme.obj
 0001:0001253c       ??_C@_0BJ@DIAPDBOF@RadarDetectionStart?9?9?9?$DO?6?$AA@ 1001353c     mlme.obj
 0001:00012558       ??_C@_0BI@EJHJLFMH@Mlme?5Thread?5Terminated?6?$AA@ 10013558     mlme.obj
 0001:00012570       ??_C@_0BH@IFKBEDCF@Mlme?5Thread?5Triggered?6?$AA@ 10013570     mlme.obj
 0001:00012588       ??_C@_1EM@MNCKGOK@?$AAM?$AAl?$AAm?$AAe?$AAT?$AAh?$AAr?$AAe?$AAa?$AAd?$AA?5?$AAh?$AAa?$AAn?$AAd?$AAl?$AAe?$AA?$DN?$AA0?$AAx?$AA?$CF?$AAx?$AA?0?$AA?5?$AAP?$AAr?$AAi?$AAo?$AAr?$AAi?$AAt?$AAy@ 10013588     mlme.obj
 0001:000125d4       ??_C@_0BD@FOEHGML@Mlme?5Thread?5Start?6?$AA@ 100135d4     mlme.obj
 0001:000125e8       ??_C@_0CP@BDGHPBED@?$DM?$DN?$DN?5MlmeFreeMemory?5?$FLIN?3?$CFd?$FN?$FLUN?3?$CFd@ 100135e8     mlme.obj
 0001:00012618       ??_C@_0FH@CDHFCHFF@MlmeFreeMemory?5Add?5it?5to?5the?5Unu@ 10013618     mlme.obj
 0001:00012670       ??_C@_0HH@HGEKCKCA@?$DMWarning?$DOFree?5memory?5faild?$CB?$CB?5mem@ 10013670     mlme.obj
 0001:000126e8       ??_C@_0BE@IBOPMBON@?$DM?$DN?$DN?5MlmeFreeMemory?6?$AA@ 100136e8     mlme.obj
 0001:00012700       ??_C@_0FI@ELLHFEGA@Mlme?5memory?5Handler?5Busy?$CB?$CB?5move?5@ 10013700     mlme.obj
 0001:00012758       ??_C@_0BE@OAOCHMJ@?$DN?$DN?$DO?5MlmeFreeMemory?6?$AA@ 10013758     mlme.obj
 0001:0001276c       ??_C@_0DC@IMDMGHCM@?$DM?$DN?$DN?5MlmeAllocateMemory?$FLIN?3?$CFd?$FN?$FLUN@ 1001376c     mlme.obj
 0001:000127a0       ??_C@_0DG@MJNLKOFL@MlmeAllocateMemory?5?$FLpMlmeMemoryS@ 100137a0     mlme.obj
 0001:000127d8       ??_C@_0EG@KMAOJKEN@MlmeAllocateMemory?0?5failed?$CB?$CB?5?$CITh@ 100137d8     mlme.obj
 0001:00012820       ??_C@_0BI@KKHFDPKB@?$DM?$DN?$DN?5MlmeAllocateMemory?6?$AA@ 10013820     mlme.obj
 0001:00012838       ??_C@_0DJ@DGPBIMOD@Mlme?5memory?5Handler?5Busy?$CB?$CB?0?5Mlme@ 10013838     mlme.obj
 0001:00012874       ??_C@_0BI@BCCIPHMG@?$DN?$DN?$DO?5MlmeAllocateMemory?6?$AA@ 10013874     mlme.obj
 0001:0001288c       ??_C@_0BE@PGBALOCM@?$DM?$DN?$DN?5MlmeInitMemory?6?$AA@ 1001388c     mlme.obj
 0001:000128a0       ??_C@_0DK@EAMLLFJN@MlmeInitMemory?5Initial?5failed?5?$FLR@ 100138a0     mlme.obj
 0001:000128dc       ??_C@_0BE@HJPBFIAI@?$DN?$DN?$DO?5MlmeInitMemory?6?$AA@ 100138dc     mlme.obj
 0001:000128f0       ??_C@_0EM@FLEJBODC@RTMPSetAGCInitValue?5?9?5Ch?$DN?$CFd?0?5Ban@ 100138f0     mlme.obj
 0001:00012940       ??_C@_0EE@DBCNKBDN@RTMPHandleMCUInterrupt?9CTS?5can?8t@ 10013940     mlme.obj
 0001:00012988       ??_C@_0GG@KBAGNFCJ@CarrierDetectTimeoutAction?3?3?5car@ 10013988     mlme.obj
 0001:000129f0       ??_C@_0CP@OOCDOMPJ@?$DO?$DO?$DOCarrierDetectTimeoutAction?$DM?$DM?$DM@ 100139f0     mlme.obj
 0001:00012a20       ??_C@_0EI@DJFELHOO@CarrierDetectTimeoutAction?3?3MCU?5@ 10013a20     mlme.obj
 0001:00012a68       ??_C@_0CM@EICPKEPE@Wait?5?$FL?$CFd?$FN?5Kick?5NULL?5frame?5?$CD1?5to?5@ 10013a68     mlme.obj
 0001:00012a94       ??_C@_0CJ@GKPNJAJL@Wait?5?$FL?$CFd?$FN?5Kick?5NULL?5frame?5?$CD1?5Pwr@ 10013a94     mlme.obj
 0001:00012ac0       ??_C@_0BN@PDGNCJPE@Wait?5?$FL?$CFd?$FN?5Polling?5TXQ?5Empty?6?$AA@ 10013ac0     mlme.obj
 0001:00012ae0       ??_C@_0EB@NCICDDCD@RTUSBFilterCalibration?5?9?5CaliBW2@ 10013ae0     mlme.obj
 0001:00012b28       ??_C@_0EP@COPHLCBF@RTUSBFilterCalibration?5?9?5can?8t?5f@ 10013b28     mlme.obj
 0001:00012b78       ??_C@_0GF@MMFMCAFM@RTUSBFilterCalibration?5BBP_R55?$DN0@ 10013b78     mlme.obj
 0001:00012be0       ??_C@_0DK@MGJLJPBJ@Capability?$DN0x?$CFx?0?5M?$DN?$CFx?0?5U?$DN?$CFx?0?5AKM@ 10013be0     mlme.obj
 0001:00012c1c       ??_C@_0BP@BOFFJLCL@SSIDLUpdateBssEntry?0?5SSID?$DN?$CFs?5?6?$AA@ 10013c1c     mlme.obj
 0001:00012c40       ??_C@_0EB@HJPBLLMP@?9?9?$DO?5AsicCheckCommanFail2?5Timeout@ 10013c40     mlme.obj
 0001:00012c84       ??_C@_0DH@NMEJCCNO@?9?9?$DO?5AsicCheckCommanFail1?5CID?5?$DN?50@ 10013c84     mlme.obj
 0001:00012cbc       ??_C@_0DL@BOOBEJGL@PSM?5?3?5?9?9?$DO?5AsicCheckCommandOk?5CID@ 10013cbc     mlme.obj
 0001:00012cf8       ??_C@_08FMKNKPCP@?$DM?9?9?9?5?$CFs?6?$AA@ 10013cf8     mlme.obj
 0001:00012d08       ??_C@_0JE@GGNNHHLP@?$CFs?3?5desiredTSSIOverHTUsingSTBC?$FL4@ 10013d08     mlme.obj
 0001:00012da0       ??_C@_0JE@GCFMEELO@?$CFs?3?5desiredTSSIOverHTUsingSTBC?$FL0@ 10013da0     mlme.obj
 0001:00012e34       ??_C@_0BB@PMALDCBB@?$CFs?3?50xEF?5?$DN?50x?$CFX?6?$AA@ 10013e34     mlme.obj
 0001:00012e48       ??_C@_0BB@BHDMIJBC@?$CFs?3?50xEE?5?$DN?50x?$CFX?6?$AA@ 10013e48     mlme.obj
 0001:00012e5c       ??_C@_0BB@PIPOOCCM@?$CFs?3?50xED?5?$DN?50x?$CFX?6?$AA@ 10013e5c     mlme.obj
 0001:00012e70       ??_C@_0BB@BKCCPJFF@?$CFs?3?50xEC?5?$DN?50x?$CFX?6?$AA@ 10013e70     mlme.obj
 0001:00012e88       ??_C@_0HA@KPNPPDO@?$CFs?3?5desiredTSSIOverHT?$FL4?$FN?5?$DN?5?$CFd?0?5d@ 10013e88     mlme.obj
 0001:00012ef8       ??_C@_0HA@MMADIKOK@?$CFs?3?5desiredTSSIOverHT?$FL0?$FN?5?$DN?5?$CFd?0?5d@ 10013ef8     mlme.obj
 0001:00012f68       ??_C@_0BB@OFIANMLH@?$CFs?3?50xE7?5?$DN?50x?$CFX?6?$AA@ 10013f68     mlme.obj
 0001:00012f7c       ??_C@_0BB@KECLHIJ@?$CFs?3?50xE6?5?$DN?50x?$CFX?6?$AA@ 10013f7c     mlme.obj
 0001:00012f90       ??_C@_0BB@OBHFAMIK@?$CFs?3?50xE5?5?$DN?50x?$CFX?6?$AA@ 10013f90     mlme.obj
 0001:00012fa4       ??_C@_0BB@OLHGHLE@?$CFs?3?50xE4?5?$DN?50x?$CFX?6?$AA@ 10013fa4     mlme.obj
 0001:00012fb8       ??_C@_0HI@FIAGLCL@?$CFs?3?5desiredTSSIOverOFDM?$FL4?$FN?5?$DN?5?$CFd?0@ 10013fb8     mlme.obj
 0001:00013030       ??_C@_0HI@JBLAGHEF@?$CFs?3?5desiredTSSIOverOFDM?$FL0?$FN?5?$DN?5?$CFd?0@ 10014030     mlme.obj
 0001:000130a8       ??_C@_0BB@DKJBHPD@?$CFs?3?50xE2?5?$DN?50x?$CFX?6?$AA@ 100140a8     mlme.obj
 0001:000130bc       ??_C@_0BB@OIJOKMPA@?$CFs?3?50xE1?5?$DN?50x?$CFX?6?$AA@ 100140bc     mlme.obj
 0001:000130d0       ??_C@_0BB@HFMMHMO@?$CFs?3?50xE0?5?$DN?50x?$CFX?6?$AA@ 100140d0     mlme.obj
 0001:000130e8       ??_C@_0HE@CFDCDLEO@?$CFs?3?5desiredTSSIOverCCK?$FL0?$FN?5?$DN?5?$CFd?0?5@ 100140e8     mlme.obj
 0001:0001315c       ??_C@_0BB@DNIFONNB@?$CFs?3?50xDF?5?$DN?50x?$CFX?6?$AA@ 1001415c     mlme.obj
 0001:00013170       ??_C@_0BB@NGLCFGNC@?$CFs?3?50xDE?5?$DN?50x?$CFX?6?$AA@ 10014170     mlme.obj
 0001:00013188       ??_C@_0EA@KPMFLIIE@?$CFs?3?5TSSIBase?5?$DN?5?$CFd?0?5TSSIStepOver2@ 10014188     mlme.obj
 0001:000131c8       ??_C@_08GCFEIJCI@?9?9?9?$DO?5?$CFs?6?$AA@ 100141c8     mlme.obj
 0001:000131d4       ??_C@_0BF@GJFGPOPP@InitDesiredTSSITable?$AA@ 100141d4     mlme.obj
 0001:000131f0       ??_C@_0EM@MCKNJMGB@?$CFs?3?5desiredTSSI?5?$DN?5?$CFd?0?5Latest?5Tx?5@ 100141f0     mlme.obj
 0001:0001323c       ??_C@_0BN@GEBMLNBD@?$CFs?3?5incorrect?5MCS?3?5MCS?5?$DN?5?$CFd?6?$AA@ 1001423c     mlme.obj
 0001:0001325c       ??_C@_0P@LEJNFLJ@GetDesiredTSSI?$AA@ 1001425c     mlme.obj
 0001:0001326c       ??_C@_0BB@HIEDCGKJ@dot11k?3?5?$DM?9?9?9?5?$CFs?6?$AA@ 1001426c     mlme.obj
 0001:00013280       ??_C@_0CF@OKCLJBOB@dot11k?3?5?$CFs?3?5BbpIPITimer?4word?5?$DN?50@ 10014280     mlme.obj
 0001:000132a8       ??_C@_0CB@BJBAEHKG@dot11k?3?5?$CFs?3?5BbpR144?4byte?5?$DN?50x?$CFX?6@ 100142a8     mlme.obj
 0001:000132cc       ??_C@_0BB@EGLKAAKO@dot11k?3?5?9?9?9?$DO?5?$CFs?6?$AA@ 100142cc     mlme.obj
 0001:000132e0       ??_C@_0P@IACEKFNG@RRMInitNHMCtrl?$AA@ 100142e0     mlme.obj
 0001:000132f0       ??_C@_0FA@PFHCCEOB@dot11k?3?5?$CFs?3?5pIPIDensityArray?$FL?$CFd?$FN@ 100142f0     mlme.obj
 0001:00013340       ??_C@_0EJ@GIIJHFMB@dot11k?3?5?$CFs?3?5?$CIASIC?5not?5ready?5or?5d@ 10014340     mlme.obj
 0001:00013390       ??_C@_0FC@FPHJCOHF@dot11k?3?5?$CFs?3?5idleTime?5?$DN?5?$CI0x?$CFX?5?$DM?$DM?5@ 10014390     mlme.obj
 0001:000133e8       ??_C@_0FM@DMFBEPAG@dot11k?3?5?$CFs?3?5IPIValueArray?$FL?$CFd?$FN?5?$DN?5@ 100143e8     mlme.obj
 0001:00013444       ??_C@_0DB@CFIJHJNH@dot11k?3?5?$CFs?3?5BbpIPITimer?4field?4BB@ 10014444     mlme.obj
 0001:00013478       ??_C@_0BD@JNFNNBCG@RRMGetIPIDensities?$AA@ 10014478     mlme.obj
 0001:00013690       ??_C@_0EK@MODKFNNA@RTMPCkipInsertCMIC?0?5Before?5to?5fo@ 10014690     rtmp_ckipmic.obj
 0001:000136e0       ??_C@_0EH@PCODGPBD@RTMPCkipCalCMIC?0?5Before?5to?5form?5@ 100146e0     rtmp_ckipmic.obj
 0001:00013728       ??_C@_0DI@JBJNPANB@Decrypt?5ERROR?5?3?3?5SN?5?$DN?5?$CFd?0?5KeyIdx@ 10014728     rtmp_ckipmic.obj
 0001:00013760       ??_C@_0DF@JINGIDAA@?6?5?9?9?5HeaderLen?$DN?$CFd?0?5L2PAD?$DN?$CFd?0?5Key@ 10014760     rtmp_ckipmic.obj
 0001:00013798       ??_C@_0EJ@IJMAIDDJ@U2M?5Can?8t?5process?5Ckip?5key?0?5Pair@ 10014798     rtmp_ckipmic.obj
 0001:000137e4       ??_C@_0BG@JMFDLJBE@keylen?5can?8t?5be?5zero?6?$AA@ 100147e4     rtmp_ckipmic.obj
 0001:00013a00       ??_C@_0DK@EDKBGDLP@Chk2?3?3?5btWifiThr?5?$DN?5?$CFd?0?5TxByteCou@ 10014a00     rtmp_cobt.obj
 0001:00013a3c       ??_C@_0DL@FAGMDPPJ@TxRxThroughputPerSeconds?5?$DN?5?$CFd?5Bp@ 10014a3c     rtmp_cobt.obj
 0001:00013a78       ??_C@_0CG@BPLKCIHN@ALL?5BT?5Profile?5Disconnected?5?4?4?5B@ 10014a78     rtmp_cobt.obj
 0001:00013aa0       ??_C@_0CM@JEAJCLGL@1?01?010000?01?01?5?$DN?$DN?$DO?5General?5Profil@ 10014aa0     rtmp_cobt.obj
 0001:00013ad0       ??_C@_0FD@KNPAAOAD@2000?0?52000?0?512000?0?52000?0?52000?5?$DN?$DN@ 10014ad0     rtmp_cobt.obj
 0001:00013b28       ??_C@_0FK@IJHBKPCF@5000?0?55000?0?512000?0?55000?0?55000?5?$DN?$DN@ 10014b28     rtmp_cobt.obj
 0001:00013b88       ??_C@_0EB@HNAHLEOH@10000?0?510000?0?520000?0?510000?0?51000@ 10014b88     rtmp_cobt.obj
 0001:00013bcc       ??_C@_0DO@NODGOMEN@200000?0?5200000?0?5200000?0?5200000?0?5@ 10014bcc     rtmp_cobt.obj
 0001:00013c10       ??_C@_0FN@IDDNILOI@200000?0?5200000?0?5200000?0?5200000?0?5@ 10014c10     rtmp_cobt.obj
 0001:00013c70       ??_C@_0CA@JAGIFMFG@?5?9?9?9?$DO?5Check?5Busy?5?$CFd?5?$CFd?5?$CFd?5?$CFd?5?$CFd?$AA@ 10014c70     rtmp_cobt.obj
 0001:00013c90       ??_C@_0CA@EMEGCFHA@?$DM?$DM?5Chk?3?3?5BT?5Initialize?5hardware?$AA@ 10014c90     rtmp_cobt.obj
 0001:00013cb0       ??_C@_0BP@CHOMMFKF@?$DO?$DO?5Chk?3?3BT?5Initialize?5hardware?$AA@ 10014cb0     rtmp_cobt.obj
 0001:00013cd0       ??_C@_0GN@MAHHMBFH@?$DO?$DOChk?3?3?5bBTSoftwareOn?5?$DN?5?$CFd?0?5bBTH@ 10014cd0     rtmp_cobt.obj
 0001:00013d40       ??_C@_0BL@OLPJENCK@?$DO?$DOChk?3?3?5nicConfig3?5?$DN0x?$CF04x?$AA@ 10014d40     rtmp_cobt.obj
 0001:00013d5c       ??_C@_0CK@IKMBFGLF@?$DO?$DOChk?3?3?5bBTCoexistence?5ON?0?5that?5@ 10014d5c     rtmp_cobt.obj
 0001:00013d88       ??_C@_0EI@PAIGLDDN@?$DO?$DOChk?3?3?5bBTSoftwareOn?5?$DN?5?$CFd?0?5bBTH@ 10014d88     rtmp_cobt.obj
 0001:00013dd0       ??_C@_0BL@EDLCGBE@?$DO?$DOChk?3?3?5nicConfig2?5?$DN0x?$CF04x?$AA@ 10014dd0     rtmp_cobt.obj
 0001:00013dec       ??_C@_0CB@IHAKAIJM@?$DO?$DOChk?3?3?5In?5InitBTCoexistence?5?4?4?4@ 10014dec     rtmp_cobt.obj
 0001:00013e10       ??_C@_0CH@CLPFCKNI@Chk9?3?3?5?4?4?4?4?4?4?4?4?4?4?4?4?4?5?9?9?5HT40?5?9?9?$DO@ 10014e10     rtmp_cobt.obj
 0001:00013e38       ??_C@_0CH@ICLNCBFF@Chk9?3?3?5?4?4?4?4?4?4?4?4?4?4?4?4?4?5?$CL?$CL?5HT40?5?9?9?$DO@ 10014e38     rtmp_cobt.obj
 0001:00013e60       ??_C@_0CL@PAHDOBGL@Chk9?3?3?5?4?4?4?4?4?4?4?4?4?4?4?4?4?5?9?9?5Delete?5B@ 10014e60     rtmp_cobt.obj
 0001:00013e8c       ??_C@_0CL@HELPLOCN@Chk9?3?3?5?4?4?4?4?4?4?4?4?4?4?4?4?4?5?$CL?$CL?5Delete?5B@ 10014e8c     rtmp_cobt.obj
 0001:00013eb8       ??_C@_0CL@IKIMHCCN@Chk9?3?3?5?4?4?4?4?4?4?4?4?4?4?4?4?4?5?9?9?5Lower?5MC@ 10014eb8     rtmp_cobt.obj
 0001:00013ee4       ??_C@_0CL@OEACNGL@Chk9?3?3?5?4?4?4?4?4?4?4?4?4?4?4?4?4?5?$CL?$CL?5Lower?5MC@ 10014ee4     rtmp_cobt.obj
 0001:00013f10       ??_C@_0DC@GDADFGBI@Chk9?3?3?5?4?4?4?4?4?4?4?4?4?4?4?4?4?5?9?9?5Lower?5BA@ 10014f10     rtmp_cobt.obj
 0001:00013f44       ??_C@_0DC@PHNOIIMP@Chk9?3?3?5?4?4?4?4?4?4?4?4?4?4?4?4?4?5?$CL?$CL?5Lower?5BA@ 10014f44     rtmp_cobt.obj
 0001:00013f78       ??_C@_0CP@INENMMDN@Chk9?3?3?5?4?4?4?4?4?4?4?4?4?4?4?4?4?5?9?9?5Lower?5BA@ 10014f78     rtmp_cobt.obj
 0001:00013fa8       ??_C@_0CP@NJEIHNCK@Chk9?3?3?5?4?4?4?4?4?4?4?4?4?4?4?4?4?5?$CL?$CL?5Lower?5BA@ 10014fa8     rtmp_cobt.obj
 0001:00013fd8       ??_C@_0DI@CGCEJDGA@Chk9?3?3?5?4?4?4?4?4?4?4?4?4?4?4?4?4?5?9?9?5Lower?5Tx@ 10014fd8     rtmp_cobt.obj
 0001:00014010       ??_C@_0DI@DBPOAPKH@Chk9?3?3?5?4?4?4?4?4?4?4?4?4?4?4?4?4?5?$CL?$CL?5Lower?5Tx@ 10015010     rtmp_cobt.obj
 0001:00014048       ??_C@_0DP@ODGCBKNJ@Chk9?3?3?5?4?4?4?4?4?4?4?4?4?4?4?4?4?5?9?9?5Lower?5LN@ 10015048     rtmp_cobt.obj
 0001:00014088       ??_C@_0CP@GEMCBAJM@Chk9?3?3?5?4?4?4?4?4?4?4?4?4?4?4?4?4?5Set?5R65?5to?5@ 10015088     rtmp_cobt.obj
 0001:000140b8       ??_C@_0CP@HPGPOIHF@Chk9?3?3?5?4?4?4?4?4?4?4?4?4?4?4?4?4?5Set?5R65?5to?5@ 100150b8     rtmp_cobt.obj
 0001:000140e8       ??_C@_0BP@FAJMNDNL@Chk9?3?3?5?4?4?4?4?4?4?4?4?4?4?4?4?4?5RSSI?5?$DN?5?$CFd?$AA@ 100150e8     rtmp_cobt.obj
 0001:00014108       ??_C@_0DP@IOPHGFDK@Chk9?3?3?5?4?4?4?4?4?4?4?4?4?4?4?4?4?5?$CL?$CL?5Lower?5LN@ 10015108     rtmp_cobt.obj
 0001:00014148       ??_C@_0BK@OKENLHCL@Chk?3?3?5Hardware?5key?5ON?$CB?$CB?$CB?$CB?$AA@ 10015148     rtmp_cobt.obj
 0001:00014168       ??_C@_0EP@OBDPAPFA@Chk?3?3?5ulBTActiveCountPastPeriod?5@ 10015168     rtmp_cobt.obj
 0001:000141b8       ??_C@_0BL@GNHNAJB@Chk?3?3?5Hardware?5key?5OFF?$CB?$CB?$CB?$CB?$AA@ 100151b8     rtmp_cobt.obj
 0001:000141d8       ??_C@_0GK@LPFKNOPE@Chk?3?3?5Method?$DN?$CFd?$CI0?$DN?$DO2?9wire?$CJ?0?5BW?$DN?$CF@ 100151d8     rtmp_cobt.obj
 0001:00014244       ??_C@_0BA@KBJCACOJ@?$DM?9?9?9?5WATCH?5TIME?$AA@ 10015244     rtmp_cobt.obj
 0001:00014254       ??_C@_0CI@BPJBAKBG@?$DO?$DO?$DO?$DO?$DO?5data?5?$DN?50x?$CF08x?0?5data_switch@ 10015254     rtmp_cobt.obj
 0001:0001427c       ??_C@_0DC@OENLBPFP@Chk9?3?3error?5RESET?0?5HALT?0?5RADIO_O@ 1001527c     rtmp_cobt.obj
 0001:000144cc       ??_C@_0DC@NJHIONIH@OID_802_11_QUERY_MANUAL_CH_LIST?5@ 100154cc     rtmp_info.obj
 0001:00014500       ??_C@_0CP@FGIEIHND@Query?3?3RT_OID_802_11_WAPI_QUERY_@ 10015500     rtmp_info.obj
 0001:00014530       ??_C@_0DK@BMOKGOBP@Query?3?3RT_OID_802_11_WAPI_QUERY_@ 10015530     rtmp_info.obj
 0001:0001456c       ??_C@_0DG@EOHJNCAK@Query?3?3RT_OID_802_11_QUERY_INITI@ 1001556c     rtmp_info.obj
 0001:000145a4       ??_C@_0DF@MMOMLCEG@Query?3?3RT_OID_802_11_QUERY_PRIVA@ 100155a4     rtmp_info.obj
 0001:000145dc       ??_C@_0CP@IEDFHOIN@Query?3?3RT_OID_802_11_QUERY_LAST_@ 100155dc     rtmp_info.obj
 0001:0001460c       ??_C@_0CP@KGMPKKHP@Query?3?3RT_OID_802_11_QUERY_LAST_@ 1001560c     rtmp_info.obj
 0001:00014640       ??_C@_0FE@LIHIFOJK@Query?3?3RT_OID_802_11_QUERY_HT_PH@ 10015640     rtmp_info.obj
 0001:00014698       ??_C@_0EP@IPIBAPCJ@Query?3?3RT_OID_802_11_QUERY_BATAB@ 10015698     rtmp_info.obj
 0001:000146e8       ??_C@_0EK@KHNAMJKM@Query?3?3RT_OID_802_11_QUERY_BATAB@ 100156e8     rtmp_info.obj
 0001:00014738       ??_C@_0EL@EFFEKPIE@Query?3?3RT_OID_802_11_QUERY_BATAB@ 10015738     rtmp_info.obj
 0001:00014788       ??_C@_0EG@HJMNIDIC@Query?3?3RT_OID_802_11_QUERY_BATAB@ 10015788     rtmp_info.obj
 0001:000147d0       ??_C@_0EK@CECBIEIK@Query?3?3RT_OID_802_11_QUERY_BATAB@ 100157d0     rtmp_info.obj
 0001:00014820       ??_C@_0EG@MNIFFOGC@Query?3?3RT_OID_802_11_QUERY_BATAB@ 10015820     rtmp_info.obj
 0001:00014868       ??_C@_0EC@GBBHCIK@?5?$CITxBAWinLimit?$DN?$CFd?$CJ?5?$CIRxBAWinLimit@ 10015868     rtmp_info.obj
 0001:000148ac       ??_C@_0DE@JPIHBBPM@Query?3?3RT_OID_802_11_QUERY_IMME_@ 100158ac     rtmp_info.obj
 0001:000148e0       ??_C@_0CH@JMPFCNON@Query?3?3RT_OID_802_11_QUERY_MAC_T@ 100158e0     rtmp_info.obj
 0001:00014908       ??_C@_0CN@FLMOEDHE@Query?3?3RT_OID_802_11_QUERY_MAC_T@ 10015908     rtmp_info.obj
 0001:00014938       ??_C@_0DD@CAABHMGK@Query?3?3RT_OID_802_11_QUERY_FIRMW@ 10015938     rtmp_info.obj
 0001:00014970       ??_C@_0EF@GHHECJJM@Query?3?3RT_OID_802_11_QUERY_HARDW@ 10015970     rtmp_info.obj
 0001:000149b8       ??_C@_0CP@NIMCLFDE@Query?3?3RT_OID_802_11_QUERY_MULTI@ 100159b8     rtmp_info.obj
 0001:000149e8       ??_C@_0CG@MADDCMLA@Query?3?3RT_OID_802_11_QUERY_WMM?5?$CI@ 100159e8     rtmp_info.obj
 0001:00014a10       ??_C@_0CO@OMCLKKIN@Query?3?3RT_OID_802_11_QUERY_AGGRE@ 10015a10     rtmp_info.obj
 0001:00014a40       ??_C@_0CN@EKNPFEBE@Query?3?3RT_OID_802_11_QUERY_IEEE8@ 10015a40     rtmp_info.obj
 0001:00014a70       ??_C@_0CK@CNDKPKCI@Query?3?3RT_OID_802_11_QUERY_PREAM@ 10015a70     rtmp_info.obj
 0001:00014a9c       ??_C@_0DD@HPHAPBAG@Query?3?3RT_OID_802_11_QUERY_TX_PO@ 10015a9c     rtmp_info.obj
 0001:00014ad0       ??_C@_0DF@NJJHAHOJ@Query?3?3RT_OID_802_11_QUERY_CURRE@ 10015ad0     rtmp_info.obj
 0001:00014b08       ??_C@_0CL@JJPLDIB@Query?3?3RT_OID_802_11_QUERY_PHY_M@ 10015b08     rtmp_info.obj
 0001:00014b38       ??_C@_0IH@JAFPDEHA@Query?3RT_OID_802_11_QUERY_COUNTR@ 10015b38     rtmp_info.obj
 0001:00014bc0       ??_C@_0CJ@MFEJFBDC@Query?3?3RT_OID_802_11_QUERY_LINK_@ 10015bc0     rtmp_info.obj
 0001:00014bec       ??_C@_0CM@KHLEIBOI@Query?3?3OID_802_11_TX_ANTENNA_SEL@ 10015bec     rtmp_info.obj
 0001:00014c18       ??_C@_0CL@OPCGEINM@Query?3?3OID_802_11_NUMBER_OF_ANTE@ 10015c18     rtmp_info.obj
 0001:00014c44       ??_C@_0CL@OAKNOPEF@Query?3?3OID_802_11_NETWORK_TYPES_@ 10015c44     rtmp_info.obj
 0001:00014c70       ??_C@_0CC@EDANKDNG@Query?3?3OID_802_11_STATISTICS?5?5?$CFx@ 10015c70     rtmp_info.obj
 0001:00014c94       ??_C@_0CH@FMGGFNCO@Query?3?3OID_802_11_TX_POWER_LEVEL@ 10015c94     rtmp_info.obj
 0001:00014cbc       ??_C@_0DA@NLFPODLE@Query?3?3OID_802_11_FRAGMENTATION_@ 10015cbc     rtmp_info.obj
 0001:00014cec       ??_C@_0CG@CDOKGMJL@Query?3?3OID_802_11_RTS_THRESHOLD?$CI@ 10015cec     rtmp_info.obj
 0001:00014d14       ??_C@_0CM@JIDKLGLC@Query?3?3OID_802_11_NETWORK_TYPE_I@ 10015d14     rtmp_info.obj
 0001:00014d40       ??_C@_0EH@DKNOICMH@Query?3?3OID_802_11_CONFIGURATION?$CI@ 10015d40     rtmp_info.obj
 0001:00014d88       ??_C@_0DL@BMOALMIA@Query?3?3OID_802_11_DESIRED_RATES?5@ 10015d88     rtmp_info.obj
 0001:00014dc4       ??_C@_0CD@NMFMFMPG@?$CFd?0?5?$CFd?0?5?$CFd?0?5?$CFd?0?5?$CFd?0?5?$CFd?0?5?$CFd?0?5?$CFd?4?4@ 10015dc4     rtmp_info.obj
 0001:00014de8       ??_C@_0CL@NIOACOAF@Query?3?3OID_802_11_SUPPORTED_RATE@ 10015de8     rtmp_info.obj
 0001:00014e14       ??_C@_0CM@OOENDMPG@Query?3?3OID_802_11_AUTHENTICATION@ 10015e14     rtmp_info.obj
 0001:00014e40       ??_C@_0CH@OBIPKPML@Query?3?3OID_802_11_PRIVACY_FILTER@ 10015e40     rtmp_info.obj
 0001:00014e68       ??_C@_0CD@JIHCFKKH@Query?3?3OID_802_11_WEP_STATUS?$CI?$DN?$CFd@ 10015e68     rtmp_info.obj
 0001:00014e8c       ??_C@_0BH@DFBEKOCK@RT_OID_VENDOR_FLIP_IQ?6?$AA@ 10015e8c     rtmp_info.obj
 0001:00014ea4       ??_C@_0CD@KOPMNEJE@RT_OID_USB_VENDOR_SWITCH_FUNCTIO@ 10015ea4     rtmp_info.obj
 0001:00014ec8       ??_C@_0BK@KDFIGBIJ@RT_OID_USB_VENDOR_UNPLUG?6?$AA@ 10015ec8     rtmp_info.obj
 0001:00014ee4       ??_C@_0BJ@NFGJLEBE@RT_OID_USB_VENDOR_RESET?6?$AA@ 10015ee4     rtmp_info.obj
 0001:00014f00       ??_C@_0CJ@OBNEAIFP@Set?3?3RT_OID_802_11_RESET_COUNTER@ 10015f00     rtmp_info.obj
 0001:00014f2c       ??_C@_0BI@FPJIPKEB@RT_OID_VENDOR_WRITE_RF?6?$AA@ 10015f2c     rtmp_info.obj
 0001:00014f44       ??_C@_0BI@LHKEGDFF@RT_OID_VENDOR_READ_BBP?6?$AA@ 10015f44     rtmp_info.obj
 0001:00014f5c       ??_C@_0BJ@HFMCKKMF@RT_OID_VENDOR_WRITE_BBP?6?$AA@ 10015f5c     rtmp_info.obj
 0001:00014f78       ??_C@_0DB@BFJLDGBK@Query?3?3RT_OID_802_11_QUERY_EEPRO@ 10015f78     rtmp_info.obj
 0001:00014fac       ??_C@_0BM@IMCMMFGP@RT_OID_USB_GET_DEVICE_DESC?6?$AA@ 10015fac     rtmp_info.obj
 0001:00014fc8       ??_C@_0CB@LIIMLHED@RT_OID_USB_VENDOR_EXIT_TESTMODE?6@ 10015fc8     rtmp_info.obj
 0001:00014fec       ??_C@_0BP@ICFJPPBE@RT_OID_USB_VENDOR_EEPROM_READ?6?$AA@ 10015fec     rtmp_info.obj
 0001:0001500c       ??_C@_0CA@LHPDKOCP@RT_OID_USB_VENDOR_EEPROM_WRITE?6?$AA@ 1001600c     rtmp_info.obj
 0001:0001502c       ??_C@_0CC@DDIKILAH@offset?5?$DN?50x?$CF04x?0?5length?5?$DN?50x?$CF04x@ 1001602c     rtmp_info.obj
 0001:00015050       ??_C@_0BI@EDHIIANO@RT_OID_MULTI_WRITE_MAC?6?$AA@ 10016050     rtmp_info.obj
 0001:00015068       ??_C@_0BM@MJFAGCN@RT_OID_VENDOR_GET_COUNTERS?6?$AA@ 10016068     rtmp_info.obj
 0001:00015084       ??_C@_0DB@GGGKDHOH@Query?3?3OID_802_3_XMIT_MORE_COLLI@ 10016084     rtmp_info.obj
 0001:000150b8       ??_C@_0CP@NDLBBAAK@Query?3?3OID_802_3_XMIT_ONE_COLLIS@ 100160b8     rtmp_info.obj
 0001:000150e8       ??_C@_0DA@ECMCLLK@Query?3?3OID_802_3_RCV_ERROR_ALIGN@ 100160e8     rtmp_info.obj
 0001:00015118       ??_C@_0CI@OANAMALP@Query?3?3OID_GEN_RCV_NO_BUFFER?5COU@ 10016118     rtmp_info.obj
 0001:00015140       ??_C@_0CE@GBJOOJHE@Query?3?3OID_GEN_RCV_ERROR?5COUNTER@ 10016140     rtmp_info.obj
 0001:00015164       ??_C@_0CF@GPADPILI@Query?3?3OID_GEN_XMIT_ERROR?5COUNTE@ 10016164     rtmp_info.obj
 0001:0001518c       ??_C@_0CB@EPMEBIOM@Query?3?3OID_GEN_RCV_OK?5COUNTERS?5?6@ 1001618c     rtmp_info.obj
 0001:000151b0       ??_C@_0CC@CGPDHM@Query?3?3OID_GEN_XMIT_OK?5COUNTERS?5@ 100161b0     rtmp_info.obj
 0001:000151d4       ??_C@_0CC@PKKLEHMG@Query?3?3OID_802_3_MULTICAST_LIST?5@ 100161d4     rtmp_info.obj
 0001:000151f8       ??_C@_0BP@IGHBJLLG@Query?3?3OID_802_3_MAC_OPTIONS?5?6?$AA@ 100161f8     rtmp_info.obj
 0001:00015218       ??_C@_0CF@JPMDLHOL@Query?3?3OID_802_3_MAXIMUM_LIST_SI@ 10016218     rtmp_info.obj
 0001:00015240       ??_C@_0CD@PEMJGHCN@Query?3?3OID_802_3_CURRENT_ADDRESS@ 10016240     rtmp_info.obj
 0001:00015264       ??_C@_0CF@GNAHHEHP@Query?3?3OID_802_3_PERMANENT_ADDRE@ 10016264     rtmp_info.obj
 0001:0001528c       ??_C@_0BP@NLHLHGCE@Query?3?3OID_PNP_CAPABILITIES?5?$AN?6?$AA@ 1001628c     rtmp_info.obj
 0001:000152ac       ??_C@_0CC@EOOOBOBL@Query?3?3OID_PNP_QUERY_POWER?5?$CI?$DN?$CFd?$CJ@ 100162ac     rtmp_info.obj
 0001:000152d0       ??_C@_0CB@MJGNDIAP@Query?3?3OID_GEN_PHYSICAL_MEDIUM?5?6@ 100162d0     rtmp_info.obj
 0001:000152f4       ??_C@_0CB@KHBFDFFE@Query?3?3OID_GEN_SUPPORTED_GUIDS?5?6@ 100162f4     rtmp_info.obj
 0001:00015318       ??_C@_0CG@IAABCDAP@Query?3?3OID_GEN_MAXIMUM_SEND_PACK@ 10016318     rtmp_info.obj
 0001:00015340       ??_C@_0CG@OGPNBFIA@Query?3?3OID_GEN_MEDIA_CONNECT_STA@ 10016340     rtmp_info.obj
 0001:00015368       ??_C@_0BN@EGEMJNPE@Query?3?3OID_GEN_MAC_OPTIONS?5?6?$AA@ 10016368     rtmp_info.obj
 0001:00015388       ??_C@_0CH@KDNCIEMI@Query?3?3OID_GEN_CURRENT_PACKET_FI@ 10016388     rtmp_info.obj
 0001:000153b0       ??_C@_0CA@PFBDKNOM@Query?3?3OID_GEN_DRIVER_VERSION?5?6?$AA@ 100163b0     rtmp_info.obj
 0001:000153d0       ??_C@_0CH@KOCBBIAE@Query?3?3OID_GEN_VENDOR_DRIVER_VER@ 100163d0     rtmp_info.obj
 0001:000153f8       ??_C@_0CE@JJDNJIPD@Query?3?3OID_GEN_VENDOR_DESCRIPTIO@ 100163f8     rtmp_info.obj
 0001:0001541c       ??_C@_0BL@GCGACEMA@Query?3?3OID_GEN_VENDOR_ID?5?6?$AA@ 1001641c     rtmp_info.obj
 0001:00015438       ??_C@_0CG@KMOOMODH@Query?3?3OID_GEN_RECEIVE_BUFFER_SP@ 10016438     rtmp_info.obj
 0001:00015460       ??_C@_0CH@CPGJOFMN@Query?3?3OID_GEN_TRANSMIT_BUFFER_S@ 10016460     rtmp_info.obj
 0001:00015488       ??_C@_0DJ@LPGMOLHE@Query?3?3OID_GEN_LINK_SPEED?5hog?5th@ 10016488     rtmp_info.obj
 0001:000154c8       ??_C@_1FM@MJABFFJL@?$AAC?$AA?3?$AA?2?$AAW?$AAi?$AAn?$AAC?$AAE?$AA6?$AA?4?$AA0?$AA?2?$AAN?$AAe?$AAw?$AA?2?$AAR?$AAT?$AA2?$AA8?$AA7?$AA0?$AA_?$AAv?$AA1?$AA?4?$AA4?$AA?4?$AA9?$AA?4?$AA0?$AA?2@ 100164c8     rtmp_info.obj
 0001:00015524       ??_C@_0BM@EGKOOEEB@Query?3?3OID_GEN_LINK_SPEED?5?6?$AA@ 10016524     rtmp_info.obj
 0001:00015540       ??_C@_0CA@LMLLKGG@Query?3?3OID_GEN_XXX_BLOCK_SIZE?5?6?$AA@ 10016540     rtmp_info.obj
 0001:00015560       ??_C@_0CE@HOFCFHAM@Query?3?3OID_GEN_MAXIMUM_FRAME_SIZ@ 10016560     rtmp_info.obj
 0001:00015584       ??_C@_0BP@HMEMEIFG@Query?3?3OID_GEN_XXX_LOOKAHEAD?5?6?$AA@ 10016584     rtmp_info.obj
 0001:000155a4       ??_C@_0BL@NHJAAPPD@Query?3?3OID_GEN_MEDIA_XXX?5?6?$AA@ 100165a4     rtmp_info.obj
 0001:000155c0       ??_C@_0CB@FAIKJOBI@Query?3?3OID_GEN_HARDWARE_STATUS?5?6@ 100165c0     rtmp_info.obj
 0001:000155e8       ??_C@_0ED@CAHJAKAD@SET?3?3RT_OID_802_11_WSC_SET_HW_PB@ 100165e8     rtmp_info.obj
 0001:00015630       ??_C@_0EK@MILKAEPC@WPS?5LED?5Mode?510?3?3Parameter?5of?5LE@ 10016630     rtmp_info.obj
 0001:00015680       ??_C@_0EG@PGCFCHKC@Set?3?3RT_OID_802_11_WPS_SET_CONNE@ 10016680     rtmp_info.obj
 0001:000156c8       ??_C@_0EB@HBFKEDDH@Set?3?3RT_OID_802_11_WPS_SET_CONNE@ 100166c8     rtmp_info.obj
 0001:0001570c       ??_C@_0CC@NODMAAGL@Set?3?3RT_OID_802_11_TEAR_IMME_BA?7@ 1001670c     rtmp_info.obj
 0001:00015730       ??_C@_0BM@CFEBIPAC@?5Set?5?3?3?5Nnot?5found?5pEntry?5?6?$AA@ 10016730     rtmp_info.obj
 0001:0001574c       ??_C@_0CO@IKMJPINH@?5Set?5?3?3?5RT_OID_802_11_TEAR_IMME_@ 1001674c     rtmp_info.obj
 0001:00015780       ??_C@_0GA@DHPAEOHO@?5Set?5?3?3?5RT_OID_802_11_TEAR_IMME_@ 10016780     rtmp_info.obj
 0001:000157e0       ??_C@_0FF@HPOHMHHM@Set?3?3RT_OID_802_11_ADD_IMME_BA?4?5@ 100167e0     rtmp_info.obj
 0001:00015838       ??_C@_0BA@GKEMMLMM@?5BA?4nMSDU?5?3?5?$CFd?6?$AA@ 10016838     rtmp_info.obj
 0001:00015848       ??_C@_0DO@PPKBMFID@RT_OID_802_11_ADD_IMME_BA?4?5break@ 10016848     rtmp_info.obj
 0001:00015888       ??_C@_0DH@OKCCHJAH@?5Set?5?3?3?5IsRecipient?5?$DN?5?$CFd?0?5BA?4nMS@ 10016888     rtmp_info.obj
 0001:000158c0       ??_C@_0EP@GAGIEIPN@?5Set?5?3?3?5RT_OID_802_11_ADD_IMME_B@ 100168c0     rtmp_info.obj
 0001:00015910       ??_C@_0CE@FFLBIIOB@Set?3?3RT_OID_802_11_ADD_IMME_BA_C@ 10016910     rtmp_info.obj
 0001:00015934       ??_C@_0BM@CAMLIFPB@Set?3?3Switch?5?$CIA?9MSDU?5?$DN?5?$CFd?$CJ?$CJ?6?$AA@ 10016934     rtmp_info.obj
 0001:00015950       ??_C@_0BH@LMNKIOMK@?$CIEntry?$FL?$CFd?$FN?4?5Flag?5?$CFx?$CJ?$CJ?6?$AA@ 10016950     rtmp_info.obj
 0001:00015968       ??_C@_0BM@MDBKKAFB@Set?3?3Switch?5?$CIMimoPs?5?$DN?5?$CFd?$CJ?$CJ?6?$AA@ 10016968     rtmp_info.obj
 0001:00015988       ??_C@_0EF@CHDNLMLI@Set?3?3?$CIMimoPs?5?$DN?5?$CFd?$CJ?$CIAmsduEnable?5?$DN@ 10016988     rtmp_info.obj
 0001:000159d0       ??_C@_0FE@HEOAGEGA@Set?3?3?$CIOrde?4AutoBA?5?$DN?5?$CFd?$CJ?5?$CIPolicy?$DN@ 100169d0     rtmp_info.obj
 0001:00015a24       ??_C@_0DD@ELMKCMHL@Set?3?3RT_OID_802_11_ADD_IMME_BA_C@ 10016a24     rtmp_info.obj
 0001:00015a58       ??_C@_0CD@LNJDNOOH@Set?3?3RT_OID_802_11_SET_WMM?5?$CI?$DN?$CFd?$CJ@ 10016a58     rtmp_info.obj
 0001:00015a7c       ??_C@_0BO@EHBACENO@InformationBufferLength?5?$DN?5?$CFd?6?$AA@ 10016a7c     rtmp_info.obj
 0001:00015aa0       ??_C@_0EB@GFIJMLDI@Set?3?3RT_OID_802_11_SET_HARDWARE_@ 10016aa0     rtmp_info.obj
 0001:00015ae4       ??_C@_0CB@COKKJBEK@Set?3?3RT_OID_802_11_SET_PREAMBLE?6@ 10016ae4     rtmp_info.obj
 0001:00015b08       ??_C@_0DG@HDAJJGEE@Set?3?3RT_OID_802_11_SET_COUNTRY_R@ 10016b08     rtmp_info.obj
 0001:00015b40       ??_C@_0DO@KNNKBJFD@Set?3?3RT_OID_802_11_SET_COUNTRY_R@ 10016b40     rtmp_info.obj
 0001:00015b80       ??_C@_0CH@FIJBBKNH@Set?3?3OID_802_11_TX_POWER_LEVEL?5?$CI@ 10016b80     rtmp_info.obj
 0001:00015ba8       ??_C@_0DA@OHCGBPIP@Set?3?3OID_802_11_FRAGMENTATION_TH@ 10016ba8     rtmp_info.obj
 0001:00015bd8       ??_C@_0CF@PPEHBBHG@Set?3?3OID_802_11_RTS_THRESHOLD?5?$CI?$DN@ 10016bd8     rtmp_info.obj
 0001:00015c00       ??_C@_0DF@IIKEPBOJ@Not?5support?5NdisDeviceStateD1?5or@ 10016c00     rtmp_info.obj
 0001:00015c38       ??_C@_0CL@KGGEDADG@NICInitializeAsic?5failed?0?5Status@ 10016c38     rtmp_info.obj
 0001:00015c64       ??_C@_0CJ@CDNEOMCG@NICLoadFirmware?5failed?0?5Status?$FL?$DN@ 10016c64     rtmp_info.obj
 0001:00015c90       ??_C@_0CA@LENPKACJ@Set?3?3OID_PNP_SET_POWER?0?5?$CFd?5?$CB?$CB?$CB?6?$AA@ 10016c90     rtmp_info.obj
 0001:00015cb0       ??_C@_0CA@OLCOHIMB@Set?3?3OID_GEN_PROTOCOL_OPTIONS?5?6?$AA@ 10016cb0     rtmp_info.obj
 0001:00015cd0       ??_C@_0GA@BIFMIPH@Set?3?3OID_GEN_CURRENT_PACKET_FILT@ 10016cd0     rtmp_info.obj
 0001:00015d30       ??_C@_0CB@HIJBKCIP@Set?3?3OID_GEN_CURRENT_LOOKAHEAD?5?6@ 10016d30     rtmp_info.obj
 0001:00015d54       ??_C@_0CD@MPEGFFOA@?$CFd?$CJ?5?$CF02x?3?$CF02x?3?$CF02x?3?$CF02x?3?$CF02x?3?$CF02@ 10016d54     rtmp_info.obj
 0001:00015d78       ??_C@_0CA@OFBOEBLA@Set?3?3OID_802_3_MULTICAST_LIST?5?6?$AA@ 10016d78     rtmp_info.obj
 0001:00015d98       ??_C@_0BH@CNLJEJGO@Query?3?3Size?5too?5short?6?$AA@ 10016d98     rtmp_info.obj
 0001:00015db0       ??_C@_0FA@BKKICDBF@Query?3?3?5RT_OID_802_11_QUERY_CCX2@ 10016db0     rtmp_info.obj
 0001:00015e00       ??_C@_0DG@CDEOOLAF@Query?3?3?5RT_OID_QUERY_CCX_RX_AIRO@ 10016e00     rtmp_info.obj
 0001:00015e38       ??_C@_0CP@LBOPAOJL@QUERY?3?3?5RT_OID_QUERY_WMM_ACM_CMD@ 10016e38     rtmp_info.obj
 0001:00015e68       ??_C@_0CE@FGILOKFG@Query?3?3RT_OID_GET_USB_VERSION?$CI?$DN?$CF@ 10016e68     rtmp_info.obj
 0001:00015e8c       ??_C@_0DH@BJOEHNBJ@Query?3?3RT_OID_802_11_QUERY_RAUI_@ 10016e8c     rtmp_info.obj
 0001:00015ec4       ??_C@_0DF@HFDALMPD@Query?3?3RT_OID_802_11_QUERY_EVENT@ 10016ec4     rtmp_info.obj
 0001:00015efc       ??_C@_0DB@EIIHENGI@Query?3?3RT_OID_802_11_QUERY_EVENT@ 10016efc     rtmp_info.obj
 0001:00015f30       ??_C@_0CP@CLPPDKLK@Query?3?3RT_OID_802_11_QUERY_EVENT@ 10016f30     rtmp_info.obj
 0001:00015f60       ??_C@_0DO@CIBIKPOK@Query?3?3RT_OID_802_11_WSC_QUERY_W@ 10016f60     rtmp_info.obj
 0001:00015fa0       ??_C@_0EM@ENBKGAMI@Query?3?3RT_OID_802_11_WSC_QUERY_W@ 10016fa0     rtmp_info.obj
 0001:00015fec       ??_C@_0DM@JPDALEKP@Query?3?3RT_OID_802_11_QUERY_PREFE@ 10016fec     rtmp_info.obj
 0001:00016028       ??_C@_0IE@MGMCBKIL@Query?3?3RT_OID_802_11_QUERY_PREFE@ 10017028     rtmp_info.obj
 0001:000160ac       ??_C@_0CN@EFPHBFAD@Query?3?3RT_OID_802_11_WSC_QUERY_H@ 100170ac     rtmp_info.obj
 0001:000160dc       ??_C@_0CI@MJCGONLC@Query?3?3RT_OID_802_11_WSC_QUERY_P@ 100170dc     rtmp_info.obj
 0001:00016104       ??_C@_0DB@HDPHGGPG@Query?3?3RT_OID_802_11_WSC_QUERY_S@ 10017104     rtmp_info.obj
 0001:00016138       ??_C@_0CG@DJDAKMEC@Query?3?3RT_OID_802_11_QUERY_DLS_P@ 10017138     rtmp_info.obj
 0001:00016160       ??_C@_0CF@OGBKOHG@Query?3?3RT_OID_802_11_QUERY_DLS?$CI?$DN@ 10017160     rtmp_info.obj
 0001:00016188       ??_C@_0CL@OIEFPHED@Query?3?3RT_OID_802_11_QUERY_APSD_@ 10017188     rtmp_info.obj
 0001:000161b8       ??_C@_0GM@OCPIODKD@Query?3?3RT_OID_802_11_QUERY_APSD_@ 100171b8     rtmp_info.obj
 0001:00016228       ??_C@_0EI@HDBPKLE@Query?3?3RT_OID_802_11_QUERY_AIRON@ 10017228     rtmp_info.obj
 0001:00016270       ??_C@_0CG@DKGPFJKC@Query?3?3OID_MH_802_1X_SUPPORTED?5?$CI@ 10017270     rtmp_info.obj
 0001:00016298       ??_C@_0BJ@LHPMNLI@Query?3?3OID_802_11_PMKID?6?$AA@ 10017298     rtmp_info.obj
 0001:000162b4       ??_C@_0BI@IPFENO@Query?3?3OID_802_11_TEST?6?$AA@ 100172b4     rtmp_info.obj
 0001:000162cc       ??_C@_0CJ@IOCANGJP@Query?3?3OID_802_11_CAPABILITY?0?5si@ 100172cc     rtmp_info.obj
 0001:000162f8       ??_C@_0DD@FNLPAPEA@Query?3?3OID_802_11_CAPABILITY?5NDI@ 100172f8     rtmp_info.obj
 0001:00016330       ??_C@_0GI@GCMLBFDM@?$CFs?3?5OID_802_11_CAPABILITY?5?$CINDIS_@ 10017330     rtmp_info.obj
 0001:00016398       ??_C@_0BE@ICGJMEHL@STAQueryInformation?$AA@ 10017398     rtmp_info.obj
 0001:000163ac       ??_C@_0CH@CDMOABJI@Query?3?3RT_OID_802_11_EXTRA_INFO?5@ 100173ac     rtmp_info.obj
 0001:000163d4       ??_C@_0CH@LOPFFCBD@Query?3?3RT_OID_802_11_QUERY_STA_C@ 100173d4     rtmp_info.obj
 0001:000163fc       ??_C@_0CO@NGAJJALN@Query?3?3RT_OID_802_11_QUERY_NOISE@ 100173fc     rtmp_info.obj
 0001:0001642c       ??_C@_0CI@NOBHOFHJ@Query?3?3RT_OID_802_11_QUERY_RADIO@ 1001742c     rtmp_info.obj
 0001:00016454       ??_C@_0DP@HCEPDJKE@Query?3?3OID_802_11_ASSOCIATION_IN@ 10017454     rtmp_info.obj
 0001:00016498       ??_C@_0EA@BHHDCCMB@Query?3?3OID_802_11_ASSOCIATION_IN@ 10017498     rtmp_info.obj
 0001:000164d8       ??_C@_0BH@MHCJOOPB@CurrBssidLength?5is?5?$CFd?6?$AA@ 100174d8     rtmp_info.obj
 0001:000164f0       ??_C@_0BN@CNGHOHBO@pBssidList?4NumberItem?5is?5?$CFd?6?$AA@ 100174f0     rtmp_info.obj
 0001:00016510       ??_C@_0EB@KAAEBOIH@Reposit?5Bssid?5List?5Test?5?$DN?$DN?$DO?5Scan@ 10017510     rtmp_info.obj
 0001:00016554       ??_C@_0BF@GOFEJDFA@Not?5Enough?5Space?$CB?$CB?$CB?6?$AA@ 10017554     rtmp_info.obj
 0001:0001656c       ??_C@_0BO@OCAAPFPE@Add?5tmpBss?5Entry?5to?5Scan?5TAB?6?$AA@ 1001756c     rtmp_info.obj
 0001:0001658c       ??_C@_0CJ@PILPEHOO@Default?5time?5expired?5time?5is?5?$CFd?5@ 1001758c     rtmp_info.obj
 0001:000165b8       ??_C@_0DE@KKJNPPGD@?$FL070706?$FN?5Query?3?3OID_802_11_BSSID@ 100175b8     rtmp_info.obj
 0001:000165f0       ??_C@_0FP@IFBKOILL@BSS?$CD?$CFd?5?9?5?$CFs?0?5Rssi?$DN?$CFd?0?5Ch?5?$CFd?$DN?$CFd?5K@ 100175f0     rtmp_info.obj
 0001:00016650       ??_C@_0CI@PDDIHPPG@Query?3?3?5BssTable?5total?5byte?5coun@ 10017650     rtmp_info.obj
 0001:00016678       ??_C@_0CE@KLLGDLJC@?$CK?$CK?$CK?$CK?5BssTable?5too?5large?5?$CI?$CFd?5byte@ 10017678     rtmp_info.obj
 0001:0001669c       ??_C@_0DE@EKHHDMNJ@Prepare?5memory?5for?5Adding?5tmpBss@ 1001769c     rtmp_info.obj
 0001:000166d0       ??_C@_0BK@OHLJJKCI@Total?5Table?5Length?5?$DN?5?$CFd?5?6?$AA@ 100176d0     rtmp_info.obj
 0001:000166ec       ??_C@_0CD@PGALJBNK@Bssid?5?$DM?$DM?$CFs?$DO?$DO?5is?5found?0?5time?5is?5?$CF@ 100176ec     rtmp_info.obj
 0001:00016710       ??_C@_0CF@MFKHAMOE@Bssid?5?$DM?$DM?$CFs?$DO?$DO?5is?5Expired?0?5time?5is@ 10017710     rtmp_info.obj
 0001:00016738       ??_C@_0BD@BFNFJMFO@Channel?5is?5legal?5?6?$AA@ 10017738     rtmp_info.obj
 0001:0001674c       ??_C@_0BC@DGFFMEAI@Channel?5is?5?$DN?5?$CFd?5?6?$AA@ 1001774c     rtmp_info.obj
 0001:00016760       ??_C@_0O@LOOIHOOC@Length?5?$DN?5?$CFd?5?6?$AA@ 10017760     rtmp_info.obj
 0001:00016770       ??_C@_0BN@GKIJJGPB@Bssid?5?$DM?$DM?$CFs?$DO?$DO?5is?5Not?5Expired?6?$AA@ 10017770     rtmp_info.obj
 0001:00016790       ??_C@_0BJ@LKCKLBCE@Scan?5Table?5Length?5?$DN?5?$CFd?5?6?$AA@ 10017790     rtmp_info.obj
 0001:000167ac       ??_C@_0DA@HAHFKKNK@Query?3?3OID_802_11_BSSID_LIST?5?$CI?$CFd@ 100177ac     rtmp_info.obj
 0001:000167e0       ??_C@_0EM@KFHGFKCO@Query?3?3OID_802_11_BSSID_LIST?5?$CI?$CFd@ 100177e0     rtmp_info.obj
 0001:0001682c       ??_C@_0CD@BLOIIOOA@Query?3?3OID_802_11_POWER_MODE?$CI?$DN?$CFd@ 1001782c     rtmp_info.obj
 0001:00016850       ??_C@_0CF@KJBKKMNK@Query?3?3OID_802_11_RSSI_TRIGGER?$CI?$DN@ 10017850     rtmp_info.obj
 0001:00016878       ??_C@_0CC@PLAAFOFM@Query?3?3OID_802_11_RSSI?$CI?$DN?$CFd?5?$DN?$CFd?5?$CJ@ 10017878     rtmp_info.obj
 0001:0001689c       ??_C@_0CK@HHECPPIH@Query?3?3OID_802_11_SSID?5?$CILen?$DN?$CFd?0?5@ 1001789c     rtmp_info.obj
 0001:000168c8       ??_C@_0CB@OAKIBHLA@Query?3?3OID_802_11_BSSID?$CI?$DNEMPTY?$CJ?6@ 100178c8     rtmp_info.obj
 0001:000168f0       ??_C@_0EL@NPHJBLJJ@Query?3?3OID_802_11_BSSID?0?5report?5@ 100178f0     rtmp_info.obj
 0001:0001693c       ??_C@_0CN@BHPMAONC@RT_OID_SET_CCX_SYSLOG_ELEM?0?5Len?$DN@ 1001793c     rtmp_info.obj
 0001:0001696c       ??_C@_0CI@LNMLMADO@Set?3?3RT_OID_SET_CCX_DIAG_ACTION?$CI@ 1001796c     rtmp_info.obj
 0001:00016994       ??_C@_0DI@CAAJGDE@Set?3?3RT_OID_SET_CCX_MFP?$CI?$DN?$CFd?$CJ?5Ign@ 10017994     rtmp_info.obj
 0001:000169cc       ??_C@_0BO@MMLBBHGK@Set?3?3RT_OID_SET_CCX_MFP?$CI?$DN?$CFd?$CJ?6?$AA@ 100179cc     rtmp_info.obj
 0001:000169ec       ??_C@_0CJ@OAGIBMAL@Set?3?3OID_MH_CCX_REMOVE_KRK?5KeyIn@ 100179ec     rtmp_info.obj
 0001:00016a18       ??_C@_0CN@JMGGJDJJ@Length?5?$DN?5?$CFlu?5KeyIndex?5?$DN?$CFlu?5KeyLe@ 10017a18     rtmp_info.obj
 0001:00016a48       ??_C@_0CJ@EBIKNGHC@Set?3?3OID_MH_CCX_ADD_KRK?5Bufferle@ 10017a48     rtmp_info.obj
 0001:00016a74       ??_C@_0CC@BDPEAPGK@Enqueue?5OID_802_11_DISASSOCIATE?5@ 10017a74     rtmp_info.obj
 0001:00016a98       ??_C@_0CP@EMAHHFPJ@RogueApTableSetEntry?0?5pAegis_Rog@ 10017a98     rtmp_info.obj
 0001:00016ac8       ??_C@_0EB@IMGILAPG@MH_CCX_RAP_NEW_CREDENTIALS?3?5Rogu@ 10017ac8     rtmp_info.obj
 0001:00016b0c       ??_C@_0CP@JJMBAOEI@OID_MH_CCX_RAP_STATUS?0?5not?5conne@ 10017b0c     rtmp_info.obj
 0001:00016b3c       ??_C@_0CL@HFIDDFNA@OID_MH_CCX_RAP_STATUS?5version?$CI?$DN?$CF@ 10017b3c     rtmp_info.obj
 0001:00016b68       ??_C@_0EB@DIGKAEIL@Set?3?3OID_MH_CCX_RAP_STATUS?$CIBSSID@ 10017b68     rtmp_info.obj
 0001:00016bac       ??_C@_0DD@DOGDKLMH@Set?3?3OID_MH_CCX_RAP_STATUS?$CIlen?$DN?$CF@ 10017bac     rtmp_info.obj
 0001:00016be0       ??_C@_0CE@PNOBMGON@Set?3?3OID_MH_CCX_8021X_RESULT?$CI?$DN?$CFl@ 10017be0     rtmp_info.obj
 0001:00016c04       ??_C@_0CO@JIMCNDDF@Set?3?3MH_OID_CCX_8021X?$CI?$DN?$CFd?$CJ?5?$CICCXC@ 10017c04     rtmp_info.obj
 0001:00016c34       ??_C@_0BM@MNMFBJHC@Set?3?3MH_OID_CCX_8021X?$CI?$DN?$CFd?$CJ?6?$AA@ 10017c34     rtmp_info.obj
 0001:00016c50       ??_C@_0DB@OKGMLHNL@Set?3?3OID_MH_CCX_MIXED_CELLS?5?$CI?$DN?$CFl@ 10017c50     rtmp_info.obj
 0001:00016c84       ??_C@_0BL@JNFCAPIH@Set?3?3OID_MH_CCX_LEAP?$CI?$DN?$CFd?$CJ?6?$AA@ 10017c84     rtmp_info.obj
 0001:00016ca0       ??_C@_0CL@OPACHLCB@Set?3?3RT_OID_SET_CCX_LEAP?$CI?$CFd?$CJ?0?5co@ 10017ca0     rtmp_info.obj
 0001:00016ccc       ??_C@_0CH@FPEFAKPL@Set?3?3RT_OID_SET_CCX_LOG_FRAME?5?$CIT@ 10017ccc     rtmp_info.obj
 0001:00016cf4       ??_C@_0CP@CDIPIGPK@Set?3?3RT_OID_SET_CCX_TX_AIRONET?5?4@ 10017cf4     rtmp_info.obj
 0001:00016d24       ??_C@_0CH@MKMPGAMC@Set?3?3?5RT_OID_WMM_ACM_CMD?$CIInfoLen@ 10017d24     rtmp_info.obj
 0001:00016d4c       ??_C@_0CN@NBJDNDNG@Set?3?3RT_OID_802_11_WAPI_SET_ADHO@ 10017d4c     rtmp_info.obj
 0001:00016d7c       ??_C@_0M@CKJMNIAA@Wapi_PN?9?$DO?5?6?$AA@ 10017d7c     rtmp_info.obj
 0001:00016d88       ??_C@_0BO@NMAEICHE@RT2870Dump?5STASetInformation?6?$AA@ 10017d88     rtmp_info.obj
 0001:00016da8       ??_C@_0N@NPDFCCCO@pWPI_Key?9?$DO?5?6?$AA@ 10017da8     rtmp_info.obj
 0001:00016db8       ??_C@_0DJ@JEFLLCNC@ktGroupKey?3?5?5lenWPIEK?5?$DN?5?$CFd?0lenWP@ 10017db8     rtmp_info.obj
 0001:00016df4       ??_C@_0CC@FEAPFGDF@?$EA?$EA_?$EA?$EAWPA_802_1X_PORT_NOT_SECURED@ 10017df4     rtmp_info.obj
 0001:00016e18       ??_C@_0CN@PADMKFEG@ktPairwiseKey?3?5?5lenWPIEK?5?$DN?5?$CFd?0le@ 10017e18     rtmp_info.obj
 0001:00016e48       ??_C@_0GC@LLHIMKHF@WAPI?3?5Can?8t?5find?5the?5desired?5BSS@ 10017e48     rtmp_info.obj
 0001:00016eac       ??_C@_0CB@NHBDPOEL@Set?3?3RT_OID_WAPI_802_11_WPI_KEY?6@ 10017eac     rtmp_info.obj
 0001:00016ed0       ??_C@_0DJ@NNIJIGFB@Set?3?3RT_OID_802_11_WAPI_SET_WAPI@ 10017ed0     rtmp_info.obj
 0001:00016f0c       ??_C@_0DH@OGNKDBEH@Set?3?3RT_OID_802_11_WAPI_SET_WAPI@ 10017f0c     rtmp_info.obj
 0001:00016f48       ??_C@_0EI@GBIEDFMP@Set?3?3RT_OID_802_11_WAPI_SET_WAPI@ 10017f48     rtmp_info.obj
 0001:00016f90       ??_C@_0EJ@MKFFINOA@Set?3?3RT_OID_802_11_WAPI_SET_WAPI@ 10017f90     rtmp_info.obj
 0001:00016fdc       ??_C@_0CL@LMEGAKM@Set?3?3RT_OID_802_11_WAPI_SET_SUPP@ 10017fdc     rtmp_info.obj
 0001:00017008       ??_C@_0DE@HIDIEDID@Set?3?3RT_OID_802_11_SET_RAUI_SETC@ 10018008     rtmp_info.obj
 0001:0001703c       ??_C@_0CM@JMHGJPCG@Set?3?3RT_OID_802_11_SET_PSPXLINK_@ 1001803c     rtmp_info.obj
 0001:00017068       ??_C@_0DK@CJOPLOND@Set?3?3RT_OID_802_11_WSC_SET_WPS_S@ 10018068     rtmp_info.obj
 0001:000170a8       ??_C@_0GD@HDIKENHC@Set?3?3RT_OID_802_11_WSC_SET_WPS_S@ 100180a8     rtmp_info.obj
 0001:0001710c       ??_C@_0DG@ODLCEFBC@Set?3?3RT_OID_802_11_SET_PREFERRED@ 1001810c     rtmp_info.obj
 0001:00017148       ??_C@_0FA@KCLHGIC@Set?3?3RT_OID_802_11_SET_PREFERRED@ 10018148     rtmp_info.obj
 0001:00017198       ??_C@_0IA@DDJKDPDM@Set?3?3RT_OID_802_11_SET_PREFERRED@ 10018198     rtmp_info.obj
 0001:00017218       ??_C@_0CL@KKGBKPLN@Set?3?3RT_OID_802_11_WSC_SET_AUTO_@ 10018218     rtmp_info.obj
 0001:00017244       ??_C@_05JIJHCBHC@?$CF02x?9?$AA@ 10018244     rtmp_info.obj
 0001:0001724c       ??_C@_0CB@IILBHDGI@Customized?5Device?5Info?$CIin?5Hex?$CJ?3?6@ 1001824c     rtmp_info.obj
 0001:00017270       ??_C@_0FM@KNLOLCBH@Set?3?3RT_OID_802_11_WSC_SET_CUSTO@ 10018270     rtmp_info.obj
 0001:000172cc       ??_C@_0CE@HNLLEFBL@Set?3?3RT_OID_802_11_WSC_SET_PROFI@ 100182cc     rtmp_info.obj
 0001:000172f0       ??_C@_0CL@OMCGLELP@Set?3?3RT_OID_802_11_WSC_SET_PROBE@ 100182f0     rtmp_info.obj
 0001:0001731c       ??_C@_0CM@BHBCJJEJ@Set?3?3RT_OID_802_11_WSC_SET_ASSOC@ 1001831c     rtmp_info.obj
 0001:00017348       ??_C@_0CO@GJLLMJJH@Set?3?3RT_OID_802_11_WSC_SET_ACTIV@ 10018348     rtmp_info.obj
 0001:00017378       ??_C@_0DB@LHBPEPKM@Set?3?3RT_OID_802_11_WSC_SET_MODE?5@ 10018378     rtmp_info.obj
 0001:000173ac       ??_C@_0CI@PDFGMIBH@Set?3?3RT_OID_802_11_WSC_SET_MODE?5@ 100183ac     rtmp_info.obj
 0001:000173d8       ??_C@_0FL@LDNEFNFM@Set?3?3RT_OID_802_11_WSC_SET_MODE?5@ 100183d8     rtmp_info.obj
 0001:00017434       ??_C@_0DI@EEGHGLGD@Set?3?3RT_OID_802_11_WSC_SET_MODE?5@ 10018434     rtmp_info.obj
 0001:0001746c       ??_C@_0DG@JOKELLCE@?$CFs?5?$CISET?3?3RT_OID_802_11_WSC_SET_M@ 1001846c     rtmp_info.obj
 0001:000174a8       ??_C@_0HI@JIAKBEHG@?$CFs?5?$CISET?3?3RT_OID_802_11_WSC_SET_M@ 100184a8     rtmp_info.obj
 0001:00017520       ??_C@_0CM@OGGBNCCI@Set?3?3RT_OID_802_11_SET_EVENT_CAP@ 10018520     rtmp_info.obj
 0001:0001754c       ??_C@_0CD@OONJEOFH@Set?3?3RT_OID_802_11_SET_DLS_PARAM@ 1001854c     rtmp_info.obj
 0001:00017570       ??_C@_0DB@GEABEIIG@Set?3?3RT_OID_802_11_SET_DLS?5?$CI?$DN?$CFd?$CJ@ 10018570     rtmp_info.obj
 0001:000175a4       ??_C@_0CP@GGPJDGJF@Free?5to?5TdlsSearchEntryFreeList?3@ 100185a4     rtmp_info.obj
 0001:000175d8       ??_C@_0EF@NEEKFPNE@TDLS?5?9?5Remove?5?$CF02x?3?$CF02x?3?$CF02x?3?$CF02@ 100185d8     rtmp_info.obj
 0001:00017620       ??_C@_0CB@HCILDFBC@Set?3?3RT_OID_802_11_SET_APSD_PSM?6@ 10018620     rtmp_info.obj
 0001:00017644       ??_C@_0DK@CIKFLBAK@Set?3?3RT_OID_802_11_SET_APSD_PSM?5@ 10018644     rtmp_info.obj
 0001:00017680       ??_C@_0GH@MLBOIPPH@Set?3?3RT_OID_802_11_SET_APSD_SETT@ 10018680     rtmp_info.obj
 0001:000176e8       ??_C@_0EA@GHMALBF@Set?3?3RT_OID_802_11_SET_HT_PHYMOD@ 100186e8     rtmp_info.obj
 0001:00017728       ??_C@_0HM@PENGKEHL@Set?3?3pHTPhyMode?5?5?$CIPhyMode?5?$DN?5?$CFd?0T@ 10018728     rtmp_info.obj
 0001:000177a4       ??_C@_0DF@PPADANAC@Set?3?3RT_OID_802_11_SET_HT_PHYMOD@ 100187a4     rtmp_info.obj
 0001:000177e0       ??_C@_0EP@GHOCLCLN@Set?3?3RT_OID_802_11_LEAP_AUTH_INF@ 100187e0     rtmp_info.obj
 0001:00017830       ??_C@_0FF@PHPCNGDF@Set?3?3RT_OID_802_11_SET_STA_CONFI@ 10018830     rtmp_info.obj
 0001:00017888       ??_C@_0DP@BCFFCFCN@Set?3?3RT_OID_802_11_SET_PHY_MODE?4@ 10018888     rtmp_info.obj
 0001:000178c8       ??_C@_0DI@FJOPHHML@Set?3?3RT_OID_802_11_SET_PHY_MODE?5@ 100188c8     rtmp_info.obj
 0001:00017900       ??_C@_0EE@MNCNNDPH@RT_OID_802_11_SET_PHY_MODE?3?5modi@ 10018900     rtmp_info.obj
 0001:00017944       ??_C@_0DE@JDKPJGDB@RT_OID_802_11_SET_PHY_MODE?3?5RFIC@ 10018944     rtmp_info.obj
 0001:00017978       ??_C@_0CE@PEMBMJJI@Set?3?3RT_OID_802_11_SET_RADIO?5?$CI?$DN?$CF@ 10018978     rtmp_info.obj
 0001:000179a0       ??_C@_0HL@KIKHIKAJ@Set?3?3FastRoamEnable?$CI?$DN?$CFd?$CJ?0?5dBmToR@ 100189a0     rtmp_info.obj
 0001:00017a1c       ??_C@_0CE@MJHFGMFC@Set?3?3RT_OID_802_11_CCX20_INFO?$CI?$DN?$CF@ 10018a1c     rtmp_info.obj
 0001:00017a40       ??_C@_0CF@GNOAPIHF@Set?3?3RT_OID_802_11_SET_AC_CAM?5?$CI?$DN@ 10018a40     rtmp_info.obj
 0001:00017a68       ??_C@_0CC@PFJIKHAG@Set?3?3OID_802_11_POWER_MODE?5?$CI?$DN?$CFd?$CJ@ 10018a68     rtmp_info.obj
 0001:00017a8c       ??_C@_0CN@NFOFPJJI@?$CB?$CB?$CB?5MLME?5busy?0?5reset?5MLME?5state?5@ 10018a8c     rtmp_info.obj
 0001:00017ac0       ??_C@_0EO@GKKILNBK@Set?3?3OID_802_11_CONFIGURATION?5?$CIS@ 10018ac0     rtmp_info.obj
 0001:00017b10       ??_C@_0CE@PNEDDMJM@Set?3?3OID_802_11_RSSI_TRIGGER?5?$CI?$DN?$CF@ 10018b10     rtmp_info.obj
 0001:00017b38       ??_C@_0JL@MKMDGCB@?$CFs?5?$CIOID_802_11_BSSID_LIST_SCAN?$CJ?3@ 10018b38     rtmp_info.obj
 0001:00017bd4       ??_C@_0BC@HHOMFNAA@STASetInformation?$AA@ 10018bd4     rtmp_info.obj
 0001:00017be8       ??_C@_0CE@BHJGACNB@Set?3?3?530sRxCnt?5?$DN?5?$CFd?5?4?5SsidLen?5?$DN?5@ 10018be8     rtmp_info.obj
 0001:00017c10       ??_C@_0EN@NDHLLGLK@Ignore?5zero?5config?5periodic?5scan@ 10018c10     rtmp_info.obj
 0001:00017c60       ??_C@_0EM@OJFEKMBG@?$CB?$CB?$CB?5Link?5UP?0?5Port?5Not?5Secured?$CB?5i@ 10018c60     rtmp_info.obj
 0001:00017cb0       ??_C@_0EE@LJCODEHF@Heavy?5traffic?5on?5TX?1RX?5ignore?5th@ 10018cb0     rtmp_info.obj
 0001:00017cf4       ??_C@_0CO@KFDMJJIF@The?5First?5Scan?5After?5Radio?5On?0?5c@ 10018cf4     rtmp_info.obj
 0001:00017d24       ??_C@_0DB@PIOHMFCJ@CCX?5enable?0?5continue?5OID_802_11_@ 10018d24     rtmp_info.obj
 0001:00017d58       ??_C@_0CO@PKNFCNOA@Set?3?3OID_802_11_BSSID_LIST_SCAN?0@ 10018d58     rtmp_info.obj
 0001:00017d88       ??_C@_0EH@LCOKEONM@Set?3?3OID_802_11_DISASSOCIATE?3?5Re@ 10018d88     rtmp_info.obj
 0001:00017dd0       ??_C@_0CA@MCHCILNG@EnqueueCmd?3?3OID_802_11_ADD_WEP?6?$AA@ 10018dd0     rtmp_info.obj
 0001:00017df0       ??_C@_0CP@JDCJONPA@CmdThread?3?3OID_802_11_ADD_WEP?0?5I@ 10018df0     rtmp_info.obj
 0001:00017e20       ??_C@_0EJ@LLDELKDE@Set?3?3OID_802_11_ADD_WEP?5?$CISkip?5th@ 10018e20     rtmp_info.obj
 0001:00017e6c       ??_C@_0CD@IAEDJABE@Update?5OID_802_11_PMKID?0?5idx?5?$DN?5?$CF@ 10018e6c     rtmp_info.obj
 0001:00017e90       ??_C@_0BH@BDEBEJJM@Set?3?3OID_802_11_PMKID?6?$AA@ 10018e90     rtmp_info.obj
 0001:00017ea8       ??_C@_0BG@IJEMAHAJ@Set?3?3OID_802_11_TEST?6?$AA@ 10018ea8     rtmp_info.obj
 0001:00017ec0       ??_C@_0CM@JLPHGGOJ@Set?3?3OID_802_11_ASSOCIATION_INFO@ 10018ec0     rtmp_info.obj
 0001:00017eec       ??_C@_0BN@CGBBMFOO@RT_OID_802_11_ADD_WPA?5Key?5?$DN?5?$AA@ 10018eec     rtmp_info.obj
 0001:00017f0c       ??_C@_0DD@JEIFOMLD@Set?3?3RT_OID_802_11_ADD_WPA?5?$CIid?$DN0@ 10018f0c     rtmp_info.obj
 0001:00017f40       ??_C@_0CM@DGLJFBPE@RT_OID_802_11_ADD_WPA?5Key?$CIWAPI?3?5@ 10018f40     rtmp_info.obj
 0001:00017f6c       ??_C@_0DA@LOFBOOKB@Set?3?3OID_802_11_ADD_KEY?5?$CIid?$DN0x?$CFx@ 10018f6c     rtmp_info.obj
 0001:00017f9c       ??_C@_0CE@LFLJLKNA@EnqueueCmd?3?3OID_802_11_ADD_KEY_W@ 10018f9c     rtmp_info.obj
 0001:00017fc0       ??_C@_0DO@DDJOJLNF@pAd?9?$DOSharedKey?$FLBSS0?$FN?$FL?$CFd?$FN?4CipherA@ 10018fc0     rtmp_info.obj
 0001:00018000       ??_C@_0CO@MHGNMEFF@RTMPWPAAddKeyProc?$DN?$DN?$DN?$DO?5pKey?9?$DOKeyI@ 10019000     rtmp_info.obj
 0001:00018030       ??_C@_0CA@GILDMKNK@EnqueueCmd?3?3OID_802_11_ADD_KEY?6?$AA@ 10019030     rtmp_info.obj
 0001:00018050       ??_C@_0CI@EAMLODAD@Set?3?3OID_802_11_ADD_KEY?0?5?5INVALI@ 10019050     rtmp_info.obj
 0001:00018078       ??_C@_0CP@DINLEMIF@Set?3?3OID_802_11_INFRASTRUCTURE_M@ 10019078     rtmp_info.obj
 0001:000180a8       ??_C@_0CN@JPHDHPDB@Set?3?3OID_802_11_INFRASTRUCTURE_M@ 100190a8     rtmp_info.obj
 0001:000180d8       ??_C@_0CO@HLOKENEC@Set?3?3OID_802_11_INFRASTRUCTURE_M@ 100190d8     rtmp_info.obj
 0001:00018108       ??_C@_0CI@EIHMKGKC@NDIS_STATUS_MEDIA_DISCONNECT?5Eve@ 10019108     rtmp_info.obj
 0001:00018130       ??_C@_0CO@HIEBKHEF@Set?3?3OID_802_11_SSID?5?$CILen?$DN?$CFd?0Ssi@ 10019130     rtmp_info.obj
 0001:00018160       ??_C@_0FN@FGMLMBEN@Set?3?3OID_802_11_SSID?5?$CISkip?5this?5@ 10019160     rtmp_info.obj
 0001:000181c0       ??_C@_0DI@KPKKMGFK@Set?3?3RT_OID_802_11_BSSID?5?$CF02x?3?$CF0@ 100191c0     rtmp_info.obj
 0001:000181f8       ??_C@_0DJ@PJGJBPJC@Set?3?3OID_802_11_BSSID?5?$CIpAd?9?$DOComm@ 100191f8     rtmp_info.obj
 0001:00018234       ??_C@_0DK@JBHEPKOJ@?$CB?$CB?$CB?$CB?$CB?$CB?$CBQueueed?5Packet?5has?5decryp@ 10019234     rtmp_info.obj
 0001:00018270       ??_C@_0BN@CFMOEBCE@?$CB?$CBWPA_802_1X_PORT_SECURED?$CB?$CB?6?$AA@ 10019270     rtmp_info.obj
 0001:00018290       ??_C@_0DO@LPDGDJNO@?5?9?9?9?9?9?9?9?9?9?9?9?9?9?9?9?9?5CCKM?$CB?$CB?5Resume?5@ 10019290     rtmp_info.obj
 0001:000182d0       ??_C@_0CN@LOAJDKNF@fRTMP_ADAPTER_ADDKEY_IN_PROGRESS@ 100192d0     rtmp_info.obj
 0001:00018300       ??_C@_0CO@DKHNDNNL@?$CFs?3?5Call?5the?5RTMPIndicateWPA2Sta@ 10019300     rtmp_info.obj
 0001:00018330       ??_C@_0BC@MCEJBBPF@RTMPWPAAddKeyProc?$AA@ 10019330     rtmp_info.obj
 0001:00018348       ??_C@_0EJ@EGDCMNBD@OID_DOT11_CIPHER_DEFAULT_KEY?3?5Se@ 10019348     rtmp_info.obj
 0001:00018394       ??_C@_0CB@ILBMEPKL@RTMPWPARemoveKeyProc?$CIKeyIdx?$DN?$CFd?$CJ?6@ 10019394     rtmp_info.obj
 0001:000183b8       ??_C@_0BL@NPGAOOHN@?9?9?9?$DO?5RTMPWPARemoveKeyProc?6?$AA@ 100193b8     rtmp_info.obj
 0001:000183d4       ??_C@_0BD@FHDILJKC@remove?5?$CFs?5key?5?$CD?$CFd?6?$AA@ 100193d4     rtmp_info.obj
 0001:000183e8       ??_C@_0DB@BFBIEKN@RTMPWPARemoveAllKeys?$CIAuthMode?$DN?$CFd@ 100193e8     rtmp_info.obj
 0001:0001841c       ??_C@_0BI@CFCOAOKA@RTMPIndicateWPA2Status?6?$AA@ 1001941c     rtmp_info.obj
 0001:00018438       ??_C@_0ID@IMGMBANH@RTMPIndicateWPA2Status?5?9?5?$CIpreaut@ 10019438     rtmp_info.obj
 0001:000184bc       ??_C@_0BO@IHHCOLPB@?$CFs?3?5Allocate?5memory?5failure?4?6?$AA@ 100194bc     rtmp_info.obj
 0001:000184dc       ??_C@_0BH@KBAJOJKM@RTMPIndicateWPA2Status?$AA@ 100194dc     rtmp_info.obj
 0001:000184f4       ??_C@_0CJ@MKGALMLC@RTMPSetPhyMode?9?$DOChannel?$DN?5?$CFd?0?5Phy@ 100194f4     rtmp_info.obj
 0001:00018520       ??_C@_0BF@GJCEOIB@RTMPSetPhyMode?$CI?$DN?$CFx?$CJ?6?$AA@ 10019520     rtmp_info.obj
 0001:00018538       ??_C@_0BI@GKGHFJBA@RFIC?$FL?$CFd?$FN?0?5Phymode?$CI?$DN?$CFx?$CJ?6?$AA@ 10019538     rtmp_info.obj
 0001:00018550       ??_C@_0CH@IAEDEJOH@RTMPSetPhyMode?5Phymode?$CI?$DN?$CFx?$CJ?4?5ret@ 10019550     rtmp_info.obj
 0001:00018578       ??_C@_0DA@CMOCJLKN@RTMPSetPhyMode?$FL?$CFd?$FN?0pAd?9?$DOCommonCf@ 10019578     rtmp_info.obj
 0001:000185a8       ??_C@_0BG@LDLAPAIO@Switch?5to?5?$CI?$DN?$CFd?$CJ?5mode?6?$AA@ 100195a8     rtmp_info.obj
 0001:000185c0       ??_C@_0CF@BJDOBHA@?$CFs?3?5pAd?9?$DOCommonCfg?4bWPSConnect?5?$DN@ 100195c0     rtmp_info.obj
 0001:000185e8       ??_C@_0BE@LIEICOHF@RTMPOPModeSwitching?$AA@ 100195e8     rtmp_info.obj
 0001:000185fc       ??_C@_03GBBBMBAD@?7?5?6?$AA@ 100195fc     rtmp_info.obj
 0001:00018600       ??_C@_04BALLJPHL@?5?$CFx?3?$AA@ 10019600     rtmp_info.obj
 0001:00018608       ??_C@_0BM@OJOLHFCK@Key?5?$FLidx?$DN?$CFx?$FN?5?$FLKeyLen?5?$DN?5?$CFd?$FN?6?$AA@ 10019608     rtmp_info.obj
 0001:00018624       ??_C@_0CN@DPJDAIOH@AddBSSIDasWCIDEntry?3?5Alg?$DN?$CFs?0?5Key@ 10019624     rtmp_info.obj
 0001:00018654       ??_C@_0CK@DFJPBECG@BSSID_WCID?5?3?5offset?5?$DN?5?$CFx?0?5WCIDAt@ 10019654     rtmp_info.obj
 0001:00018680       ??_C@_0CC@PKCINAPI@?7RxMic?5?$DN?5?$CF02x?3?$CF02x?3?$CF02x?3?$CF02x?3?4?4?4@ 10019680     rtmp_info.obj
 0001:000186a4       ??_C@_0CD@MKOJODFD@?7TxMIC?5?5?$DN?5?$CF02x?3?$CF02x?3?$CF02x?3?$CF02x?3?4?4@ 100196a4     rtmp_info.obj
 0001:000186c8       ??_C@_0CA@CBGAIPEG@RTMPAddBSSIDCipher?$DN?$DN?$DO?5Aid?5?$DN?5?$CFd?6?$AA@ 100196c8     rtmp_info.obj
 0001:000186e8       ??_C@_0DA@LHFLOEDN@?5RTMPSetHT?$DM?9?9?9ExtOffset?5?$DN?5?$CFd?4?5AM@ 100196e8     rtmp_info.obj
 0001:00018718       ??_C@_0DE@LAEALALN@RTMPSetHT?9?9?9?9?9?$DO?$CIMimoPs?5?$DN?5?$CFd?$CJ?5?$CIRx@ 10019718     rtmp_info.obj
 0001:0001874c       ??_C@_0DI@KAPJOECG@RTMPSetHT?5?9?$CIRxBAWinLimit?$DN?5?$CFd?$CJ?0?5?$CI@ 1001974c     rtmp_info.obj
 0001:00018784       ??_C@_09IAKMBOIK@RTMPSetHT?$AA@ 10019784     rtmp_info.obj
 0001:00018790       ??_C@_0BD@MGEGNHBO@RTMPSetHT?9?9?9?9?9?$DO?5?5?6?$AA@ 10019790     rtmp_info.obj
 0001:000187a4       ??_C@_0BF@IHIJPPO@RTMPUpdateHTIE?5?$DM?$DN?$DN?5?6?$AA@ 100197a4     rtmp_info.obj
 0001:000187bc       ??_C@_0BI@JPBOGBGO@?$CFs?3?5LED_WPS_IN_PROCESS?6?$AA@ 100197bc     rtmp_info.obj
 0001:000187d4       ??_C@_0BK@OBMCFH@?$CFs?3?5LED_WPS_TURN_LED_OFF?6?$AA@ 100197d4     rtmp_info.obj
 0001:000187f0       ??_C@_0BD@OHEPIBDN@LEDConnectionStart?$AA@ 100197f0     rtmp_info.obj
 0001:00018804       ??_C@_0BI@ENIFDAPA@LEDConnectionCompletion?$AA@ 10019804     rtmp_info.obj
 0001:0001881c       ??_C@_0BJ@EHGKCNN@Entry?$CD?$CFd?5?9?5no?5beacon?4?4?4?6?$AA@ 1001981c     rtmp_info.obj
 0001:00018838       ??_C@_0CF@GAAKJKGB@Deauth?5received?5from?5adhoc?5entry@ 10019838     rtmp_info.obj
 0001:00018860       ??_C@_1BE@GIGCBHND@?$AAC?$AAh?$AA1?$AA4?$AAB?$AAO?$AAn?$AAl?$AAy?$AA?$AA@ 10019860     rtmp_init.obj
 0001:00018874       ??_C@_1CA@MPGMFPNC@?$AAB?$AAT?$AAC?$AAo?$AAn?$AAf?$AAi?$AAg?$AAu?$AAr?$AAa?$AAt?$AAi?$AAo?$AAn?$AA?$AA@ 10019874     rtmp_init.obj
 0001:00018894       ??_C@_1BK@CJJNEDPG@?$AAB?$AAT?$AAS?$AAo?$AAf?$AAt?$AAw?$AAa?$AAr?$AAe?$AAO?$AAn?$AA?$AA@ 10019894     rtmp_init.obj
 0001:000188b0       ??_C@_1BK@BABIKIEF@?$AAG?$AAa?$AAi?$AAn?$AAP?$AAr?$AAo?$AAS?$AAp?$AAe?$AAe?$AAd?$AA?$AA@ 100198b0     rtmp_init.obj
 0001:000188cc       ??_C@_1CC@GCNEADEG@?$AAB?$AAs?$AAs?$AAi?$AAd?$AAR?$AAe?$AAp?$AAo?$AAs?$AAi?$AAt?$AAT?$AAi?$AAm?$AAe?$AA?$AA@ 100198cc     rtmp_init.obj
 0001:000188f0       ??_C@_1CC@KKEIICNE@?$AAP?$AAr?$AAo?$AAh?$AAi?$AAb?$AAi?$AAt?$AAT?$AAK?$AAI?$AAP?$AAo?$AAn?$AAH?$AAT?$AA?$AA@ 100198f0     rtmp_init.obj
 0001:00018914       ??_C@_19EIBINHIL@?$AAW?$AAA?$AAP?$AAI?$AA?$AA@ 10019914     rtmp_init.obj
 0001:00018920       ??_C@_19DICJPJO@?$AAT?$AAE?$AAS?$AAT?$AA?$AA@ 10019920     rtmp_init.obj
 0001:0001892c       ??_C@_1BO@LFECHPJM@?$AAC?$AAo?$AAu?$AAn?$AAt?$AAr?$AAy?$AAT?$AAx?$AAP?$AAw?$AAr?$AA5?$AAG?$AA?$AA@ 1001992c     rtmp_init.obj
 0001:0001894c       ??_C@_1BK@ENDJOIGJ@?$AAC?$AAo?$AAu?$AAn?$AAt?$AAr?$AAy?$AAT?$AAx?$AAP?$AAw?$AAr?$AA?$AA@ 1001994c     rtmp_init.obj
 0001:00018968       ??_C@_1BI@LGPNEEJB@?$AAL?$AAE?$AAD?$AAP?$AAo?$AAl?$AAa?$AAr?$AAi?$AAt?$AAy?$AA?$AA@ 10019968     rtmp_init.obj
 0001:00018980       ??_C@_1O@PFJDAPJC@?$AAL?$AAE?$AAD?$AAA?$AAc?$AAt?$AA?$AA@ 10019980     rtmp_init.obj
 0001:00018990       ??_C@_1BE@IFGCHPPB@?$AAL?$AAE?$AAD?$AAC?$AAo?$AAn?$AAf?$AAi?$AAg?$AA?$AA@ 10019990     rtmp_init.obj
 0001:000189a4       ??_C@_1BA@JBHFPAPB@?$AAL?$AAE?$AAD?$AAM?$AAo?$AAd?$AAe?$AA?$AA@ 100199a4     rtmp_init.obj
 0001:000189b4       ??_C@_1BG@PLJAEAAM@?$AAL?$AAE?$AAD?$AAC?$AAt?$AAl?$AAB?$AAy?$AAS?$AAW?$AA?$AA@ 100199b4     rtmp_init.obj
 0001:000189cc       ??_C@_1CA@LJPPBOF@?$AAL?$AAi?$AAn?$AAk?$AAS?$AAp?$AAe?$AAe?$AAd?$AAS?$AAt?$AAa?$AAt?$AAu?$AAs?$AA?$AA@ 100199cc     rtmp_init.obj
 0001:000189ec       ??_C@_1DC@LFKLGNPI@?$AAS?$AAo?$AAf?$AAt?$AAA?$AAP?$AAF?$AAo?$AAr?$AAc?$AAe?$AAM?$AAu?$AAl?$AAt?$AAi?$AAc?$AAa?$AAs?$AAt?$AAR?$AAa?$AAt?$AAe?$AA?$AA@ 100199ec     rtmp_init.obj
 0001:00018a20       ??_C@_1BC@OGAKBKDE@?$AAI?$AAd?$AAl?$AAe?$AAT?$AAi?$AAm?$AAe?$AA?$AA@ 10019a20     rtmp_init.obj
 0001:00018a34       ??_C@_1BG@IINBLCLB@?$AAD?$AAt?$AAi?$AAm?$AAP?$AAe?$AAr?$AAi?$AAo?$AAd?$AA?$AA@ 10019a34     rtmp_init.obj
 0001:00018a4c       ??_C@_1CE@PCANMBOM@?$AAA?$AAu?$AAt?$AAo?$AAC?$AAh?$AAa?$AAn?$AAn?$AAe?$AAl?$AAS?$AAe?$AAl?$AAe?$AAc?$AAt?$AA?$AA@ 10019a4c     rtmp_init.obj
 0001:00018a70       ??_C@_1BE@NOKFBOKB@?$AAP?$AAS?$AAC?$AAo?$AAn?$AAt?$AAr?$AAo?$AAl?$AA?$AA@ 10019a70     rtmp_init.obj
 0001:00018a84       ??_C@_1BE@DBKPDCJJ@?$AAS?$AAm?$AAa?$AAr?$AAt?$AAS?$AAc?$AAa?$AAn?$AA?$AA@ 10019a84     rtmp_init.obj
 0001:00018a98       ??_C@_1BE@IINHAOJL@?$AAR?$AAs?$AAs?$AAi?$AAD?$AAe?$AAl?$AAt?$AAa?$AA?$AA@ 10019a98     rtmp_init.obj
 0001:00018aac       ??_C@_1CI@CFGDGLJB@?$AAC?$AAC?$AAX?$AAP?$AAk?$AAt?$AAL?$AAo?$AAs?$AAs?$AAL?$AAi?$AAm?$AAi?$AAt?$AAT?$AAi?$AAm?$AAe?$AA?$AA@ 10019aac     rtmp_init.obj
 0001:00018ad4       ??_C@_1CA@KIMCJOKE@?$AAC?$AAA?$AAC?$AAD?$AAr?$AAo?$AAp?$AAC?$AAr?$AAi?$AAt?$AAe?$AAr?$AAi?$AAa?$AA?$AA@ 10019ad4     rtmp_init.obj
 0001:00018af4       ??_C@_1BM@PHBOPLGB@?$AAC?$AAA?$AAC?$AAD?$AAr?$AAo?$AAp?$AAP?$AAe?$AAr?$AAi?$AAo?$AAd?$AA?$AA@ 10019af4     rtmp_init.obj
 0001:00018b10       ??_C@_1BK@PJKHDBMG@?$AAC?$AAC?$AAX?$AAD?$AAb?$AAm?$AAO?$AAf?$AAf?$AAs?$AAe?$AAt?$AA?$AA@ 10019b10     rtmp_init.obj
 0001:00018b2c       ??_C@_1BC@GBGBNBCD@?$AAC?$AAL?$AAF?$AAa?$AAc?$AAt?$AAo?$AAr?$AA?$AA@ 10019b2c     rtmp_init.obj
 0001:00018b40       ??_C@_1BC@EGPLFCEP@?$AAN?$AAH?$AAF?$AAa?$AAc?$AAt?$AAo?$AAr?$AA?$AA@ 10019b40     rtmp_init.obj
 0001:00018b54       ??_C@_1BI@GKAHDKBF@?$AAC?$AAC?$AAX?$AA2?$AAC?$AAo?$AAn?$AAt?$AAr?$AAo?$AAl?$AA?$AA@ 10019b54     rtmp_init.obj
 0001:00018b6c       ??_C@_1O@LPLILBCD@?$AAP?$AAS?$AAM?$AAo?$AAd?$AAe?$AA?$AA@ 10019b6c     rtmp_init.obj
 0001:00018b7c       ??_C@_1CO@GMOLFAC@?$AAA?$AAd?$AAh?$AAo?$AAc?$AAN?$AA1?$AA4?$AAC?$AAh?$AA4?$AA0?$AAM?$AAH?$AAz?$AAA?$AAl?$AAl?$AAo?$AAw?$AAe?$AAd?$AA?$AA@ 10019b7c     rtmp_init.obj
 0001:00018bac       ??_C@_1CG@JEBJJGB@?$AAA?$AAd?$AAh?$AAo?$AAc?$AAN?$AA4?$AA0?$AAM?$AAH?$AAz?$AAA?$AAl?$AAl?$AAo?$AAw?$AAe?$AAd?$AA?$AA@ 10019bac     rtmp_init.obj
 0001:00018bd4       ??_C@_1BO@GPLOFEO@?$AAA?$AAd?$AAh?$AAo?$AAc?$AA5?$AAG?$AAD?$AAi?$AAs?$AAa?$AAb?$AAl?$AAe?$AA?$AA@ 10019bd4     rtmp_init.obj
 0001:00018bf4       ??_C@_1DC@PEAJAPLG@?$AAA?$AAd?$AAh?$AAo?$AAc?$AAN?$AAF?$AAo?$AAr?$AAc?$AAe?$AAM?$AAu?$AAl?$AAt?$AAi?$AAc?$AAa?$AAs?$AAt?$AAR?$AAa?$AAt?$AAe?$AA?$AA@ 10019bf4     rtmp_init.obj
 0001:00018c28       ??_C@_1BG@HIJECENL@?$AAA?$AAd?$AAh?$AAo?$AAc?$AAN?$AAM?$AAo?$AAd?$AAe?$AA?$AA@ 10019c28     rtmp_init.obj
 0001:00018c40       ??_C@_1BE@KABNOABI@?$AAA?$AAd?$AAh?$AAo?$AAc?$AAO?$AAf?$AAd?$AAm?$AA?$AA@ 10019c40     rtmp_init.obj
 0001:00018c54       ??_C@_1BI@FJLDDKCH@?$AAN?$AAe?$AAt?$AAw?$AAo?$AAr?$AAk?$AAT?$AAy?$AAp?$AAe?$AA?$AA@ 10019c54     rtmp_init.obj
 0001:00018c6c       ??_C@_1BM@EFMHHLJG@?$AAA?$AAu?$AAt?$AAo?$AAR?$AAe?$AAc?$AAo?$AAn?$AAn?$AAe?$AAc?$AAt?$AA?$AA@ 10019c6c     rtmp_init.obj
 0001:00018c88       ??_C@_1BO@MJECKBG@?$AAS?$AAh?$AAo?$AAw?$AAH?$AAi?$AAd?$AAd?$AAe?$AAn?$AAS?$AAS?$AAI?$AAD?$AA?$AA@ 10019c88     rtmp_init.obj
 0001:00018ca8       ??_C@_1M@HCFAIFML@?$AAR?$AAa?$AAd?$AAi?$AAo?$AA?$AA@ 10019ca8     rtmp_init.obj
 0001:00018cb4       ??_C@_1BC@CKIBMGHF@?$AAP?$AAS?$AAP?$AAX?$AAl?$AAi?$AAn?$AAk?$AA?$AA@ 10019cb4     rtmp_init.obj
 0001:00018cc8       ??_C@_1BG@LDMHCIGI@?$AAD?$AAi?$AAr?$AAe?$AAc?$AAt?$AAM?$AAo?$AAd?$AAe?$AA?$AA@ 10019cc8     rtmp_init.obj
 0001:00018ce0       ??_C@_1BG@LEFEDPAE@?$AAD?$AAL?$AAS?$AAC?$AAa?$AAp?$AAa?$AAb?$AAl?$AAe?$AA?$AA@ 10019ce0     rtmp_init.obj
 0001:00018cf8       ??_C@_1CA@EFEMNLAK@?$AAT?$AAr?$AAa?$AAn?$AAs?$AAm?$AAi?$AAt?$AAS?$AAe?$AAt?$AAt?$AAi?$AAn?$AAg?$AA?$AA@ 10019cf8     rtmp_init.obj
 0001:00018d18       ??_C@_1BK@JLNNNNCD@?$AAB?$AAA?$AAC?$AAa?$AAp?$AAa?$AAb?$AAi?$AAl?$AAi?$AAt?$AAy?$AA?$AA@ 10019d18     rtmp_init.obj
 0001:00018d34       ??_C@_1BI@HGMLCLKI@?$AAM?$AAu?$AAl?$AAt?$AAi?$AAp?$AAl?$AAe?$AAI?$AAR?$AAP?$AA?$AA@ 10019d34     rtmp_init.obj
 0001:00018d4c       ??_C@_1BI@FBEBBJAC@?$AAM?$AAa?$AAx?$AAS?$AAP?$AAL?$AAe?$AAn?$AAg?$AAt?$AAh?$AA?$AA@ 10019d4c     rtmp_init.obj
 0001:00018d64       ??_C@_1BE@MGPCNCPB@?$AAA?$AAP?$AAS?$AAD?$AAA?$AAC?$AA_?$AAV?$AAO?$AA?$AA@ 10019d64     rtmp_init.obj
 0001:00018d78       ??_C@_1BE@ODJJINCN@?$AAA?$AAP?$AAS?$AAD?$AAA?$AAC?$AA_?$AAV?$AAI?$AA?$AA@ 10019d78     rtmp_init.obj
 0001:00018d8c       ??_C@_1BE@NBNHAFCL@?$AAA?$AAP?$AAS?$AAD?$AAA?$AAC?$AA_?$AAB?$AAK?$AA?$AA@ 10019d8c     rtmp_init.obj
 0001:00018da0       ??_C@_1BE@DBAIHCBI@?$AAA?$AAP?$AAS?$AAD?$AAA?$AAC?$AA_?$AAB?$AAE?$AA?$AA@ 10019da0     rtmp_init.obj
 0001:00018db4       ??_C@_1BI@LOMHIPGP@?$AAA?$AAP?$AAS?$AAD?$AAC?$AAa?$AAp?$AAa?$AAb?$AAl?$AAe?$AA?$AA@ 10019db4     rtmp_init.obj
 0001:00018dcc       ??_C@_1BG@HGDCKNNC@?$AAW?$AAM?$AAM?$AAC?$AAa?$AAp?$AAa?$AAb?$AAl?$AAe?$AA?$AA@ 10019dcc     rtmp_init.obj
 0001:00018de4       ??_C@_1BI@OECFHPPP@?$AAT?$AAG?$AAn?$AAW?$AAi?$AAf?$AAi?$AAT?$AAe?$AAs?$AAt?$AA?$AA@ 10019de4     rtmp_init.obj
 0001:00018dfc       ??_C@_1BA@FANIFMBI@?$AAT?$AAX?$AAB?$AAu?$AAr?$AAs?$AAt?$AA?$AA@ 10019dfc     rtmp_init.obj
 0001:00018e0c       ??_C@_1BM@GOCPLMJI@?$AAC?$AAa?$AAr?$AAr?$AAi?$AAe?$AAr?$AAD?$AAe?$AAt?$AAe?$AAc?$AAt?$AA?$AA@ 10019e0c     rtmp_init.obj
 0001:00018e28       ??_C@_1BG@BPJAKMMA@?$AAI?$AAE?$AAE?$AAE?$AA8?$AA0?$AA2?$AA1?$AA1?$AAH?$AA?$AA@ 10019e28     rtmp_init.obj
 0001:00018e40       ??_C@_1CC@CENNGNJ@?$AAF?$AAr?$AAa?$AAm?$AAe?$AAA?$AAg?$AAg?$AAr?$AAe?$AAg?$AAa?$AAt?$AAi?$AAo?$AAn?$AA?$AA@ 10019e40     rtmp_init.obj
 0001:00018e64       ??_C@_1BE@CJFJGBPC@?$AAS?$AAh?$AAo?$AAr?$AAt?$AAS?$AAl?$AAo?$AAt?$AA?$AA@ 10019e64     rtmp_init.obj
 0001:00018e78       ??_C@_1BK@KPPOILKG@?$AAB?$AAG?$AAP?$AAr?$AAo?$AAt?$AAe?$AAc?$AAt?$AAi?$AAo?$AAn?$AA?$AA@ 10019e78     rtmp_init.obj
 0001:00018e94       ??_C@_1CA@PGBNFBEB@?$AAM?$AAa?$AAx?$AAP?$AAk?$AAt?$AAO?$AAn?$AAe?$AAT?$AAx?$AAB?$AAu?$AAl?$AAk?$AA?$AA@ 10019e94     rtmp_init.obj
 0001:00018eb4       ??_C@_1BC@IOGOHBPE@?$AAT?$AAB?$AAF?$AAa?$AAc?$AAt?$AAo?$AAr?$AA?$AA@ 10019eb4     rtmp_init.obj
 0001:00018ec8       ??_C@_1BC@IABCMNHB@?$AAR?$AAB?$AAF?$AAa?$AAc?$AAt?$AAo?$AAr?$AA?$AA@ 10019ec8     rtmp_init.obj
 0001:00018edc       ??_C@_1BO@HGPPFMIN@?$AAN?$AAe?$AAt?$AAw?$AAo?$AAr?$AAk?$AAA?$AAd?$AAd?$AAr?$AAe?$AAs?$AAs?$AA?$AA@ 10019edc     rtmp_init.obj
 0001:00018efc       ??_C@_1BA@HCLACGFM@?$AAW?$AAE?$AAP?$AAK?$AAe?$AAy?$AA4?$AA?$AA@ 10019efc     rtmp_init.obj
 0001:00018f0c       ??_C@_1BA@OPGHBOOF@?$AAW?$AAE?$AAP?$AAK?$AAe?$AAy?$AA3?$AA?$AA@ 10019f0c     rtmp_init.obj
 0001:00018f1c       ??_C@_1BA@FHNLHJIA@?$AAW?$AAE?$AAP?$AAK?$AAe?$AAy?$AA2?$AA?$AA@ 10019f1c     rtmp_init.obj
 0001:00018f2c       ??_C@_1BA@EFGONGGO@?$AAW?$AAE?$AAP?$AAK?$AAe?$AAy?$AA1?$AA?$AA@ 10019f2c     rtmp_init.obj
 0001:00018f3c       ??_C@_1BG@OHMGBAFO@?$AAW?$AAP?$AAS?$AAD?$AAe?$AAv?$AAN?$AAa?$AAm?$AAe?$AA?$AA@ 10019f3c     rtmp_init.obj
 0001:00018f54       ??_C@_1BG@OIMBEMPB@?$AAV?$AAe?$AAn?$AAd?$AAo?$AAr?$AAD?$AAe?$AAs?$AAc?$AA?$AA@ 10019f54     rtmp_init.obj
 0001:00018f6c       ??_C@_19KJNOMKCJ@?$AAS?$AAS?$AAI?$AAD?$AA?$AA@ 10019f6c     rtmp_init.obj
 0001:00018f78       ??_C@_17BPNEPMND@?$AAR?$AAD?$AAG?$AA?$AA@ 10019f78     rtmp_init.obj
 0001:00018f80       ??_C@_1BE@HKNKOMJL@?$AAW?$AAE?$AAP?$AAK?$AAe?$AAy?$AAU?$AAs?$AAe?$AA?$AA@ 10019f80     rtmp_init.obj
 0001:00018f94       ??_C@_1BG@CLENCLJC@?$AAA?$AAu?$AAt?$AAh?$AAe?$AAn?$AAT?$AAy?$AAp?$AAe?$AA?$AA@ 10019f94     rtmp_init.obj
 0001:00018fac       ??_C@_1BG@MHEIMMBG@?$AAE?$AAn?$AAc?$AAr?$AAy?$AAp?$AAt?$AAi?$AAo?$AAn?$AA?$AA@ 10019fac     rtmp_init.obj
 0001:00018fc4       ??_C@_1BG@CPCOBECG@?$AAF?$AAr?$AAa?$AAg?$AAT?$AAh?$AAr?$AAe?$AAs?$AAh?$AA?$AA@ 10019fc4     rtmp_init.obj
 0001:00018fdc       ??_C@_1BE@NCNOFIOB@?$AAR?$AAt?$AAs?$AAT?$AAh?$AAr?$AAe?$AAs?$AAh?$AA?$AA@ 10019fdc     rtmp_init.obj
 0001:00018ff0       ??_C@_1BA@DLAHBHMC@?$AAC?$AAh?$AAa?$AAn?$AAn?$AAe?$AAl?$AA?$AA@ 10019ff0     rtmp_init.obj
 0001:00019000       ??_C@_1BK@CMGABJAK@?$AAW?$AAi?$AAr?$AAe?$AAl?$AAe?$AAs?$AAs?$AAM?$AAo?$AAd?$AAe?$AA?$AA@ 1001a000     rtmp_init.obj
 0001:0001901c       ??_C@_1CG@FHJPKHBD@?$AAC?$AAo?$AAu?$AAn?$AAt?$AAr?$AAy?$AAR?$AAe?$AAg?$AAi?$AAo?$AAn?$AAA?$AAB?$AAa?$AAn?$AAd?$AA?$AA@ 1001a01c     rtmp_init.obj
 0001:00019044       ??_C@_1BM@PHDEHLBE@?$AAC?$AAo?$AAu?$AAn?$AAt?$AAr?$AAy?$AAR?$AAe?$AAg?$AAi?$AAo?$AAn?$AA?$AA@ 1001a044     rtmp_init.obj
 0001:00019060       ??_C@_1CA@PGOEGKAH@?$AAU?$AAs?$AAe?$AAR?$AAa?$AAS?$AAu?$AAp?$AAp?$AAl?$AAi?$AAc?$AAa?$AAn?$AAt?$AA?$AA@ 1001a060     rtmp_init.obj
 0001:00019080       ??_C@_1O@OADBDALB@?$AAO?$AAp?$AAM?$AAo?$AAd?$AAe?$AA?$AA@ 1001a080     rtmp_init.obj
 0001:00019090       ??_C@_07BDGAECLF@CKIP128?$AA@ 1001a090     rtmp_init.obj
 0001:00019098       ??_C@_07LMFBNJNH@CKIP104?$AA@ 1001a098     rtmp_init.obj
 0001:000190a0       ??_C@_06HHMNOKIF@CKIP64?$AA@ 1001a0a0     rtmp_init.obj
 0001:000190a8       ??_C@_03BKNEFOAH@AES?$AA@  1001a0a8     rtmp_init.obj
 0001:000190ac       ??_C@_06JCFAKCMD@wep128?$AA@ 1001a0ac     rtmp_init.obj
 0001:000190b4       ??_C@_05PJDLFBFB@wep64?$AA@ 1001a0b4     rtmp_init.obj
 0001:000190bc       ??_C@_04CGFJFPFD@none?$AA@ 1001a0bc     rtmp_init.obj
 0001:000192c8       ccitt_16Table              1001a2c8     rtmp_init.obj
 0001:000194c8       ??_C@_0CG@OCNACBOC@?$DM?9?9?5RTMPAllocAdapterBlock?0?5Statu@ 1001a4c8     rtmp_init.obj
 0001:000194f0       ??_C@_0CF@OKIAKFAA@Failed?5to?5allocate?5memory?5?9?5ADAP@ 1001a4f0     rtmp_init.obj
 0001:00019518       ??_C@_0BL@JGKILNFB@?9?9?$DO?5RTMPAllocAdapterBlock?6?$AA@ 1001a518     rtmp_init.obj
 0001:00019534       ??_C@_0BF@MLMMNDCF@?$DM?9?9?5NICInitTransmit?6?$AA@ 1001a534     rtmp_init.obj
 0001:0001954c       ??_C@_0CH@GEIBMAME@PsPoll?5Context?5?3?5sizeof?$CITX_BUFFE@ 1001a54c     rtmp_init.obj
 0001:00019574       ??_C@_0DD@ONNCDAOJ@?$DM?9?9?5ERROR?5in?5Alloc?5TX?5PsPollCont@ 1001a574     rtmp_init.obj
 0001:000195a8       ??_C@_0CE@OAEMILFG@RTS?5Context?5?3?5sizeof?$CITX_BUFFER?$CJ?$DN@ 1001a5a8     rtmp_init.obj
 0001:000195cc       ??_C@_0DA@KGPAPHEL@?$DM?9?9?5ERROR?5in?5Alloc?5TX?5RTSContext@ 1001a5cc     rtmp_init.obj
 0001:000195fc       ??_C@_0CF@KEPBHPDC@Null?5Context?5?3?5sizeof?$CITX_BUFFER?$CJ@ 1001a5fc     rtmp_init.obj
 0001:00019624       ??_C@_0DB@GHKDFEHD@?$DM?9?9?5ERROR?5in?5Alloc?5TX?5NullContex@ 1001a624     rtmp_init.obj
 0001:00019658       ??_C@_0DF@CLCCHGFA@?$DM?9?9?5ERROR?5in?5Alloc?5TX?5MLMEContex@ 1001a658     rtmp_init.obj
 0001:00019690       ??_C@_0DL@EPENJHFN@TX?5Ring?3?5total?5?$CFd?5entry?5allocate@ 1001a690     rtmp_init.obj
 0001:000196cc       ??_C@_0DD@JKNKBBIM@?$DM?9?9?5ERROR?5in?5Alloc?5TX?5TxContext?$FL@ 1001a6cc     rtmp_init.obj
 0001:00019700       ??_C@_0BJ@FEOFJHDA@ERROR?5pAd?9?$DOnonpagedlist?6?$AA@ 1001a700     rtmp_init.obj
 0001:0001971c       ??_C@_0BP@IJJKCPFK@ERROR?5pAd?9?$DOBulkOutTempBuf?$FL?$CFd?$FN?6?$AA@ 1001a71c     rtmp_init.obj
 0001:0001973c       ??_C@_0BF@KPOGPPPE@?9?9?$DO?5NICInitTransmit?6?$AA@ 1001a73c     rtmp_init.obj
 0001:00019758       ??_C@_1EK@NLLLCOO@?$AAR?$AAT?$AA2?$AA8?$AA7?$AA0?$AA?3?$AA?5?$AAC?$AAr?$AAe?$AAa?$AAt?$AAe?$AA?5?$AAJ?$AAu?$AAn?$AAk?$AAT?$AAh?$AAr?$AAe?$AAa?$AAd?$AA?5?$AAe?$AAr?$AAr?$AAo?$AAr?$AA?3@ 1001a758     rtmp_init.obj
 0001:000197a8       ??_C@_1EK@GGPKIICH@?$AAR?$AAT?$AA2?$AA8?$AA7?$AA0?$AA?3?$AA?5?$AAC?$AAr?$AAe?$AAa?$AAt?$AAe?$AA?5?$AAM?$AAl?$AAm?$AAe?$AAT?$AAh?$AAr?$AAe?$AAa?$AAd?$AA?5?$AAe?$AAr?$AAr?$AAo?$AAr?$AA?3@ 1001a7a8     rtmp_init.obj
 0001:000197f8       ??_C@_1FC@HEJAOJKG@?$AAR?$AAT?$AA2?$AA8?$AA7?$AA0?$AA?3?$AA?5?$AAC?$AAr?$AAe?$AAa?$AAt?$AAe?$AA?5?$AAR?$AAT?$AAU?$AAS?$AAB?$AAC?$AAm?$AAd?$AAT?$AAh?$AAr?$AAe?$AAa?$AAd?$AA?5?$AAe?$AAr@ 1001a7f8     rtmp_init.obj
 0001:00019850       ??_C@_0HE@FLGGNENA@Rx?5Reordering?5buffer?3?5total?5?$CFd?5e@ 1001a850     rtmp_init.obj
 0001:000198c4       ??_C@_0DH@CNLLOJCA@RX?5Ring?3?5total?5?$CFd?5entry?5allocate@ 1001a8c4     rtmp_init.obj
 0001:000198fc       ??_C@_0BJ@FDDDKNNF@?$DM?9?9?5RTUSBBulkReceiveDPC?6?$AA@ 1001a8fc     rtmp_init.obj
 0001:00019918       ??_C@_0BJ@NJDIKFME@?9?9?$DO?5RTUSBBulkReceiveDPC?6?$AA@ 1001a918     rtmp_init.obj
 0001:00019934       ??_C@_0BG@EBKOFMAH@?$DM?9?9?5RTUSBRxPacketDPC?6?$AA@ 1001a934     rtmp_init.obj
 0001:0001994c       ??_C@_0BG@LABOJEGJ@?9?9?$DO?5RTUSBRxPacketDPC?6?$AA@ 1001a94c     rtmp_init.obj
 0001:00019964       ??_C@_0BJ@GFFAJBKC@?$DM?9?9?5RTUSBKickbulkoutDPC?6?$AA@ 1001a964     rtmp_init.obj
 0001:00019980       ??_C@_0DO@OGOEGODD@?9?9?$DO?5RTUSBKickbulkoutDPC?5?0pAd?9?$DOSe@ 1001a980     rtmp_init.obj
 0001:000199c0       ??_C@_0CF@BPCDNDPB@?$DM?9?9?5RTMPInitAdapterBlock?0?5Status@ 1001a9c0     rtmp_init.obj
 0001:000199e8       ??_C@_1BG@KDOEMPEF@?$AAJ?$AAu?$AAn?$AAk?$AA?5?$AAE?$AAv?$AAe?$AAn?$AAt?$AA?$AA@ 1001a9e8     rtmp_init.obj
 0001:00019a00       ??_C@_1BG@EEMGAPFL@?$AAM?$AAL?$AAM?$AAE?$AA?5?$AAE?$AAv?$AAe?$AAn?$AAt?$AA?$AA@ 1001aa00     rtmp_init.obj
 0001:00019a18       ??_C@_1FM@BJNLCDGL@?$AAC?$AA?3?$AA?2?$AAW?$AAi?$AAn?$AAC?$AAE?$AA6?$AA?4?$AA0?$AA?2?$AAN?$AAe?$AAw?$AA?2?$AAR?$AAT?$AA2?$AA8?$AA7?$AA0?$AA_?$AAv?$AA1?$AA?4?$AA4?$AA?4?$AA9?$AA?4?$AA0?$AA?2@ 1001aa18     rtmp_init.obj
 0001:00019a74       ??_C@_1BM@IBPGOOAH@?$AAC?$AAo?$AAn?$AAt?$AAr?$AAo?$AAl?$AA?5?$AAE?$AAv?$AAe?$AAn?$AAt?$AA?$AA@ 1001aa74     rtmp_init.obj
 0001:00019a90       ??_C@_0BK@DJIKAFOI@?9?9?$DO?5RTMPInitAdapterBlock?6?$AA@ 1001aa90     rtmp_init.obj
 0001:00019aac       ??_C@_0BF@BGEGKJLJ@?$DM?9?9?9?5ReleaseAdapter?6?$AA@ 1001aaac     rtmp_init.obj
 0001:00019ac4       ??_C@_0BF@GFNLJLB@?9?9?9?$DO?5ReleaseAdapter?6?$AA@ 1001aac4     rtmp_init.obj
 0001:00019adc       ??_C@_0BK@JJJBMFJM@?$DM?9?9?5RTMPReadTxPwrPerRate?6?$AA@ 1001aadc     rtmp_init.obj
 0001:00019af8       ??_C@_0CF@NPOAKLDF@?$CFx?0?5?5Adata40M?5?$DN?5?$CFx?0?5?5Gdata40M?5?$DN?5@ 1001aaf8     rtmp_init.obj
 0001:00019b20       ??_C@_0CC@MABMGGC@Gpwrdelta?5?$DN?5?$CFx?0?5Apwrdelta?5?$DN?5?$CFx?5?4@ 1001ab20     rtmp_init.obj
 0001:00019b44       ??_C@_0BC@OKEKFALL@Txpower?5per?5Rate?6?$AA@ 1001ab44     rtmp_init.obj
 0001:00019b58       ??_C@_0DO@KFAKEAH@E2PROM?3?5TxPower?$FL?$CF03d?$FN?0?5Channel?5?$DN@ 1001ab58     rtmp_init.obj
 0001:00019b98       ??_C@_1EG@INAMCIGM@?$AAp?$AAA?$AAd?$AA?9?$AA?$DO?$AAT?$AAx?$AAP?$AAo?$AAw?$AAe?$AAr?$AA?5?$AAb?$AAu?$AAf?$AAf?$AAe?$AAr?$AA?5?$AAm?$AAi?$AAg?$AAh?$AAt?$AA?5?$AAo?$AAv?$AAe?$AAr?$AAf?$AAl@ 1001ab98     rtmp_init.obj
 0001:00019be0       ??_C@_0BL@IDIACGIH@bAdhocNMode?5Support?5?$DN?$FL?$CFd?$FN?6?$AA@ 1001abe0     rtmp_init.obj
 0001:00019bfc       ??_C@_0BD@CKMOPGMM@NumOfBulkInIRP?$DN?$CFd?6?$AA@ 1001abfc     rtmp_init.obj
 0001:00019c10       ??_C@_0BL@DDFFGHBD@WmmCapable?$DN?$CFd?4?5rdg?5?$DN?5?$CFd?4?5?6?$AA@ 1001ac10     rtmp_init.obj
 0001:00019c2c       ??_C@_0CM@HIECLJEN@WPS?5Device?5Name?5?$CILen?$DN?$CFd?0?5WPSDevN@ 1001ac2c     rtmp_init.obj
 0001:00019c58       ??_C@_0CL@FCFMHIIM@Local?5MAC?5?$DN?5?$CF02x?3?$CF02x?3?$CF02x?3?$CF02x?3@ 1001ac58     rtmp_init.obj
 0001:00019c84       ??_C@_0BO@OJJINGMM@NHFactori?5?$DN?$CFd?0?5CLFactor?5?$DN?5?$CFd?6?$AA@ 1001ac84     rtmp_init.obj
 0001:00019ca4       ??_C@_0BE@JCOFMPI@CCXControl?5is?5?$CF08x?6?$AA@ 1001aca4     rtmp_init.obj
 0001:00019cb8       ??_C@_0BI@IKJPMJHO@WindowsPowerMode?5is?5?$CFd?6?$AA@ 1001acb8     rtmp_init.obj
 0001:00019cd0       ??_C@_0BG@MEHMEPLP@Software?5Radio?5is?5on?6?$AA@ 1001acd0     rtmp_init.obj
 0001:00019ce8       ??_C@_0BH@CFIMCAHD@Software?5Radio?5is?5off?6?$AA@ 1001ace8     rtmp_init.obj
 0001:00019d00       ??_C@_0CL@JBBHAABC@Soft?5AP?5mode?0?5Software?5Radio?5is?5@ 1001ad00     rtmp_init.obj
 0001:00019d2c       ??_C@_0DC@HJKOLOLJ@WEP?5key?$CI?$CFd?$CJ?3?5KeyLen?$DN?$CFd?0?5?$CF02x?3?$CF02@ 1001ad2c     rtmp_init.obj
 0001:00019d60       ??_C@_0CP@MKHFOGKI@Vendor?5Description?5?$CILen?$DN?$CFd?0?5Vend@ 1001ad60     rtmp_init.obj
 0001:00019d90       ??_C@_0BL@CNHLFECN@SSID?5?$CILen?$DN?$CFd?0?5ssid?$DN?$CFs?4?4?4?$CJ?6?$AA@ 1001ad90     rtmp_init.obj
 0001:00019db0       ??_C@_0EN@OBCDPHJB@BACapability?5?$DN?50x?$CFx?4?5MpduDensity@ 1001adb0     rtmp_init.obj
 0001:00019e00       ??_C@_0DH@EKBJJCEA@MaxPktOneTxBulk?$DN?$CFd?0?5TxBulkFactor@ 1001ae00     rtmp_init.obj
 0001:00019e38       ??_C@_0FB@LDFMCABB@TransmitSetting?5?$DN?50x?$CFx?4?5BW?$DN?$CFd?0?5H@ 1001ae38     rtmp_init.obj
 0001:00019e90       ??_C@_0GH@KBODAAFM@BACapability?5?$DN?50x?$CFx?4?5MpduDensity@ 1001ae90     rtmp_init.obj
 0001:00019ef8       ??_C@_0DF@JMOKDCCF@?5PhyMode?$DN?$CFd?0?5BW?5?$DN?$CFd?5?5MCS?5?$DN?$CFd?5?5Sh@ 1001aef8     rtmp_init.obj
 0001:00019f30       ??_C@_0FI@PPCNBIIP@AP?$DN?$CFd?0?5Channel?$DN?$CFd?0?5Rts?$DN?$CFd?0?5Frag?$DN@ 1001af30     rtmp_init.obj
 0001:00019f88       ??_C@_0BF@PHFIBNDC@Bogus?5field?5size?5?$CFd?6?$AA@ 1001af88     rtmp_init.obj
 0001:00019fa0       ??_C@_0BC@FICEFMOJ@?$DN?50x?$CFx?5?$CIdefault?$CJ?6?$AA@ 1001afa0     rtmp_init.obj
 0001:00019fb4       ??_C@_0M@BIPEIMIP@?5?9?9?5failed?6?$AA@ 1001afb4     rtmp_init.obj
 0001:00019fc0       ??_C@_0CF@LBJHNGKL@?$DM?9?9?5NICReadRegParameters?0?5Status@ 1001afc0     rtmp_init.obj
 0001:00019fe8       ??_C@_0BO@DPMOFAFD@NdisOpenConfiguration?5failed?6?$AA@ 1001afe8     rtmp_init.obj
 0001:0001a008       ??_C@_0BK@PGIONEIM@?9?9?$DO?5NICReadRegParameters?6?$AA@ 1001b008     rtmp_init.obj
 0001:0001a024       ??_C@_0BN@NAMNKJBM@?$DM?9?9?5NICReadEEPROMParameters?6?$AA@ 1001b024     rtmp_init.obj
 0001:0001a044       ??_C@_0BN@NOKEAOOO@E2PROM?3?5RF?5freq?5offset?$DN0x?$CFx?6?$AA@ 1001b044     rtmp_init.obj
 0001:0001a068       ??_C@_0EO@HCMFKNAH@E2PROM?3?5A?5Tssi?$FL?94?5?4?4?5?$CL4?$FN?5?$DN?5?$CFd?5?$CFd@ 1001b068     rtmp_init.obj
 0001:0001a0b8       ??_C@_0EO@HOOADKDM@E2PROM?3?5G?5Tssi?$FL?94?5?4?4?5?$CL4?$FN?5?$DN?5?$CFd?5?$CFd@ 1001b0b8     rtmp_init.obj
 0001:0001a108       ??_C@_0CB@BMBCHDKC@A?5Band?5Manual?5Ch1?5value?5is?50x?$CFx?6@ 1001b108     rtmp_init.obj
 0001:0001a12c       ??_C@_0CB@JLLELIOB@A?5Band?5Manual?5Ch0?5value?5is?50x?$CFx?6@ 1001b12c     rtmp_init.obj
 0001:0001a150       ??_C@_0CB@EJFGMPMN@BG?5Band?5Manual?5Ch?5value?5is?50x?$CFx?6@ 1001b150     rtmp_init.obj
 0001:0001a174       ??_C@_0CH@IMCJKMIN@E2PROM?3?5Version?5?$DN?5?$CFd?0?5FAE?5releas@ 1001b174     rtmp_init.obj
 0001:0001a19c       ??_C@_0BN@NIOCHLKL@?9?9?$DO?5NICReadEEPROMParameters?6?$AA@ 1001b19c     rtmp_init.obj
 0001:0001a1bc       ??_C@_0BG@JBMACHBJ@3xxx?$DL?5RT30xxInitAsic?6?$AA@ 1001b1bc     rtmp_init.obj
 0001:0001a1d4       ??_C@_0BL@DMFFKKPO@?$DM?9?9?5NICInitAsicFromEEPROM?6?$AA@ 1001b1d4     rtmp_init.obj
 0001:0001a1f0       ??_C@_0DA@GMOGHAJI@TxPath?5?$DN?5?$CFd?0?5RxPath?5?$DN?5?$CFd?0?5RFIC?$DN?$CF@ 1001b1f0     rtmp_init.obj
 0001:0001a220       ??_C@_0CO@FKEBOFFH@Use?5Hw?5Radio?5Control?5Pin?$DN?$CFd?$DL?5if?5@ 1001b220     rtmp_init.obj
 0001:0001a250       ??_C@_0DP@DOILJLBJ@RT3071?5Update?5RF?5Registers?5from?5@ 1001b250     rtmp_init.obj
 0001:0001a290       ??_C@_0EC@OHJEFLLI@RT3071?5Update?5BBP?5Registers?5from@ 1001b290     rtmp_init.obj
 0001:0001a2d4       ??_C@_0CK@HFGAHGBC@?$CFs?3?5pAd?9?$DOTxPowerCtrl?4bInternalTx@ 1001b2d4     rtmp_init.obj
 0001:0001a300       ??_C@_0BG@OPGKKLPJ@NICInitAsicFromEEPROM?$AA@ 1001b300     rtmp_init.obj
 0001:0001a318       ??_C@_0CD@PJFFOMCJ@pAd?9?$DORfIcType?5?$DN?5?$CFd?0?5RealRxPath?$DN?$CF@ 1001b318     rtmp_init.obj
 0001:0001a33c       ??_C@_0CD@EOKJGJHI@E2PROM?5error?0?5hard?5code?5as?50x?$CF04@ 1001b33c     rtmp_init.obj
 0001:0001a360       ??_C@_0BL@GBFHILNH@?9?9?$DO?5NICInitAsicFromEEPROM?6?$AA@ 1001b360     rtmp_init.obj
 0001:0001a37c       ??_C@_07KHJCGGJL@?$DM?9?9?5?$CFs?6?$AA@ 1001b37c     rtmp_init.obj
 0001:0001a388       ??_C@_0FH@ODFIMEIC@?$CFs?3?5BBPR106?3?5BBPR106?4field?4Short@ 1001b388     rtmp_init.obj
 0001:0001a3e0       ??_C@_0IG@PJEOFGKJ@?$CFs?3?5BBP_R105?3?5BBPR105?4field?4Enab@ 1001b3e0     rtmp_init.obj
 0001:0001a468       ??_C@_07JCMBCHBL@?9?9?$DO?5?$CFs?6?$AA@ 1001b468     rtmp_init.obj
 0001:0001a470       ??_C@_0BG@FIHHOJHB@PostBBPInitialization?$AA@ 1001b470     rtmp_init.obj
 0001:0001a488       ??_C@_0BF@OEGKMHKJ@PostRFInitialization?$AA@ 1001b488     rtmp_init.obj
 0001:0001a4a0       ??_C@_0BH@DHLGCAAF@?$DM?9?9?5NICInitializeAsic?6?$AA@ 1001b4a0     rtmp_init.obj
 0001:0001a4b8       ??_C@_0BA@NIANNCKD@buseEfuse?5?$DN?5?$CFd?6?$AA@ 1001b4b8     rtmp_init.obj
 0001:0001a4c8       ??_C@_0P@FBPDPAL@Set?5Radio?5Off?6?$AA@ 1001b4c8     rtmp_init.obj
 0001:0001a4d8       ??_C@_0BC@LPJHJHGI@BBP?5version?5?$DN?5?$CFd?6?$AA@ 1001b4d8     rtmp_init.obj
 0001:0001a4ec       ??_C@_0BN@KHEHKLMH@MAC_CSR0?5?5?$FL?5Ver?3Rev?$DN0x?$CF08x?$FN?6?$AA@ 1001b4ec     rtmp_init.obj
 0001:0001a50c       ??_C@_0BH@JNENNMJC@?9?9?$DO?5NICInitializeAsic?6?$AA@ 1001b50c     rtmp_init.obj
 0001:0001a524       ??_C@_0DP@OFJCBOEH@?$DM?$DN?$DN?$DN?$DN?5NICLoadFirmware?$CIWrite?5Firm@ 1001b524     rtmp_init.obj
 0001:0001a564       ??_C@_0CL@JGLJOCGF@NICLoadFirmware?5Failed?$CB?5?$CIntStatu@ 1001b564     rtmp_init.obj
 0001:0001a590       ??_C@_0BB@PJNJINLK@MAC_CSR0?5?$DN?50x?$CFx?6?$AA@ 1001b590     rtmp_init.obj
 0001:0001a5a8       ??_C@_0FC@KLIBEFGN@NICLoadFirmware?3?5Ver?$DN?$CFd?0?5local?5V@ 1001b5a8     rtmp_init.obj
 0001:0001a600       ??_C@_0EA@PGMHJBNG@NICLoadFirmware?3?5Ver?$DN?$CFd?0?5local?5V@ 1001b600     rtmp_init.obj
 0001:0001a640       ??_C@_0BN@FMPJLHFP@CRC?5OK?$DN0x?$CF02x?50x?$CF02x?5ver?$DN?$CFd?6?$AA@ 1001b640     rtmp_init.obj
 0001:0001a660       ??_C@_0GH@JGEKOIJM@NICLoadFirmware?3?5CRC?5?$DN?50x?$CF02x?50x@ 1001b660     rtmp_init.obj
 0001:0001a6c8       ??_C@_0BL@GFGNPMFI@NdisMapFile?5FileLength?$DN?$CFd?6?$AA@ 1001b6c8     rtmp_init.obj
 0001:0001a6e8       ??_C@_0FE@NBNKIGIH@NICLoadFirmware?3?5NdisOpenFile?$CIrt@ 1001b6e8     rtmp_init.obj
 0001:0001a73c       ??_C@_0L@KBGDKEEF@rt2870?4bin?$AA@ 1001b73c     rtmp_init.obj
 0001:0001a748       ??_C@_0BH@JFDPKNGF@?$DN?$DN?$DN?$DN?$DO?5NICFirmwareMode?6?$AA@ 1001b748     rtmp_init.obj
 0001:0001a760       ??_C@_0BK@MHDDAMDP@?$DN?$DN?$DN?$DN?$DO?5NICFirmwareMode?$DN?$CFx?6?$AA@ 1001b760     rtmp_init.obj
 0001:0001a77c       ??_C@_0CN@IFCGGFNK@NICLoadFirmware?0?5Invalid?5MAC?5Ver@ 1001b77c     rtmp_init.obj
 0001:0001a7ac       ??_C@_0BN@JHIJEKBJ@?$CFs?3?5EEPROM?$FL0x?$CF02X?$FN?5?$DN?50x?$CF02X?6?$AA@ 1001b7ac     rtmp_init.obj
 0001:0001a7cc       ??_C@_0BF@FMEIFCPO@?$CFs?3?5FileLength?5?$DN?5?$CFd?6?$AA@ 1001b7cc     rtmp_init.obj
 0001:0001a7e8       ??_C@_0EP@IMBEFFLI@?$CFs?3?5?$CK?$CK?$CK?$CK?$CK?$CK?$CK?$CK?$CK?$CK?$CK?$CK?$CK?$CK?$CK?$CK?$CK?$CK?$CK?$CK?$CK?$CK?$CK?$CK?$CK?$CK?$CK?$CK@ 1001b7e8     rtmp_init.obj
 0001:0001a838       ??_C@_0CN@JHNCHDKE@?$CFs?3?5NdisOpenFile?5?$CIRT3xUsbEeprom?4@ 1001b838     rtmp_init.obj
 0001:0001a868       ??_C@_0BI@GMBKIMOJ@LoadExternalEEPROMImage?$AA@ 1001b868     rtmp_init.obj
 0001:0001a880       ??_C@_0BC@FFMOBLFK@RT3xUsbEeprom?4bin?$AA@ 1001b880     rtmp_init.obj
 0001:0001a894       ??_C@_0BB@PHIIJONB@?$DM?9?9?5UserCfgInit?6?$AA@ 1001b894     rtmp_init.obj
 0001:0001a8a8       ??_C@_0M@HGGDHBHP@UserCfgInit?$AA@ 1001b8a8     rtmp_init.obj
 0001:0001a8b4       ??_C@_0CG@PDPIIEAA@?9?9?$DO?5UserCfgInit?4?5BACapability?5?$DN?5@ 1001b8b4     rtmp_init.obj
 0001:0001a8dc       ??_C@_0CF@CNMNLCOM@?9?9?$DOsizeof?$CIFRAME_ADDBA_RSP?$CJ?$DN?$CFd?0?5?5@ 1001b8dc     rtmp_init.obj
 0001:0001a904       ??_C@_0BB@DCGADJNJ@?9?9?$DO?5UserCfgInit?6?$AA@ 1001b904     rtmp_init.obj
 0001:0001a918       ??_C@_0DE@CCCAEEKK@RTMPSetTimer?5failed?0?5Timer?5hasn?8@ 1001b918     rtmp_init.obj
 0001:0001a94c       ??_C@_0DI@GHCOIHIK@NdisMCancelTimer?5failed?0?5Timer?5h@ 1001b94c     rtmp_init.obj
 0001:0001a984       ??_C@_0DE@KKIECLAA@RTMPSetLED?3?3Mode?$DN?$CFd?0HighByte?$DN0x?$CF@ 1001b984     rtmp_init.obj
 0001:0001a9b8       ??_C@_0BP@LEONMOCE@RTMPSetLED?3?3Unknown?5Status?5?$CFd?6?$AA@ 1001b9b8     rtmp_init.obj
 0001:0001a9d8       ??_C@_0BN@HBHBMLBJ@?$CFs?3?5LED_WPS_MODE10_TURN_OFF?6?$AA@ 1001b9d8     rtmp_init.obj
 0001:0001a9f8       ??_C@_0BK@HCCPHCOE@?$CFs?3?5LED_WPS_MODE10_FLASH?6?$AA@ 1001b9f8     rtmp_init.obj
 0001:0001aa14       ??_C@_0BM@HCEECIOL@?$CFs?3?5LED_WPS_MODE10_TURN_ON?6?$AA@ 1001ba14     rtmp_init.obj
 0001:0001aa30       ??_C@_0DB@HIHJGBAN@?$CFs?3?5LINK_STATUS_NORMAL_CONNECTIO@ 1001ba30     rtmp_init.obj
 0001:0001aa64       ??_C@_0DE@PCJAOLOC@?$CFs?3?5LINK_STATUS_NORMAL_CONNECTIO@ 1001ba64     rtmp_init.obj
 0001:0001aa98       ??_C@_0BO@KOMGPIK@?$CFs?3?5LED_WPS_TURN_ON_BLUE_LED?6?$AA@ 1001ba98     rtmp_init.obj
 0001:0001aab8       ??_C@_0CP@CNFBIBPA@?$CFs?3?5LED_WPS_SUCCESS?5?$CIIncorrect?5L@ 1001bab8     rtmp_init.obj
 0001:0001aae8       ??_C@_0DA@GDCNIFBD@?$CFs?3?5LED_WPS_SUCCESS?5?$CILINK_STATUS@ 1001bae8     rtmp_init.obj
 0001:0001ab18       ??_C@_0EA@NFJOHOD@?$CFs?3?5LED_WPS_SUCCESS?5?$CILINK_STATUS@ 1001bb18     rtmp_init.obj
 0001:0001ab58       ??_C@_0DN@FAPMHJBH@?$CFs?3?5LED_WPS_SUCCESS?5?$CILINK_STATUS@ 1001bb58     rtmp_init.obj
 0001:0001ab98       ??_C@_0CG@MJOBOEIC@?$CFs?3?5LED_WPS_SESSION_OVERLAP_DETE@ 1001bb98     rtmp_init.obj
 0001:0001abc0       ??_C@_0BD@BHHHBJHC@?$CFs?3?5LED_WPS_ERROR?6?$AA@ 1001bbc0     rtmp_init.obj
 0001:0001abd4       ??_C@_0L@LHOBCDB@RTMPSetLED?$AA@ 1001bbd4     rtmp_init.obj
 0001:0001abe0       ??_C@_0BE@BFGNJMED@?$DM?$DN?$DN?5RTMPEnableRxTx?6?$AA@ 1001bbe0     rtmp_init.obj
 0001:0001abf4       ??_C@_0DC@JFGJKEGF@UsbCfg?4field?4RxBulkAggLmt?$DN?$CFd?0?5Us@ 1001bbf4     rtmp_init.obj
 0001:0001ac28       ??_C@_0CD@CPEEBDBG@?$DM?$DN?$DN?5WRITE?5DMA?5offset?50x208?5?$DN?50x?$CF@ 1001bc28     rtmp_init.obj
 0001:0001ac4c       ??_C@_0CC@OKNNFFHF@?$DM?$DN?$DN?5READ?5DMA?5offset?50x208?5?$DN?50x?$CFx@ 1001bc4c     rtmp_init.obj
 0001:0001ac70       ??_C@_0BE@JKIMHKGH@?$DN?$DN?$DO?5RTMPEnableRxTx?6?$AA@ 1001bc70     rtmp_init.obj
 0001:0001ac84       ??_C@_0CO@GMHAPCPK@RTMPReadSafelyRemoveFlag?0?5Safely@ 1001bc84     rtmp_init.obj
 0001:0001acb4       ??_C@_1CA@EGHOFHML@?$AAS?$AAa?$AAf?$AAe?$AAl?$AAy?$AAR?$AAe?$AAm?$AAo?$AAv?$AAe?$AAO?$AAf?$AAf?$AA?$AA@ 1001bcb4     rtmp_init.obj
 0001:0001acd4       ??_C@_0BJ@PFBFHACM@?$DN?$DN?$DO?5RTMPPrepareCTSFrame?6?$AA@ 1001bcd4     rtmp_init.obj
 0001:0001acf0       ??_C@_0DD@PAFLMHNH@RTMPSetMessageEvent?0?5Indicate?5Ev@ 1001bcf0     rtmp_init.obj
 0001:0001ad24       ??_C@_0CD@IGPEFKPC@RTMPSetMessageEvent?0?5Message?5ful@ 1001bd24     rtmp_init.obj
 0001:0001ad48       ??_C@_03OFAPEBGM@?$CFs?6?$AA@ 1001bd48     rtmp_init.obj
 0001:0001ad4c       ??_C@_0N@GFACJJGM@AsicRadioOff?$AA@ 1001bd4c     rtmp_init.obj
 0001:0001ad5c       ??_C@_0CM@NPFBJLAJ@PSM?5?3ASIC?50x31?5WakeUp?5Cmd?5may?5Fa@ 1001bd5c     rtmp_init.obj
 0001:0001ad88       ??_C@_0CC@MOADAFIO@PSM?5?3WakeUp?5Cmd?5Failed?0?5retry?5?$CFd@ 1001bd88     rtmp_init.obj
 0001:0001afb0       ??_C@_0BO@GKEDAOEO@?$DM?$DN?$DN?$DN?$DN?5DriverEntry?0?5Status?$DN?$CFx?6?$AA@ 1001bfb0     rtmp_main.obj
 0001:0001afd0       ??_C@_0CC@OMMKENOM@Calling?5NdisMRegisterMiniport?4?4?4@ 1001bfd0     rtmp_main.obj
 0001:0001aff4       ??_C@_0DE@ILKGMENG@?$DM?$DN?$DN?$DN?$DN?5DriverEntry?5failed?5to?5Init@ 1001bff4     rtmp_main.obj
 0001:0001b028       ??_C@_0CI@DNBGGCBB@Build?5Date?3?5Dec?5?54?52009?5Time?3?517@ 1001c028     rtmp_main.obj
 0001:0001b050       ??_C@_0DC@OEKGBEFC@?$DN?$DN?$DN?$DN?$DN?$DN?$DN?$DN?$DN?$DN?$DN?$DN?$DN?$DN?$DN?$DN?$DN?$DN?$DN?$DN?$DN?$DN?$DN?$DN?$DN?$DN?$DN?$DN?$DN?$DN?$DN?$DN@ 1001c050     rtmp_main.obj
 0001:0001b084       ??_C@_0BD@ENJGEEKK@?$DN?$DN?$DN?$DN?$DO?5DriverEntry?6?$AA@ 1001c084     rtmp_main.obj
 0001:0001b098       ??_C@_0CB@IJCDNANJ@?$DM?$DN?$DN?$DN?$DN?5RTMPInitialize?0?5Status?$DN?$CFx?6@ 1001c098     rtmp_main.obj
 0001:0001b0bc       ??_C@_0CE@LPPMBONH@pAd?9?$DOCommonCfg?4NumOfBulkInIRP?5?$DN?$CF@ 1001c0bc     rtmp_main.obj
 0001:0001b0e0       ??_C@_0BD@EOHFKIGJ@RTUSBBulkReceive?$CB?6?$AA@ 1001c0e0     rtmp_main.obj
 0001:0001b0f8       ??_C@_1FM@JPJIBOOC@?$AAC?$AA?3?$AA?2?$AAW?$AAi?$AAn?$AAC?$AAE?$AA6?$AA?4?$AA0?$AA?2?$AAN?$AAe?$AAw?$AA?2?$AAR?$AAT?$AA2?$AA8?$AA7?$AA0?$AA_?$AAv?$AA1?$AA?4?$AA4?$AA?4?$AA9?$AA?4?$AA0?$AA?2@ 1001c0f8     rtmp_main.obj
 0001:0001b154       ??_C@_0CI@BFPAOAGH@Create?5Threads?5failed?0?5Status?$FL?$DN0@ 1001c154     rtmp_main.obj
 0001:0001b17c       ??_C@_0CC@FDCOMGPL@MlmeInit?5failed?0?5Status?$FL?$DN0x?$CF08x?$FN@ 1001c17c     rtmp_main.obj
 0001:0001b1a0       ??_C@_0BM@NJJFCGIK@2070?3?5Remove?511n?5parameter?6?$AA@ 1001c1a0     rtmp_main.obj
 0001:0001b1bc       ??_C@_0BO@LCAOMCND@2pAd?9?$DOCommonCfg?4PhyMode?$FL?$DN?$CFd?$FN?6?$AA@ 1001c1bc     rtmp_main.obj
 0001:0001b1dc       ??_C@_0CO@JBPFLHDN@NICReadRegParameters?5failed?0?5Sta@ 1001c1dc     rtmp_main.obj
 0001:0001b20c       ??_C@_0DK@CHFMMCPC@pAd?9?$DORepositBssidList?4pBssidList@ 1001c20c     rtmp_main.obj
 0001:0001b248       ??_C@_0DF@LEEABLAA@?$CK?$CK?$CK?$CK?5Can?5not?5allocate?5memory?5for@ 1001c248     rtmp_main.obj
 0001:0001b280       ??_C@_0BL@PKLGKDIC@USB_InterfaceStart?5failed?6?$AA@ 1001c280     rtmp_main.obj
 0001:0001b29c       ??_C@_0CO@GCEAKGBJ@RTMPInitAdapterBlock?5failed?0?5Sta@ 1001c29c     rtmp_main.obj
 0001:0001b2cc       ??_C@_0BP@MLFMABFF@NdisMGetDeviceProperty?5failed?6?$AA@ 1001c2cc     rtmp_main.obj
 0001:0001b2ec       ??_C@_0CP@LFACBFEF@RTMPAllocAdapterBlock?5failed?0?5St@ 1001c2ec     rtmp_main.obj
 0001:0001b31c       ??_C@_0CF@BKLPFPFO@RTMPAllocAdapterBlock?5Sizeof?$FL?5?$DN?5@ 1001c31c     rtmp_main.obj
 0001:0001b344       ??_C@_0CM@FOFIOPBB@Expected?5media?5?$CI?$CFx?$CJ?5is?5not?5in?5Me@ 1001c344     rtmp_main.obj
 0001:0001b370       ??_C@_0BG@NIGEMMBH@?$DN?$DN?$DN?$DN?$DO?5RTMPInitialize?6?$AA@ 1001c370     rtmp_main.obj
 0001:0001b388       ??_C@_0BI@PPPKMGJG@?$DM?$DN?$DN?$DN?$DN?5RTMPCheckForHang?6?$AA@ 1001c388     rtmp_main.obj
 0001:0001b3a0       ??_C@_0DN@MKHJFMDH@Packet?$CIs?$CJ?5are?5pended?5for?5a?5while@ 1001c3a0     rtmp_main.obj
 0001:0001b3e0       ??_C@_0BI@NBHGOOHL@?$DN?$DN?$DN?$DN?$DO?5RTMPCheckForHang?6?$AA@ 1001c3e0     rtmp_main.obj
 0001:0001b3f8       ??_C@_0BA@LJBIDOBK@?$DM?$DN?$DN?$DN?$DN?5RTMPHalt?6?$AA@ 1001c3f8     rtmp_main.obj
 0001:0001b408       ??_C@_0CL@JKGIAEDF@Halt?5wait?5for?5SCAN_CHANNEL_IN_PR@ 1001c408     rtmp_main.obj
 0001:0001b434       ??_C@_0CJ@BOGICMLC@Halt?5wait?5for?5RESET_PIPE_IN_PROG@ 1001c434     rtmp_main.obj
 0001:0001b460       ??_C@_0BA@BAJOCMCN@PendingRx?5?$DN?5?$CFd?6?$AA@ 1001c460     rtmp_main.obj
 0001:0001b470       ??_C@_0CM@LCNDGKAE@Halt?5wait?5for?5MlmeThread?$CB?$CB?$CB?$FLQueu@ 1001c470     rtmp_main.obj
 0001:0001b49c       ??_C@_0BO@KLPONHN@Halt?5wait?5for?5hJunkThread?$CB?$CB?$CB?6?$AA@ 1001c49c     rtmp_main.obj
 0001:0001b4bc       ??_C@_0CP@FCPGJNKN@Halt?5wait?5for?5ControlThread?$CB?$CB?$CB?$FLQ@ 1001c4bc     rtmp_main.obj
 0001:0001b4ec       ??_C@_0BD@ELKKCIOH@Terminate?5Threads?6?$AA@ 1001c4ec     rtmp_main.obj
 0001:0001b500       ??_C@_0CP@JFLKGALI@pAd?9?$DORepositBssidList?4pBssidList@ 1001c500     rtmp_main.obj
 0001:0001b530       ??_C@_0DH@KNMLJDHF@RTMPHalt?3?3?5Device?5has?5been?5remov@ 1001c530     rtmp_main.obj
 0001:0001b568       ??_C@_0BA@GAOOHNHL@?$DN?$DN?$DN?$DN?$DO?5RTMPHalt?6?$AA@ 1001c568     rtmp_main.obj
 0001:0001b578       ??_C@_0P@LEBEILCN@?$DM?9?9?9RTMPReset?6?$AA@ 1001c578     rtmp_main.obj
 0001:0001b588       ??_C@_0P@DCALPAIG@?9?9?9?$DORTMPReset?6?$AA@ 1001c588     rtmp_main.obj
 0001:0001b598       ??_C@_0BI@NBOMLCPL@?$DM?$DN?$DN?$DN?$DN?5RTMPTransferData?6?$AA@ 1001c598     rtmp_main.obj
 0001:0001b5b0       ??_C@_0BI@PPGAJKBG@?$DN?$DN?$DN?$DN?$DO?5RTMPTransferData?6?$AA@ 1001c5b0     rtmp_main.obj
 0001:0001b5c8       ??_C@_0BK@MOOEFMFE@?$DM?$DN?$DN?$DN?$DN?5RTMPPnPEventNotify?6?$AA@ 1001c5c8     rtmp_main.obj
 0001:0001b5e4       ??_C@_0CP@GPELIKKA@RTMPPnPEventNotify?3?5unsupported?5@ 1001c5e4     rtmp_main.obj
 0001:0001b614       ??_C@_0CO@CFIHJMCN@RTMPPnPEventNotify?3?5NdisPowerPro@ 1001c614     rtmp_main.obj
 0001:0001b644       ??_C@_0CN@MLNPNADH@RTMPPnPEventNotify?3?5NdisPowerPro@ 1001c644     rtmp_main.obj
 0001:0001b674       ??_C@_0DL@EJJFAAF@RTMPPnPEventNotify?3?5NdisDevicePn@ 1001c674     rtmp_main.obj
 0001:0001b6b0       ??_C@_0DH@GADDADJI@RTMPPnPEventNotify?3?5NdisDevicePn@ 1001c6b0     rtmp_main.obj
 0001:0001b6e8       ??_C@_0BK@BAIBFHID@?$DN?$DN?$DN?$DN?$DO?5RTMPPnPEventNotify?6?$AA@ 1001c6e8     rtmp_main.obj
 0001:0001b704       ??_C@_0BC@OCCJCLCM@?$DM?$DN?$DN?$DN?$DN?5MPShutdown?6?$AA@ 1001c704     rtmp_main.obj
 0001:0001b718       ??_C@_0BC@HBBKLIBG@?$DN?$DN?$DN?$DN?$DO?5MPShutdown?6?$AA@ 1001c718     rtmp_main.obj
 0001:0001b72c       ??_C@_0CO@KMCPLDLJ@?$CK?$CK?$CK?$CK?$CK?$CK?$CK?$CK?$CK?5Junk?5Thread?5Terminated@ 1001c72c     rtmp_main.obj
 0001:0001b75c       ??_C@_0BG@EIPOHEHI@Junk?5Event?5Triggered?6?$AA@ 1001c75c     rtmp_main.obj
 0001:0001b774       ??_C@_0BD@OKGCBEFK@Junk?5Thread?5Start?6?$AA@ 1001c774     rtmp_main.obj
 0001:0001b988       ??_C@_0BH@MJMAGBCI@Calculated?5MIC?5value?5?$DN?$AA@ 1001c988     rtmp_tkip.obj
 0001:0001b9a0       ??_C@_0BB@DICCCLEK@Orig?5MIC?5value?5?$DN?$AA@ 1001c9a0     rtmp_tkip.obj
 0001:0001b9b4       ??_C@_0BE@CBHOODBL@?$CB?5TKIP?5MIC?5Error?5?$CB?6?$AA@ 1001c9b4     rtmp_tkip.obj
 0001:0001b9c8       ??_C@_0CF@BIOAILID@RTMPSoftEncryptTKIP?5Encrypt?5done@ 1001c9c8     rtmp_tkip.obj
 0001:0001b9f0       ??_C@_0DG@JNFKCOBK@CCX?9MFP?3?5Append?5MHDRIE?5behind?5th@ 1001c9f0     rtmp_tkip.obj
 0001:0001ba28       ??_C@_0DC@LDPGLIDJ@RTMPSoftEncryptTKIP?$CB?5?$CIIncorrect?5@ 1001ca28     rtmp_tkip.obj
 0001:0001ba5c       ??_C@_0DO@OMDCJHCC@RTMPSoftEncryptTKIP?5failed?$CB?5?$CIKey@ 1001ca5c     rtmp_tkip.obj
 0001:0001ba9c       ??_C@_0CE@HJOKLGPO@RTMPSoftDecryptTKIP?5Decrypt?5done@ 1001ca9c     rtmp_tkip.obj
 0001:0001bac0       ??_C@_0CH@KIIEBHOI@RTMPSoftDecryptTKIP?0?5invalid?5MHD@ 1001cac0     rtmp_tkip.obj
 0001:0001bae8       ??_C@_0DD@GEAOAEMJ@RTMPSoftDecryptTKIP?5failed?$CB?5?$CIWEP@ 1001cae8     rtmp_tkip.obj
 0001:0001bb1c       ??_C@_0DO@CONJGANN@RTMPSoftDecryptTKIP?5failed?$CB?5?$CIKey@ 1001cb1c     rtmp_tkip.obj
 0001:0001bb5c       ??_C@_0DJ@KDBJNPHK@RTMPSoftDecryptTKIP?5failed?$CB?5?$CIInc@ 1001cb5c     rtmp_tkip.obj
 0001:0001bb98       ??_C@_0CD@HINLBHHL@RTMPSoftEncryptAES?5Encrypt?5done?$CB@ 1001cb98     rtmp_tkip.obj
 0001:0001bbbc       ??_C@_0DB@GMBKMJPM@RTMPSoftEncryptAES?$CB?5?$CIIncorrect?5d@ 1001cbbc     rtmp_tkip.obj
 0001:0001bbf0       ??_C@_0DN@PNPJNGAG@RTMPSoftEncryptAES?5failed?$CB?5?$CIKeyI@ 1001cbf0     rtmp_tkip.obj
 0001:0001bc30       ??_C@_0CD@MBLFPLBB@RTMPSoftDecryptAES?5Decrypt?5done?$CB@ 1001cc30     rtmp_tkip.obj
 0001:0001bc54       ??_C@_0CK@PAGKAPFG@RTMPSoftDecryptAES?0?5WEP?5Data?5MIC@ 1001cc54     rtmp_tkip.obj
 0001:0001bc80       ??_C@_0DL@FCMIAKLL@RTMPSoftDecryptAES?5failed?$CB?$CIKeyID@ 1001cc80     rtmp_tkip.obj
 0001:0001bcbc       ??_C@_0DI@OKDFOOCM@RTMPSoftDecryptAES?5failed?$CB?5?$CIInco@ 1001ccbc     rtmp_tkip.obj
 0001:0001bcf8       ??_C@_1FM@NEHKBGLG@?$AAC?$AA?3?$AA?2?$AAW?$AAi?$AAn?$AAC?$AAE?$AA6?$AA?4?$AA0?$AA?2?$AAN?$AAe?$AAw?$AA?2?$AAR?$AAT?$AA2?$AA8?$AA7?$AA0?$AA_?$AAv?$AA1?$AA?4?$AA4?$AA?4?$AA9?$AA?4?$AA0?$AA?2@ 1001ccf8     rtmp_tkip.obj
 0001:0001bd54       ??_C@_0CH@FHOJIOKK@RTMPSoftEncryptMgmtAES?5Encrypt?5d@ 1001cd54     rtmp_tkip.obj
 0001:0001bd7c       ??_C@_0BG@HNBJBPLM@Set?5AES?5key?5failed?5?$CB?6?$AA@ 1001cd7c     rtmp_tkip.obj
 0001:0001bd94       ??_C@_0DC@HGELGCFP@RTMPSoftEncryptMgmtAES?$CB?5?$CIIncorre@ 1001cd94     rtmp_tkip.obj
 0001:0001bdc8       ??_C@_0EB@HGHHALPB@RTMPSoftEncryptMgmtAES?5failed?$CB?5?$CI@ 1001cdc8     rtmp_tkip.obj
 0001:0001be0c       ??_C@_0CH@FFEFGKAN@RTMPSoftDecryptMgmtAES?5Decrypt?5d@ 1001ce0c     rtmp_tkip.obj
 0001:0001be34       ??_C@_0CO@PMDIBKKE@RTMPSoftDecryptMgmtAES?0?5WEP?5Data@ 1001ce34     rtmp_tkip.obj
 0001:0001be64       ??_C@_0DP@MIFILIOB@RTMPSoftDecryptMgmtAES?5failed?$CB?$CIK@ 1001ce64     rtmp_tkip.obj
 0001:0001bea4       ??_C@_0DJ@FLCKIDDG@RTMPSoftDecryptMgmtAES?5failed?$CB?5?$CI@ 1001cea4     rtmp_tkip.obj
 0001:0001c0e0       ??_C@_0CG@MHBIIBFI@CKIP_KP_ON?5?9?9?5?$CB?5WEP?5Data?5CRC?5Err@ 1001d0e0     rtmp_wep.obj
 0001:0001c108       ??_C@_0BI@BNDFFBGF@?$CB?5WEP?5Data?5CRC?5Error?5?$CB?6?$AA@ 1001d108     rtmp_wep.obj
 0001:0001c320       ??_C@_1FO@FFACIBBA@?$AAC?$AA?3?$AA?2?$AAW?$AAi?$AAn?$AAC?$AAE?$AA6?$AA?4?$AA0?$AA?2?$AAN?$AAe?$AAw?$AA?2?$AAR?$AAT?$AA2?$AA8?$AA7?$AA0?$AA_?$AAv?$AA1?$AA?4?$AA4?$AA?4?$AA9?$AA?4?$AA0?$AA?2@ 1001d320     rtusb_bulk.obj
 0001:0001c380       ??_C@_0HP@MIKBFDND@h1?91?5?5TmpBulkPos?5?$DN?5?$CFd?0?5TmpBulkEn@ 1001d380     rtusb_bulk.obj
 0001:0001c400       ??_C@_0HN@FENCCGGG@h2?5?5TmpBulkPos?5?$DN?5?$CFd?0?5TmpBulkEndP@ 1001d400     rtusb_bulk.obj
 0001:0001c480       ??_C@_0CN@PAFOHEMP@CONVERT_2_AMSDU_HEADER?5?$DN?500?3?5?$CFx?5@ 1001d480     rtusb_bulk.obj
 0001:0001c4b0       ??_C@_0BN@MODLDGD@?$DM?9?9?9RTUSBBulkOutDataPacket?5?6?$AA@ 1001d4b0     rtusb_bulk.obj
 0001:0001c4d0       ??_C@_0BO@DKMCJLE@No?5Pending?0?5Irp?5?$CFx?0?5Index?5?$CFd?6?$AA@ 1001d4d0     rtusb_bulk.obj
 0001:0001c4f0       ??_C@_0EM@MEBMDBJN@RTUSBBulkOutDataPacket?5IoCallDri@ 1001d4f0     rtusb_bulk.obj
 0001:0001c53c       ??_C@_0CB@JLMBIMED@RT2870?3?5USB_TRANSFER?5is?5NULL?$CB?$CB?$CB?6@ 1001d53c     rtusb_bulk.obj
 0001:0001c560       ??_C@_0CB@IFOMLPFF@?$CFx?5?5?$CFx?5?5?$CFx?5?5?$CFx?5?5?$CFx?5?5?$CFx?5?5?$CFx?5?5?$CFx?5?6@ 1001d560     rtusb_bulk.obj
 0001:0001c588       ??_C@_0FM@NGAHNOKO@h?9e2?5?5USBDMATxPktLen?5?$DN?$DN?50?5?9?9?$DO?5Si@ 1001d588     rtusb_bulk.obj
 0001:0001c5e8       ??_C@_0FG@BNBHFOKI@RTUSBBulkOutDataPacket?5?9?9?$DO?5COPY?5@ 1001d5e8     rtusb_bulk.obj
 0001:0001c640       ??_C@_0CL@OJNKCAHK@allzero?5?3?5?$CFx?5?5?$CFx?5?5?$CFx?5?5?$CFx?5?5?$CFx?5?5?$CFx@ 1001d640     rtusb_bulk.obj
 0001:0001c66c       ??_C@_0CE@PGEKMKFL@?$DM?9?9?9RTUSBBulkOutDataPacketComple@ 1001d66c     rtusb_bulk.obj
 0001:0001c690       ??_C@_0FH@NEDOBMLP@BulkOutComplete?$CISTATUS_CANCELLED@ 1001d690     rtusb_bulk.obj
 0001:0001c6e8       ??_C@_0BM@KOOHGLKG@?$DM?9?9?9RTUSBBulkOutNullFrame?5?6?$AA@ 1001d6e8     rtusb_bulk.obj
 0001:0001c708       ??_C@_0EL@LGOAFBND@RTUSBBulkOutNullFrame?5IoCallDriv@ 1001d708     rtusb_bulk.obj
 0001:0001c754       ??_C@_0BM@NJPHNGFG@?9?9?9?$DORTUSBBulkOutNullFrame?5?6?$AA@ 1001d754     rtusb_bulk.obj
 0001:0001c770       ??_C@_0CD@IEOAJDHL@?$DM?9?9?9RTUSBBulkOutNullFrameComplet@ 1001d770     rtusb_bulk.obj
 0001:0001c794       ??_C@_0BM@IHGAMGPL@Bulk?5Out?5Null?5Frame?5Failed?6?$AA@ 1001d794     rtusb_bulk.obj
 0001:0001c7b0       ??_C@_0CD@NAMCKGKO@?9?9?9?$DORTUSBBulkOutNullFrameComplet@ 1001d7b0     rtusb_bulk.obj
 0001:0001c7d4       ??_C@_0BL@ILIJPNBA@?$DM?9?9?9RTUSBBulkOutRTSFrame?5?6?$AA@ 1001d7d4     rtusb_bulk.obj
 0001:0001c7f0       ??_C@_0EK@JBAEPNAD@RTUSBBulkOutRTSFrame?5IoCallDrive@ 1001d7f0     rtusb_bulk.obj
 0001:0001c83c       ??_C@_0BL@JMAEJLBB@?9?9?9?$DORTUSBBulkOutRTSFrame?5?6?$AA@ 1001d83c     rtusb_bulk.obj
 0001:0001c858       ??_C@_0CC@LNJEIKJP@?$DM?9?9?9RTUSBBulkOutRTSFrameComplete@ 1001d858     rtusb_bulk.obj
 0001:0001c87c       ??_C@_0CC@EBPGHGGJ@?9?9?9?$DORTUSBBulkOutRTSFrameComplete@ 1001d87c     rtusb_bulk.obj
 0001:0001c8a0       ??_C@_0BN@BIHJLFKO@?$DM?9?9?9RTUSBBulkOutMLMEPacket?5?6?$AA@ 1001d8a0     rtusb_bulk.obj
 0001:0001c8c0       ??_C@_0EM@FIDHLONF@RTUSBBulkOutMLMEPacket?5IoCallDri@ 1001d8c0     rtusb_bulk.obj
 0001:0001c910       ??_C@_0HK@LCCAOENE@RTUSBBulkOutMLME?3?3PrioRingFirstI@ 1001d910     rtusb_bulk.obj
 0001:0001c98c       ??_C@_0CE@MJBECIHE@?$DM?9?9?9RTUSBBulkOutMLMEPacketComple@ 1001d98c     rtusb_bulk.obj
 0001:0001c9b0       ??_C@_0II@NHBAPID@RTUSBBulkOutMLMEPacketComplete?3?3@ 1001d9b0     rtusb_bulk.obj
 0001:0001ca38       ??_C@_1LM@DGIIDKDA@?$AAR?$AAT?$AA2?$AA8?$AA7?$AA0?$AA?3?$AA?5?$AA?$CK?$AA?$CK?$AA?$CK?$AAD?$AAu?$AAm?$AAp?$AA?3?$AA?5?$AAA?$AAf?$AAt?$AAe?$AAr?$AA?5?$AA?3?$AA?5?$AAR?$AAT?$AAU?$AAS?$AAB?$AAE?$AAn@ 1001da38     rtusb_bulk.obj
 0001:0001caf8       ??_C@_1LM@NKJIMFHB@?$AAR?$AAT?$AA2?$AA8?$AA7?$AA0?$AA?3?$AA?5?$AA?$CK?$AA?$CK?$AA?$CK?$AAD?$AAu?$AAm?$AAp?$AA?3?$AA?5?$AAB?$AAe?$AAf?$AAo?$AAr?$AAe?$AA?3?$AA?5?$AAR?$AAT?$AAU?$AAS?$AAB?$AAE?$AAn@ 1001daf8     rtusb_bulk.obj
 0001:0001cbb4       ??_C@_0CD@BDGNEPAH@Bulk?5Out?5MLME?5Failed?4?5Status?5?$DN?5?$CF@ 1001dbb4     rtusb_bulk.obj
 0001:0001cbd8       ??_C@_0BJ@NNDMBPEG@?$DM?9?9?9RTUSBBulkOutPsPoll?5?6?$AA@ 1001dbd8     rtusb_bulk.obj
 0001:0001cbf8       ??_C@_0EI@BDPKCLL@RTUSBBulkOutPsPoll?5IoCallDriver?5@ 1001dbf8     rtusb_bulk.obj
 0001:0001cc40       ??_C@_0CA@JAFMDLIB@?$DM?9?9?9RTUSBBulkOutPsPollComplete?6?$AA@ 1001dc40     rtusb_bulk.obj
 0001:0001cc60       ??_C@_0DB@CCPKNLIF@?9?9?9?$DORTUSBBulkOutPsPollComplete?5S@ 1001dc60     rtusb_bulk.obj
 0001:0001cc94       ??_C@_0BI@LPBJIB@Bulk?5Out?5PSPoll?5Failed?6?$AA@ 1001dc94     rtusb_bulk.obj
 0001:0001ccb0       ??_C@_0EG@GKDHPBIH@RTUSBBulkReceive?5IoCallDriver?5re@ 1001dcb0     rtusb_bulk.obj
 0001:0001ccf8       ??_C@_0DF@IFALOFHD@pRxContext?$FL?$CFd?$FN?5?4pRxContext?9?$DORead@ 1001dcf8     rtusb_bulk.obj
 0001:0001cd30       ??_C@_0CG@HLLELKMO@pRxContext?$FL?$CFd?$FN?5InUse?5?$DN?5?$CFd?4?4?5?5Ret@ 1001dd30     rtusb_bulk.obj
 0001:0001cd58       ??_C@_0DA@EFMPCDNF@pAd?9?$DONextRxBulkInPosition?5?$DN?50x?$CFx@ 1001dd58     rtusb_bulk.obj
 0001:0001cd88       ??_C@_0FD@NGEAOACK@?$DN?$DN?$DONextRxBulkInIndex?$DN0x?$CFx?0?5NextR@ 1001dd88     rtusb_bulk.obj
 0001:0001cddc       ??_C@_0BP@EPMILLCN@Bulk?5In?5Failed?4?5Status?5?$DN?50x?$CFx?6?$AA@ 1001dddc     rtusb_bulk.obj
 0001:0001cdfc       ??_C@_0CB@NNJKMMDI@IoCancelIrp?5RTUSBBulkRxComplete?6@ 1001ddfc     rtusb_bulk.obj
 0001:0001ce20       ??_C@_0CM@GEEMFPAO@RTUSBKickBulkOut?5return?9?9?9?$DOpAd?9?$DO@ 1001de20     rtusb_bulk.obj
 0001:0001ce4c       ??_C@_0BG@CAHADCAD@?9?9?9?$DORTUSBKickBulkOut?6?$AA@ 1001de4c     rtusb_bulk.obj
 0001:0001ce64       ??_C@_0BN@GDHDOJHH@?$DM?9?9?9CleanUpDataBulkOutQueue?6?$AA@ 1001de64     rtusb_bulk.obj
 0001:0001ce84       ??_C@_0BN@NOLJALNG@?9?9?9?$DOCleanUpDataBulkOutQueue?6?$AA@ 1001de84     rtusb_bulk.obj
 0001:0001cea4       ??_C@_0BN@IJLHHALC@?$DM?9?9?9CleanUpMLMEBulkOutQueue?6?$AA@ 1001dea4     rtusb_bulk.obj
 0001:0001cec4       ??_C@_0BN@DEHNJCBD@?9?9?9?$DOCleanUpMLMEBulkOutQueue?6?$AA@ 1001dec4     rtusb_bulk.obj
 0001:0001cee4       ??_C@_0CO@PBCKPAM@?$DM?9?9IoCancelIrp?5pTxContext?9?$DOpIrp?$FL@ 1001dee4     rtusb_bulk.obj
 0001:0001cf14       ??_C@_0CE@HHNPFMI@?9?9?$DOIoCancelIrp?5pTxContext?9?$DOpIrp?$FL@ 1001df14     rtusb_bulk.obj
 0001:0001cf38       ??_C@_0CO@JCBNEOHK@?$DM?9?9IoCancelIrp?5pTxContext?9?$DOpIrp?$FL@ 1001df38     rtusb_bulk.obj
 0001:0001cf68       ??_C@_0CE@LPMBJCKN@?9?9?$DOIoCancelIrp?5pTxContext?9?$DOpIrp?$FL@ 1001df68     rtusb_bulk.obj
 0001:0001cf8c       ??_C@_02JJDEPCGB@54?$AA@   1001df8c     rtusb_data.obj
 0001:0001cf90       ??_C@_02DEEDNHFK@48?$AA@   1001df90     rtusb_data.obj
 0001:0001cf94       ??_C@_02KPIPOMFB@36?$AA@   1001df94     rtusb_data.obj
 0001:0001cf98       ??_C@_02JMHLOEOE@24?$AA@   1001df98     rtusb_data.obj
 0001:0001cf9c       ??_C@_02DCIIBFLB@18?$AA@   1001df9c     rtusb_data.obj
 0001:0001cfa0       ??_C@_02MIGHPNDL@12?$AA@   1001dfa0     rtusb_data.obj
 0001:0001cfa4       ??_C@_01LAKCGALK@9?$AA@    1001dfa4     rtusb_data.obj
 0001:0001cfa8       ??_C@_01DHDKHMHF@6?$AA@    1001dfa8     rtusb_data.obj
 0001:0001d1b0       ??_C@_0CM@OKGHKGKF@Sniff2BytesFromNdisBuffer?$CIoffset@ 1001e1b0     rtusb_data.obj
 0001:0001d1e0       ??_C@_0EH@PHFANPFA@Drop?5Packet?5for?5CCX?5test?3?5NdisMS@ 1001e1e0     rtusb_data.obj
 0001:0001d228       ??_C@_0BI@HGBFLCFD@?$DO?$DO?$DO?5One?5Packet?5Pending?6?$AA@ 1001e228     rtusb_data.obj
 0001:0001d240       ??_C@_0ED@NEGKHJAG@RTMPSendPacket?5?9?$DO?5Enqueue?5Airone@ 1001e240     rtusb_data.obj
 0001:0001d284       ??_C@_0CF@OKLLCBGL@Infrastructure?5?9?$DO?5Enqueue?5one?5fr@ 1001e284     rtusb_data.obj
 0001:0001d2ac       ??_C@_0DC@MNPDMEGA@RTMPSendPacket?5QueIdx?5?$DN?5?$CFd?0?5StaC@ 1001e2ac     rtusb_data.obj
 0001:0001d2e0       ??_C@_0FH@OMANPLFO@Drop?5Packets?5in?5RTMPSendPacket?$CIU@ 1001e2e0     rtusb_data.obj
 0001:0001d338       ??_C@_0CF@NAOBINAP@Number?5of?5fragments?5include?5RTS?5@ 1001e338     rtusb_data.obj
 0001:0001d360       ??_C@_0EI@FGIEPOCI@RTMPSendPacket?9?$DOCannot?5find?5pEnt@ 1001e360     rtusb_data.obj
 0001:0001d3a8       ??_C@_0BF@GNHDENIC@?$DN?$DN?$DN?$DO?5RTMPSendPacket?6?$AA@ 1001e3a8     rtusb_data.obj
 0001:0001d3c0       ??_C@_0DE@OFNBLBBC@?9?9RTMPDeQueuePacket?5?$CFd?5queue?5ful@ 1001e3c0     rtusb_data.obj
 0001:0001d3f4       ??_C@_0BP@PECHPFME@NDIS_STATUS_ADAPTER_NOT_READY?6?$AA@ 1001e3f4     rtusb_data.obj
 0001:0001d414       ??_C@_0CC@ENBHKDHL@RESOURSE?5NOT?5ENOUGH?5pPacket?5?$DN?5?$CFX@ 1001e414     rtusb_data.obj
 0001:0001d438       ??_C@_0CP@BBDGDJCM@?9?9RTMPDeQueuePacket?5?$CFd?5reset?9in?9@ 1001e438     rtusb_data.obj
 0001:0001d468       ??_C@_0DE@PMMLONJB@?9?9RTMPDeQueuePacket?5?$CFd?5queue?5ful@ 1001e468     rtusb_data.obj
 0001:0001d49c       ??_C@_0CL@MFGAFFNH@?9?9?9?$DORTUSBFreeDescriptorRequest?$CI?$CJ@ 1001e49c     rtusb_data.obj
 0001:0001d4c8       ??_C@_0DC@ELCKMAIC@s3?5?9?9?$DO?5Cur?5?$DN?5?$CFd?0?5Next?5?$DN?5?$CFd?0Enext@ 1001e4c8     rtusb_data.obj
 0001:0001d4fc       ??_C@_0DC@MEHCOPJB@s2?5?9?9?$DO?5Cur?5?$DN?5?$CFd?0?5Next?5?$DN?5?$CFd?0Enext@ 1001e4fc     rtusb_data.obj
 0001:0001d530       ??_C@_0EF@NPOBJBGD@RTUSBFreeD?5s1?5?9?9?$DO?5CurWritePositi@ 1001e530     rtusb_data.obj
 0001:0001d578       ??_C@_0FK@PEIGPAEK@?$DM?9?9?9RejectPendingPackets?0?5Pendin@ 1001e578     rtusb_data.obj
 0001:0001d5d8       ??_C@_0FK@OHBCANO@?9?9?9?$DORejectPendingPackets?0?5Pendin@ 1001e5d8     rtusb_data.obj
 0001:0001d634       ??_C@_0BP@KOLEFIHD@Suspend?5MSDU?5transmission?5?4?4?4?6?$AA@ 1001e634     rtusb_data.obj
 0001:0001d654       ??_C@_0DD@CKMHGHHK@RTUSBResumeMsduTransmission?0?5R66@ 1001e654     rtusb_data.obj
 0001:0001d688       ??_C@_0BO@HNNCBLPD@Resume?5MSDU?5transmission?5?4?4?4?6?$AA@ 1001e688     rtusb_data.obj
 0001:0001d6a8       ??_C@_0CP@NBIGJBNN@RTMPWriteTxWI?3?5RFIC_3020?1RFIC_20@ 1001e6a8     rtusb_data.obj
 0001:0001d6d8       ??_C@_0CP@LNBACPBG@?$DO?$DO?$DO?$DO?$DO?5Chk?3?3?5dynamic?5BA?5?$DN?5?$CFd?0?5reg@ 1001e6d8     rtusb_data.obj
 0001:0001d708       ??_C@_0DL@FAPHJHLM@?$DO?$DO?$DO?$DO?$DO?5Chk?3?3?5dynamic?5BA?5interval?$DN@ 1001e708     rtusb_data.obj
 0001:0001d744       ??_C@_0CK@FFAANDB@?$DN?$DN?$DN?$DN?$DO?5QueueSel?5?$CB?$DN?5FIFO_EDCA?$DM?$DN?$DN?$DN?$DN@ 1001e744     rtusb_data.obj
 0001:0001d770       ??_C@_0BF@KDCDAHJM@RELASE?5NDIS?5PACKET?5?6?$AA@ 1001e770     rtusb_data.obj
 0001:0001d788       ??_C@_0FB@JAOHBPIG@MLME?5?9?5disassociate?5with?5current@ 1001e788     rtusb_data.obj
 0001:0001d7e0       ??_C@_0IA@JKPMFOA@Error?3?5Force?5multicast?5rate?5to?51@ 1001e7e0     rtusb_data.obj
 0001:0001d860       ??_C@_0IB@COAIPFNB@Error?3?5Force?5multicast?5rate?5to?52@ 1001e860     rtusb_data.obj
 0001:0001d8e4       ??_C@_0CL@MAGGOLHL@CCX?9MFP?3?5Data?0?5RTMPSoftEncryptTK@ 1001e8e4     rtusb_data.obj
 0001:0001d910       ??_C@_0CK@IFCJJMNI@CCX?9MFP?3?5Data?0?5RTMPSoftEncryptAE@ 1001e910     rtusb_data.obj
 0001:0001d940       ??_C@_0EI@BBFAEKAC@?5RTUSBHardTransmit?3?5?5SMS4?5DataSi@ 1001e940     rtusb_data.obj
 0001:0001d988       ??_C@_0FP@DEMDFIOG@?5RTUSBHardTransmit?3?5?5SMS4?5TxSize@ 1001e988     rtusb_data.obj
 0001:0001d9e8       ??_C@_0BO@KIPACKMM@RT2870Dump?5RTUSBHardTransmit?6?$AA@ 1001e9e8     rtusb_data.obj
 0001:0001da08       ??_C@_09MJFEDBKH@Tx?5IVSeq?6?$AA@ 1001ea08     rtusb_data.obj
 0001:0001da14       ??_C@_0BK@OGKKMGAG@?$FLSMS4?$FN?5TX?3?5KeyIdx?5?$DN?5?$FL?$CFd?$FN?6?$AA@ 1001ea14     rtusb_data.obj
 0001:0001da30       ??_C@_0EM@CIOOOAFC@RTUSBHardTransmit?5c4?5?9?9?$DO?5CurWrit@ 1001ea30     rtusb_data.obj
 0001:0001da7c       ??_C@_0DC@ELKPAKA@RTMPHardTransmit?$CIbEAP?$DN?$CFd?$CJ?5?9?5?$CFs?5k@ 1001ea7c     rtusb_data.obj
 0001:0001dab0       ??_C@_1FO@HGHMBPB@?$AAC?$AA?3?$AA?2?$AAW?$AAi?$AAn?$AAC?$AAE?$AA6?$AA?4?$AA0?$AA?2?$AAN?$AAe?$AAw?$AA?2?$AAR?$AAT?$AA2?$AA8?$AA7?$AA0?$AA_?$AAv?$AA1?$AA?4?$AA4?$AA?4?$AA9?$AA?4?$AA0?$AA?2@ 1001eab0     rtusb_data.obj
 0001:0001db10       ??_C@_0DG@MBCCNOND@RTMPHardTransmit?3?5?$FLWPI_SMS4?$FN?5Pac@ 1001eb10     rtusb_data.obj
 0001:0001db48       ??_C@_0CD@FOEAHKCC@bWAIFrame?5packet?5will?5use?5nonQoS@ 1001eb48     rtusb_data.obj
 0001:0001db6c       ??_C@_0CC@JIKHHCPL@Low?5rate?5packet?5will?5use?5nonQoS?4@ 1001eb6c     rtusb_data.obj
 0001:0001db90       ??_C@_0CD@MGCMENOJ@RTMPHardEncrypt?3MCS?$DN?$CFd?0?5bTXBA?$DN?$CFd@ 1001eb90     rtusb_data.obj
 0001:0001dbb4       ??_C@_0CL@CLDCLCBO@RTMPHardEncrypt?5?9?9?$DO?5Originator_W@ 1001ebb4     rtusb_data.obj
 0001:0001dbe0       ??_C@_0EH@KGHILHHG@RTMPHardEncrypt?5?9?9?$DO?5Drop?5non?5bWA@ 1001ebe0     rtusb_data.obj
 0001:0001dc28       ??_C@_0DJ@DBCNFLON@RTMPHardEncrypt?5?9?9?$DO?5Drop?5packet?5@ 1001ec28     rtusb_data.obj
 0001:0001dc68       ??_C@_0ED@BPOOMAOH@?$CB?$CB?$CB?$CB?5fRTMP_ADAPTER_ADDKEY_IN_PRO@ 1001ec68     rtusb_data.obj
 0001:0001dcac       ??_C@_0BE@DFNODCMN@Send?5WAIFrame?$CB?$CB?$CB?$CB?$CB?6?$AA@ 1001ecac     rtusb_data.obj
 0001:0001dcc0       ??_C@_0GB@HLPEELMB@RTMPHardEncrypt?3?5Session?5Timeout@ 1001ecc0     rtusb_data.obj
 0001:0001dd24       ??_C@_0CP@INNEDCIN@KeyType?$FL?$CFd?$FN?5Secure?$FL?$CFd?$FN?5Request?$FL?$CF@ 1001ed24     rtusb_data.obj
 0001:0001dd54       ??_C@_0CO@OBJBOIBM@Tx?5EAPOL?5Frame?3?5Group?5Key?5Handsh@ 1001ed54     rtusb_data.obj
 0001:0001dd84       ??_C@_0CL@JEHADDH@Tx?5EAPOL?5Frame?3?54?9Way?5Handshake?5@ 1001ed84     rtusb_data.obj
 0001:0001ddb0       ??_C@_0CK@HKHMEFII@Tx?5EAPOL?5Frame?3?54?9Way?5Handshake?5@ 1001edb0     rtusb_data.obj
 0001:0001dddc       ??_C@_0BN@IGPKKMK@Tx?5EAPOL?5Frame?3?5ProType?$FL?$CFd?$FN?6?$AA@ 1001eddc     rtusb_data.obj
 0001:0001de00       ??_C@_0GB@GADCAFOM@?5ADHOC?5MCAST?3?5find?5out?5the?5lowes@ 1001ee00     rtusb_data.obj
 0001:0001de64       ??_C@_0DL@HJKHAKDC@CCX?9MFP?3?5Drop?5non?9encrypted?5mgmt@ 1001ee64     rtusb_data.obj
 0001:0001dea0       ??_C@_0EC@DFLIGLAA@CCX?9MFP?3?5Drop?5non?9specified?5ACTI@ 1001eea0     rtusb_data.obj
 0001:0001dee4       ??_C@_0CJ@JKDKLKKP@CCX?9MFP?3?5AES?0?5Decrypt?5mgmt?5frame@ 1001eee4     rtusb_data.obj
 0001:0001df10       ??_C@_0DN@CEIADBIN@CCX?9MFP?3?5AES?0?5Decrypt?5mgmt?5frame@ 1001ef10     rtusb_data.obj
 0001:0001df50       ??_C@_0CK@FOIINJFF@CCX?9MFP?3?5TKIP?0?5Decrypt?5mgmt?5fram@ 1001ef50     rtusb_data.obj
 0001:0001df7c       ??_C@_0DO@FDOEHGML@CCX?9MFP?3?5TKIP?0?5Decrypt?5mgmt?5fram@ 1001ef7c     rtusb_data.obj
 0001:0001dfbc       ??_C@_0DC@MJDCHCHB@?$CB?$CB?$CB?5report?5DATA?5?$CIfragmented?$CJ?5to?5@ 1001efbc     rtusb_data.obj
 0001:0001dff0       ??_C@_0FG@CNAKIJMA@?$CB?$CB?$CB?5report?5EAPOL?1AIRONET?5DATA?5to@ 1001eff0     rtusb_data.obj
 0001:0001e048       ??_C@_0FJ@LKHAOFPJ@DataSize?5?$DN?5?$FL?$CFd?$FN?5pWpaKey?9?$DORxMic?$FL0@ 1001f048     rtusb_data.obj
 0001:0001e0a4       ??_C@_0DM@GPEFJNEG@Find?5another?5LLC?5at?5Middle?5or?5En@ 1001f0a4     rtusb_data.obj
 0001:0001e0e0       ??_C@_0FG@JJKGJCFO@Ndis802_11AuthModeWAI_CERT?3?5?$CB?$CB?$CB?5@ 1001f0e0     rtusb_data.obj
 0001:0001e138       ??_C@_0CB@EJDLLAEN@Queue?5This?5Rx?5EAPOL?5Frame?5SN?$DN?$CFd?6@ 1001f138     rtusb_data.obj
 0001:0001e160       ??_C@_0EM@LIAJIFJA@?$CB?$CB?$CB?5report?5EAPOL?1AIRONET?5DATA?5to@ 1001f160     rtusb_data.obj
 0001:0001e1b0       ??_C@_0GJ@KKLHJBNN@?$CB?$CB?$CB?5report?5BCASTDATA?5?$CIno?5frag?$CJ?5t@ 1001f1b0     rtusb_data.obj
 0001:0001e21c       ??_C@_0CG@IPOCHKNF@duplicate?5frame?5?$FL?$CFd?$FN?5B?1Mcast?5?$FL?$CFd@ 1001f21c     rtusb_data.obj
 0001:0001e244       ??_C@_0DE@LDNEFIBG@?$CFs?3?5SHOULD?5NOT?5HAPPENED?$CB?$CB?5?$CIpHead@ 1001f244     rtusb_data.obj
 0001:0001e278       ??_C@_0CC@NGPJBMOL@2?9Way?3?3RTMPSoftDecryptAES?5Failed@ 1001f278     rtusb_data.obj
 0001:0001e29c       ??_C@_0CE@IGCIAGJB@2?9Way?3?3RTMPSoftDecryptAES?5Comple@ 1001f29c     rtusb_data.obj
 0001:0001e2c0       ??_C@_0CJ@NLDFDOJB@?6?5Queue?5This?5Rx?52?9way?5frame?5Fram@ 1001f2c0     rtusb_data.obj
 0001:0001e2ec       ??_C@_0CD@HPOFFKON@2?9Way?3?3RTMPSoftDecryptTKIP?5Faile@ 1001f2ec     rtusb_data.obj
 0001:0001e310       ??_C@_0CF@EPMNOMKO@2?9Way?3?3RTMPSoftDecryptTKIP?5Compl@ 1001f310     rtusb_data.obj
 0001:0001e338       ??_C@_0CL@PPGELBB@CCX?9MFP?3?5Data?0?5RTMPSoftDecryptTK@ 1001f338     rtusb_data.obj
 0001:0001e364       ??_C@_0CK@KIAPDFNO@CCX_MFP?3?5Data?0?5RTMPSoftDecryptAE@ 1001f364     rtusb_data.obj
 0001:0001e390       ??_C@_0BI@BFEENHKE@RTMPCkipDecrypt?5failed?6?$AA@ 1001f390     rtusb_data.obj
 0001:0001e3a8       ??_C@_0BD@CCCCLMCA@Get?5WAIFrame?$CB?$CB?$CB?$CB?$CB?6?$AA@ 1001f3a8     rtusb_data.obj
 0001:0001e3bc       ??_C@_0CO@DIBDAJGO@Rx?5EAPOL?5Frame?3?5Group?5Key?5Handsh@ 1001f3bc     rtusb_data.obj
 0001:0001e3f0       ??_C@_0EN@POKFOMHN@Rx?5EAPOL?5Frame?3?54?9Way?5Handshake?5@ 1001f3f0     rtusb_data.obj
 0001:0001e440       ??_C@_0CK@IENONDH@Rx?5EAPOL?5Frame?3?54?9Way?5Handshake?5@ 1001f440     rtusb_data.obj
 0001:0001e46c       ??_C@_0BN@JJAOHKFD@Rx?5EAPOL?5Frame?3?5ProType?$FL?$CFd?$FN?6?$AA@ 1001f46c     rtusb_data.obj
 0001:0001e48c       ??_C@_0CL@NJAHLBMI@?$FLRX?$FN?5case?$CIb?4?$CJ?5parse?5Msdu2Size?5si@ 1001f48c     rtusb_data.obj
 0001:0001e4b8       ??_C@_0DH@CODKMFNJ@?$CFs?3?5Do?5not?5drop?5this?5packet?5?$CIpHe@ 1001f4b8     rtusb_data.obj
 0001:0001e4f0       ??_C@_0O@KEPILHA@RTUSBRxPacket?$AA@ 1001f4f0     rtusb_data.obj
 0001:0001e500       ??_C@_0EA@LJNNCDPK@RxDone?9?5drop?5NULL?5frame?$CIsubtype?$DN@ 1001f500     rtusb_data.obj
 0001:0001e540       ??_C@_0EM@OIPPFHPA@no?5cipherErr?0?5will?5update?5Privat@ 1001f540     rtusb_data.obj
 0001:0001e58c       ??_C@_0DM@GKBCBEOC@RX?5err?5filtered1?5?$FLMPDUtotalByteC@ 1001f58c     rtusb_data.obj
 0001:0001e5c8       ??_C@_0GK@CNBACDCL@?$CF02x?3?$CF02x?3?$CF02x?3?$CF02x?5?9?3?$CF02x?3?$CF02x?3@ 1001f5c8     rtusb_data.obj
 0001:0001e638       ??_C@_0GI@HOOPEOPC@BulkIn?5TransferBufLen?$CI?$CFd?$CJ?4?5ThisF@ 1001f638     rtusb_data.obj
 0001:0001e6a0       ??_C@_0DC@BFDNPCIO@bIsBulkINFail?5?$CFd?5ThisFrameLen?5?$CFd@ 1001f6a0     rtusb_data.obj
 0001:0001e6d8       ??_C@_0EF@FACCLILN@RXDMALen?5not?5multiple?5of?54?4?5?$FL?$CFu?$FN@ 1001f6d8     rtusb_data.obj
 0001:0001e720       ??_C@_0IA@POPBAFCN@RTUSBDequeueMLMEPacket?3?3PrioRing@ 1001f720     rtusb_data.obj
 0001:0001e7a0       ??_C@_0DK@KCGIBGDJ@not?5enough?5space?5in?5PrioRing?$FLpAd@ 1001f7a0     rtusb_data.obj
 0001:0001e7dc       ??_C@_0DB@CLMDDHIN@?$DM?9?9?9RTUSBDequeueMLMEPacket?5?3?5DeM@ 1001f7dc     rtusb_data.obj
 0001:0001e810       ??_C@_0BK@MKFDOFDK@?$DM?9?9?9CleanUpMLMEWaitQueue?6?$AA@ 1001f810     rtusb_data.obj
 0001:0001e82c       ??_C@_0BK@PAILKHKE@?9?9?9?$DOCleanUpMLMEWaitQueue?6?$AA@ 1001f82c     rtusb_data.obj
 0001:0001e848       ??_C@_0BI@BACCDPCM@?$DM?9?9?9?5MiniportMMRequest?6?$AA@ 1001f848     rtusb_data.obj
 0001:0001e860       ??_C@_0CG@FHEFMLON@MiniportMMRequest?5?$CIerror?3?3?5NULL?5@ 1001f860     rtusb_data.obj
 0001:0001e888       ??_C@_0CM@DIPODIBD@MiniportMMRequest?0?5MFP?5is?5enable@ 1001f888     rtusb_data.obj
 0001:0001e8b4       ??_C@_0CL@PAFEGNOE@MiniportMMRequest?5?$CIerror?3?3?5MgmtR@ 1001f8b4     rtusb_data.obj
 0001:0001e8e0       ??_C@_0BI@NOJGLFDJ@?9?9?9?$DO?5MiniportMMRequest?6?$AA@ 1001f8e0     rtusb_data.obj
 0001:0001e8f8       ??_C@_0CE@GKPOGJOK@not?9to?9me?5unicast?5?0RxInfo?5?$DN?50x?$CF0@ 1001f8f8     rtusb_data.obj
 0001:0001e91c       ??_C@_0DA@JIGHBGOJ@Accept?5multicast?5?$CF02x?3?$CF02x?3?$CF02x?3@ 1001f91c     rtusb_data.obj
 0001:0001e94c       ??_C@_0DN@EJDAJKJM@Rx?5MCAST?5?$CF02x?3?$CF02x?3?$CF02x?3?$CF02x?3?$CF02@ 1001f94c     rtusb_data.obj
 0001:0001e98c       ??_C@_0BP@LDCLPLJJ@Rx?5MCAST?5dropped?5by?5RX_FILTER?6?$AA@ 1001f98c     rtusb_data.obj
 0001:0001e9ac       ??_C@_0BP@LKINOACC@Rx?5BCAST?5dropped?5by?5RX_FILTER?6?$AA@ 1001f9ac     rtusb_data.obj
 0001:0001e9cc       ??_C@_0BN@PJJLECKM@Rx?5U2M?5dropped?5by?5RX_FILTER?6?$AA@ 1001f9cc     rtusb_data.obj
 0001:0001e9ec       ??_C@_0CC@CLIOIPBG@Rx?5dropped?5by?5MIC?5countermeasure@ 1001f9ec     rtusb_data.obj
 0001:0001ea10       ??_C@_0CF@PBEOHMJM@pRxD?5ERROR?3?5ICV?5Err?5state?5change@ 1001fa10     rtusb_data.obj
 0001:0001ea38       ??_C@_0BE@EPBKBMD@Rx?5MIC?5Value?5error?6?$AA@ 1001fa38     rtusb_data.obj
 0001:0001ea4c       ??_C@_0BD@PNDILBF@CIPHER?5error?5?$DN?5?$CFd?6?$AA@ 1001fa4c     rtusb_data.obj
 0001:0001ea60       ??_C@_0DF@FNOAADPE@Prevent?5ReportMicError?$FL?$CFd?$FN?1?$FL?$CFd?$FN?1@ 1001fa60     rtusb_data.obj
 0001:0001ea98       ??_C@_0DO@GMIJMNNG@WepStatus?$FL?$CFd?$FN?5but?5get?5CipherErr?$FL@ 1001fa98     rtusb_data.obj
 0001:0001ead8       ??_C@_0BK@GHKAJGCP@received?5packet?5too?5long?6?$AA@ 1001fad8     rtusb_data.obj
 0001:0001eaf4       ??_C@_0N@PEOLAIF@Err?$DLFC?4ToDs?6?$AA@ 1001faf4     rtusb_data.obj
 0001:0001eb08       ??_C@_0GI@EJNENLM@The?5second?5MIC?5error?5was?5detecte@ 1001fb08     rtusb_data.obj
 0001:0001eb70       ??_C@_0BG@NMJIJKNE@?$DM?9?9?9MlmeHardTransmit?6?$AA@ 1001fb70     rtusb_data.obj
 0001:0001eb88       ??_C@_0CP@JOAMMDML@CCX?9MFP?3?5Mgmt?0?5RTMPSoftEncryptMg@ 1001fb88     rtusb_data.obj
 0001:0001ebb8       ??_C@_0CL@HJDJMOAE@CCX?9MFP?3?5Mgmt?0?5RTMPSoftEncryptTK@ 1001fbb8     rtusb_data.obj
 0001:0001ebe4       ??_C@_0DB@CMPDOBIF@RTUSBMlmeHardTransmit?5?9?9?$DO?5carrie@ 1001fbe4     rtusb_data.obj
 0001:0001ec18       ??_C@_0DP@KMMFANBM@RTUSBMlmeHardTransmit?5?9?9?$DO?5radar?5@ 1001fc18     rtusb_data.obj
 0001:0001ec58       ??_C@_0BG@NCFDAJPG@?9?9?9?$DOMlmeHardTransmit?6?$AA@ 1001fc58     rtusb_data.obj
 0001:0001ec70       ??_C@_0CI@ODOHLLG@SYNC?5?9?5send?5QoS?5NULL?5Frame?5?$EA?$CFd?5M@ 1001fc70     rtusb_data.obj
 0001:0001ec98       ??_C@_0DK@DBLDNCKJ@RTMPSendNullFrameForDirect?5?9?5sen@ 1001fc98     rtusb_data.obj
 0001:0001ecd4       ??_C@_0DO@LDHMGGM@RTMPSendNullFrameForDirect?5?9?5sen@ 1001fcd4     rtusb_data.obj
 0001:0001ed14       ??_C@_0BO@PAHCEHOK@RTMPCheckTxSIPPacket?5?4?4?4BYE?5?6?$AA@ 1001fd14     rtusb_data.obj
 0001:0001ed34       ??_C@_08DLGAODGK@BYE?5sip?3?$AA@ 1001fd34     rtusb_data.obj
 0001:0001ed40       ??_C@_0CB@FIMHANPA@RTMPCheckTxSIPPacket?5?4?4?4CANCEL?5?6@ 1001fd40     rtusb_data.obj
 0001:0001ed64       ??_C@_0M@NPADNAGD@CANCEL?5sip?3?$AA@ 1001fd64     rtusb_data.obj
 0001:0001ed70       ??_C@_0CB@MBOLJFLF@RTMPCheckTxSIPPacket?5?4?4?4INVITE?5?6@ 1001fd70     rtusb_data.obj
 0001:0001ed94       ??_C@_0M@CCBCPDCA@INVITE?5sip?3?$AA@ 1001fd94     rtusb_data.obj
 0001:0001eda0       ??_C@_0BO@GEPECCM@RTMPCheckRxSIPPacket?5?4?4?4BYE?5?6?$AA@ 1001fda0     rtusb_data.obj
 0001:0001edc0       ??_C@_0CB@OIPKFPKA@RTMPCheckRxSIPPacket?5?4?4?4CANCEL?5?6@ 1001fdc0     rtusb_data.obj
 0001:0001ede4       ??_C@_0CB@HBNGMHOF@RTMPCheckRxSIPPacket?5?4?4?4INVITE?5?6@ 1001fde4     rtusb_data.obj
 0001:0001ee08       ??_C@_0CA@JLGHGEKO@MailBoxTOExec?5read?5code?5?3?50x?$CFx?6?$AA@ 1001fe08     rtusb_data.obj
 0001:0001ee28       ??_C@_0CG@FBPOAMCP@MailBoxTOExec?5read?5command?5id?5?3?5@ 1001fe28     rtusb_data.obj
 0001:0001ee50       ??_C@_0EA@OOFLGLOH@DUPCHECK?5?9?5replace?5Entry?5?$CFd?0?5MAC@ 1001fe50     rtusb_data.obj
 0001:0001ee90       ??_C@_0DM@DAOJGCKM@DUPCHECK?5?9?5Add?5Entry?5?$CFd?0?5MAC?$DN?$CF02@ 1001fe90     rtusb_data.obj
 0001:0001eecc       ??_C@_0CA@KBLLJNLP@?$CFs?3?$DM?9?9?5MCS?$FL?$CFd?$FN?5BW?$FL?$CFd?$FN?5MODE?$FL?$CFd?$FN?6?$AA@ 1001fecc     rtusb_data.obj
 0001:0001eeec       ??_C@_0BL@HLGNPNBG@?$CFs?3BulkOut?5Reach?5CurWrite?6?$AA@ 1001feec     rtusb_data.obj
 0001:0001ef08       ??_C@_0EG@JINCOBFB@RTMPSendBAR?5c3?5?9?9?$DO?5CurWritePosit@ 1001ff08     rtusb_data.obj
 0001:0001ef50       ??_C@_0EG@IAHIDDDF@RTMPSendBAR?5c2?5?9?9?$DO?5CurWritePosit@ 1001ff50     rtusb_data.obj
 0001:0001ef98       ??_C@_0EG@NDIGNOGN@RTMPSendBAR?5c4?5?9?9?$DO?5CurWritePosit@ 1001ff98     rtusb_data.obj
 0001:0001efe0       ??_C@_0EG@KJIHEFJJ@RTMPSendBAR?5c1?5?9?9?$DO?5CurWritePosit@ 1001ffe0     rtusb_data.obj
 0001:0001f028       ??_C@_0CI@BHLNAJFI@packetsize?3?$CFd?0?5PhysicalBufferCou@ 10020028     rtusb_data.obj
 0001:0001f050       ??_C@_0BE@EPFPDABJ@?$CFs?3?5?9?9?$DO?5QueIdx?$FL?$CFd?$FN?6?$AA@ 10020050     rtusb_data.obj
 0001:0001f064       ??_C@_0M@BBLIPOJE@RTMPSendBAR?$AA@ 10020064     rtusb_data.obj
 0001:0001f070       ??_C@_0CI@FOGMPHIE@?$CFs?3RTMPSendTxWaitQueue?3?5New?5Ndis@ 10020070     rtusb_data.obj
 0001:0001f098       ??_C@_0CK@HKEGELG@?$CFs?3RTMPSendTxWaitQueue?3?5packet?5t@ 10020098     rtusb_data.obj
 0001:0001f0c4       ??_C@_0BM@BMLABEPL@?$CFs?3alloc?5ndis?5buffer?5?5fail?6?$AA@ 100200c4     rtusb_data.obj
 0001:0001f0e0       ??_C@_0BL@DONKIIGM@?$CFs?3alloc?5ndis?5packet?5fail?6?$AA@ 100200e0     rtusb_data.obj
 0001:0001f0fc       ??_C@_0BE@EOIKHOKO@RTMPSendTxWaitQueue?$AA@ 100200fc     rtusb_data.obj
 0001:0001f310       ??_C@_0BA@BJAGMFGL@InitEFuseConfig?$AA@ 10020310     rtusb_io.obj
 0001:0001f320       ??_C@_0CB@KDJMGMEA@FlashInstallationWith8KBFirmware@ 10020320     rtusb_io.obj
 0001:0001f344       ??_C@_0BF@BFHOPAB@?$DM?9?9RTUSBVenderReset?6?$AA@ 10020344     rtusb_io.obj
 0001:0001f35c       ??_C@_0BF@GFHNMDNA@?9?9?$DORTUSBVenderReset?6?$AA@ 1002035c     rtusb_io.obj
 0001:0001f374       ??_C@_0BI@OJMICEDB@BBP?5read?5R?$CFd?$DN0x?$CFx?5fail?6?$AA@ 10020374     rtusb_io.obj
 0001:0001f390       ??_C@_0EF@EJEFIALG@?$CK?$CK?$CK?$CK?$CK?$CK?5BBP_Write_Latch?5Buffer?5?$CIi@ 10020390     rtusb_io.obj
 0001:0001f3d8       ??_C@_0BJ@PEJLMMEE@BBP?5write?5R?$CFd?$DN0x?$CFx?5fail?6?$AA@ 100203d8     rtusb_io.obj
 0001:0001f3f4       ??_C@_0CM@NIGPMLOI@Retry?5count?5exhausted?5or?5device?5@ 100203f4     rtusb_io.obj
 0001:0001f420       ??_C@_0CF@LPBAFGMA@RF?5read?5R?$CFd?$DN0x?$CFx?5fail?0?5i?$FL?$CFd?$FN?0?5k?$FL@ 10020420     rtusb_io.obj
 0001:0001f448       ??_C@_0CD@EMBHHPKF@Not?5bWriteSuccess?5new?5BlkNum?5?$DN?5?$CF@ 10020448     rtusb_io.obj
 0001:0001f46c       ??_C@_0BP@OBGAJELB@Not?5bWriteSuccess?5BlkNum?5?$DN?5?$CFd?6?$AA@ 1002046c     rtusb_io.obj
 0001:0001f48c       ??_C@_0DC@FHKPFOPF@eFuseWriteRegisters?3?5out?5of?5free@ 1002048c     rtusb_io.obj
 0001:0001f4c0       ??_C@_0CC@OPKMEOC@eFuseWriteRegisters?5BlkNum?5?$DN?5?$CFd?5@ 100204c0     rtusb_io.obj
 0001:0001f4e4       ??_C@_0CJ@NLFNLHGA@eFuseWriteRegisters?5Offset?$DN?$CFx?0?5p@ 100204e4     rtusb_io.obj
 0001:0001f510       ??_C@_0BM@PBPPKPNH@Sleep?5Mailbox?5testvalue?5?$CFx?6?$AA@ 10020510     rtusb_io.obj
 0001:0001f530       ??_C@_0IA@GKJGAIHK@Fail?3?5RTUSBEnqueueCmdFromNdis?3?3A@ 10020530     rtusb_io.obj
 0001:0001f5b0       ??_C@_0HC@GCICHLNJ@Fail?3?5RTUSBEnqueueCmdFromNdis?3?3?5@ 100205b0     rtusb_io.obj
 0001:0001f624       ??_C@_0BN@BALDHKEF@?$DM?9?9?9RTUSBEnqueueInternalCmd?6?$AA@ 10020624     rtusb_io.obj
 0001:0001f648       ??_C@_0GH@BBBMKEEB@Fail?3?5RTUSBEnqueueInternalCmd?3?3A@ 10020648     rtusb_io.obj
 0001:0001f6b0       ??_C@_0HC@JLOLNIJF@Fail?3?5RTUSBEnqueueInternalCmd?3?3?5@ 100206b0     rtusb_io.obj
 0001:0001f724       ??_C@_0BN@KNHJJIOE@?9?9?9?$DORTUSBEnqueueInternalCmd?6?$AA@ 10020724     rtusb_io.obj
 0001:0001f748       ??_C@_1FA@NHKKMGPJ@?$AAR?$AAe?$AAt?$AAr?$AAy?$AA?3?$AA?5?$AAR?$AAe?$AAs?$AAe?$AAt?$AAD?$AAe?$AAf?$AAa?$AAu?$AAl?$AAt?$AAE?$AAn?$AAd?$AAp?$AAo?$AAi?$AAn?$AAt?$AA?0?$AA?5?$AAd?$AAw?$AAE@ 10020748     rtusb_io.obj
 0001:0001f798       ??_C@_1BM@HHJCCGJE@?$AAE?$AAR?$AAR?$AAO?$AAR?$AA_?$AA?$DP?$AA?$DP?$AA?$DP?$AA?$DP?$AA?$DP?$AA?$AN?$AA?6?$AA?$AA@ 10020798     rtusb_io.obj
 0001:0001f7b4       ??_C@_1DE@LANJFFNJ@?$AAE?$AAR?$AAR?$AAO?$AAR?$AA_?$AAI?$AAN?$AAV?$AAA?$AAL?$AAI?$AAD?$AA_?$AAP?$AAA?$AAR?$AAA?$AAM?$AAE?$AAT?$AAE?$AAR?$AA?$AN?$AA?6?$AA?$AA@ 100207b4     rtusb_io.obj
 0001:0001f7e8       ??_C@_1CI@IOGAENCH@?$AAE?$AAR?$AAR?$AAO?$AAR?$AA_?$AAG?$AAE?$AAN?$AA_?$AAF?$AAA?$AAI?$AAL?$AAU?$AAR?$AAE?$AA?$AN?$AA?6?$AA?$AA@ 100207e8     rtusb_io.obj
 0001:0001f810       ??_C@_1CA@CEAOKJKM@?$AAE?$AAR?$AAR?$AAO?$AAR?$AA_?$AAT?$AAI?$AAM?$AAE?$AAO?$AAU?$AAT?$AA?$AN?$AA?6?$AA?$AA@ 10020810     rtusb_io.obj
 0001:0001f830       ??_C@_1CA@MCLMAGAP@?$AAE?$AAR?$AAR?$AAO?$AAR?$AA_?$AAS?$AAU?$AAC?$AAC?$AAE?$AAS?$AAS?$AA?$AN?$AA?6?$AA?$AA@ 10020830     rtusb_io.obj
 0001:0001f850       ??_C@_1JG@JIFNMJMG@?$AAV?$AAe?$AAn?$AAd?$AAe?$AAr?$AAR?$AAe?$AAq?$AA?4?$AAb?$AAm?$AAR?$AAe?$AAq?$AAu?$AAe?$AAs?$AAt?$AAT?$AAy?$AAp?$AAe?$AA?$DN?$AA0?$AAx?$AA?$CF?$AA0?$AA2?$AAx?$AA?0?$AA?5@ 10020850     rtusb_io.obj
 0001:0001f8e8       ??_C@_1LO@MIJFMEEH@?$AAR?$AAT?$AA2?$AA8?$AA7?$AA0?$AA?3?$AA?5?$AAI?$AAs?$AAs?$AAu?$AAe?$AAV?$AAe?$AAn?$AAd?$AAo?$AAr?$AAT?$AAr?$AAa?$AAn?$AAs?$AAf?$AAe?$AAr?$AA?5?$AAe?$AAr?$AAr?$AA?$CB@ 100208e8     rtusb_io.obj
 0001:0001f9a8       ??_C@_1GA@IEJFCPAO@?$AA?5?$AAR?$AAT?$AAU?$AAS?$AAB?$AA_?$AAV?$AAe?$AAn?$AAd?$AAo?$AAr?$AAR?$AAe?$AAq?$AAu?$AAe?$AAs?$AAt?$AA?5?$AAC?$AAo?$AAm?$AAm?$AAa?$AAn?$AAd?$AAT?$AAr?$AAa?$AAn@ 100209a8     rtusb_io.obj
 0001:0001fa08       ??_C@_1FK@PBEMMNHI@?$AAC?$AA?3?$AA?2?$AAW?$AAi?$AAn?$AAC?$AAE?$AA6?$AA?4?$AA0?$AA?2?$AAN?$AAe?$AAw?$AA?2?$AAR?$AAT?$AA2?$AA8?$AA7?$AA0?$AA_?$AAv?$AA1?$AA?4?$AA4?$AA?4?$AA9?$AA?4?$AA0?$AA?2@ 10020a08     rtusb_io.obj
 0001:0001fa64       ??_C@_0BC@LJKEACAO@?$DM?9?9USB_ResetPipe?6?$AA@ 10020a64     rtusb_io.obj
 0001:0001fa78       ??_C@_0BC@LHLKGCJL@?9?9?$DOUSB_ResetPipe?6?$AA@ 10020a78     rtusb_io.obj
 0001:0001fa8c       ??_C@_0BO@ICALAGIK@?$DM?9?9?9USB_ResetDevice?5?$CI0x?$CF08x?$CJ?6?$AA@ 10020a8c     rtusb_io.obj
 0001:0001faac       ??_C@_0BP@INKCKCHE@IoCallDriver?$CIUSB_ResetDevice?$CJ?6?$AA@ 10020aac     rtusb_io.obj
 0001:0001facc       ??_C@_0BF@JOOEBDOD@?9?9?9?$DOUSB_ResetDevice?6?$AA@ 10020acc     rtusb_io.obj
 0001:0001fae4       ??_C@_0CG@LPNJFEHN@?$DM?9?9?9RTUSB_AbortPipe?0?5ntStatus?$DN0x@ 10020ae4     rtusb_io.obj
 0001:0001fb0c       ??_C@_0CA@MDGKNOFA@?9?9?9?$DORTUSB_AbortPipe?0?5PipeId?$DN?$CFd?6?$AA@ 10020b0c     rtusb_io.obj
 0001:0001fb2c       ??_C@_0BL@HOHCKNIA@?5RTUSB_ReadVersion?5?$CI0x?$CFx?$CJ?6?$AA@ 10020b2c     rtusb_io.obj
 0001:0001fb48       ??_C@_0CM@LAKOLIPE@?$DM?9?9?9RTUSB_GetPortStatus?0?5PortSta@ 10020b48     rtusb_io.obj
 0001:0001fb74       ??_C@_0BJ@NGBKIDD@?9?9?9?$DORTUSB_GetPortStatus?6?$AA@ 10020b74     rtusb_io.obj
 0001:0001fb90       ??_C@_0DL@IGIMLDPP@RTUSB_EndpointUsage?5?9?5?5?$CFd?3?$CFd?3?$CFd?3@ 10020b90     rtusb_io.obj
 0001:0001fbd0       ??_C@_0EK@IIKNPBME@Re?5RTUSBBulkOutDataPacket?5EP?$CD?$CFd?5@ 10020bd0     rtusb_io.obj
 0001:0001fc1c       ??_C@_0CI@MGNHJNJP@?5All?5pTxContext?9?$DOIRPPending?5is?5p@ 10020c1c     rtusb_io.obj
 0001:0001fc44       ??_C@_0CN@IHDFKPKC@?5SavedPad?5?3?5?$CFx?5?5?$CFx?5?5?$CFx?5?5?$CFx?5?5?$CFx?5?5@ 10020c44     rtusb_io.obj
 0001:0001fc74       ??_C@_0CM@IHHKMBLB@?$CL?5?$CL?5?$CL?5?$CL?5Control?5Thread?5Terminate@ 10020c74     rtusb_io.obj
 0001:0001fca0       ??_C@_0EP@MADONNPL@APSetInformation?3?5Channel?5change@ 10020ca0     rtusb_io.obj
 0001:0001fcf0       ??_C@_0BJ@BELCHNHN@Command?5Thread?5Finished?6?$AA@ 10020cf0     rtusb_io.obj
 0001:0001fd0c       ??_C@_0CI@JNLPEPJF@Device?5not?5connect?5or?5Halt?5in?5pr@ 10020d0c     rtusb_io.obj
 0001:0001fd34       ??_C@_0CO@HJOIIIGI@?9?9?$DO?5Control?5Thread?5?$CB?$CB?5ERROR?5?$CB?$CB?5d@ 10020d34     rtusb_io.obj
 0001:0001fd64       ??_C@_0CF@CMKNBM@WPS?5LED?5mode?510?3?3?5No?5this?5status@ 10020d64     rtusb_io.obj
 0001:0001fd8c       ??_C@_0CK@JABMHLCF@WPS?5LED?5mode?510?3?3ON?5or?5Flash?5or?5@ 10020d8c     rtusb_io.obj
 0001:0001fdb8       ??_C@_0DD@PKAKPOD@?$CFs?3?5RT_CMD_SET_WPS_LED_STATUS?5?$CIW@ 10020db8     rtusb_io.obj
 0001:0001fdf0       ??_C@_0FC@MNJGHLP@CmdThread?3?3RT_OID_CCX_SEND_PLM_M@ 10020df0     rtusb_io.obj
 0001:0001fe48       ??_C@_0EJ@LGBEFGPF@CmdThread?3?3?5RT_OID_MH_LEAP_SEND_@ 10020e48     rtusb_io.obj
 0001:0001fe94       ??_C@_0CB@MAFIIHKB@?9?9?$DO?5RT_OID_802_11_TEAR_IMME_BA?5?6@ 10020e94     rtusb_io.obj
 0001:0001feb8       ??_C@_0CA@CEMLAKCJ@?9?9?$DO?5RT_OID_802_11_ADD_IMME_BA?5?6?$AA@ 10020eb8     rtusb_io.obj
 0001:0001fed8       ??_C@_0CM@OJPEJLKH@CmdThread?3?3RT_OID_802_11_SET_APS@ 10020ed8     rtusb_io.obj
 0001:0001ff04       ??_C@_0CH@ONFEJEIA@CmdThread?3?3RT_OID_SET_PSM_BIT_AC@ 10020f04     rtusb_io.obj
 0001:0001ff2c       ??_C@_0CI@FLEPJCPM@CmdThread?3?3OID_802_11_POWER_MODE@ 10020f2c     rtusb_io.obj
 0001:0001ff54       ??_C@_0CO@OAHBNICP@CmdThread?3?3OID_802_11_STATISTICS@ 10020f54     rtusb_io.obj
 0001:0001ff84       ??_C@_0CC@FAPBEIDK@Query?3?3RT_OID_802_11_RSSI_2?$CI?$DN?$CFd?$CJ@ 10020f84     rtusb_io.obj
 0001:0001ffa8       ??_C@_0CC@NOHOEPNJ@Query?3?3RT_OID_802_11_RSSI_1?$CI?$DN?$CFd?$CJ@ 10020fa8     rtusb_io.obj
 0001:0001ffcc       ??_C@_0DA@PLOIOHOD@CmdThread?3?3AsicRemoveSharedKeyEn@ 10020fcc     rtusb_io.obj
 0001:0001fffc       ??_C@_0DJ@EFBAEIOP@CmdThread?3?3OID_802_11_REMOVE_KEY@ 10020ffc     rtusb_io.obj
 0001:00020038       ??_C@_0CB@JCEACAEE@CmdThread?3?3RTMPWPARemoveKeyProc?6@ 10021038     rtusb_io.obj
 0001:0002005c       ??_C@_0BP@FJJJFOOO@CmdThread?3?3OID_802_11_ADD_KEY?6?$AA@ 1002105c     rtusb_io.obj
 0001:00020080       ??_C@_0EI@OJGHFCDO@CmdThread?3?3OID_802_11_ADD_KEY_WE@ 10021080     rtusb_io.obj
 0001:000200c8       ??_C@_0DK@BCMPHKKK@CmdThread?3?3OID_802_11_ADD_KEY_WE@ 100210c8     rtusb_io.obj
 0001:00020104       ??_C@_0CO@MDNHJEFM@CmdThread?3?3OID_802_11_REMOVE_WEP@ 10021104     rtusb_io.obj
 0001:00020134       ??_C@_0DJ@OHADAOII@CmdThread?3?3OID_802_11_REMOVE_WEP@ 10021134     rtusb_io.obj
 0001:00020170       ??_C@_0DC@MIAFOFP@CmdThread?3?3OID_802_11_REMOVE_WEP@ 10021170     rtusb_io.obj
 0001:000201a4       ??_C@_0DI@OMKJEDIG@CmdThread?3?3OID_802_11_ADD_WEP?5?$CIK@ 100211a4     rtusb_io.obj
 0001:000201dc       ??_C@_0CO@FLIMMGLO@BSS0Mcast_WCID?5?3?5offset?5?$DN?5?$CFx?0?5WC@ 100211dc     rtusb_io.obj
 0001:0002020c       ??_C@_0CB@OMGNIOPD@CmdThread?3?3OID_802_11_ADD_WEP?5?5?6@ 1002120c     rtusb_io.obj
 0001:00020230       ??_C@_0IP@KFIGDLGG@Set?3?3RT_OID_802_11_SET_HT_PHYMOD@ 10021230     rtusb_io.obj
 0001:000202c0       ??_C@_0CK@PEGEDMKG@SetCMD?3?3RT_OID_802_11_SET_PHY_MO@ 100212c0     rtusb_io.obj
 0001:000202ec       ??_C@_0CH@OLGPNPC@Set?3?3RT_OID_802_11_SET_PREAMBLE?5@ 100212ec     rtusb_io.obj
 0001:00020314       ??_C@_0O@PNBKBNAD@I?1Q?5Not?5Flip?6?$AA@ 10021314     rtusb_io.obj
 0001:00020324       ??_C@_09BIFAHHDL@I?1Q?5Flip?6?$AA@ 10021324     rtusb_io.obj
 0001:00020330       ??_C@_0DB@IIOOOMJF@RT_OID_VENDOR_SWITCH_FUNCTION?5?9?9@ 10021330     rtusb_io.obj
 0001:00020364       ??_C@_0BA@HFIMNODF@value?5?$DN?50x?$CF08x?6?$AA@ 10021364     rtusb_io.obj
 0001:00020374       ??_C@_0BA@BKDBDOFB@value?5?$DN?50x?$CF02x?6?$AA@ 10021374     rtusb_io.obj
 0001:00020384       ??_C@_0BB@OELIFODF@offset?5?$DN?50x?$CF02x?6?$AA@ 10021384     rtusb_io.obj
 0001:00020398       ??_C@_0BG@JJBBNCK@BBPCurrentBW?5?$DN?5BW_20?6?$AA@ 10021398     rtusb_io.obj
 0001:000203b0       ??_C@_0BK@LPCAFBIE@?$FL070507?$FN?5register?5set?4?4?4?6?$AA@ 100213b0     rtusb_io.obj
 0001:000203cc       ??_C@_0BG@CMPKECPG@BBPCurrentBW?5?$DN?5BW_40?6?$AA@ 100213cc     rtusb_io.obj
 0001:000203e4       ??_C@_0BM@FDIHPOEA@?5extoffset?5?$DN?$DN?5EXTCHA_ABOVE?6?$AA@ 100213e4     rtusb_io.obj
 0001:00020400       ??_C@_0BM@KHJMBLO@?5extoffset?5?$DN?$DN?5EXTCHA_BELOW?6?$AA@ 10021400     rtusb_io.obj
 0001:0002041c       ??_C@_0BP@OKPIJGFJ@2?9offset?5?$DN?5?$CFx?5?0?5MACValue?$DN?5?$CFx?0?6?$AA@ 1002141c     rtusb_io.obj
 0001:0002043c       ??_C@_0DN@LNOJPNJO@Cmd?5?3?5RT_CMD_SET_ASIC_WCID_CIPHE@ 1002143c     rtusb_io.obj
 0001:0002047c       ??_C@_0BB@CGFNCKLH@2?9MACValue?$DN?5?$CFx?0?6?$AA@ 1002147c     rtusb_io.obj
 0001:00020490       ??_C@_0BB@HFMHHBDD@1?9MACValue?$DN?5?$CFx?0?6?$AA@ 10021490     rtusb_io.obj
 0001:000204a8       ??_C@_0EH@EBNLGMIF@Cmd?5?3?5RT_CMD_SET_ASIC_WCID?5?3?5WCI@ 100214a8     rtusb_io.obj
 0001:000204f0       ??_C@_0CA@PPNMHDPK@offset?5?$DN?50x?$CF02x?7value?5?$DN?50x?$CF02x?6?$AA@ 100214f0     rtusb_io.obj
 0001:00020510       ??_C@_0CG@PJEPDILG@Send?5Disassoc?5to?5Peer?5?$CF02x?3?$CF02x?3@ 10021510     rtusb_io.obj
 0001:00020538       ??_C@_0EH@PMIHONHN@?$CFs?3?5RT_OID_LINK_DOWN?3?5Send?5the?5d@ 10021538     rtusb_io.obj
 0001:00020580       ??_C@_0P@JJKDMOCF@RTUSBCmdThread?$AA@ 10021580     rtusb_io.obj
 0001:00020590       ??_C@_0BM@PGBKONNJ@LinkDown?$CIRT_OID_LINK_DOWN?$CJ?6?$AA@ 10021590     rtusb_io.obj
 0001:000205ac       ??_C@_0CE@NFPGIPEL@bPromiscuous?$CI?5switch?5channel?5?$DN?5?$CF@ 100215ac     rtusb_io.obj
 0001:000205d0       ??_C@_0GJ@HOLEJFNE@Set?3?3RT_OID_802_11_SET_AP_CONFIG@ 100215d0     rtusb_io.obj
 0001:00020640       ??_C@_0HB@DLJIEBEO@CmdThread?3?3RT_OID_802_11_SET_STA@ 10021640     rtusb_io.obj
 0001:000206b4       ??_C@_0DI@IGLHAIHL@CmdThread?3?3RT_OID_802_11_SET_STA@ 100216b4     rtusb_io.obj
 0001:000206ec       ??_C@_07DKHDFDA@BW_20?5?6?$AA@ 100216ec     rtusb_io.obj
 0001:000206f4       ??_C@_07IMOHMAJA@BW_40?5?6?$AA@ 100216f4     rtusb_io.obj
 0001:000206fc       ??_C@_0CL@OOBNNMBH@CmdThread?5?3?5RT_OID_USB_RESET_BUL@ 100216fc     rtusb_io.obj
 0001:00020728       ??_C@_0BH@HDHELPPH@Read?5Register?5Failed?$CB?6?$AA@ 10021728     rtusb_io.obj
 0001:00020740       ??_C@_0BJ@DIIMHJBG@Device?5has?5been?5removed?6?$AA@ 10021740     rtusb_io.obj
 0001:0002075c       ??_C@_0BA@JECDGBEA@?3RTUSBRxPacket?6?$AA@ 1002175c     rtusb_io.obj
 0001:0002076c       ??_C@_0BD@BCEOHJNN@?3RTUSBBulkReceive?6?$AA@ 1002176c     rtusb_io.obj
 0001:00020780       ??_C@_0DB@PIINCAMK@NextRxBulkInReadIndex?$FL?$CFd?$FN?5NextRx@ 10021780     rtusb_io.obj
 0001:000207b8       ??_C@_0KN@CFPBHGBO@?$FL4?$FN?5IRPPending?$DN?$CFd?3?5?5InUse?$DN?$CFd?3?5Re@ 100217b8     rtusb_io.obj
 0001:00020868       ??_C@_0KN@GKLKJEOC@?$FL0?$FN?5IRPPending?$DN?$CFd?3?5?5InUse?$DN?$CFd?3?5Re@ 10021868     rtusb_io.obj
 0001:00020918       ??_C@_0CE@PJEMEBEA@0x?$CFx?10x?$CFx?1?50x?$CFx?4?5?3?3x?$CFx?10x?$CFx?1?50x?$CF@ 10021918     rtusb_io.obj
 0001:0002093c       ??_C@_0CO@PCBANGBA@RTUSBReadMACRegister?5MAC_CSR0?5Ti@ 1002193c     rtusb_io.obj
 0001:00020970       ??_C@_0GB@BBCMAAOJ@CmdThread?5?3?5RT_OID_USB_RESET_BUL@ 10021970     rtusb_io.obj
 0001:000209d4       ??_C@_0CL@KEPBHMNI@CmdThread?5?3?5RT_OID_USB_RESET_BUL@ 100219d4     rtusb_io.obj
 0001:00020a00       ??_C@_0CG@NAGALCCJ@Clear?5fRTMP_ADAPTER_BULKOUT_RESE@ 10021a00     rtusb_io.obj
 0001:00020a28       ??_C@_0EO@NGHGHNHD@EP?$CD?$CFd?4?5PendingIRP?5number?5?$DN?51?0?5An@ 10021a28     rtusb_io.obj
 0001:00020a78       ??_C@_0GE@LNFCACAA@EP?$CD?$CFd?4?5PendingIRP?5number?5?$DN?52?0?5An@ 10021a78     rtusb_io.obj
 0001:00020ae0       ??_C@_0EG@DCGAPHCP@AnotherPendingTx?5?$DN?50x?$CF02X?0?5First@ 10021ae0     rtusb_io.obj
 0001:00020b28       ??_C@_0ED@FNPPLEHD@Prepare?5ReBulkOut?5the?5ResetPipeI@ 10021b28     rtusb_io.obj
 0001:00020b6c       ??_C@_0DC@LACBJOJO@Set?50x2a0?5bit19?4?5Clear?5USB?5DMA?5T@ 10021b6c     rtusb_io.obj
 0001:00020ba0       ??_C@_0GP@OJCPENAL@CmdThread?5?3?5RT_OID_USB_RESET_BUL@ 10021ba0     rtusb_io.obj
 0001:00020c10       ??_C@_0DC@BLCNIGOD@RT_OID_MULTI_WRITE_MAC?5?3?5Offset?5@ 10021c10     rtusb_io.obj
 0001:00020c44       ??_C@_0CP@CAPHLOFG@CMD?3Pending?5this?5OID?$FL?$DN0x?$CF08x?$FN?5to@ 10021c44     rtusb_io.obj
 0001:00020c74       ??_C@_0BG@FPFDEMHJ@IBSS?5Sync?3?5IBSS?5mode?6?$AA@ 10021c74     rtusb_io.obj
 0001:00020c8c       ??_C@_0BE@HNJJPECA@IBSS?5Sync?3?5AP?5mode?6?$AA@ 10021c8c     rtusb_io.obj
 0001:00020ca0       ??_C@_0FP@NBIHNCGE@RT_OID_BA_DELETE_REC_ENTRY?5?3Fini@ 10021ca0     rtusb_io.obj
 0001:00020d00       ??_C@_0DG@OPOOFDEO@RT_OID_BA_DELETE_REC_ENTRY?5Idx?$FL?$CF@ 10021d00     rtusb_io.obj
 0001:00020d38       ??_C@_0CH@MBJCAJPM@?$CIEntry?$FL?$CFd?$FN?4?5MacTab?8s?5MmpsMode?5?$DN?5@ 10021d38     rtusb_io.obj
 0001:00020d60       ??_C@_0EB@JKHEKPHJ@RT_OID_SEND_PSMP_ACTION_FRAME?3?5A@ 10021d60     rtusb_io.obj
 0001:00020da8       ??_C@_0EK@CAPDAKIA@RX?5URB?5no?5responding?0?5RXQPCNT?$DN0x@ 10021da8     rtusb_io.obj
 0001:00020df4       ??_C@_0BG@GCJCDGBH@?$CB?$CB?$CB?5WPS?5?9?5HW?5PBC?5?$CB?$CB?$CB?6?$AA@ 10021df4     rtusb_io.obj
 0001:00020e0c       ??_C@_0DC@CHDNKOCE@disassociate?5with?5current?5AP?5bef@ 10021e0c     rtusb_io.obj
 0001:00020e40       ??_C@_0BD@MHJIODPL@?$CB?$CB?$CB?5Radio?5Off?5?$CB?$CB?$CB?6?$AA@ 10021e40     rtusb_io.obj
 0001:00020e54       ??_C@_0BC@OGANFKK@?$CB?$CB?$CB?5Radio?5On?5?$CB?$CB?$CB?6?$AA@ 10021e54     rtusb_io.obj
 0001:00020e68       ??_C@_0BL@LBIJFMJL@?$CB?$CB?$CB?5RT_OID_CHECK_GPIO?5?$CB?$CB?$CB?6?$AA@ 10021e68     rtusb_io.obj
 0001:00020e84       ??_C@_09BBAMGPBN@Cmd?5?$DN?5?$CFx?6?$AA@ 10021e84     rtusb_io.obj
 0001:00020e90       ??_C@_1EK@BBBCJCFM@?$AAC?$AAm?$AAd?$AAT?$AAh?$AAr?$AAe?$AAa?$AAd?$AA?5?$AAh?$AAa?$AAn?$AAd?$AAl?$AAe?$AA?$DN?$AA0?$AAx?$AA?$CF?$AAx?$AA?0?$AA?5?$AAP?$AAr?$AAi?$AAo?$AAr?$AAi?$AAt?$AAy?$AA?$DN@ 10021e90     rtusb_io.obj
 0001:00020edc       ??_C@_0BK@ILEKEOEG@Command?5Thread?5Triggered?6?$AA@ 10021edc     rtusb_io.obj
 0001:00020ef8       ??_C@_0BJ@OAHPGHNF@EEP?3ID?$FL0x?$CF04x?$FN?$DN?$FL0x?$CF04x?$FN?6?$AA@ 10021ef8     rtusb_io.obj
 0001:00020f14       ??_C@_0BI@JKCDOABM@RF?3ID?$FL0x?$CF02x?$FN?$DN?$FL0x?$CF02x?$FN?6?$AA@ 10021f14     rtusb_io.obj
 0001:00020f2c       ??_C@_0CA@LIKHBIBK@RF?5type?$DN?$CFd?0?5not?5support?5access?6?$AA@ 10021f2c     rtusb_io.obj
 0001:00020f4c       ??_C@_0BJ@GILFBCBM@BBP?3ID?$FL0x?$CF02x?$FN?$DN?$FL0x?$CF02x?$FN?6?$AA@ 10021f4c     rtusb_io.obj
 0001:00020f68       ??_C@_0BN@DMNNPFEH@MAC?3Offset?$FL0x?$CF04x?$FN?$DN?$FL0x?$CF04x?$FN?6?$AA@ 10021f68     rtusb_io.obj
 0001:00020f88       ??_C@_0DB@BLDOOIEJ@OID?5has?5been?5reset?5and?5can?8t?5acc@ 10021f88     rtusb_io.obj
 0001:00020fbc       ??_C@_0CF@BGCABFBJ@?$CFs?3?5Skip?5the?5EEPROM?5write?5operat@ 10021fbc     rtusb_io.obj
 0001:00020fe4       ??_C@_0BC@OIOEAJAE@AGGREGATION?5?$DN?5?$CFd?6?$AA@ 10021fe4     rtusb_io.obj
 0001:00020ff8       ??_C@_0BB@POPOLHKA@ACK?5policy?5?$DN?5?$CFs?6?$AA@ 10021ff8     rtusb_io.obj
 0001:0002100c       ??_C@_09CFPFIELH@BLOCK?9ACK?$AA@ 1002200c     rtusb_io.obj
 0001:00021018       ??_C@_0BA@HHLPELHL@NO?9EXPLICIT?9ACK?$AA@ 10022018     rtusb_io.obj
 0001:00021028       ??_C@_06PDABOHKG@NO?9ACK?$AA@ 10022028     rtusb_io.obj
 0001:00021030       ??_C@_06IOJAGNKJ@NORMAL?$AA@ 10022030     rtusb_io.obj
 0001:00021038       ??_C@_0BL@POKGBEJK@HTCEnable?5?$DN?5?$CFd?5?0?5RDG?5?$DN?5?$CFd?6?$AA@ 10022038     rtusb_io.obj
 0001:00021054       ??_C@_0CB@OFDPEMHH@pAd?9?$DOBbpTuning?4bEnable?5?$DN?5FALSE?5?6@ 10022054     rtusb_io.obj
 0001:00021078       ??_C@_0CA@EGNBFGFC@pAd?9?$DOBbpTuning?4bEnable?5?$DN?5TRUE?5?6?$AA@ 10022078     rtusb_io.obj
 0001:00021098       ??_C@_0CC@ELPOJBLN@bEnableAutoAntennaCheck?5?$DN?5FALSE?5@ 10022098     rtusb_io.obj
 0001:000210bc       ??_C@_0CB@FGGGNGLK@bEnableAutoAntennaCheck?5?$DN?5TRUE?5?6@ 100220bc     rtusb_io.obj
 0001:000210e0       ??_C@_0DB@JONKJNPH@Bulk?5Out?5Reset?5on?5Pipe?$FL?$DN?$CFd?$FN?5Fail@ 100220e0     rtusb_io.obj
 0001:00021114       ??_C@_0CH@PPPNEPAJ@Bulk?5Out?5Reset?5on?5Pipe?$FL?$DN?$CFd?$FN?5Succ@ 10022114     rtusb_io.obj
 0001:0002113c       ??_C@_0BE@IJHOFHLN@USB_RESET_BULK_OUT?6?$AA@ 1002213c     rtusb_io.obj
 0001:00021150       ??_C@_0CC@PMCOHKBA@Bulk?5In?5Reset?5Failed?$CBStatus?$DN0x?$CFx@ 10022150     rtusb_io.obj
 0001:00021174       ??_C@_0BC@OHIOCJJF@RTUSBBulkReceive?6?$AA@ 10022174     rtusb_io.obj
 0001:00021188       ??_C@_0BJ@HGAHBILG@Bulk?5In?5Reset?5Successed?6?$AA@ 10022188     rtusb_io.obj
 0001:000211a4       ??_C@_0CB@PKOLCNCP@Stop?5RX?5failed?0?5ntStatus?$DN0x?$CF08x?6@ 100221a4     rtusb_io.obj
 0001:000211c8       ??_C@_0CK@OAMFMGFN@BulkIn?5IRP?5Pending?0?5pAd?9?$DOPending@ 100221c8     rtusb_io.obj
 0001:000211f4       ??_C@_0BD@FMIJNHBA@USB_RESET_BULK_IN?6?$AA@ 100221f4     rtusb_io.obj
 0001:00021208       ??_C@_0CB@FDNEKIJD@?5BSSID_WCID?4MpduDensity?5?$DN?50x?$CFd?5?6@ 10022208     rtusb_io.obj
 0001:0002122c       ??_C@_0BM@PKMANIME@?5HTPhyMode?4ShortGI?5?$DN?50x?$CFd?5?6?$AA@ 1002222c     rtusb_io.obj
 0001:00021248       ??_C@_0BH@HCJJMAMI@?5HTPhyMode?4BW?5?$DN?50x?$CFd?5?6?$AA@ 10022248     rtusb_io.obj
 0001:00021260       ??_C@_0BI@FACDMPEL@?5HTPhyMode?4MCS?5?$DN?50x?$CFd?5?6?$AA@ 10022260     rtusb_io.obj
 0001:00021278       ??_C@_0BJ@KIKHBHGI@?5HTPhyMode?4MODE?5?$DN?50x?$CFd?5?6?$AA@ 10022278     rtusb_io.obj
 0001:00021294       ??_C@_0CL@CPOFCAIH@DRS?3?5STBC?$DN?$CFd?0?5ShortGI?$DN?$CFd?0?5MODE?$DN?$CF@ 10022294     rtusb_io.obj
 0001:000212c0       ??_C@_0BK@DBAPPPPK@Enable?5antenna?5diversity?6?$AA@ 100222c0     rtusb_io.obj
 0001:000212dc       ??_C@_0BL@JNDJLGNE@Disable?5antenna?5diversity?6?$AA@ 100222dc     rtusb_io.obj
 0001:000212f8       ??_C@_0CB@BCPHCKFJ@Antenna?5diversity?0?5antenna?5?$DN?5?$CFd?6@ 100222f8     rtusb_io.obj
 0001:0002131c       ??_C@_0BE@MHKEALOJ@?5mlme?4word?5?$DN?50x?$CFx?5?6?$AA@ 1002231c     rtusb_io.obj
 0001:00021330       ??_C@_0CB@DHELICI@?5MacTab?4Content?$FL0?$FN?4word?5?$DN?50x?$CFx?5?6@ 10022330     rtusb_io.obj
 0001:00021354       ??_C@_0CB@IENCHDGL@?5MacTab?4Content?$FL1?$FN?4word?5?$DN?50x?$CFx?5?6@ 10022354     rtusb_io.obj
 0001:00021378       ??_C@_0BH@HKCIBPPE@pAd?9?$DOQuickTimerP?5?$DN?5?$CFd?6?$AA@ 10022378     rtusb_io.obj
 0001:00021390       ??_C@_0BD@EPLHMCFO@RTUSBBulkReceive?5?6?$AA@ 10022390     rtusb_io.obj
 0001:000213a4       ??_C@_0BD@FAALMAMI@Normal?5SCANNING?4?5?6?$AA@ 100223a4     rtusb_io.obj
 0001:000213b8       ??_C@_0BF@OPGIKLNA@Send?5a?5NULL?5frame?4?5?6?$AA@ 100223b8     rtusb_io.obj
 0001:000213d0       ??_C@_0BI@LHPLPKDF@Send?5a?5Ps?9Poll?5frame?4?5?6?$AA@ 100223d0     rtusb_io.obj
 0001:000213e8       ??_C@_0CA@EENJOMMG@Force?5Disable?5autowakeup?5?$DN?$CFd?4?5?6?$AA@ 100223e8     rtusb_io.obj
 0001:00021408       ??_C@_0CJ@IOGAPGCO@pAd?9?$DOMacTab?4Content?$FL1?$FN?4HTPhyMode@ 10022408     rtusb_io.obj
 0001:00021434       ??_C@_0CL@KCGLHKAB@MlmeSet?5TbttNumToNextWakeUp?$DN?$CFd?4?5@ 10022434     rtusb_io.obj
 0001:00021460       ??_C@_0CC@FLMFADNG@QUERY?5POWER?5Mailbox?5testvalue?5?$CFx@ 10022460     rtusb_io.obj
 0001:00021484       ??_C@_0BA@EKKIIINA@?5Clear?5Command?6?$AA@ 10022484     rtusb_io.obj
 0001:00021494       ??_C@_0CH@KJPMKMBA@MailBoxTOExec?5read?50x701c?5code?5?3@ 10022494     rtusb_io.obj
 0001:000214bc       ??_C@_0CN@DDBHFDCO@MailBoxTOExec?5read?50x7014?5comman@ 100224bc     rtusb_io.obj
 0001:000214ec       ??_C@_0CB@LJDFNHHJ@SignalStr?5Mailbox?5test?5value?5?$CFx?6@ 100224ec     rtusb_io.obj
 0001:00021510       ??_C@_0BL@CDIDEMBN@LED?5Mailbox?5test?5value?5?$CFx?6?$AA@ 10022510     rtusb_io.obj
 0001:0002152c       ??_C@_0BM@PFCFKFJF@Wakeup?5Mailbox?5testvalue?$CFx?6?$AA@ 1002252c     rtusb_io.obj
 0001:00021548       ??_C@_0CP@PLEDMFNP@?$FL?$CFd?$FN?5IRPPending?$DN?$CFd?3?5?5InUse?$DN?$CFd?3?5R@ 10022548     rtusb_io.obj
 0001:00021578       ??_C@_0DO@DOLMEHOL@?$DO?$DOBulkInReq?$DN0x?$CFx?0?5BulkInComplete@ 10022578     rtusb_io.obj
 0001:000215b8       ??_C@_0FL@EHFCJKKB@NextRxBulkInIndex?5?$DN?50x?$CFx?0?5NextRx@ 100225b8     rtusb_io.obj
 0001:00021614       ??_C@_0DJ@JIFCLFJO@?5?9?9?$DO?5CurWritePosition?5?$DN?5?$CFd?4?5?5Nex@ 10022614     rtusb_io.obj
 0001:00021650       ??_C@_0DJ@JPHLLDHJ@?$DO?$DOBulkOutCompleteCancel?$DN0x?$CFx?0?5Bu@ 10022650     rtusb_io.obj
 0001:0002168c       ??_C@_0CJ@DEGELNPI@?$DO?$DOBulkOutReq?$DN0x?$CFx?0?5BulkOutComple@ 1002268c     rtusb_io.obj
 0001:000216b8       ??_C@_0FL@JKLIDOBM@?$FL?$CFd?$FN?5IRPPending?$DN?$CFd?3?5?5InUse?$DN?$CFd?3?5b@ 100226b8     rtusb_io.obj
 0001:00021714       ??_C@_0CF@KOIJMGHA@?$DN?$DN?$DN?$DN?$DN?$DN?$DN?$DN?$DN?$DN?$DN?$DN?$DNMLME?$DN?$DN?$DN?$DN?$DN?$DN?$DN?$DN?$DN?$DN?$DN?$DN?$DN?$DN?$DN@ 10022714     rtusb_io.obj
 0001:00021740       ??_C@_0EF@BDBBJOKO@pAd?9?$DOPrioRingFirstIndex?5?$DN?5?$CFd?0?5Po@ 10022740     rtusb_io.obj
 0001:00021788       ??_C@_0CG@DOOMPOMN@pAd?9?$DOFlags?$DN0x?$CFx?0?5pAd?9?$DOBulkFlags?$DN@ 10022788     rtusb_io.obj
 0001:000217b0       ??_C@_0CM@KKCJOCLG@?$DN?$DN?$DN?$DN?$DN?$DN?$DN?$DN?$DN?$DN?$DN?$DN?$DN?$DN?$DN?$DN?$DN?$DN?$DN?$DN?$DN?$DN?$DN?$DN?$DN?$DN?$DN?$DN?$DN?$DN?$DN?$DN@ 100227b0     rtusb_io.obj
 0001:000217dc       ??_C@_0BF@LAKBGEGJ@bForcePrintRX?5?$DN?5?$CFd?5?6?$AA@ 100227dc     rtusb_io.obj
 0001:000217f4       ??_C@_0BF@LNLPBECO@bForcePrintTX?5?$DN?5?$CFd?5?6?$AA@ 100227f4     rtusb_io.obj
 0001:0002180c       ??_C@_0BD@FLJKFCJL@Not?5support?5Efuse?6?$AA@ 1002280c     rtusb_io.obj
 0001:00021820       ??_C@_0M@NMHAFGMO@?$CF02x?3?5?$CF02x?6?$AA@ 10022820     rtusb_io.obj
 0001:0002182c       ??_C@_0BN@IMGMAKFC@Dump?5Efuse?5mapping?5address?3?6?$AA@ 1002282c     rtusb_io.obj
 0001:00021850       ??_C@_0FB@JCNDEDAH@CmdThread?3?3RT_OID_802_11_SET_HAR@ 10022850     rtusb_io.obj
 0001:00021aa8       ??_C@_0DE@FHCBIKLJ@MlmeScanReqSanity?5fail?5?9?5wrong?5B@ 10022aa8     sanity.obj
 0001:00021adc       ??_C@_0CN@EEOAAFHE@MlmeStartReqSanity?5fail?5?9?5wrong?5@ 10022adc     sanity.obj
 0001:00021b0c       ??_C@_0CK@GILPPNOI@MlmeAuthReqSanity?5fail?5?9?5wrong?5a@ 10022b0c     sanity.obj
 0001:00021b38       ??_C@_0DD@DHNIMLGH@PeerAssocRspSanity?5?9?5ignore?5unre@ 10022b38     sanity.obj
 0001:00021b6c       ??_C@_0DK@CJBCAKBC@CCX?5CAC?5EDCA?5Lifetime?5TSID?$DN?50x?$CFx@ 10022b6c     sanity.obj
 0001:00021ba8       ??_C@_0CN@GDJPCPMD@CCX?5CAC?5TSRATE?5TSID?$DN?50x?$CFx?0?5Rate?$DN@ 10022ba8     sanity.obj
 0001:00021bd8       ??_C@_0CC@KONJNLFC@AssocRsp?0?5CCX?5version?5match?5?$DN?5?$CFx@ 10022bd8     sanity.obj
 0001:00021bfc       ??_C@_0DE@INFEHLGD@PeerAssocRspSanity?5?9?5wrong?5IE_NE@ 10022bfc     sanity.obj
 0001:00021c30       ??_C@_0CI@HLFEJCHN@PeerAssocRspSanity?5?9?5wrong?5IE_AD@ 10022c30     sanity.obj
 0001:00021c58       ??_C@_0CI@HIKBNHAJ@PeerAssocRspSanity?5?9?5wrong?5IE_HT@ 10022c58     sanity.obj
 0001:00021c80       ??_C@_0DD@BAJFBEKN@PeerAssocRspSanity?5fail?5?9?5wrong?5@ 10022c80     sanity.obj
 0001:00021cb4       ??_C@_0CH@BIPFCJDM@PeerAuthSanity?5fail?5?9?5wrong?5algo@ 10022cb4     sanity.obj
 0001:00021cdc       ??_C@_0CC@EGKFAAHJ@PeerAuthSanity?5fail?5?9?5wrong?5Seq?$CD@ 10022cdc     sanity.obj
 0001:00021d00       ??_C@_0EB@IMPCBFEO@PeerProbeReqSanity?5fail?5?9?5wrong?5@ 10022d00     sanity.obj
 0001:00021d44       ??_C@_0DJ@FMKPGFHG@PeerProbeReqSanity?5fail?5?9?5wrong?5@ 10022d44     sanity.obj
 0001:00021d80       ??_C@_0DM@KELBNLBJ@PeerBeaconAndProbeRspSanity?5?9?5mi@ 10022d80     sanity.obj
 0001:00021dc0       ??_C@_0ED@DBKKONJK@TPC?3?5?$CFs?3?5The?5maximum?5transmit?5po@ 10022dc0     sanity.obj
 0001:00021e08       ??_C@_0GK@JMMHNFOE@TPC?3?5?$CFs?3?5?$CIBSSID?5?$DN?5?$CF02X?3?$CF02X?3?$CF02X@ 10022e08     sanity.obj
 0001:00021e78       ??_C@_0EK@JFBEEOAG@TPC?3?5?$CFs?3?5Search?5the?5maximum?5tran@ 10022e78     sanity.obj
 0001:00021ec4       ??_C@_0DF@ENLIANNN@PeerBeaconAndProbeRspSanity?5?9?5un@ 10022ec4     sanity.obj
 0001:00021f00       ??_C@_0FA@BLDIGCCB@TPC?3?5?$CFs?3?5Power?5constraint?5IE?0?5pP@ 10022f00     sanity.obj
 0001:00021f50       ??_C@_0DJ@DDPPIAHH@TPC?3?5?$CFs?3?5Country?5IE?0?5pCountryIE?9@ 10022f50     sanity.obj
 0001:00021f8c       ??_C@_0DF@GMLEFHIN@TPC?3?5?$CFs?3?5Country?5IE?5is?5too?5short@ 10022f8c     sanity.obj
 0001:00021fc4       ??_C@_0BM@NICDGDMO@PeerBeaconAndProbeRspSanity?$AA@ 10022fc4     sanity.obj
 0001:00021fe0       ??_C@_0BE@JGMOOONG@IE_RSN?5length?5?$DN?5?$CFd?6?$AA@ 10022fe0     sanity.obj
 0001:00021ff4       ??_C@_0CO@GGNNNAAG@PeerBeaconAndProbeRspSanity?5?9?5Re@ 10022ff4     sanity.obj
 0001:00022024       ??_C@_0CD@CBLJPALM@Unknown?5CISCO_OUI?0?5CCX?5IE?5ID?$DN0x?$CF@ 10023024     sanity.obj
 0001:00022048       ??_C@_0DN@IDOFAGDM@PeerBeaconAndProbeRspSanity?0?5CIS@ 10023048     sanity.obj
 0001:00022088       ??_C@_0DC@HFLCAEOC@PeerBeaconAndProbeRspSanity?5?9?5wr@ 10023088     sanity.obj
 0001:000220bc       ??_C@_0DA@PMMJHGGB@PeerBeaconAndProbeRspSanity?5?9?5wr@ 100230bc     sanity.obj
 0001:000220ec       ??_C@_0DJ@BBLNEPEJ@PeerBeaconAndProbeRspSanity?5?9?5wr@ 100230ec     sanity.obj
 0001:00022128       ??_C@_0DI@NLKPHPBJ@PeerBeaconAndProbeRspSanity?5?9?5wr@ 10023128     sanity.obj
 0001:00022160       ??_C@_0CK@HBCJAKBG@PeerBeaconAndProbeRspSanity?$CIIE_F@ 10023160     sanity.obj
 0001:0002218c       ??_C@_0DN@JFLJPABG@PeerBeaconAndProbeRspSanity?5?9?5wr@ 1002318c     sanity.obj
 0001:000221cc       ??_C@_0DB@IJDKOKKO@PeerBeaconAndProbeRspSanity?5?9?5wr@ 100231cc     sanity.obj
 0001:00022200       ??_C@_0DP@PEOJJOPK@PeerBeaconAndProbeRspSanity?5?9?5wr@ 10023200     sanity.obj
 0001:00022240       ??_C@_0DA@BIALMAIJ@PeerBeaconAndProbeRspSanity?5?9?5IE@ 10023240     sanity.obj
 0001:00022270       ??_C@_0DM@OJHKFFDL@PeerBeaconAndProbeRspSanity?5?9?5wr@ 10023270     sanity.obj
 0001:000222ac       ??_C@_0DG@EACFIODC@PeerBeaconAndProbeRspSanity?5?9?5wr@ 100232ac     sanity.obj
 0001:000222e8       ??_C@_0FK@IFKNOOMO@PeerBeaconAndProbeRspSanity?5?9?5Va@ 100232e8     sanity.obj
 0001:00022348       ??_C@_0EC@NPLEEJDJ@PeerBeaconAndProbeRspSanity?5?9?5IE@ 10023348     sanity.obj
 0001:00022390       ??_C@_0EG@ILGIGFEI@PeerBeaconAndProbeRspSanity?5?9?5wr@ 10023390     sanity.obj
 0001:000223d8       ??_C@_0EA@ECPGHPEJ@PeerBeaconAndProbeRspSanity?5?9?5wr@ 100233d8     sanity.obj
 0001:00022418       ??_C@_0DG@KGKOAMPJ@MlmeEnqueueForRecv?3?5ADDBA?5Reques@ 10023418     sanity.obj
 0001:00022450       ??_C@_0CO@NJLDPLMC@ADDBA?5Request?4?5tid?$DN?$CFx?0?5Bufsize?$DN?$CF@ 10023450     sanity.obj
 0001:00022480       ??_C@_0DN@HKGILDBD@MlmeEnqueueForRecv?3?5ADDBA?5Reques@ 10023480     sanity.obj
 0001:000224c0       ??_C@_0EE@KMGPNPCK@MlmeEnqueueForRecv?3?5ADDBA?5Reques@ 100234c0     sanity.obj
 0001:00022504       ??_C@_0DN@FNAMPHPK@PeerAddBARspActionSanity?3?5ADDBA?5@ 10023504     sanity.obj
 0001:00022544       ??_C@_0DO@EAPBKADN@MlmeEnqueueForRecv?3?5ADDBA?5Respon@ 10023544     sanity.obj
 0001:00022588       ??_C@_0EL@BDHGNGGO@PeerAddBARspActionSanity?3?5ADDBA?5@ 10023588     sanity.obj
 0001:000225d4       ??_C@_0DA@BHNABLLJ@RTMPWPAWepKeySanity?3?5GroupKey?5bu@ 100235d4     sanity.obj
 0001:00022608       ??_C@_0ED@OFFNJFKJ@RTMPWPAWepKeySanity?3?5Pairwisekey@ 10023608     sanity.obj
 0001:0002264c       ??_C@_0DP@OOMFANPH@RTMPWPAWepKeySanity?3?5Pairwisekey@ 1002364c     sanity.obj
 0001:0002268c       ??_C@_0DO@DPDCPKNH@RTMPWPAWepKeySanity?3?5Pairwisekey@ 1002368c     sanity.obj
 0001:000226cc       ??_C@_0DG@CLCODGBD@RTMPWPAWepKeySanity?3?5Pairwisekey@ 100236cc     sanity.obj
 0001:00022704       ??_C@_0DD@CNFKBPMD@RTMPWPAWepKeySanity?3?5Pairwisekey@ 10023704     sanity.obj
 0001:00022738       ??_C@_0DM@NNPCKDPE@MlmeAddBAReqSanity?5fail?5?9?5broadc@ 10023738     sanity.obj
 0001:00022778       ??_C@_0EL@HMHKEJEL@MlmeAddBAReqSanity?5fail?5?9?5Rx?5Reo@ 10023778     sanity.obj
 0001:000227c4       ??_C@_0DP@GHGPELOD@MlmeAddBAReqSanity?5fail?5?9?5The?5pe@ 100237c4     sanity.obj
 0001:00022804       ??_C@_0DH@IFBMGPAF@MlmeAddBAReqSanity?5fail?5?9?5messag@ 10023804     sanity.obj
 0001:0002283c       ??_C@_0DG@BJPLBJCA@MlmeDelBAReqSanity?5fail?5?9?5The?5pe@ 1002383c     sanity.obj
 0001:00022874       ??_C@_0DP@PPPDMDCE@MlmeDelBAReqSanity?5fail?5?9?5The?5pe@ 10023874     sanity.obj
 0001:000228b4       ??_C@_0DH@PEONCKLH@MlmeDelBAReqSanity?5fail?5?9?5messag@ 100238b4     sanity.obj
 0001:000228ec       ??_C@_0DA@DPENODEN@PeerTdlsSetupReqSanity?5?9?5unrecog@ 100238ec     sanity.obj
 0001:00022920       ??_C@_0EC@FHEEFOAC@PeerTdlsSetupReqSanity?5?9?9?$DO?5Invai@ 10023920     sanity.obj
 0001:00022964       ??_C@_0DE@JBAOPGAN@PeerTdlsSetupReqSanity?5?9?9?$DO?5It?8s?5@ 10023964     sanity.obj
 0001:00022998       ??_C@_0CO@JGEKCKEI@PeerTdlsSetupReqSanity?5?9?9?$DO?5It?8s?5@ 10023998     sanity.obj
 0001:000229c8       ??_C@_0EH@OOCNJIAJ@PeerTdlsSetupReqSanity?5?9?9?$DO?5Invai@ 100239c8     sanity.obj
 0001:00022a10       ??_C@_0EE@BLDIIKFM@PeerTdlsSetupReqSanity?5?9?9?$DO?5Invai@ 10023a10     sanity.obj
 0001:00022a58       ??_C@_0EF@EAGJAGG@PeerTdlsSetupReqSanity?5?9?9?$DO?5Invai@ 10023a58     sanity.obj
 0001:00022aa0       ??_C@_0DA@PHAEIMKJ@PeerTdlsSetupRspSanity?5?9?5unrecog@ 10023aa0     sanity.obj
 0001:00022ad0       ??_C@_0DE@DPJMBCLB@PeerTdlsSetupRspSanity?5?9?9?$DO?5It?8s?5@ 10023ad0     sanity.obj
 0001:00022b04       ??_C@_0CO@MMLLLLEP@PeerTdlsSetupRspSanity?5?9?9?$DO?5It?8s?5@ 10023b04     sanity.obj
 0001:00022b38       ??_C@_0EH@PBJKEGIH@PeerTdlsSetupRspSanity?5?9?9?$DO?5Invai@ 10023b38     sanity.obj
 0001:00022b80       ??_C@_0EE@HKGHFEMJ@PeerTdlsSetupRspSanity?5?9?9?$DO?5Invai@ 10023b80     sanity.obj
 0001:00022bc8       ??_C@_0ED@GKKJGPOM@PeerTdlsSetupRspSanity?5?9?9?$DO?5Invai@ 10023bc8     sanity.obj
 0001:00022c10       ??_C@_0EF@IEACKIHD@PeerTdlsSetupRspSanity?5?9?9?$DO?5Invai@ 10023c10     sanity.obj
 0001:00022c58       ??_C@_0DB@GKDJKBCO@PeerTdlsSetupConfSanity?5?9?5unreco@ 10023c58     sanity.obj
 0001:00022c8c       ??_C@_0DF@JLNBOOMH@PeerTdlsSetupConfSanity?5?9?9?$DO?5It?8s@ 10023c8c     sanity.obj
 0001:00022cc4       ??_C@_0CP@EDIDBEAM@PeerTdlsSetupConfSanity?5?9?9?$DO?5It?8s@ 10023cc4     sanity.obj
 0001:00022cf8       ??_C@_0EI@LPHJPLIJ@PeerTdlsSetupConfSanity?5?9?9?$DO?5Inva@ 10023cf8     sanity.obj
 0001:00022d40       ??_C@_0EF@NOFAIOBJ@PeerTdlsSetupConfSanity?5?9?9?$DO?5Inva@ 10023d40     sanity.obj
 0001:00022d88       ??_C@_0EE@IMLHNCIK@PeerTdlsSetupConfSanity?5?9?9?$DO?5Inva@ 10023d88     sanity.obj
 0001:00022dd0       ??_C@_0EG@CHFENHN@PeerTdlsSetupConfSanity?5?9?9?$DO?5Inva@ 10023dd0     sanity.obj
 0001:00022e18       ??_C@_0CO@JHHCFIJO@PeerTdlsTearDownSanity?5?9?9?$DO?5It?8s?5@ 10023e18     sanity.obj
 0001:00022e48       ??_C@_0EH@KBLKGDEE@PeerTdlsTearDownSanity?5?9?9?$DO?5Invai@ 10023e48     sanity.obj
 0001:00022e90       ??_C@_0ED@FLONFMOO@PeerTdlsTearDownSanity?5?9?9?$DO?5Invai@ 10023e90     sanity.obj
 0001:00022ed8       ??_C@_0EF@OMLDMNGF@PeerTdlsTearDownSanity?5?9?9?$DO?5Invai@ 10023ed8     sanity.obj
 0001:00023120       ??_C@_0BO@KOHMAOLC@STAWapiWAIPacketAction?5?$DM?$DN?$DN?$DN?5?6?$AA@ 10024120     Sta_wapi.obj
 0001:00023140       ??_C@_0DN@MBEKBCC@STAWapiWAIPacketAction?3?5STA?5don?8@ 10024140     Sta_wapi.obj
 0001:00023180       ??_C@_0DG@NDGJKKOJ@STAWapiWAIPacketAction?3?5STA?5get?5@ 10024180     Sta_wapi.obj
 0001:000231b8       ??_C@_0DG@DLAEBELO@STAWapiWAIPacketAction?3?5STA?5get?5@ 100241b8     Sta_wapi.obj
 0001:000231f0       ??_C@_0DE@PFLAFFCE@STAWapiWAIPacketAction?3?5STA?5get?5@ 100241f0     Sta_wapi.obj
 0001:00023224       ??_C@_0CG@IGBGNFHJ@STAWapiWAIPacketAction?3uSubType?5@ 10024224     Sta_wapi.obj
 0001:0002324c       ??_C@_0DJ@FDEIJNGN@STAWapiWAIPacketAction?3?5?$FLIBSS?$FN?5W@ 1002424c     Sta_wapi.obj
 0001:00023288       ??_C@_0HB@PDPHDGKG@STAWapiWAIPacketAction?3?5Wapi_IBS@ 10024288     Sta_wapi.obj
 0001:00023300       ??_C@_0GF@GGIHGMKO@STAWapiWAIPacketAction?3?5Can?8t?5fi@ 10024300     Sta_wapi.obj
 0001:00023368       ??_C@_0BN@OLMALACC@STAWapiWAIPacketAction?5?$DN?$DN?$DN?$DO?6?$AA@ 10024368     Sta_wapi.obj
 0001:00023388       ??_C@_0CI@LGBGDFCJ@STAWapiWAIPacket_HandleMBcastReq@ 10024388     Sta_wapi.obj
 0001:000233b0       ??_C@_0FC@JFJINLDN@?$EA?$EASTAWapiWAIPacket_HandleMBcastR@ 100243b0     Sta_wapi.obj
 0001:00023404       ??_C@_0BI@DNOHIMKK@Peer?5STA?8s?5MAC?5address?6?$AA@ 10024404     Sta_wapi.obj
 0001:00023420       ??_C@_0GL@OAPNMLLN@STAWapiWAIPacket_HandleMBcastReq@ 10024420     Sta_wapi.obj
 0001:00023490       ??_C@_0IO@BAHNGIMD@STAWapiWAIPacket_HandleMBcastReq@ 10024490     Sta_wapi.obj
 0001:00023520       ??_C@_0CN@CEFHJNLE@Below?5are?5GROUP?5KEY?$CB?$CB?$CB?5Cipher?5Da@ 10024520     Sta_wapi.obj
 0001:00023550       ??_C@_0DE@BBMPMJAN@STAWapiWAIPacket_HandleMBcastReq@ 10024550     Sta_wapi.obj
 0001:00023584       ??_C@_0CN@LEDNFMCK@RT2870Dump?5STAWapiWAIPacket_Hand@ 10024584     Sta_wapi.obj
 0001:000235b8       ??_C@_0ED@EGHCLAIJ@STAWapiWAIPacket_HandleMBcastReq@ 100245b8     Sta_wapi.obj
 0001:000235fc       ??_C@_0DF@FOFEGNNL@STAWapiWAIPacket_HandleMBcastReq@ 100245fc     Sta_wapi.obj
 0001:00023634       ??_C@_0DE@DIJOGNNH@STAWapiWAIPacket_HandleMBcastReq@ 10024634     Sta_wapi.obj
 0001:00023668       ??_C@_0CI@CNEJBHD@STAWapiWAIPacket_HandleMBcastReq@ 10024668     Sta_wapi.obj
 0001:00023690       ??_C@_0CJ@DLMDAMMM@STAWapiWAIPacket_HandleUnicastRe@ 10024690     Sta_wapi.obj
 0001:000236bc       ??_C@_0BL@OODMECFB@Below?5are?5PAIRWISE?5KEY?$CB?$CB?$CB?6?$AA@ 100246bc     Sta_wapi.obj
 0001:000236d8       ??_C@_0DD@LBNMINHM@STAWapiWAIPacket_HandleUnicastRe@ 100246d8     Sta_wapi.obj
 0001:0002370c       ??_C@_0DH@PHGCHFDM@STAWapiWAIPacket_HandleUnicastRe@ 1002470c     Sta_wapi.obj
 0001:00023744       ??_C@_0DL@PKMOELCH@STAWapiWAIPacket_HandleUnicastRe@ 10024744     Sta_wapi.obj
 0001:00023780       ??_C@_0DC@GFGOOAJE@STAWapiWAIPacket_HandleUnicastRe@ 10024780     Sta_wapi.obj
 0001:000237b8       ??_C@_0GE@JIIICJML@STAWapiWAIPacket_HandleUnicastRe@ 100247b8     Sta_wapi.obj
 0001:00023820       ??_C@_0GB@LNKBPDEH@STAWapiWAIPacket_HandleUnicastRe@ 10024820     Sta_wapi.obj
 0001:00023884       ??_C@_0CO@CALEOPEB@RT2870Dump?5STAWapiWAIPacket_Hand@ 10024884     Sta_wapi.obj
 0001:000238b4       ??_C@_08EMFKKEDI@My?5BKID?6?$AA@ 100248b4     Sta_wapi.obj
 0001:000238c0       ??_C@_0CJ@IPABKIJG@STAWapiWAIPacket_HandleUnicastRe@ 100248c0     Sta_wapi.obj
 0001:000238f0       ??_C@_0EO@NIICAHME@STAWapiWAIPacket_HandleUnicastCo@ 100248f0     Sta_wapi.obj
 0001:00023940       ??_C@_0EK@DIENAPBB@?$FL?$CB?$CB?$CB?$CBFinished?5Unicast?5rekey?$CB?$CB?$CB?$CB?$FN@ 10024940     Sta_wapi.obj
 0001:00023990       ??_C@_0EK@KOGNEFAK@STAWapiWAIPacket_HandleUnicastCo@ 10024990     Sta_wapi.obj
 0001:000239dc       ??_C@_0CP@DAJJJBHB@RT2870Dump?5STAWapiWAIPacket_Hand@ 100249dc     Sta_wapi.obj
 0001:00023a10       ??_C@_0HJ@DGJCLIMH@STAWapiWAIPacket_HandleUnicastCo@ 10024a10     Sta_wapi.obj
 0001:00023a8c       ??_C@_0DE@LHICHCMF@STAWapiWAIPacket_HandleUnicastCo@ 10024a8c     Sta_wapi.obj
 0001:00023ac0       ??_C@_0DD@INCEEGNB@STAWapiWAIPacket_HandleUnicastCo@ 10024ac0     Sta_wapi.obj
 0001:00023af8       ??_C@_0EF@ENFAACFC@STAWapiWAIPacket_HandleUnicastCo@ 10024af8     Sta_wapi.obj
 0001:00023b40       ??_C@_0EH@JICKPPIN@STAWapiWAIPacket_HandleUnicastCo@ 10024b40     Sta_wapi.obj
 0001:00023b88       ??_C@_0CK@MIDBDLBM@STAWapiWAIPacket_HandleUnicastCo@ 10024b88     Sta_wapi.obj
 0001:00023bb4       ??_C@_0CK@OEDEPCKB@STAWapiSend_MBcastKeyNegotiate_R@ 10024bb4     Sta_wapi.obj
 0001:00023be0       ??_C@_0EB@DPODNFCN@STAWapiWAIPacket_HandleUnicastRe@ 10024be0     Sta_wapi.obj
 0001:00023c24       ??_C@_0CK@FAPGFGPL@STAWapiSend_MBcastKeyNegotiate_R@ 10024c24     Sta_wapi.obj
 0001:00023c50       ??_C@_0DL@DHJKJDDJ@STAWapiSend_UnicastKeyNegotiate_@ 10024c50     Sta_wapi.obj
 0001:00023c8c       ??_C@_0CL@PJGOEFCP@STAWapiSend_UnicastKeyNegotiate_@ 10024c8c     Sta_wapi.obj
 0001:00023cb8       ??_C@_0DO@IMGLLBNK@?$DM?9?9STAWapi_RxSMS4Decrypt?3?5Receiv@ 10024cb8     Sta_wapi.obj
 0001:00023cf8       ??_C@_0EB@LEHNNPFB@RTUSBRxPacket?3?5SMS4?5decrypt?5fail@ 10024cf8     Sta_wapi.obj
 0001:00023d3c       ??_C@_0O@KDKOPKCH@After?5decrypt?$AA@ 10024d3c     Sta_wapi.obj
 0001:00023d4c       ??_C@_0DN@DNKAAJKK@RTUSBRxPacket?3?5SMS4?5decrypt?5fail@ 10024d4c     Sta_wapi.obj
 0001:00023d8c       ??_C@_0CL@KNFNPCIJ@RTUSBRxPacket?3?5But?5have?5LLC?0?5so?5@ 10024d8c     Sta_wapi.obj
 0001:00023db8       ??_C@_0DG@OLDCMHNN@RTUSBRxPacket?3?5SMS4?5decrypt?5fail@ 10024db8     Sta_wapi.obj
 0001:00023df0       ??_C@_0DO@DHFONKEH@?$FLSMS4?$FN?5Is?5Qos?5Packet?0?5AAD?5len?5is@ 10024df0     Sta_wapi.obj
 0001:00023e30       ??_C@_0BK@HLHGMNBF@?$FLSMS4?$FN?5RX?3?5KeyIdx?5?$DN?5?$FL?$CFd?$FN?6?$AA@ 10024e30     Sta_wapi.obj
 0001:00023e4c       ??_C@_0DB@FOBEGNNG@?$FLSMS4?$FN?5Rx?5IV?5is?5less?5or?5equal?5th@ 10024e4c     Sta_wapi.obj
 0001:00023e80       ??_C@_0CC@LPOIAHHE@RT2870Dump?5STAWapi_RxSMS4Decrypt@ 10024e80     Sta_wapi.obj
 0001:00023ea4       ??_C@_0P@PPFEFBDP@LocalRx?5IVSeq?6?$AA@ 10024ea4     Sta_wapi.obj
 0001:00023eb4       ??_C@_0DB@EMKBMCDI@?$FLSMS4?$FN?5Rx?5IV?5is?5less?5or?5equal?5th@ 10024eb4     Sta_wapi.obj
 0001:00023ee8       ??_C@_0CE@KLAEOCLD@?$FLSMS4?$FN?5I?5am?5ASUE?3?5Rx?5IV?5is?5not?5o@ 10024ee8     Sta_wapi.obj
 0001:00023f0c       ??_C@_0CD@GBBOJEHG@?$FLSMS4?$FN?5I?5am?5AE?3?5Rx?5IV?5is?5not?5eve@ 10024f0c     Sta_wapi.obj
 0001:00023f30       ??_C@_0EH@NIEMIOKM@?9?9?$DOSTAWapi_RxSMS4Decrypt?3?5Receiv@ 10024f30     Sta_wapi.obj
 0001:00024178       ??_C@_0BG@OKHOMMNN@SYNC?5?9?5BeaconTimeout?6?$AA@ 10025178     sync.obj
 0001:00024190       ??_C@_0BG@HLPCBHKO@SYNC?5?9?5Scan?5Timeout?5?6?$AA@ 10025190     sync.obj
 0001:000241a8       ??_C@_0DD@FBBOHEJC@AYNC?5?9?5InvalidStateNullFunction?$CI@ 100251a8     sync.obj
 0001:000241dc       ??_C@_0CO@OPEIFMNL@SYNC?5?9?5MlmeScanReqAction?$CI?$CJ?5sanit@ 100251dc     sync.obj
 0001:0002420c       ??_C@_0BK@GAFEFHPL@SYNC?5?9?5BBP?5R4?5to?520MHz?4l?6?$AA@ 1002520c     sync.obj
 0001:00024228       ??_C@_0CD@EGMEANAP@SCAN?5AST?3?5pAd?9?$DOMlmeAux?4Channel?$DN?$CF@ 10025228     sync.obj
 0001:00024250       ??_C@_0ED@ONPCMCFI@?$CFs?3?5Scan?5the?5remaining?5channel?5l@ 10025250     sync.obj
 0001:00024294       ??_C@_0BC@HKPBHFEE@MlmeScanReqAction?$AA@ 10025294     sync.obj
 0001:000242a8       ??_C@_0CH@GMBGBFED@Cisco?5AST?5Scan?3?5set?5RtyLimit?5to?5@ 100252a8     sync.obj
 0001:000242d0       ??_C@_0DJ@LIDEBBLA@SYNC?5?9?5MlmeScanReqAction?0?5Mlme?4S@ 100252d0     sync.obj
 0001:00024310       ??_C@_0EI@JIDFLIDB@SYNC?5?9?5Switch?5to?5ch?5?$CFd?0?5Wait?5BEA@ 10025310     sync.obj
 0001:00024358       ??_C@_0CL@CELIKACI@SYNC?5?9?5send?5ProbeReq?5?$EA?5channel?$DN?$CF@ 10025358     sync.obj
 0001:00024388       ??_C@_0HF@DHGMFJLI@SYNC?5?9?5?$CI802?411h?5and?1or?5Carrier?5D@ 10025388     sync.obj
 0001:00024400       ??_C@_0FL@GICINNGM@To?5avoid?5disturbing?5the?5associat@ 10025400     sync.obj
 0001:0002445c       ??_C@_0BK@LBELJNOP@?$CB?$CB?$CBto?520MHz?5?4?4?4?4?4?4?4?5?$CB?$CB?$CB?5?6?$AA@ 1002545c     sync.obj
 0001:00024478       ??_C@_0DD@PBMBBKBL@SYNC?5?9?5CCX?5Roaming?0?5Stay?5at?5the?5@ 10025478     sync.obj
 0001:000244ac       ??_C@_0CD@HIEFMEBE@SYNC?5?9?5MlmeJoinReqAction?$CIBSS?5?$CD?$CFd@ 100254ac     sync.obj
 0001:000244d0       ??_C@_0DA@NGBBKGMA@SYNC?5?9?5MlmeStartReqAction?$CI?$CJ?5sani@ 100254d0     sync.obj
 0001:00024500       ??_C@_0DP@NACCAHKL@SYNC?5?9?5MlmeStartReqAction?$CIch?$DN?5?$CFd@ 10025500     sync.obj
 0001:00024540       ??_C@_0DF@LCMPNHGJ@MlmeStartReqAction?5pAd?9?$DOMlmeAux?4@ 10025540     sync.obj
 0001:00024578       ??_C@_0DG@LMLEEOJF@SYNC?5?9pAd?9?$DOStaActive?4SupportedHt@ 10025578     sync.obj
 0001:000245b0       ??_C@_0DE@LEHLJFKE@?$CFs?3?5Break?5scanning?0?5since?5we?5fin@ 100255b0     sync.obj
 0001:000245e4       ??_C@_0BH@GIDJJMCM@PeerBeaconAtScanAction?$AA@ 100255e4     sync.obj
 0001:000245fc       ??_C@_0CN@HMDGOGPC@SSIDL?3?5Update?5ScanTab?$FL?$CFd?$FN?5?$DN?$DN?$DO?5Ti@ 100255fc     sync.obj
 0001:0002462c       ??_C@_0DO@NCCEMJFG@BssTableSetEntry?5for?5SSIDL?0?5SSID@ 1002562c     sync.obj
 0001:0002466c       ??_C@_0DI@MGDNBOAN@PeerBeaconAtJoinAction?0?5after?5JO@ 1002566c     sync.obj
 0001:000246a4       ??_C@_0DB@DECJICF@SYNC?5?9?5after?5JOIN?0?5SupRateLen?$DN?$CFd@ 100256a4     sync.obj
 0001:000246d8       ??_C@_0BL@HICOICLC@SYNC?5?9?5EdcaParm?4bValid?$DN?$CFd?6?$AA@ 100256d8     sync.obj
 0001:000246f4       ??_C@_0DK@EOOHEAPL@PeerBeaconAtJoinAction?$CB?$CB?$CB?5?5?$CI?5BW?$DN@ 100256f4     sync.obj
 0001:00024730       ??_C@_0ED@FLLDHPJI@PeerBeaconAtJoinAction?$CB?$CB?$CB?5?5?$CI?5Mpd@ 10025730     sync.obj
 0001:00024778       ??_C@_0JB@KKBKDED@?$CFs?$DN?$DN?$DOThe?5connected?5AP?5is?5Cisco?5A@ 10025778     sync.obj
 0001:0002480c       ??_C@_0BH@BMGGCEPE@PeerBeaconAtJoinAction?$AA@ 1002580c     sync.obj
 0001:00024828       ??_C@_0EN@GMIIPOJO@PeerBeaconAtJoinAction?5HT?$DN?$DN?$DN?$DOCen@ 10025828     sync.obj
 0001:00024878       ??_C@_0FA@CFDPLIJG@SYNC?5?9?5JoinWaitBeacon?5?4?4?4?5Beacon@ 10025878     sync.obj
 0001:000248c8       ??_C@_0EB@MBFGCIM@SYNC?5?9?5receive?5desired?5BEACON?5at@ 100258c8     sync.obj
 0001:00024910       ??_C@_0FC@CBBNDBHG@PeerBeacon?5?9?5AP?5added?5to?5ScanTab@ 10025910     sync.obj
 0001:00024964       ??_C@_0DC@OHLNNLPI@Drastic?5Roaming?5Case?3?5Update?5the@ 10025964     sync.obj
 0001:00024998       ??_C@_0CE@GIMPGLHE@indicate?5IBSS_INSERTED_EVENT_ID?4@ 10025998     sync.obj
 0001:000249bc       ??_C@_0DF@GNEOKGDC@?$EA?$EAWAPI?3?5IBSS?3?5Peer?5MAC?5address?5i@ 100259bc     sync.obj
 0001:000249f4       ??_C@_0BP@CLOBMGBP@?$CF02X?3?$CF02X?3?$CF02X?3?$CF02X?3?$CF02X?3?$CF02X?6?$AA@ 100259f4     sync.obj
 0001:00024a14       ??_C@_0BB@IIFCAKEG@DUMP?5PeerBeacon?6?$AA@ 10025a14     sync.obj
 0001:00024a28       ??_C@_0CD@GHBBHFGD@?$EA?$EAWAPI?3?5IBSS?3?5peer?5MAC?5address?5?$DN@ 10025a28     sync.obj
 0001:00024a50       ??_C@_0EP@IOGMOEBC@?$EA?$EAWAPI?3?5IBSS?3?5should?5not?5happen?$CB@ 10025a50     sync.obj
 0001:00024aa0       ??_C@_0DB@NNGFJMOI@?$EA?$EAWAPI?3?5IBSS?3?5peer?5STA?5will?5be?5A@ 10025aa0     sync.obj
 0001:00024ad4       ??_C@_0DK@OCPMLLCK@PeerBeacon?5?9?5Send?5AP_WAPI_MT2_UN@ 10025ad4     sync.obj
 0001:00024b10       ??_C@_0DB@KIOAJKHA@?$EA?$EAWAPI?3?5IBSS?3?5our?5STA?5will?5be?5AE@ 10025b10     sync.obj
 0001:00024b44       ??_C@_0DM@PCOLLFKN@ADHOC?5?9?5BA?5BaSizeInUse?5?$DN?5?$CFd?0?5TXB@ 10025b44     sync.obj
 0001:00024b80       ??_C@_0BL@JDLLNIJG@ADHOC?5?9?5Add?5Entry?5failed?4?6?$AA@ 10025b80     sync.obj
 0001:00024b9c       ??_C@_0CM@GAFKKKHD@ADHOC?5?$CFx?3?$CFx?3?$CFx?3?$CFx?3?$CFx?3?$CFx?5?5join?5in@ 10025b9c     sync.obj
 0001:00024bc8       ??_C@_0CE@LNEKLANK@?$CB?$CB?$CB?5Adhoc?5LINK?5UP?5and?5Update?5RTS@ 10025bc8     sync.obj
 0001:00024bec       ??_C@_0CL@OHGONHHD@SYNC?5?9?5PHY?5sleeps?5for?5?$CFd?5TBTT?0?5D@ 10025bec     sync.obj
 0001:00024c18       ??_C@_0DG@MGHEGBJN@SYNC?5?9?5outgoing?5frame?5in?5TxRing?1@ 10025c18     sync.obj
 0001:00024c50       ??_C@_0DD@LJHIBKDP@SYNC?5?9?5AP?5backlog?5broadcast?1mult@ 10025c50     sync.obj
 0001:00024c84       ??_C@_0DK@IMBEEHE@SYNC?5?9?5AP?5backlog?5unicast?9to?9me?0@ 10025c84     sync.obj
 0001:00024cc0       ??_C@_0EA@NEAIJBHG@?$CFs?3?5if?5Supported?5MCS?5change?0?5sho@ 10025cc0     sync.obj
 0001:00024d00       ??_C@_0L@JNBADIJI@PeerBeacon?$AA@ 10025d00     sync.obj
 0001:00024d0c       ??_C@_0DB@POMPAEFO@SYNC?5?9?5AP?5change?5EDCA?5parameters@ 10025d0c     sync.obj
 0001:00024d40       ??_C@_0CH@LMIDECJO@SYNC?5?9?5AP?5forced?5to?5use?5LONG?5pre@ 10025d40     sync.obj
 0001:00024d68       ??_C@_0DL@CPMOMOMM@SYNC?5?9?5AP?5change?5to?5OperaionMode@ 10025d68     sync.obj
 0001:00024da4       ??_C@_0CI@NKMHKFBH@SYNC?5?9?5AP?5changed?5B?1G?5protection@ 10025da4     sync.obj
 0001:00024dcc       ??_C@_0CA@CCOBGKC@SYNC?5?9?5Turn?5Off?5BG?5Protection?5?6?$AA@ 10025dcc     sync.obj
 0001:00024dec       ??_C@_0BP@JMKBNGAM@SYNC?5?9?5Turn?5On?5BG?5Protection?5?6?$AA@ 10025dec     sync.obj
 0001:00024e0c       ??_C@_0O@GANGOBDF@Rx?5My?5BEACON?6?$AA@ 10025e0c     sync.obj
 0001:00024e20       ??_C@_0EO@CJMLMEDG@SYNC?5?9?5PeerBeacon?5from?5?$CF02x?3?$CF02x@ 10025e20     sync.obj
 0001:00024e70       ??_C@_0EK@HECKCKCK@SYNC?5?9?5merge?5to?5the?5IBSS?5with?5bi@ 10025e70     sync.obj
 0001:00024ebc       ??_C@_0CF@LDKJHFHA@SYNC?5?9?5Not?5matched?5wep?5status?5?$CFd@ 10025ebc     sync.obj
 0001:00024ee4       ??_C@_0DL@HIDLGPHM@PeerBeacon?$CIcan?5not?5find?5New?5Chan@ 10025ee4     sync.obj
 0001:00024f20       ??_C@_0EL@BLHDMLMA@PeerBeacon?5?9?5STA?5receive?5channel@ 10025f20     sync.obj
 0001:00024f70       ??_C@_0FD@NMKEIBMC@SYNC?5?9?5New?5AP?5added?5to?5SsidBssTa@ 10025f70     sync.obj
 0001:00024fc4       ??_C@_0BK@OGBCFFEJ@BeaconTimeoutAtJoinAction?$AA@ 10025fc4     sync.obj
 0001:00024fe0       ??_C@_0ED@KKDIGNBO@BeaconTimeoutAtJoinAction?0?5resto@ 10025fe0     sync.obj
 0001:00025024       ??_C@_0CC@HKMEIBBD@SYNC?5?9?5BeaconTimeoutAtJoinAction@ 10026024     sync.obj
 0001:00025048       ??_C@_0CK@EHHPJOME@?$CFs?3?5Found?5the?5desired?5connection@ 10026048     sync.obj
 0001:00025078       ??_C@_0GB@OAGNEHDO@?$CFs?3?5Preserve?5the?5last?5scan?5chann@ 10026078     sync.obj
 0001:000250e0       ??_C@_0FC@PGHONEML@?$CFs?5?9?5Active?5scan?5for?5hidden?5APs?5@ 100260e0     sync.obj
 0001:00025134       ??_C@_0BC@PCLPDOII@ScanTimeoutAction?$AA@ 10026134     sync.obj
 0001:00025148       ??_C@_0EO@EKNEPBCO@?$CFs?3?5This?5is?5a?5hidden?5AP?5?$CIChannel@ 10026148     sync.obj
 0001:00025198       ??_C@_0BJ@OPPOGFNL@HasHiddenAPAtThisChannel?$AA@ 10026198     sync.obj
 0001:000251b4       ??_C@_0CP@DFNCKPDJ@SYNC?5?9?5ScanNextChannel?$CI?$CJ?5allocat@ 100261b4     sync.obj
 0001:000251e8       ??_C@_0GJ@GAEAOGOC@SYNC?5?9?5send?5an?5additional?5ProbeR@ 100261e8     sync.obj
 0001:00025258       ??_C@_0FK@OPLOGPIL@?$CFs?3?5SYNC?9?5The?5pAd?9?$DOMlmeAux?4AutoR@ 10026258     sync.obj
 0001:000252b8       ??_C@_0FL@LFGICNGP@SYNC?5?9?5send?5ProbeReq?5?$EA?5channel?$DN?$CF@ 100262b8     sync.obj
 0001:00025314       ??_C@_0CI@COAIAGKO@?$CFs?3?5SYNC?5?9?5Active?5scan?5for?5hidde@ 10026314     sync.obj
 0001:00025340       ??_C@_0HD@MJFCIKOH@SYNC?5?9?5?$CI802?411h?5and?1or?5Carrier?5D@ 10026340     sync.obj
 0001:000253b4       ??_C@_0CM@ONALHAIP@SYNC?5?9?5global?5domain?0?5passive?5sc@ 100263b4     sync.obj
 0001:000253e0       ??_C@_0BO@NDJIEHCP@SYNC?5?9?5Skip?5the?5channel?5?$CD?5?$CFd?6?$AA@ 100263e0     sync.obj
 0001:00025400       ??_C@_0DG@MNJANJDF@?$CK?$CK?$CK?$CK?$CK?$CK?$CK?$CK?$CK?$CK?$CK?$CK?$CK?$CK?$CK?$CK?5Scan?5Complete?5?$CK@ 10026400     sync.obj
 0001:00025438       ??_C@_0EE@KONNBGA@bFastRoamingScan?5?$HO?$HO?$HO?$HO?$HO?$HO?$HO?$HO?$HO?$HO?$HO?$HO?$HO?5G@ 10026438     sync.obj
 0001:00025480       ??_C@_0GJ@OLPFBJPO@CntlChannelWidth?3?5SYNC?5?9?5End?5of?5@ 10026480     sync.obj
 0001:000254ec       ??_C@_0BA@FCBNCJDJ@ScanNextChannel?$AA@ 100264ec     sync.obj
 0001:000254fc       ??_C@_0DM@CLGDNDLE@SYNC?5?9?5End?5of?5SCAN?0?5restore?5to?5c@ 100264fc     sync.obj
 0001:00025538       ??_C@_0DN@GPFBCMLM@MlmeScanReqAction?5?9?9?5Send?5PSM?5Da@ 10026538     sync.obj
 0001:00025578       ??_C@_0BK@JCBMFILD@SYNC?5?9?5MlmeScanReqAction?6?$AA@ 10026578     sync.obj
 0001:00025594       ??_C@_0DL@DPPLBMBC@AYNC?5?9?5InvalidStateWhenScan?$CIstat@ 10026594     sync.obj
 0001:000255d0       ??_C@_0FA@JPDCMJMC@?$FL070625?$FNSYNC?5?9?5Switch?5to?5ch?5?$CFd?0?5@ 100265d0     sync.obj
 0001:00025620       ??_C@_0DE@DGDDDOIA@InvalidStateWhenJoin?$CIstate?$DN?$CFd?$CJ?4?5@ 10026620     sync.obj
 0001:00025654       ??_C@_0DF@GOPKNNOJ@InvalidStateWhenStart?$CIstate?$DN?$CFd?$CJ?4@ 10026654     sync.obj
 0001:0002568c       ??_C@_0BO@NPMEEBDG@?$CF08x?3?3?5?$CF08x?3?3?5?$CF08x?3?3?5?$CF08x?3?3?5?6?$AA@ 1002668c     sync.obj
 0001:000256ac       ??_C@_0BH@KKMOOIKP@SYNC?5?9?5send?5PsPoll?5?4?4?4?$AA@ 100266ac     sync.obj
 0001:000256c4       ??_C@_0CJ@BDIPLDPB@EnqueueBeaconFrame?5allocate?5memo@ 100266c4     sync.obj
 0001:000256f0       ??_C@_0CH@NBEFGGIA@SYNC?5?9?5driver?5sent?5BEACON?5?$CIlen?$DN?$CF@ 100266f0     sync.obj
 0001:00025718       ??_C@_0BO@BLKMMEKG@force?5out?5a?5ProbeRequest?5?4?4?4?6?$AA@ 10026718     sync.obj
 0001:00025738       ??_C@_04HFIMANJO@?5?$CD?$CFd?$AA@ 10026738     sync.obj
 0001:00025740       ??_C@_0DP@CLKBLMHF@country?5code?$DN?$CFd?1?$CFd?0?5RFIC?$DN?$CFd?0?5PHY@ 10026740     sync.obj
 0001:00025780       ??_C@_0BI@EDHDJIGL@pManualChList?$FL?$CFd?$FN?5?$DN?5?$CFd?6?$AA@ 10026780     sync.obj
 0001:00025798       ??_C@_0BN@POGCCCPH@countryregion?$DN?$CFd?5not?5support?$AA@ 10026798     sync.obj
 0001:000257b8       ??_C@_09LGMEEGCL@num?5?$DN?5?$CFd?6?$AA@ 100267b8     sync.obj
 0001:000257c4       ??_C@_0CK@OIFCNHFM@EEPROMManualChannelList_A_Band_1@ 100267c4     sync.obj
 0001:000257f0       ??_C@_0CK@CJNMAIJM@EEPROMManualChannelList_A_Band_0@ 100267f0     sync.obj
 0001:0002581c       ??_C@_0BG@JPDIKGL@index?5?$DN?5?$CFd?0?5num?5?$DN?5?$CFd?6?$AA@ 1002681c     sync.obj
 0001:00025834       ??_C@_0DA@EIDBDMIG@BuildChannelList?5?9?9?5Region_30_A_@ 10026834     sync.obj
 0001:00025864       ??_C@_0BE@OEOBABJC@index?$CFd?5?$DN?5TxPower?$CFd?$AA@ 10026864     sync.obj
 0001:00025878       ??_C@_0BP@KMBKBFHN@EEPROMManualChannelList?5?$DN?5?$CF04x?$AA@ 10026878     sync.obj
 0001:00025898       ??_C@_0DB@GDOHNDJC@BuildChannelList?5?9?9?5Region_30_BG@ 10026898     sync.obj
 0001:000258cc       ??_C@_0BH@GBHCIFCO@?$DO?$DOBuildChannelList?5?$DM?$DM?6?$AA@ 100268cc     sync.obj
 0001:000258e4       ??_C@_0BM@IFABOGJG@?5EffectedChannel?$FL?$CFd?$FN?$CI?5?$DN?$CFd?$CJ?6?$AA@ 100268e4     sync.obj
 0001:00025900       ??_C@_0EA@NNMPILNL@BuildEffectedChannelList?$CBLowerCh@ 10026900     sync.obj
 0001:00025940       ??_C@_0CL@HJJKJGGD@LinkUP?51?5BuildEffectedChannelLis@ 10026940     sync.obj
 0001:0002596c       ??_C@_0CL@OMOKECPG@LinkUP?50?5BuildEffectedChannelLis@ 1002696c     sync.obj
 0001:00025998       ??_C@_0EB@FLENGLOC@RTMPCheckBWOffset?3?3?5Current?5Chan@ 10026998     sync.obj
 0001:000259e0       ??_C@_0GN@NHIHJNJA@StaAdhocUpdateMacTableEntry?5?9?5Ai@ 100269e0     sync.obj
 0001:00025a50       ??_C@_0FM@KJMPDIMJ@StaAdhocUpdateMacTableEntry?5?9?5Su@ 10026a50     sync.obj
 0001:00025ab0       ??_C@_0FC@GDDOOOKO@StaAdhocUpdateMacTableEntry?5?9?5No@ 10026ab0     sync.obj
 0001:00025b08       ??_C@_0FA@HKCMBHHP@StaAdhocUpdateMacTableEntry?5?9?5No@ 10026b08     sync.obj
 0001:00025b58       ??_C@_0CK@FAIKMEOH@StaAdhocUpdateMacTableEntry?5?9?5NU@ 10026b58     sync.obj
 0001:00025b84       ??_C@_0BN@LHJJJEHG@MlmeProbeInactiveStation?4?4?4?6?$AA@ 10026b84     sync.obj
 0001:00025da8       ??_C@_1CM@BHHLIDEJ@?$AAR?$AAT?$AA2?$AA8?$AA7?$AA0?$AA?3?$AA?$DM?$AA?$DN?$AA?$DN?$AA?5?$AAD?$AAl?$AAl?$AAE?$AAn?$AAt?$AAr?$AAy?$AA?$AN?$AA?6?$AA?$AA@ 10026da8     wince.obj
 0001:00025dd4       ??_C@_1DK@HDOFPFHO@?$AAR?$AAT?$AA2?$AA8?$AA7?$AA0?$AA?3?$AA?5?$AAD?$AAL?$AAL?$AA_?$AAP?$AAR?$AAO?$AAC?$AAE?$AAS?$AAS?$AA_?$AAD?$AAE?$AAT?$AAA?$AAC?$AAH?$AA?$AN?$AA?6?$AA?$AA@ 10026dd4     wince.obj
 0001:00025e10       ??_C@_1DO@GPGHCGLL@?$AAD?$AAr?$AAi?$AAv?$AAe?$AAr?$AA?5?$AAV?$AAe?$AAr?$AAs?$AAi?$AAo?$AAn?$AA?3?$AA?5?$AA0?$AAx?$AA?$CF?$AA0?$AA8?$AAx?$AA?5?$AA?$CI?$AAD?$AAB?$AAG?$AA?$CJ?$AA?$AN?$AA?6?$AA?$AA@ 10026e10     wince.obj
 0001:00025e50       ??_C@_1FC@FAPOEMAG@?$AAB?$AAu?$AAi?$AAl?$AAd?$AA?5?$AAD?$AAa?$AAt?$AAe?$AA?3?$AA?5?$AAD?$AAe?$AAc?$AA?5?$AA?5?$AA4?$AA?5?$AA2?$AA0?$AA0?$AA9?$AA?5?$AAT?$AAi?$AAm?$AAe?$AA?3?$AA?5?$AA1?$AA7@ 10026e50     wince.obj
 0001:00025ea4       ??_C@_1DK@NPFADLJG@?$AAR?$AAT?$AA2?$AA8?$AA7?$AA0?$AA?3?$AA?5?$AAD?$AAL?$AAL?$AA_?$AAP?$AAR?$AAO?$AAC?$AAE?$AAS?$AAS?$AA_?$AAA?$AAT?$AAT?$AAA?$AAC?$AAH?$AA?$AN?$AA?6?$AA?$AA@ 10026ea4     wince.obj
 0001:00025ee0       ??_C@_1CM@NJEMINLJ@?$AAR?$AAT?$AA2?$AA8?$AA7?$AA0?$AA?3?$AA?$DN?$AA?$DN?$AA?$DO?$AA?5?$AAD?$AAl?$AAl?$AAE?$AAn?$AAt?$AAr?$AAy?$AA?$AN?$AA?6?$AA?$AA@ 10026ee0     wince.obj
 0001:00025f0c       ??_C@_1DI@MCOKAIFC@?$AAC?$AAl?$AAo?$AAs?$AAe?$AA?5?$AAP?$AAi?$AAp?$AAe?$AA?5?$AAh?$AAa?$AAn?$AAd?$AAl?$AAe?$AA?$DN?$AA0?$AAx?$AA?$CF?$AA0?$AA8?$AAx?$AA?$CB?$AA?$AN?$AA?6?$AA?$AA@ 10026f0c     wince.obj
 0001:00025f48       ??_C@_1GA@CIFDECFB@?$AAR?$AAT?$AA2?$AA8?$AA7?$AA0?$AA?3?$AA?5?$AAR?$AAT?$AAU?$AAS?$AAB?$AAC?$AAE?$AA_?$AAC?$AAl?$AAo?$AAs?$AAe?$AAP?$AAi?$AAp?$AAe?$AA?5?$AA?9?$AAI?$AAn?$AAv?$AAa?$AAl@ 10026f48     wince.obj
 0001:00025fa8       ??_C@_1FC@DBOLHIBH@?$AAR?$AAT?$AA2?$AA8?$AA7?$AA0?$AA?3?$AA?$DM?$AA?$DN?$AA?$DN?$AA?5?$AAR?$AAT?$AAU?$AAS?$AAB?$AAC?$AAE?$AA_?$AAR?$AAe?$AAm?$AAo?$AAv?$AAe?$AAD?$AAe?$AAv?$AAi?$AAc?$AAe?$AAC@ 10026fa8     wince.obj
 0001:00025ffc       ??_C@_1CI@JMPKHPDN@?$AAI?$AAn?$AAv?$AAa?$AAl?$AAi?$AAd?$AA?5?$AAP?$AAa?$AAr?$AAa?$AAm?$AAe?$AAt?$AAe?$AAr?$AA?$AN?$AA?6?$AA?$AA@ 10026ffc     wince.obj
 0001:00026028       ??_C@_1FK@IKIAOPHK@?$AAR?$AAT?$AA2?$AA8?$AA7?$AA0?$AA?3?$AA?$DN?$AA?$DN?$AA?$DO?$AA?5?$AAR?$AAT?$AAU?$AAS?$AAB?$AAC?$AAE?$AA_?$AAR?$AAe?$AAm?$AAo?$AAv?$AAe?$AAD?$AAe?$AAv?$AAi?$AAc?$AAe?$AAC@ 10027028     wince.obj
 0001:00026084       ??_C@_1O@ECGDNAC@?$AAR?$AAT?$AA2?$AA8?$AA7?$AA0?$AA?$AA@ 10027084     wince.obj
 0001:00026098       ??_C@_1EE@KHLKJEBK@?$AAR?$AAT?$AA2?$AA8?$AA7?$AA0?$AA?3?$AA?$DM?$AA?$DN?$AA?$DN?$AA?5?$AAR?$AAT?$AAU?$AAS?$AAB?$AAC?$AAE?$AA_?$AAD?$AAe?$AAv?$AAi?$AAc?$AAe?$AAN?$AAo?$AAt?$AAi?$AAf?$AAy?$AA?$AN@ 10027098     wince.obj
 0001:000260e0       ??_C@_1FG@OBPKCICF@?$AAR?$AAT?$AAU?$AAS?$AAB?$AAC?$AAE?$AA_?$AAD?$AAe?$AAv?$AAi?$AAc?$AAe?$AAN?$AAo?$AAt?$AAi?$AAf?$AAy?$AA?5?$AA?9?$AA?5?$AAU?$AAn?$AAh?$AAa?$AAn?$AAd?$AAl?$AAe?$AAd@ 100270e0     wince.obj
 0001:00026138       ??_C@_1HE@KIPPELHN@?$AAW?$AAa?$AAr?$AAn?$AAi?$AAn?$AAg?$AA?0?$AA?5?$AAu?$AAn?$AAa?$AAb?$AAl?$AAe?$AA?5?$AAt?$AAo?$AA?5?$AAN?$AAd?$AAi?$AAs?$AAD?$AAe?$AAr?$AAe?$AAg?$AAi?$AAs?$AAt?$AAe@ 10027138     wince.obj
 0001:000261b0       ??_C@_1EA@FBJJOBOM@?$AAR?$AAT?$AA2?$AA8?$AA7?$AA0?$AA?3?$AA?5?$AAN?$AAd?$AAi?$AAs?$AAD?$AAe?$AAr?$AAe?$AAg?$AAi?$AAs?$AAt?$AAe?$AAr?$AAA?$AAd?$AAa?$AAp?$AAt?$AAe?$AAr?$AA?$AN?$AA?6?$AA?$AA@ 100271b0     wince.obj
 0001:000261f0       ??_C@_1BA@CCMJLFHB@?$AAR?$AAT?$AA2?$AA8?$AA7?$AA0?$AA1?$AA?$AA@ 100271f0     wince.obj
 0001:00026200       ??_C@_1CG@FMKAPCIC@?$AAM?$AAl?$AAm?$AAe?$AAT?$AAh?$AAr?$AAe?$AAa?$AAd?$AA?5?$AAc?$AAl?$AAo?$AAs?$AAe?$AA?$AN?$AA?6?$AA?$AA@ 10027200     wince.obj
 0001:00026228       ??_C@_1EM@POODPMPJ@?$AAM?$AAl?$AAm?$AAe?$AAT?$AAh?$AAr?$AAe?$AAa?$AAd?$AA?5?$AAs?$AAt?$AAi?$AAl?$AAl?$AA?5?$AAa?$AAl?$AAi?$AAv?$AAe?$AA?0?$AAt?$AAe?$AAr?$AAm?$AAi?$AAn?$AAa?$AAt?$AAe@ 10027228     wince.obj
 0001:00026274       ??_C@_1CM@EFKKOIOI@?$AAC?$AAo?$AAn?$AAt?$AAr?$AAo?$AAl?$AAT?$AAh?$AAr?$AAe?$AAa?$AAd?$AA?5?$AAc?$AAl?$AAo?$AAs?$AAe?$AA?$AN?$AA?6?$AA?$AA@ 10027274     wince.obj
 0001:000262a0       ??_C@_1FC@CNLEOJHJ@?$AAC?$AAo?$AAn?$AAt?$AAr?$AAo?$AAl?$AAT?$AAh?$AAr?$AAe?$AAa?$AAd?$AA?5?$AAs?$AAt?$AAi?$AAl?$AAl?$AA?5?$AAa?$AAl?$AAi?$AAv?$AAe?$AA?0?$AAt?$AAe?$AAr?$AAm?$AAi?$AAn@ 100272a0     wince.obj
 0001:000262f8       ??_C@_1HA@JDPIIGPN@?$AAR?$AAT?$AAU?$AAS?$AAB?$AAC?$AAE?$AA_?$AAD?$AAe?$AAv?$AAi?$AAc?$AAe?$AAN?$AAo?$AAt?$AAi?$AAf?$AAy?$AA?5?$AA?9?$AA?5?$AAU?$AAS?$AAB?$AA_?$AAC?$AAL?$AAO?$AAS?$AAE@ 100272f8     wince.obj
 0001:00026368       ??_C@_1DM@EHELCDIJ@?$AAd?$AAw?$AAC?$AAo?$AAd?$AAe?$AA?$DN?$AAU?$AAS?$AAB?$AA_?$AAC?$AAL?$AAO?$AAS?$AAE?$AA_?$AAD?$AAE?$AAV?$AAI?$AAC?$AAE?$AA?$CI?$AA?$CF?$AAd?$AA?$CJ?$AA?$AN?$AA?6?$AA?$AA@ 10027368     wince.obj
 0001:000263a8       ??_C@_1FE@OLNIAGLP@?$AA?$CF?$AAs?$AA?3?$AA?5?$AAC?$AAo?$AAd?$AAe?$AA?5?$AAC?$AAo?$AAv?$AAe?$AAr?$AAa?$AAg?$AAe?$AA?5?$AAT?$AAr?$AAa?$AAp?$AA?5?$AAi?$AAn?$AA?3?$AA?5?$AA?$CF?$AAs?$AA?0?$AA?5?$AAL@ 100273a8     wince.obj
 0001:000263fc       ??_C@_1BG@PKPPFBOC@?$AAR?$AAT?$AA2?$AA8?$AA7?$AA0?$AA?4?$AAD?$AAL?$AAL?$AA?$AA@ 100273fc     wince.obj
 0001:00026418       ??_C@_1FE@JDEOPNLJ@?$AAC?$AA?3?$AA?2?$AAW?$AAi?$AAn?$AAC?$AAE?$AA6?$AA?4?$AA0?$AA?2?$AAN?$AAe?$AAw?$AA?2?$AAR?$AAT?$AA2?$AA8?$AA7?$AA0?$AA_?$AAv?$AA1?$AA?4?$AA4?$AA?4?$AA9?$AA?4?$AA0?$AA?2@ 10027418     wince.obj
 0001:00026470       ??_C@_1FE@HNNNIJPA@?$AAR?$AAT?$AAU?$AAS?$AAB?$AAC?$AAE?$AA_?$AAD?$AAe?$AAv?$AAi?$AAc?$AAe?$AAN?$AAo?$AAt?$AAi?$AAf?$AAy?$AA?5?$AA?9?$AA?5?$AAI?$AAn?$AAv?$AAa?$AAl?$AAi?$AAd?$AA?5?$AAC@ 10027470     wince.obj
 0001:000264c8       ??_C@_1FK@MPMFIHKK@?$AAR?$AAT?$AA2?$AA8?$AA7?$AA0?$AA?3?$AA?$DN?$AA?$DN?$AA?$DO?$AA?5?$AAR?$AAT?$AAU?$AAS?$AAB?$AAC?$AAE?$AA_?$AAD?$AAe?$AAv?$AAi?$AAc?$AAe?$AAN?$AAo?$AAt?$AAi?$AAf?$AAy?$AA?0@ 100274c8     wince.obj
 0001:00026528       ??_C@_1EK@ODHOLCLP@?$AAR?$AAT?$AA2?$AA8?$AA7?$AA0?$AA?3?$AA?$DM?$AA?$DN?$AA?$DN?$AA?5?$AAR?$AAT?$AAU?$AAS?$AAB?$AAC?$AAE?$AA_?$AAC?$AAo?$AAn?$AAf?$AAi?$AAg?$AAu?$AAr?$AAe?$AAD?$AAe?$AAv?$AAi@ 10027528     wince.obj
 0001:00026578       ??_C@_1FA@JFLELJBE@?$AAR?$AAT?$AA2?$AA8?$AA7?$AA0?$AA?5?$AAi?$AAs?$AA?5?$AAc?$AAo?$AAn?$AAf?$AAi?$AAg?$AAr?$AAe?$AAd?$AA?5?$AAi?$AAn?$AA?5?$AA2?$AA?5?$AAp?$AAi?$AAp?$AAe?$AAs?$AA?4?$AA?4@ 10027578     wince.obj
 0001:000265c8       ??_C@_1EM@KHEIHJPL@?$AAR?$AAT?$AA2?$AA8?$AA7?$AA0?$AA?5?$AAi?$AAs?$AA?5?$AAc?$AAo?$AAn?$AAf?$AAi?$AAg?$AAr?$AAe?$AAd?$AA?5?$AAi?$AAn?$AA?5?$AA2?$AA?5?$AAp?$AAi?$AAp?$AAe?$AAs?$AA?4?$AA?4@ 100275c8     wince.obj
 0001:00026618       ??_C@_1FA@CDDPKMPK@?$AAR?$AAT?$AA2?$AA8?$AA7?$AA0?$AA?5?$AAi?$AAs?$AA?5?$AAc?$AAo?$AAn?$AAf?$AAi?$AAg?$AAr?$AAe?$AAd?$AA?5?$AAi?$AAn?$AA?5?$AA7?$AA?5?$AAp?$AAi?$AAp?$AAe?$AAs?$AA?4?$AA?4@ 10027618     wince.obj
 0001:00026668       ??_C@_1EM@GKKLBGND@?$AAR?$AAT?$AA2?$AA8?$AA7?$AA0?$AA?5?$AAi?$AAs?$AA?5?$AAc?$AAo?$AAn?$AAf?$AAi?$AAg?$AAr?$AAe?$AAd?$AA?5?$AAi?$AAn?$AA?5?$AA7?$AA?5?$AAp?$AAi?$AAp?$AAe?$AAs?$AA?4?$AA?4@ 10027668     wince.obj
 0001:000266b8       ??_C@_1EI@EEPCIFC@?$AAB?$AAu?$AAl?$AAk?$AAI?$AAn?$AA?5?$AAI?$AAn?$AAd?$AAe?$AAx?$AA?$DN?$AA?$CF?$AAd?$AA?0?$AA?5?$AAM?$AAa?$AAx?$AAP?$AAa?$AAc?$AAk?$AAe?$AAt?$AAS?$AAi?$AAz?$AAe?$AA?$DN?$AA?$CF@ 100276b8     wince.obj
 0001:00026700       ??_C@_1DC@BGEMFGOP@?$AAO?$AAp?$AAe?$AAn?$AA?5?$AAB?$AAu?$AAl?$AAk?$AA?5?$AAI?$AAn?$AA?5?$AAP?$AAi?$AAp?$AAe?$AA?4?$AA?4?$AA?4?$AA?$AN?$AA?6?$AA?$AN?$AA?6?$AA?$AA@ 10027700     wince.obj
 0001:00026734       ??_C@_1CK@CAEIPOEK@?$AAO?$AAp?$AAe?$AAn?$AAP?$AAi?$AAp?$AAe?$AA?5?$AAe?$AAr?$AAr?$AAo?$AAr?$AA?3?$AA?5?$AA?$CF?$AAd?$AA?$AN?$AA?6?$AA?$AA@ 10027734     wince.obj
 0001:00026760       ??_C@_1EK@JFHIKHEJ@?$AAB?$AAu?$AAl?$AAk?$AAO?$AAu?$AAt?$AA?5?$AAI?$AAn?$AAd?$AAe?$AAx?$AA?$DN?$AA?$CF?$AAd?$AA?0?$AA?5?$AAM?$AAa?$AAx?$AAP?$AAa?$AAc?$AAk?$AAe?$AAt?$AAS?$AAi?$AAz?$AAe?$AA?$DN@ 10027760     wince.obj
 0001:000267ac       ??_C@_1DG@IMDGOLBA@?$AAO?$AAp?$AAe?$AAn?$AA?5?$AAB?$AAu?$AAl?$AAk?$AA?5?$AAO?$AAu?$AAt?$AA?5?$AAP?$AAi?$AAp?$AAe?$AA?5?$AA?$CF?$AAd?$AA?4?$AA?$AN?$AA?6?$AA?$AN?$AA?6?$AA?$AA@ 100277ac     wince.obj
 0001:000267e4       ??_C@_1CI@DCGFFIOH@?$AAO?$AAp?$AAe?$AAn?$AAP?$AAi?$AAp?$AAe?$AA?5?$AAe?$AAr?$AAr?$AAo?$AAr?$AA?3?$AA?$CF?$AAd?$AA?$AN?$AA?6?$AA?$AA@ 100277e4     wince.obj
 0001:0002680c       ??_C@_15JNBOKNOG@?$AA?$AN?$AA?6?$AA?$AA@ 1002780c     wince.obj
 0001:00026814       ??_C@_1CE@HCABCFIA@?$AAb?$AAI?$AAn?$AAt?$AAe?$AAr?$AAv?$AAa?$AAl?$AA?3?$AA?5?$AA0?$AAx?$AA?$CF?$AAx?$AA?$AN?$AA?6?$AA?$AA@ 10027814     wince.obj
 0001:00026838       ??_C@_1CO@LIHJEKO@?$AAw?$AAM?$AAa?$AAx?$AAP?$AAa?$AAc?$AAk?$AAe?$AAt?$AAS?$AAi?$AAz?$AAe?$AA?3?$AA?5?$AA0?$AAx?$AA?$CF?$AAx?$AA?$AN?$AA?6?$AA?$AA@ 10027838     wince.obj
 0001:00026868       ??_C@_1CK@KLMMILPK@?$AAb?$AAm?$AAA?$AAt?$AAt?$AAr?$AAi?$AAb?$AAu?$AAt?$AAe?$AAs?$AA?3?$AA?5?$AA0?$AAx?$AA?$CF?$AAx?$AA?$AN?$AA?6?$AA?$AA@ 10027868     wince.obj
 0001:00026894       ??_C@_1DC@GOKDAOKL@?$AAb?$AAE?$AAn?$AAd?$AAp?$AAo?$AAi?$AAn?$AAt?$AAA?$AAd?$AAd?$AAr?$AAe?$AAs?$AAs?$AA?3?$AA?5?$AA0?$AAx?$AA?$CF?$AAx?$AA?$AN?$AA?6?$AA?$AA@ 10027894     wince.obj
 0001:000268c8       ??_C@_1DA@EEFFIAIE@?$AAb?$AAD?$AAe?$AAs?$AAc?$AAr?$AAi?$AAp?$AAt?$AAo?$AAr?$AAT?$AAy?$AAp?$AAe?$AA?3?$AA?5?$AA0?$AAx?$AA?$CF?$AAx?$AA?$AN?$AA?6?$AA?$AA@ 100278c8     wince.obj
 0001:000268f8       ??_C@_1CA@CLOOEKHC@?$AAb?$AAL?$AAe?$AAn?$AAg?$AAt?$AAh?$AA?3?$AA?5?$AA0?$AAx?$AA?$CF?$AAx?$AA?$AN?$AA?6?$AA?$AA@ 100278f8     wince.obj
 0001:00026918       ??_C@_1EA@ENBBADGH@?$AA?9?$AA?9?$AA?9?$AA?9?$AA?9?$AA?9?$AA?9?$AA?9?$AA?9?$AA?9?$AA?9?$AA?9?$AA?9?$AA?9?$AA?9?$AA?9?$AA?9?$AA?9?$AA?9?$AA?9?$AA?9?$AA?9?$AA?9?$AA?9?$AA?9?$AA?9?$AA?9?$AA?9?$AA?9?$AA?$AN?$AA?6?$AA?$AA@ 10027918     wince.obj
 0001:00026958       ??_C@_1DG@FBHCDIOA@?$AAU?$AAS?$AAB?$AA_?$AAE?$AAN?$AAD?$AAP?$AAO?$AAI?$AAN?$AAT?$AA_?$AAD?$AAE?$AAS?$AAC?$AAR?$AAI?$AAP?$AAT?$AAO?$AAR?$AA?3?$AA?$AN?$AA?6?$AA?$AA@ 10027958     wince.obj
 0001:00026990       ??_C@_1DG@HEMLHFHK@?$AAS?$AAe?$AAt?$AAU?$AAs?$AAb?$AAI?$AAn?$AAt?$AAe?$AAr?$AAf?$AAa?$AAc?$AAe?$AA?5?$AAe?$AAr?$AAr?$AAo?$AAr?$AA?3?$AA?$CF?$AAd?$AA?$AN?$AA?6?$AA?$AA@ 10027990     wince.obj
 0001:000269c8       ??_C@_0DC@PLDICDGE@pUsbInterface?9?$DODescriptor?4bInter@ 100279c8     wince.obj
 0001:000269fc       ??_C@_1CI@GCCMIBEH@?$AAI?$AAn?$AAv?$AAa?$AAl?$AAi?$AAd?$AA?5?$AAp?$AAa?$AAr?$AAa?$AAm?$AAe?$AAt?$AAe?$AAr?$AA?$AN?$AA?6?$AA?$AA@ 100279fc     wince.obj
 0001:00026a28       ??_C@_1EK@PBCAIEJ@?$AAR?$AAT?$AA2?$AA8?$AA7?$AA0?$AA?3?$AA?$DN?$AA?$DN?$AA?$DO?$AA?5?$AAR?$AAT?$AAU?$AAS?$AAB?$AAC?$AAE?$AA_?$AAC?$AAo?$AAn?$AAf?$AAi?$AAg?$AAu?$AAr?$AAe?$AAD?$AAe?$AAv?$AAi@ 10027a28     wince.obj
 0001:00026a78       ??_C@_1EI@DFDHJAIB@?$AAR?$AAT?$AA2?$AA8?$AA7?$AA0?$AA?3?$AA?$DM?$AA?$DN?$AA?$DN?$AA?5?$AAR?$AAT?$AAU?$AAS?$AAB?$AAC?$AAE?$AA_?$AAI?$AAn?$AAt?$AAe?$AAr?$AAf?$AAa?$AAc?$AAe?$AAS?$AAt?$AAa?$AAr@ 10027a78     wince.obj
 0001:00026ac0       ??_C@_1CC@JJHBOMBA@?$AAR?$AAT?$AA2?$AA8?$AA7?$AA0?$AA?3?$AA?5?$AAR?$AAe?$AAa?$AAd?$AAy?$AA?4?$AA?$AN?$AA?6?$AA?$AA@ 10027ac0     wince.obj
 0001:00026ae8       ??_C@_1EO@NFLONBLC@?$AAR?$AAe?$AAg?$AAi?$AAs?$AAt?$AAe?$AAr?$AAN?$AAo?$AAt?$AAi?$AAf?$AAi?$AAc?$AAa?$AAt?$AAi?$AAo?$AAn?$AAR?$AAo?$AAu?$AAt?$AAi?$AAn?$AAe?$AA?5?$AAe?$AAr?$AAr?$AAo@ 10027ae8     wince.obj
 0001:00026b38       ??_C@_1EE@OFMHELFL@?$AAR?$AAT?$AAU?$AAS?$AAB?$AAC?$AAE?$AA_?$AAC?$AAo?$AAn?$AAf?$AAi?$AAg?$AAu?$AAr?$AAe?$AAD?$AAe?$AAv?$AAi?$AAc?$AAe?$AA?5?$AAf?$AAa?$AAi?$AAl?$AAe?$AAd?$AA?4?$AA?$AN@ 10027b38     wince.obj
 0001:00026b80       ??_C@_1EI@HNBOGFMI@?$AAR?$AAT?$AA2?$AA8?$AA7?$AA0?$AA?3?$AA?$DN?$AA?$DN?$AA?$DO?$AA?5?$AAR?$AAT?$AAU?$AAS?$AAB?$AAC?$AAE?$AA_?$AAI?$AAn?$AAt?$AAe?$AAr?$AAf?$AAa?$AAc?$AAe?$AAS?$AAt?$AAa?$AAr@ 10027b80     wince.obj
 0001:00026bc8       ??_C@_1DK@BDGINGDP@?$AAR?$AAT?$AA2?$AA8?$AA7?$AA0?$AA?3?$AA?$DM?$AA?$DN?$AA?$DN?$AA?5?$AAU?$AAS?$AAB?$AAD?$AAe?$AAv?$AAi?$AAc?$AAe?$AAA?$AAt?$AAt?$AAa?$AAc?$AAh?$AA?$AN?$AA?6?$AA?$AA@ 10027bc8     wince.obj
 0001:00026c08       ??_C@_1EM@PBMPPJBH@?$AAR?$AAT?$AA2?$AA8?$AA7?$AA0?$AA?3?$AA?5?$AAD?$AAa?$AAt?$AAa?$AA?5?$AAc?$AAa?$AAc?$AAh?$AAe?$AA?9?$AAl?$AAi?$AAn?$AAe?$AA?5?$AAb?$AAo?$AAu?$AAn?$AAd?$AAa?$AAr?$AAy@ 10027c08     wince.obj
 0001:00026c54       ??_C@_1DC@EKFFGEO@?$AAR?$AAT?$AA2?$AA8?$AA7?$AA0?$AA?5?$AAR?$AAe?$AAg?$AAi?$AAs?$AAt?$AAe?$AAr?$AAA?$AAd?$AAa?$AAp?$AAt?$AAe?$AAr?$AA?4?$AA?6?$AA?$AA@ 10027c54     wince.obj
 0001:00026c88       ??_C@_1GO@PFOBFKOM@?$AAR?$AAT?$AA2?$AA8?$AA7?$AA0?$AA?3?$AA?5?$AAU?$AAn?$AAa?$AAb?$AAl?$AAe?$AA?5?$AAt?$AAo?$AA?5?$AAN?$AAd?$AAi?$AAs?$AAR?$AAe?$AAg?$AAi?$AAs?$AAt?$AAe?$AAr?$AAA?$AAd@ 10027c88     wince.obj
 0001:00026cf8       ??_C@_1GK@MPKDPBBO@?$AAP?$AAa?$AAr?$AAs?$AAe?$AAU?$AAs?$AAb?$AAD?$AAe?$AAs?$AAc?$AAr?$AAi?$AAp?$AAt?$AAo?$AAr?$AAs?$AA?5?$AAf?$AAa?$AAi?$AAl?$AAe?$AAd?$AA?$CB?$AA?5?$AAR?$AAT?$AA2?$AA8@ 10027cf8     wince.obj
 0001:00026d64       ??_C@_1DI@HDPCPAKC@?$AAR?$AAT?$AA2?$AA8?$AA7?$AA0?$AA?3?$AA?5?$AAD?$AAe?$AAv?$AAi?$AAc?$AAe?$AA?5?$AAC?$AAl?$AAa?$AAs?$AAs?$AA?3?$AA0?$AAx?$AA?$CF?$AAx?$AA?$AN?$AA?6?$AA?$AA@ 10027d64     wince.obj
 0001:00026d9c       ??_C@_1DO@HCENPNHL@?$AAD?$AAe?$AAa?$AAf?$AAu?$AAl?$AAt?$AA?5?$AAU?$AAS?$AAB?$AA?5?$AAI?$AAn?$AAt?$AAe?$AAr?$AAf?$AAa?$AAc?$AAe?$AA?$DN?$AA0?$AAx?$AA?$CF?$AA0?$AA8?$AAx?$AA?$AN?$AA?6?$AA?$AA@ 10027d9c     wince.obj
 0001:00026de0       ??_C@_1EO@DGHMMBND@?$AAF?$AAo?$AAu?$AAn?$AAd?$AA?5?$AAa?$AA?5?$AAU?$AAS?$AAB?$AA?5?$AAI?$AAn?$AAt?$AAe?$AAr?$AAf?$AAa?$AAc?$AAe?$AA?$DN?$AA0?$AAx?$AA?$CF?$AA0?$AA8?$AAx?$AA?0?$AA?5?$AAi?$AAd@ 10027de0     wince.obj
 0001:00026e30       ??_C@_1DK@GDKJCNPA@?$AAU?$AAS?$AAB?$AA?5?$AAI?$AAn?$AAt?$AAe?$AAr?$AAf?$AAa?$AAc?$AAe?$AA?5?$AAS?$AAe?$AAa?$AAr?$AAc?$AAh?$AAi?$AAn?$AAg?$AA?4?$AA?4?$AA?4?$AA?$AN?$AA?6?$AA?$AA@ 10027e30     wince.obj
 0001:00026e70       ??_C@_1FC@HLOHLBOG@?$AAR?$AAT?$AA2?$AA8?$AA7?$AA0?$AA?3?$AA?$DN?$AA?$DN?$AA?$DO?$AA?5?$AAU?$AAS?$AAB?$AAD?$AAe?$AAv?$AAi?$AAc?$AAe?$AAA?$AAt?$AAt?$AAa?$AAc?$AAh?$AA?5?$AA?5?$AA?$CI?$AA0?$AAx?$AA?$CF@ 10027e70     wince.obj
 0001:00026ec4       ??_C@_1DM@LDDABILD@?$AAR?$AAT?$AA2?$AA8?$AA7?$AA0?$AA?3?$AA?$DM?$AA?$DN?$AA?$DN?$AA?5?$AAU?$AAS?$AAB?$AAI?$AAn?$AAs?$AAt?$AAa?$AAl?$AAl?$AAD?$AAr?$AAi?$AAv?$AAe?$AAr?$AA?$AN?$AA?6?$AA?$AA@ 10027ec4     wince.obj
 0001:00026f00       ??_C@_1EE@MHNANKFI@?$AAR?$AAe?$AAg?$AAi?$AAs?$AAt?$AAe?$AAr?$AAC?$AAl?$AAi?$AAe?$AAn?$AAt?$AAS?$AAe?$AAt?$AAt?$AAi?$AAn?$AAg?$AAs?$AA?5?$AAe?$AAr?$AAr?$AAo?$AAr?$AA?3?$AA?$CF?$AAd?$AA?$AN@ 10027f00     wince.obj
 0001:00026f48       ??_C@_1EE@PHEKIMBI@?$AAR?$AAe?$AAg?$AAi?$AAs?$AAt?$AAe?$AAr?$AAC?$AAl?$AAi?$AAe?$AAn?$AAt?$AAD?$AAr?$AAi?$AAv?$AAe?$AAr?$AAI?$AAD?$AA?5?$AAe?$AAr?$AAr?$AAo?$AAr?$AA?3?$AA?$CF?$AAd?$AA?$AN@ 10027f48     wince.obj
 0001:00026f8c       ??_C@_1DM@PEMCAIFD@?$AAR?$AAT?$AA2?$AA8?$AA7?$AA0?$AA?3?$AA?$DN?$AA?$DN?$AA?$DO?$AA?5?$AAU?$AAS?$AAB?$AAI?$AAn?$AAs?$AAt?$AAa?$AAl?$AAl?$AAD?$AAr?$AAi?$AAv?$AAe?$AAr?$AA?$AN?$AA?6?$AA?$AA@ 10027f8c     wince.obj
 0001:00026fc8       ??_C@_1EG@JIBDDOML@?$AAR?$AAT?$AA2?$AA8?$AA7?$AA0?$AA?3?$AA?$DM?$AA?$DN?$AA?$DN?$AA?5?$AAU?$AAS?$AAB?$AAU?$AAn?$AAI?$AAn?$AAs?$AAt?$AAa?$AAl?$AAl?$AAD?$AAr?$AAi?$AAv?$AAe?$AAr?$AA?3?$AA?$CF?$AAd@ 10027fc8     wince.obj
 0001:00027010       ??_C@_1EA@NJGNPFMN@?$AAR?$AAT?$AA2?$AA8?$AA7?$AA0?$AA?3?$AA?$DN?$AA?$DN?$AA?$DO?$AA?5?$AAU?$AAS?$AAB?$AAU?$AAn?$AAI?$AAn?$AAs?$AAt?$AAa?$AAl?$AAl?$AAD?$AAr?$AAi?$AAv?$AAe?$AAr?$AA?$AN?$AA?6?$AA?$AA@ 10028010     wince.obj
 0001:00027050       ??_C@_1EC@HLGADALB@?$AAR?$AAT?$AA2?$AA8?$AA7?$AA0?$AA?3?$AA?$DM?$AA?$DN?$AA?$DN?$AA?5?$AAL?$AAo?$AAa?$AAd?$AAV?$AAI?$AAD?$AAF?$AAr?$AAo?$AAm?$AAR?$AAe?$AAg?$AAi?$AAs?$AAt?$AAr?$AAy?$AA?$AN?$AA?6@ 10028050     wince.obj
 0001:00027094       ??_C@_1CO@KEGAEHEH@?$AAO?$AAp?$AAe?$AAn?$AA?5?$AAR?$AAe?$AAg?$AAi?$AAs?$AAt?$AAr?$AAy?$AA?5?$AAF?$AAa?$AAi?$AAl?$AAe?$AAd?$AA?$AN?$AA?6?$AA?$AA@ 10028094     wince.obj
 0001:000270c8       ??_C@_1EI@LIHOANKL@?$AAL?$AAo?$AAa?$AAd?$AA?5?$AAV?$AAI?$AAD?$AA?1?$AAP?$AAI?$AAD?$AA?5?$AAF?$AAr?$AAo?$AAm?$AA?5?$AAR?$AAe?$AAg?$AAi?$AAs?$AAt?$AAr?$AAy?$AA?5?$AAF?$AAa?$AAi?$AAl?$AAe@ 100280c8     wince.obj
 0001:00027110       ??_C@_1CE@DNCGOPOI@?$AAL?$AAo?$AAa?$AAd?$AA?5?$AAP?$AAI?$AAD?$AA?$DN?$AA0?$AAx?$AA?$CF?$AA0?$AA4?$AAx?$AA?$AN?$AA?6?$AA?$AA@ 10028110     wince.obj
 0001:00027134       ??_C@_1CE@CPIDCFJ@?$AAL?$AAo?$AAa?$AAd?$AA?5?$AAV?$AAI?$AAD?$AA?$DN?$AA0?$AAx?$AA?$CF?$AA0?$AA4?$AAx?$AA?$AN?$AA?6?$AA?$AA@ 10028134     wince.obj
 0001:00027158       ??_C@_1BM@OOGBHLFH@?$AAC?$AAu?$AAs?$AAt?$AAo?$AAm?$AAi?$AAz?$AAe?$AAd?$AAP?$AAI?$AAD?$AA?$AA@ 10028158     wince.obj
 0001:00027174       ??_C@_1BM@CIAOHCNA@?$AAC?$AAu?$AAs?$AAt?$AAo?$AAm?$AAi?$AAz?$AAe?$AAd?$AAV?$AAI?$AAD?$AA?$AA@ 10028174     wince.obj
 0001:00027190       ??_C@_1IE@HNGICLPE@?$AAC?$AAu?$AAs?$AAt?$AAo?$AAm?$AAi?$AAz?$AAe?$AAd?$AAC?$AAo?$AAn?$AAt?$AAr?$AAo?$AAl?$AAF?$AAl?$AAa?$AAg?$AA?$DO?$AA?$DN?$AA2?$AA?0?$AA?5?$AAL?$AAo?$AAa?$AAd?$AA?5?$AAB@ 10028190     wince.obj
 0001:00027218       ??_C@_1GC@CPKHJOL@?$AAC?$AAu?$AAs?$AAt?$AAo?$AAm?$AAi?$AAz?$AAe?$AAd?$AAC?$AAo?$AAn?$AAt?$AAr?$AAo?$AAl?$AAF?$AAl?$AAa?$AAg?$AA?$DN?$AA1?$AA?0?$AA?5?$AAL?$AAo?$AAa?$AAd?$AA?5?$AAE?$AAx@ 10028218     wince.obj
 0001:00027280       ??_C@_1GC@MHAPECCA@?$AAC?$AAu?$AAs?$AAt?$AAo?$AAm?$AAi?$AAz?$AAe?$AAd?$AAC?$AAo?$AAn?$AAt?$AAr?$AAo?$AAl?$AAF?$AAl?$AAa?$AAg?$AA?$DN?$AA0?$AA?0?$AA?5?$AAL?$AAo?$AAa?$AAd?$AA?5?$AAI?$AAn@ 10028280     wince.obj
 0001:000272e8       ??_C@_1HC@GLOCAGIO@?$AAL?$AAo?$AAa?$AAd?$AA?5?$AAC?$AAu?$AAs?$AAt?$AAo?$AAm?$AAi?$AAz?$AAe?$AAd?$AAC?$AAo?$AAn?$AAt?$AAr?$AAo?$AAl?$AAF?$AAl?$AAa?$AAg?$AA?5?$AAF?$AAa?$AAi?$AAl?$AAe@ 100282e8     wince.obj
 0001:0002735c       ??_C@_1CM@CEPJCBLC@?$AAC?$AAu?$AAs?$AAt?$AAo?$AAm?$AAi?$AAz?$AAe?$AAd?$AAC?$AAo?$AAn?$AAt?$AAr?$AAo?$AAl?$AAF?$AAl?$AAa?$AAg?$AA?$AA@ 1002835c     wince.obj
 0001:00027388       ??_C@_1CG@GEIBFOOG@?$AAC?$AAo?$AAm?$AAm?$AA?2?$AAR?$AAT?$AA2?$AA8?$AA7?$AA0?$AA1?$AA?2?$AAP?$AAa?$AAr?$AAm?$AAs?$AA?$AA@ 10028388     wince.obj
 0001:000273b0       ??_C@_1EC@FEHOPJNI@?$AAR?$AAT?$AA2?$AA8?$AA7?$AA0?$AA?3?$AA?$DN?$AA?$DN?$AA?$DO?$AA?5?$AAL?$AAo?$AAa?$AAd?$AAV?$AAI?$AAD?$AAF?$AAr?$AAo?$AAm?$AAR?$AAe?$AAg?$AAi?$AAs?$AAt?$AAr?$AAy?$AA?$AN?$AA?6@ 100283b0     wince.obj
 0001:000273f8       ??_C@_1HO@BFALFBNM@?$AAR?$AAT?$AA2?$AA8?$AA7?$AA0?$AA?3?$AA?$DM?$AA?$DN?$AA?$DN?$AA?5?$AAP?$AAa?$AAr?$AAs?$AAe?$AAU?$AAs?$AAb?$AAD?$AAe?$AAs?$AAc?$AAr?$AAi?$AAp?$AAt?$AAo?$AAr?$AAs?$AA?4?$AA?5@ 100283f8     wince.obj
 0001:00027478       ??_C@_1FI@LMMNFLHH@?$AAR?$AAT?$AA2?$AA8?$AA7?$AA0?$AA?3?$AAF?$AAo?$AAu?$AAn?$AAd?$AA?5?$AAU?$AAs?$AAb?$AA?5?$AAi?$AAn?$AAt?$AAe?$AAr?$AAf?$AAa?$AAc?$AAe?$AA?$DN?$AA0?$AAx?$AA?$CF?$AA0?$AA8@ 10028478     wince.obj
 0001:000274d0       ??_C@_1CG@IFLAKLCK@?$AAi?$AAI?$AAn?$AAt?$AAe?$AAr?$AAf?$AAa?$AAc?$AAe?$AA?3?$AA?5?$AA0?$AAx?$AA?$CF?$AAx?$AA?$AN?$AA?6?$AA?$AA@ 100284d0     wince.obj
 0001:000274f8       ??_C@_1DG@PIHIEECL@?$AAb?$AAI?$AAn?$AAt?$AAe?$AAr?$AAf?$AAa?$AAc?$AAe?$AAP?$AAr?$AAo?$AAt?$AAo?$AAc?$AAo?$AAl?$AA?3?$AA?5?$AA0?$AAx?$AA?$CF?$AAx?$AA?$AN?$AA?6?$AA?$AA@ 100284f8     wince.obj
 0001:00027530       ??_C@_1DG@KDHFAFM@?$AAb?$AAI?$AAn?$AAt?$AAe?$AAr?$AAf?$AAa?$AAc?$AAe?$AAS?$AAu?$AAb?$AAC?$AAl?$AAa?$AAs?$AAs?$AA?3?$AA?5?$AA0?$AAx?$AA?$CF?$AAx?$AA?$AN?$AA?6?$AA?$AA@ 10028530     wince.obj
 0001:00027568       ??_C@_1DA@EDEFDCHL@?$AAb?$AAI?$AAn?$AAt?$AAe?$AAr?$AAf?$AAa?$AAc?$AAe?$AAC?$AAl?$AAa?$AAs?$AAs?$AA?3?$AA?5?$AA0?$AAx?$AA?$CF?$AAx?$AA?$AN?$AA?6?$AA?$AA@ 10028568     wince.obj
 0001:00027598       ??_C@_1CM@IIKLFHEC@?$AAb?$AAN?$AAu?$AAm?$AAE?$AAn?$AAd?$AAp?$AAo?$AAi?$AAn?$AAt?$AAs?$AA?3?$AA?5?$AA0?$AAx?$AA?$CF?$AAx?$AA?$AN?$AA?6?$AA?$AA@ 10028598     wince.obj
 0001:000275c4       ??_C@_1DE@NHAPNLFD@?$AAb?$AAA?$AAl?$AAt?$AAe?$AAr?$AAn?$AAa?$AAt?$AAe?$AAS?$AAe?$AAt?$AAt?$AAi?$AAn?$AAg?$AA?3?$AA?5?$AA0?$AAx?$AA?$CF?$AAx?$AA?$AN?$AA?6?$AA?$AA@ 100285c4     wince.obj
 0001:000275f8       ??_C@_1DC@MEMNJHBF@?$AAb?$AAI?$AAn?$AAt?$AAe?$AAr?$AAf?$AAa?$AAc?$AAe?$AAN?$AAu?$AAm?$AAb?$AAe?$AAr?$AA?3?$AA?5?$AA0?$AAx?$AA?$CF?$AAx?$AA?$AN?$AA?6?$AA?$AA@ 100285f8     wince.obj
 0001:0002762c       ??_C@_1DI@ICGGBIHH@?$AA?9?$AA?9?$AA?9?$AA?9?$AA?9?$AA?9?$AA?9?$AA?9?$AA?9?$AA?9?$AA?9?$AA?9?$AA?9?$AA?9?$AA?9?$AA?9?$AA?9?$AA?9?$AA?9?$AA?9?$AA?9?$AA?9?$AA?9?$AA?9?$AA?9?$AA?$AN?$AA?6?$AA?$AA@ 1002862c     wince.obj
 0001:00027668       ??_C@_1EA@HIDJGMKA@?$AAU?$AAS?$AAB?$AA_?$AAI?$AAN?$AAT?$AAE?$AAR?$AAF?$AAA?$AAC?$AAE?$AA_?$AAD?$AAE?$AAS?$AAC?$AAR?$AAI?$AAP?$AAT?$AAO?$AAR?$AA?$FL?$AA?$CF?$AAd?$AA?$FN?$AA?3?$AA?$AN?$AA?6?$AA?$AA@ 10028668     wince.obj
 0001:000276a8       ??_C@_1CM@CJAJFOCN@?$AAU?$AAS?$AAB?$AA?5?$AAC?$AAo?$AAn?$AAf?$AAi?$AAg?$AA?5?$AAI?$AAn?$AAd?$AAe?$AAx?$AA?$DN?$AA?$CF?$AAd?$AA?$AN?$AA?6?$AA?$AA@ 100286a8     wince.obj
 0001:000276d8       ??_C@_1GK@EFNNGGDG@?$AAD?$AAe?$AAv?$AAi?$AAc?$AAe?$AA?5?$AAi?$AAs?$AA?5?$AAn?$AAo?$AAt?$AA?5?$AAm?$AAa?$AAt?$AAc?$AAh?$AAe?$AAd?$AA?5?$AAc?$AAu?$AAs?$AAt?$AAo?$AAm?$AAe?$AAr?$AA?8?$AAs@ 100286d8     wince.obj
 0001:00027744       ??_C@_1DM@GIKJLEAJ@?$AAD?$AAe?$AAv?$AAi?$AAc?$AAe?$AA?$CI?$AAV?$AAI?$AAD?$AA?$DN?$AA0?$AAx?$AA?$CF?$AA0?$AA4?$AAx?$AA?0?$AA?5?$AAP?$AAI?$AAD?$AA?$DN?$AA0?$AAx?$AA?$CF?$AA4?$AAx?$AA?$CJ?$AA?$AA@ 10028744     wince.obj
 0001:00027780       ??_C@_1HM@IGPJLFMJ@?$AAT?$AAh?$AAi?$AAs?$AA?5?$AAd?$AAe?$AAv?$AAi?$AAc?$AAe?$AA?5?$AAi?$AAs?$AA?5?$AAn?$AAo?$AAt?$AA?5?$AAf?$AAo?$AAu?$AAn?$AAd?$AA?5?$AAi?$AAn?$AA?5?$AAt?$AAh?$AAe?$AA?5@ 10028780     wince.obj
 0001:00027800       ??_C@_1GG@JEDMGKLO@?$AAF?$AAo?$AAu?$AAn?$AAd?$AA?5?$AAa?$AA?5?$AAs?$AAu?$AAp?$AAp?$AAo?$AAr?$AAt?$AAe?$AAd?$AA?5?$AAd?$AAe?$AAv?$AAi?$AAc?$AAe?$AA?$CI?$AAV?$AAI?$AAD?$AA?$DN?$AA0?$AAx?$AA?$CF@ 10028800     wince.obj
 0001:00027868       ??_C@_1EE@GOOOCJCF@?$AAT?$AAo?$AAt?$AAa?$AAl?$AA?5?$AAs?$AAu?$AAp?$AAp?$AAo?$AAr?$AAt?$AAe?$AAd?$AA?5?$AA?$CF?$AAd?$AA?5?$AAU?$AAS?$AAB?$AA?5?$AAd?$AAe?$AAv?$AAi?$AAc?$AAe?$AAs?$AA?4?$AA?$AN@ 10028868     wince.obj
 0001:000278ac       ??_C@_1CC@LOPFMING@?$AAM?$AAa?$AAx?$AAP?$AAo?$AAw?$AAe?$AAr?$AA?3?$AA?5?$AA0?$AAx?$AA?$CF?$AAx?$AA?$AN?$AA?6?$AA?$AA@ 100288ac     wince.obj
 0001:000278d0       ??_C@_1CO@DCDGKEKI@?$AAi?$AAC?$AAo?$AAn?$AAf?$AAi?$AAg?$AAu?$AAr?$AAa?$AAt?$AAi?$AAo?$AAn?$AA?3?$AA?5?$AA0?$AAx?$AA?$CF?$AAx?$AA?$AN?$AA?6?$AA?$AA@ 100288d0     wince.obj
 0001:00027900       ??_C@_1DI@BMBGEIBL@?$AAb?$AAC?$AAo?$AAn?$AAf?$AAi?$AAg?$AAu?$AAr?$AAa?$AAt?$AAi?$AAo?$AAn?$AAV?$AAa?$AAl?$AAu?$AAe?$AA?3?$AA?5?$AA0?$AAx?$AA?$CF?$AAx?$AA?$AN?$AA?6?$AA?$AA@ 10028900     wince.obj
 0001:00027938       ??_C@_1CO@OKPNEMPD@?$AAb?$AAN?$AAu?$AAm?$AAI?$AAn?$AAt?$AAe?$AAr?$AAf?$AAa?$AAc?$AAe?$AAs?$AA?3?$AA?5?$AA0?$AAx?$AA?$CF?$AAx?$AA?$AN?$AA?6?$AA?$AA@ 10028938     wince.obj
 0001:00027968       ??_C@_1CK@DFEDICHM@?$AAw?$AAT?$AAo?$AAt?$AAa?$AAl?$AAL?$AAe?$AAn?$AAg?$AAt?$AAh?$AA?3?$AA?5?$AA0?$AAx?$AA?$CF?$AAx?$AA?$AN?$AA?6?$AA?$AA@ 10028968     wince.obj
 0001:00027998       ??_C@_1EA@MIJDAJH@?$AAU?$AAS?$AAB?$AA_?$AAC?$AAO?$AAN?$AAF?$AAI?$AAG?$AAU?$AAR?$AAA?$AAT?$AAI?$AAO?$AAN?$AA_?$AAD?$AAE?$AAS?$AAC?$AAR?$AAI?$AAP?$AAT?$AAO?$AAR?$AA?3?$AA?$AN?$AA?6?$AA?$AA@ 10028998     wince.obj
 0001:000279d8       ??_C@_1DG@IJKOLLI@?$AAb?$AAN?$AAu?$AAm?$AAC?$AAo?$AAn?$AAf?$AAi?$AAg?$AAu?$AAr?$AAa?$AAt?$AAi?$AAo?$AAn?$AAs?$AA?3?$AA?5?$AA0?$AAx?$AA?$CF?$AAx?$AA?$AN?$AA?6?$AA?$AA@ 100289d8     wince.obj
 0001:00027a10       ??_C@_1CM@DCJDIHK@?$AAi?$AAS?$AAe?$AAr?$AAi?$AAa?$AAl?$AAN?$AAu?$AAm?$AAb?$AAe?$AAr?$AA?3?$AA?5?$AA0?$AAx?$AA?$CF?$AAx?$AA?$AN?$AA?6?$AA?$AA@ 10028a10     wince.obj
 0001:00027a3c       ??_C@_1CC@FNMHHDBN@?$AAi?$AAP?$AAr?$AAo?$AAd?$AAu?$AAc?$AAt?$AA?3?$AA?5?$AA0?$AAx?$AA?$CF?$AAx?$AA?$AN?$AA?6?$AA?$AA@ 10028a3c     wince.obj
 0001:00027a60       ??_C@_1CM@EAIDCOFA@?$AAi?$AAM?$AAa?$AAn?$AAu?$AAf?$AAa?$AAc?$AAt?$AAu?$AAr?$AAe?$AAr?$AA?3?$AA?5?$AA0?$AAx?$AA?$CF?$AAx?$AA?$AN?$AA?6?$AA?$AA@ 10028a60     wince.obj
 0001:00027a8c       ??_C@_1CE@KFOJIAEC@?$AAb?$AAc?$AAd?$AAD?$AAe?$AAv?$AAi?$AAc?$AAe?$AA?3?$AA?5?$AA0?$AAx?$AA?$CF?$AAx?$AA?$AN?$AA?6?$AA?$AA@ 10028a8c     wince.obj
 0001:00027ab0       ??_C@_1CK@PEANKDAO@?$AAi?$AAd?$AAP?$AAr?$AAo?$AAd?$AAu?$AAc?$AAt?$AA?3?$AA?5?$AA?$CF?$AAd?$AA?$DN?$AA0?$AAx?$AA?$CF?$AAx?$AA?$AN?$AA?6?$AA?$AA@ 10028ab0     wince.obj
 0001:00027adc       ??_C@_1CI@FEAGFPDG@?$AAi?$AAd?$AAV?$AAe?$AAn?$AAd?$AAo?$AAr?$AA?3?$AA?5?$AA?$CF?$AAd?$AA?$DN?$AA0?$AAx?$AA?$CF?$AAx?$AA?$AN?$AA?6?$AA?$AA@ 10028adc     wince.obj
 0001:00027b04       ??_C@_1DA@OGKOKEJB@?$AAb?$AAM?$AAa?$AAx?$AAP?$AAa?$AAc?$AAk?$AAe?$AAt?$AAS?$AAi?$AAz?$AAe?$AA0?$AA?3?$AA?5?$AA0?$AAx?$AA?$CF?$AAx?$AA?$AN?$AA?6?$AA?$AA@ 10028b04     wince.obj
 0001:00027b34       ??_C@_1DA@PPLCGINE@?$AAb?$AAD?$AAe?$AAv?$AAi?$AAc?$AAe?$AAP?$AAr?$AAo?$AAt?$AAo?$AAc?$AAo?$AAl?$AA?3?$AA?5?$AA0?$AAx?$AA?$CF?$AAx?$AA?$AN?$AA?6?$AA?$AA@ 10028b34     wince.obj
 0001:00027b64       ??_C@_1DA@NPNHMKD@?$AAb?$AAD?$AAe?$AAv?$AAi?$AAc?$AAe?$AAS?$AAu?$AAb?$AAC?$AAl?$AAa?$AAs?$AAs?$AA?3?$AA?5?$AA0?$AAx?$AA?$CF?$AAx?$AA?$AN?$AA?6?$AA?$AA@ 10028b64     wince.obj
 0001:00027b94       ??_C@_1CK@HMHKELPA@?$AAb?$AAD?$AAe?$AAv?$AAi?$AAc?$AAe?$AAC?$AAl?$AAa?$AAs?$AAs?$AA?3?$AA?5?$AA0?$AAx?$AA?$CF?$AAx?$AA?$AN?$AA?6?$AA?$AA@ 10028b94     wince.obj
 0001:00027bc0       ??_C@_1BO@KIOIBPFP@?$AAb?$AAc?$AAd?$AAU?$AAS?$AAB?$AA?3?$AA?5?$AA0?$AAx?$AA?$CF?$AAx?$AA?$AN?$AA?6?$AA?$AA@ 10028bc0     wince.obj
 0001:00027be0       ??_C@_1DC@EKFFFINH@?$AA?9?$AA?9?$AA?9?$AA?9?$AA?9?$AA?9?$AA?9?$AA?9?$AA?9?$AA?9?$AA?9?$AA?9?$AA?9?$AA?9?$AA?9?$AA?9?$AA?9?$AA?9?$AA?9?$AA?9?$AA?9?$AA?9?$AA?$AN?$AA?6?$AA?$AA@ 10028be0     wince.obj
 0001:00027c14       ??_C@_1DC@BCNGPCJI@?$AAU?$AAS?$AAB?$AA_?$AAD?$AAE?$AAV?$AAI?$AAC?$AAE?$AA_?$AAD?$AAE?$AAS?$AAC?$AAR?$AAI?$AAP?$AAT?$AAO?$AAR?$AA?3?$AA?$AN?$AA?6?$AA?$AA@ 10028c14     wince.obj
 0001:00027c48       ??_C@_1DC@GNDMFOKL@?$AAG?$AAe?$AAt?$AAD?$AAe?$AAv?$AAi?$AAc?$AAe?$AAI?$AAn?$AAf?$AAo?$AA?5?$AAe?$AAr?$AAr?$AAo?$AAr?$AA?3?$AA?$CF?$AAd?$AA?$AN?$AA?6?$AA?$AA@ 10028c48     wince.obj
 0001:00027c80       ??_C@_1EA@LBCNPIEL@?$AAI?$AAn?$AAv?$AAa?$AAl?$AAi?$AAd?$AA?5?$AAp?$AAa?$AAr?$AAa?$AAm?$AAe?$AAt?$AAe?$AAr?$AA?3?$AAC?$AAo?$AAn?$AAf?$AAi?$AAg?$AAI?$AAn?$AAd?$AAe?$AAx?$AA?$AN?$AA?6?$AA?$AA@ 10028c80     wince.obj
 0001:00027cc0       ??_C@_1EC@BLMAJBLK@?$AAI?$AAn?$AAv?$AAa?$AAl?$AAi?$AAd?$AA?5?$AAp?$AAa?$AAr?$AAa?$AAm?$AAe?$AAt?$AAe?$AAr?$AA?3?$AAC?$AAu?$AAr?$AAI?$AAn?$AAt?$AAe?$AAr?$AAf?$AAa?$AAc?$AAe?$AA?$AN?$AA?6@ 10028cc0     wince.obj
 0001:00027d04       ??_C@_1DK@KILCHDCF@?$AAI?$AAn?$AAv?$AAa?$AAl?$AAi?$AAd?$AA?5?$AAp?$AAa?$AAr?$AAa?$AAm?$AAe?$AAt?$AAe?$AAr?$AA?3?$AAU?$AAs?$AAb?$AAF?$AAu?$AAn?$AAc?$AAs?$AA?$AN?$AA?6?$AA?$AA@ 10028d04     wince.obj
 0001:00027d40       ??_C@_1DO@BDDPKKG@?$AAI?$AAn?$AAv?$AAa?$AAl?$AAi?$AAd?$AA?5?$AAp?$AAa?$AAr?$AAa?$AAm?$AAe?$AAt?$AAe?$AAr?$AA?3?$AAh?$AAU?$AAs?$AAb?$AAD?$AAe?$AAv?$AAi?$AAc?$AAe?$AA?$AN?$AA?6?$AA?$AA@ 10028d40     wince.obj
 0001:00027d80       ??_C@_1EC@PFIPFCG@?$AAR?$AAT?$AA2?$AA8?$AA7?$AA0?$AA?3?$AA?$DN?$AA?$DN?$AA?$DO?$AA?5?$AAP?$AAa?$AAr?$AAs?$AAe?$AAU?$AAs?$AAb?$AAD?$AAe?$AAs?$AAc?$AAr?$AAi?$AAp?$AAt?$AAo?$AAr?$AAs?$AA?$AN?$AA?6@ 10028d80     wince.obj
 0001:00027dc4       ??_C@_07BNCCFNNE@?$CF4?44x?5?5?$AA@ 10028dc4     wince.obj
 0001:00027dcc       ??_C@_0BA@MCNGBKFE@?$DN?$DN?$DO?5?$CFs?$CI?$CFd?$CJ?5?$DM?$DN?$DN?6?$AA@ 10028dcc     wince.obj
 0001:00027ddc       ??_C@_0BB@JCEFLFJE@0123456789abcdef?$AA@ 10028ddc     wince.obj
 0001:00027df0       ??_C@_1FK@DMAEMGGE@?$AAC?$AAa?$AAs?$AAe?$AA?5?$AA2?$AA?9?$AA2?$AA?$CI?$AAp?$AAS?$AAr?$AAc?$AA?$DN?$AAp?$AAD?$AAe?$AAs?$AAt?$AA?$CL?$AA1?$AA6?$AA?$CJ?$AA?3?$AA?3?$AAR?$AAt?$AAl?$AAM?$AAo?$AAv?$AAe@ 10028df0     wince.obj
 0001:00027e50       ??_C@_1GC@NGOPGHFM@?$AAC?$AAa?$AAs?$AAe?$AA?5?$AA2?$AA?9?$AA2?$AA?$CI?$AAp?$AAS?$AAr?$AAc?$AA?$DN?$AAp?$AAD?$AAe?$AAs?$AAt?$AA?$CL?$AA1?$AA6?$AA?$CJ?$AA?3?$AA?3?$AAR?$AAt?$AAl?$AAM?$AAo?$AAv?$AAe@ 10028e50     wince.obj
 0001:00027eb4       ??_C@_0BC@GFDKHKNI@Case?52?92?4?5Orginal?$AA@ 10028eb4     wince.obj
 0001:00027ec8       ??_C@_1FM@EPHGPOHD@?$AAC?$AAa?$AAs?$AAe?$AA?5?$AA2?$AA?9?$AA1?$AA?$CI?$AAp?$AAS?$AAr?$AAc?$AA?$DN?$AAp?$AAD?$AAe?$AAs?$AAt?$AA?$CL?$AA1?$AA6?$AA?$CJ?$AA?3?$AA?3?$AAN?$AAd?$AAi?$AAs?$AAM?$AAo?$AAv@ 10028ec8     wince.obj
 0001:00027f28       ??_C@_1GE@MDIFICIO@?$AAC?$AAa?$AAs?$AAe?$AA?5?$AA2?$AA?9?$AA1?$AA?$CI?$AAp?$AAS?$AAr?$AAc?$AA?$DN?$AAp?$AAD?$AAe?$AAs?$AAt?$AA?$CL?$AA1?$AA6?$AA?$CJ?$AA?3?$AA?3?$AAN?$AAd?$AAi?$AAs?$AAM?$AAo?$AAv@ 10028f28     wince.obj
 0001:00027f8c       ??_C@_0BC@PMNIBMNJ@Case?52?91?4?5Orginal?$AA@ 10028f8c     wince.obj
 0001:00027fa0       ??_C@_1FK@NKIDCHLA@?$AAC?$AAa?$AAs?$AAe?$AA?5?$AA1?$AA?9?$AA2?$AA?$CI?$AAp?$AAD?$AAe?$AAs?$AAt?$AA?$DN?$AAp?$AAS?$AAr?$AAc?$AA?$CL?$AA1?$AA6?$AA?$CJ?$AA?3?$AA?3?$AAR?$AAt?$AAl?$AAM?$AAo?$AAv?$AAe@ 10028fa0     wince.obj
 0001:00028000       ??_C@_1GC@FFEOKEAG@?$AAC?$AAa?$AAs?$AAe?$AA?5?$AA1?$AA?9?$AA2?$AA?$CI?$AAp?$AAD?$AAe?$AAs?$AAt?$AA?$DN?$AAp?$AAS?$AAr?$AAc?$AA?$CL?$AA1?$AA6?$AA?$CJ?$AA?3?$AA?3?$AAR?$AAt?$AAl?$AAM?$AAo?$AAv?$AAe@ 10029000     wince.obj
 0001:00028064       ??_C@_0BE@KCBFLJGD@After?5RtlMoveMemory?$AA@ 10029064     wince.obj
 0001:00028078       ??_C@_0BC@NIPABGBG@Case?51?92?4?5Orginal?$AA@ 10029078     wince.obj
 0001:00028090       ??_C@_1FM@HNCPMKAB@?$AAC?$AAa?$AAs?$AAe?$AA?5?$AA1?$AA?9?$AA1?$AA?$CI?$AAp?$AAD?$AAe?$AAs?$AAt?$AA?$DN?$AAp?$AAS?$AAr?$AAc?$AA?$CL?$AA1?$AA6?$AA?$CJ?$AA?3?$AA?3?$AAN?$AAd?$AAi?$AAs?$AAM?$AAo?$AAv@ 10029090     wince.obj
 0001:000280f0       ??_C@_1GE@IBLMCHPL@?$AAC?$AAa?$AAs?$AAe?$AA?5?$AA1?$AA?9?$AA1?$AA?$CI?$AAp?$AAD?$AAe?$AAs?$AAt?$AA?$DN?$AAp?$AAS?$AAr?$AAc?$AA?$CL?$AA1?$AA6?$AA?$CJ?$AA?3?$AA?3?$AAN?$AAd?$AAi?$AAs?$AAM?$AAo?$AAv@ 100290f0     wince.obj
 0001:00028154       ??_C@_0BF@NDIEOGBM@After?5NdisMoveMemory?$AA@ 10029154     wince.obj
 0001:0002816c       ??_C@_0BL@ENACGPHD@pSrc?$DN0x?$CF08x?0?5pDest?$DN0x?$CF08x?6?$AA@ 1002916c     wince.obj
 0001:00028188       ??_C@_09OGLAPBDF@Reference?$AA@ 10029188     wince.obj
 0001:00028194       ??_C@_0BC@EBBCHABH@Case?51?91?4?5Orginal?$AA@ 10029194     wince.obj
 0001:000281a8       ??_C@_1DG@BCJAAIHH@?$AA?9?$AA?9?$AA?$DN?$AA?$DN?$AA?5?$AAT?$AAe?$AAs?$AAt?$AAM?$AAo?$AAv?$AAe?$AAM?$AAe?$AAm?$AAo?$AAr?$AAy?$AA?5?$AA?$DN?$AA?$DN?$AA?9?$AA?9?$AA?$AN?$AA?6?$AA?$AA@ 100291a8     wince.obj
 0001:000281e0       ??_C@_1DC@LKOADMHA@?$AAP?$AAr?$AAo?$AAc?$AAe?$AAs?$AAs?$AAo?$AAr?$AAR?$AAe?$AAv?$AAi?$AAs?$AAi?$AAo?$AAn?$AA?$DN?$AA?$CF?$AA0?$AA4?$AAx?$AA?$AN?$AA?6?$AA?$AA@ 100291e0     wince.obj
 0001:00028214       ??_C@_1CI@BKHJAAEJ@?$AAP?$AAr?$AAo?$AAc?$AAe?$AAs?$AAs?$AAo?$AAr?$AAL?$AAe?$AAv?$AAe?$AAl?$AA?$DN?$AA?$CF?$AAd?$AA?$AN?$AA?6?$AA?$AA@ 10029214     wince.obj
 0001:0002823c       ??_C@_1BM@KHHDMGEP@?$AAP?$AAa?$AAg?$AAe?$AAS?$AAi?$AAz?$AAe?$AA?$DN?$AA?$CF?$AAd?$AA?$AN?$AA?6?$AA?$AA@ 1002923c     wince.obj
 0001:00028258       ??_C@_1BM@EJAINDLO@?$AAC?$AAP?$AAU?$AA?$DN?$AAU?$AAN?$AAK?$AAN?$AAO?$AAW?$AAN?$AA?$AN?$AA?6?$AA?$AA@ 10029258     wince.obj
 0001:00028274       ??_C@_1BE@EEFFOFNO@?$AAC?$AAP?$AAU?$AA?$DN?$AAS?$AAH?$AA4?$AA?$AN?$AA?6?$AA?$AA@ 10029274     wince.obj
 0001:00028288       ??_C@_1BE@CHOFANCH@?$AAC?$AAP?$AAU?$AA?$DN?$AAA?$AAR?$AAM?$AA?$AN?$AA?6?$AA?$AA@ 10029288     wince.obj
 0001:0002829c       ??_C@_1BI@LDGJLFJC@?$AAC?$AAP?$AAU?$AA?$DN?$AAM?$AAI?$AAP?$AAS?$AA?5?$AA?$AN?$AA?6?$AA?$AA@ 1002929c     wince.obj
 0001:000282b4       ??_C@_1BI@MPBJOOFH@?$AAC?$AAP?$AAU?$AA?$DN?$AAI?$AAn?$AAt?$AAe?$AAl?$AA?$AN?$AA?6?$AA?$AA@ 100292b4     wince.obj
 0001:000284d0       ??_C@_0CC@FBIOIOKB@WpaMsgTypeSubst?5?3?5return?5FALSE?$DL?5@ 100294d0     wpa.obj
 0001:000284f4       ??_C@_0BK@FCFKDKFN@?$DM?9?9?9?9?9?5WpaEAPOLKeyAction?6?$AA@ 100294f4     wpa.obj
 0001:00028510       ??_C@_0CD@NEKIIEKD@Receive?5EAPOL?5Key?5Group?5Message?5@ 10029510     wpa.obj
 0001:00028534       ??_C@_0CG@MOEKGKHL@Receive?5EAPOL?5Key?5Pairwise?5Messa@ 10029534     wpa.obj
 0001:0002855c       ??_C@_0CG@MNMOLOBF@Receive?5EAPOL?5Key?5Pairwise?5Messa@ 1002955c     wpa.obj
 0001:00028584       ??_C@_0CK@NJMGNMDI@?7?5Key?5descripter?7version?7not?7mat@ 10029584     wpa.obj
 0001:000285b0       ??_C@_0CJ@CMKNHCCA@?7?5Key?5descripter?7version?7not?5mat@ 100295b0     wpa.obj
 0001:000285dc       ??_C@_0DA@DABEDLHK@?7?5Key?5descripter?7does?5not?5match?5@ 100295dc     wpa.obj
 0001:0002860c       ??_C@_0P@CLMDLOPL@KeyInfo?5DL?5?$CFd?6?$AA@ 1002960c     wpa.obj
 0001:0002861c       ??_C@_0BE@NLFFPJBE@KeyInfo?5Request?5?$CFd?6?$AA@ 1002961c     wpa.obj
 0001:00028630       ??_C@_0BC@EDNACAIN@KeyInfo?5Error?5?$CFd?6?$AA@ 10029630     wpa.obj
 0001:00028644       ??_C@_0BD@EKMAOFCC@KeyInfo?5Secure?5?$CFd?6?$AA@ 10029644     wpa.obj
 0001:00028658       ??_C@_0BE@FOAJNOFO@KeyInfo?5Key?5MIC?5?$CFd?6?$AA@ 10029658     wpa.obj
 0001:0002866c       ??_C@_0BE@IJJECKJI@KeyInfo?5Key?5Ack?5?$CFd?6?$AA@ 1002966c     wpa.obj
 0001:00028680       ??_C@_0BE@GMCJJBPH@KeyInfo?5Install?5?$CFd?6?$AA@ 10029680     wpa.obj
 0001:00028694       ??_C@_0BG@BPKLHODP@KeyInfo?5Key?5Index?5?$CFd?6?$AA@ 10029694     wpa.obj
 0001:000286ac       ??_C@_0BF@JMNDEIOC@KeyInfo?5Key?5Type?5?$CFd?6?$AA@ 100296ac     wpa.obj
 0001:000286c4       ??_C@_0CE@EGIDKOC@KeyInfo?5Key?5Description?5Version?5@ 100296c4     wpa.obj
 0001:000286e8       ??_C@_0BK@CPOPFHLN@?9?9?9?9?9?$DO?5WpaEAPOLKeyAction?6?$AA@ 100296e8     wpa.obj
 0001:00028704       ??_C@_0BK@JAFFONEP@WpaPairMsg1Action?5?$DM?9?9?9?9?9?6?$AA@ 10029704     wpa.obj
 0001:00028720       ??_C@_0BB@HHEOGBJL@?6?5FrameLen?5?$DN?5?$CFd?6?$AA@ 10029720     wpa.obj
 0001:00028734       ??_C@_08PHECDEMI@?6?5PTK?5?$DN?5?$AA@ 10029734     wpa.obj
 0001:00028740       ??_C@_04BABGPLLL@?$CF2x?9?$AA@ 10029740     wpa.obj
 0001:00028748       ??_C@_07MFJOCGMC@?5PMK?5?$DN?5?$AA@ 10029748     wpa.obj
 0001:00028750       ??_C@_0BK@DOCEMBND@WpaPairMsg1Action?5?9?9?9?9?9?$DO?6?$AA@ 10029750     wpa.obj
 0001:0002876c       ??_C@_0BK@BHPFMICM@WpaPairMsg3Action?5?$DM?9?9?9?9?9?6?$AA@ 1002976c     wpa.obj
 0001:00028788       ??_C@_0DD@LFNKAODL@?5MIC?5VALID?5in?5msg?53?5of?54?9way?5han@ 10029788     wpa.obj
 0001:000287bc       ??_C@_0DH@FFNOHOGI@?5MIC?5Different?5in?5msg?53?5of?54?9way@ 100297bc     wpa.obj
 0001:000287f4       ??_C@_0DI@KIDEAJOH@?5RSN?5IE?5matched?5in?5msg?53?5of?54?9wa@ 100297f4     wpa.obj
 0001:0002882c       ??_C@_0DI@LNMJCNFK@?5RSN?5IE?5mismatched?5msg?53?5of?54?9wa@ 1002982c     wpa.obj
 0001:00028864       ??_C@_0BK@LJIEOELA@WpaPairMsg3Action?5?9?9?9?9?9?$DO?6?$AA@ 10029864     wpa.obj
 0001:00028880       ??_C@_0BL@HNEAFNIJ@WpaGroupMsg1Action?5?$DM?9?9?9?9?9?6?$AA@ 10029880     wpa.obj
 0001:0002889c       ??_C@_06OAHPBHNA@PTK?5?$DN?5?$AA@ 1002989c     wpa.obj
 0001:000288a4       ??_C@_0DJ@HCPLAPHD@?5MIC?5VALID?5in?5group?5msg?51?5of?52?9w@ 100298a4     wpa.obj
 0001:000288e0       ??_C@_0DN@CHLDNCBC@?5MIC?5Different?5in?5group?5msg?51?5of@ 100298e0     wpa.obj
 0001:00028920       ??_C@_0BL@NDDBHBBF@WpaGroupMsg1Action?5?9?9?9?9?9?$DO?6?$AA@ 10029920     wpa.obj
 0001:0002893c       ??_C@_0CD@OEBOOBJF@WpaGroupMsg1Action?5?9?9?9?9?9?$DOlen?5?$DN?5?$CF@ 1002993c     wpa.obj
 0001:00028b60       ??_C@_0BF@NCIECBDG@?$DM?9?9?9?9?9?5WscEAPAction?6?$AA@ 10029b60     wsc.obj
 0001:00028b78       ??_C@_0CI@EACFNEIJ@WscEAPAction?3?5Received?5MsgType?$DN?5@ 10029b78     wsc.obj
 0001:00028ba0       ??_C@_0BF@MJFFDKCI@?9?9?9?9?9?$DO?5WscEAPAction?6?$AA@ 10029ba0     wsc.obj
 0001:00028bb8       ??_C@_0CN@KNKDEAAO@?5Error?5handling?5?$DM?9?9?9?9?9?5WscEAPEnr@ 10029bb8     wsc.obj
 0001:00028be8       ??_C@_0CN@LHMDIEPN@WscEAPEnrolleeAction?5?3?5Unsupport@ 10029be8     wsc.obj
 0001:00028c18       ??_C@_0CE@PDOCECIA@WscEAPEnrolleeAction?5?3?5Rx?5EAP?9FA@ 10029c18     wsc.obj
 0001:00028c3c       ??_C@_0CO@CBHMIAOL@?5Error?5handling?5?$DM?9?9?9?9?9?5WscEAPReg@ 10029c3c     wsc.obj
 0001:00028c6c       ??_C@_0CO@MCFFHDNM@WscEAPRegistrarAction?5?3?5Unsuppor@ 10029c6c     wsc.obj
 0001:00028c9c       ??_C@_0CF@FHFOFOBN@WscEAPRegistrarAction?5?3?5Rx?5EAP?9F@ 10029c9c     wsc.obj
 0001:00028cc4       ??_C@_0DA@NGDGKLMG@WscRxMsgType?5?3?5Not?5supposed?5to?5r@ 10029cc4     wsc.obj
 0001:00028cf4       ??_C@_0CO@CICJMHJA@WscRxMsgType?5?3?5Unsupported?5EAP?5C@ 10029cf4     wsc.obj
 0001:00028d24       ??_C@_0DB@CJOGPKCO@WscRxMsgType?5?3?5EAP?5length?5is?5too@ 10029d24     wsc.obj
 0001:00028d58       ??_C@_0CK@FPOBPFIA@WscMsgTypeSubst?5?3?5unsupported?5EA@ 10029d58     wsc.obj
 0001:00028d84       ??_C@_0CK@LFNGCEML@WscMsgTypeSubst?5?3?5unsupported?5EA@ 10029d84     wsc.obj
 0001:00028db0       ??_C@_0CH@MMIPFLI@WscConnectTimeout?5?9?9?$DO?5Fail?5to?5co@ 10029db0     wsc.obj
 0001:00028dd8       ??_C@_0CL@PMDHEHIH@?$CFs?3?5Last?5WPS?5LED?5status?5is?5LED_W@ 10029dd8     wsc.obj
 0001:00028e08       ??_C@_0FG@CMDDCMFK@?$CFs?3?5The?5NIC?5using?5PIN?5method?5fai@ 10029e08     wsc.obj
 0001:00028e60       ??_C@_0BC@BIDAAPHA@WscConnectTimeout?$AA@ 10029e60     wsc.obj
 0001:00028e74       ??_C@_0CF@GOLHLGBO@WscConnectTimeout?5?9?9?$DO?5Connection@ 10029e74     wsc.obj
 0001:00028e9c       ??_C@_0BI@GKOEOLIK@?$CB?$CB?$CB?5WscScanTimeout?5?$CB?$CB?$CB?6?$AA@ 10029e9c     wsc.obj
 0001:00028eb4       ??_C@_0BH@JGGBMBJK@?$CB?$CB?$CB?5WscPBCTimeout?5?$CB?$CB?$CB?6?$AA@ 10029eb4     wsc.obj
 0001:00028ecc       ??_C@_0BH@PPGPBHDP@?$CB?$CB?$CB?5WscPINTimeout?5?$CB?$CB?$CB?6?$AA@ 10029ecc     wsc.obj
 0001:00028ee4       ??_C@_0CF@PPPBLJLD@Disassociate?5with?5current?5WPS?5AP@ 10029ee4     wsc.obj
 0001:00028f0c       ??_C@_0BJ@CPDDKJJO@?$CB?$CB?$CB?5WscEAPRxTimeout?5?$CB?$CB?$CB?6?$AA@ 10029f0c     wsc.obj
 0001:00028f28       ??_C@_0CB@LEFLFBIJ@?$CB?$CB?$CB?5WscM8WaitEapFailTimeout?5?$CB?$CB?$CB?6@ 10029f28     wsc.obj
 0001:00028f4c       ??_C@_0BJ@JFMLJBKB@?$CB?$CB?$CB?5WscEapM2Timeout?5?$CB?$CB?$CB?6?$AA@ 10029f4c     wsc.obj
 0001:00028f68       ??_C@_0DO@LGOIFODI@?$CFs?3?5LED_WPS_SESSION_OVERLAP_DETE@ 10029f68     wsc.obj
 0001:00028fa8       ??_C@_0EM@CMFKBCJE@?$CFs?3?5LED_WPS_ERROR?1LED_WPS_SESSIO@ 10029fa8     wsc.obj
 0001:00028ff4       ??_C@_0DC@NJJAPBPK@?$CFs?3?5LED_WPS_TURN_LED_OFF?5?$DN?$DO?5LED_@ 10029ff4     wsc.obj
 0001:00029028       ??_C@_0DG@FKOLNHFM@?$CFs?3?5LED_WPS_TURN_LED_OFF?5?$DN?$DO?5LED_@ 1002a028     wsc.obj
 0001:00029060       ??_C@_0CN@HDHIFGOC@?$CFs?3?5LED_WPS_SUCCESS?5?$DN?$DO?5LED_WPS_T@ 1002a060     wsc.obj
 0001:00029090       ??_C@_0CO@GHMLLKGD@?$CFs?3?5Turn?5off?5the?5WPS?5successful?5@ 1002a090     wsc.obj
 0001:000290c0       ??_C@_0M@OBCCAONO@WscLEDTimer?$AA@ 1002a0c0     wsc.obj
 0001:000290cc       ??_C@_0DC@OBGABKHF@?$CFs?3?5Allow?5the?5NIC?5to?5turn?5off?5th@ 1002a0cc     wsc.obj
 0001:00029100       ??_C@_0BH@HFJEHHMC@WscSkipTurnOffLEDTimer?$AA@ 1002a100     wsc.obj
 0001:00029118       ??_C@_0BJ@KFDGBPKH@?$DM?9?9?9?9?9?5WscPushPBCAction?6?$AA@ 1002a118     wsc.obj
 0001:00029134       ??_C@_0BJ@BHMFEOCI@?9?9?9?9?9?$DO?5WscPushPBCAction?6?$AA@ 1002a134     wsc.obj
 0001:00029150       ??_C@_0BF@MCGCIODF@?$CB?$CB?$CB?5WscScanExec?5?$CB?$CB?$CB?6?$AA@ 1002a150     wsc.obj
 0001:00029168       ??_C@_0DM@JEGNDCDM@?$CB?$CB?$CB?5WscPBCExec?5?9?9?$DO?5MLME?5busy?0?5re@ 1002a168     wsc.obj
 0001:000291a4       ??_C@_0DC@JFIKMKNC@WscPBCExec?5?9?9?$DO?5AP?5list?5is?5?$CFd?0?5wa@ 1002a1a4     wsc.obj
 0001:000291d8       ??_C@_0DL@FFJJJNDI@?$CFs?3?5Skip?5the?5WPS?5session?5overlap@ 1002a1d8     wsc.obj
 0001:00029214       ??_C@_0L@IMEHIEPP@WscPBCExec?$AA@ 1002a214     wsc.obj
 0001:00029220       ??_C@_0CM@ECDFBJFJ@WscPBCBssTableSort?5?3?5Total?5?$CFd?5PB@ 1002a220     wsc.obj
 0001:0002924c       ??_C@_0CO@PNHKHPNI@?$CFs?3?5PREFERRED_WPS_AP_PHY_TYPE_AU@ 1002a24c     wsc.obj
 0001:00029280       ??_C@_0EN@CAPOHLFH@?$CFs?3?5Choice?52?44G?5WPS?5APs?5instead?5@ 1002a280     wsc.obj
 0001:000292d0       ??_C@_0BM@CPDNOFJA@?$CFs?3?5Choice?55G?5WPS?5APs?5only?6?$AA@ 1002a2d0     wsc.obj
 0001:000292ec       ??_C@_0CJ@IINGLFMJ@?$CFs?3?5PREFERRED_WPS_AP_PHY_TYPE_5_@ 1002a2ec     wsc.obj
 0001:00029318       ??_C@_0EL@LHJPGODE@?$CFs?3?5Choice?55G?5WPS?5APs?5instead?5or@ 1002a318     wsc.obj
 0001:00029364       ??_C@_0BO@IFPPPBIP@?$CFs?3?5Choice?52?44G?5WPS?5APs?5only?6?$AA@ 1002a364     wsc.obj
 0001:00029384       ??_C@_0CN@CLHBCEMM@?$CFs?3?5PREFERRED_WPS_AP_PHY_TYPE_2D@ 1002a384     wsc.obj
 0001:000293b4       ??_C@_0BD@DBPNECAE@WscPBCBssTableSort?$AA@ 1002a3b4     wsc.obj
 0001:000293c8       ??_C@_06CDMPDAMA@?$CF02x?5?5?$AA@ 1002a3c8     wsc.obj
 0001:000293d0       ??_C@_08FFADHLMB@UUID?9E?$DN?5?$AA@ 1002a3d0     wsc.obj
 0001:000293dc       ??_C@_0DM@ILOLICOL@?$CD?$CFd?5?5Bssid?5?$CF02x?3?$CF02x?3?$CF02x?3?$CF02x?3?$CF@ 1002a3dc     wsc.obj
 0001:00029418       ??_C@_0CB@BDLFACIN@PBC?5Found?5by?5Probe?5Response?9?9?$DO?5?6@ 1002a418     wsc.obj
 0001:0002943c       ??_C@_0CK@HPBMMDDO@?$CD?$CFd?5?5Bssid?5?$CF02x?3?$CF02x?3?$CF02x?3?$CF02x?3?$CF@ 1002a43c     wsc.obj
 0001:00029468       ??_C@_0BJ@DGPCJHMD@PBC?5Found?5by?5Beacon?9?9?$DO?5?6?$AA@ 1002a468     wsc.obj
 0001:00029484       ??_C@_0DA@KPEFAEHE@WscPBCBssTableSort?5?3?5DevicePassw@ 1002a484     wsc.obj
 0001:000294b4       ??_C@_0CM@GILOONGB@WscPBCModeAPSearch?5?3?5Total?5?$CFd?5PB@ 1002a4b4     wsc.obj
 0001:000294e0       ??_C@_0DA@CLNLIHGA@WscPBCModeAPSearch?5?3?5DevicePassw@ 1002a4e0     wsc.obj
 0001:00029510       ??_C@_0CK@CIMIDBJJ@WscPBCModeAPSearch?5?3?5Found?5desir@ 1002a510     wsc.obj
 0001:0002953c       ??_C@_0CM@PHBABGJM@WscPINModeAPSearch?5?3?5Total?5?$CFd?5PI@ 1002a53c     wsc.obj
 0001:00029568       ??_C@_0CB@HLPJDDHL@PIN?5Found?5by?5Probe?5Response?9?9?$DO?5?6@ 1002a568     wsc.obj
 0001:0002958c       ??_C@_0BJ@CHHHAKDE@PIN?5Found?5by?5Beacon?9?9?$DO?5?6?$AA@ 1002a58c     wsc.obj
 0001:000295a8       ??_C@_0DA@KLCJMNK@WscPINModeAPSearch?5?3?5DevicePassw@ 1002a5a8     wsc.obj
 0001:000295d8       ??_C@_0CK@OAEECHLG@WscPINModeAPSearch?5?3?5Found?5desir@ 1002a5d8     wsc.obj
 0001:00029608       ??_C@_0IL@ONDEGMEI@?$CFs?3?5This?5is?5the?5T?9Home?5W?5303V?5WP@ 1002a608     wsc.obj
 0001:00029698       ??_C@_0EN@EPAMHIMI@?$CFs?3?5This?5is?5a?5WPS?5AP?5?$CIBSSID?5?$DN?5?$CF0@ 1002a698     wsc.obj
 0001:000296e8       ??_C@_0O@EDAIOEHK@WscCheckWPSAP?$AA@ 1002a6e8     wsc.obj
 0001:000296f8       ??_C@_0BH@PJKOMMGN@?$DM?9?9?9?9?9?5WscStartAction?6?$AA@ 1002a6f8     wsc.obj
 0001:00029710       ??_C@_0BM@MBNIODPG@Send?5EAPOL?9START?5size?5?$DN?5?$CFd?6?$AA@ 1002a710     wsc.obj
 0001:0002972c       ??_C@_0BH@KHIKCBIP@?9?9?9?9?9?$DO?5WscStartAction?6?$AA@ 1002a72c     wsc.obj
 0001:00029744       ??_C@_0BN@CINKKLGC@?$DM?9?9?9?9?9?5WscInitRegistrarPair?6?$AA@ 1002a744     wsc.obj
 0001:00029764       ??_C@_0BN@OKGACJFG@?9?9?9?9?9?$DO?5WscInitRegistrarPair?6?$AA@ 1002a764     wsc.obj
 0001:00029784       ??_C@_0BI@DKKALIKK@?$DM?9?9?9?9?9?5MakeWSCEAPFrame?6?$AA@ 1002a784     wsc.obj
 0001:0002979c       ??_C@_0BI@HEPKBPBD@?9?9?9?9?9?$DO?5MakeWSCEAPFrame?6?$AA@ 1002a79c     wsc.obj
 0001:000297b4       ??_C@_0BI@PAJLLEMN@?$DM?9?9?9?9?9?5WscSendEapRspId?6?$AA@ 1002a7b4     wsc.obj
 0001:000297cc       ??_C@_0BI@LOMBBDHE@?9?9?9?9?9?$DO?5WscSendEapRspId?6?$AA@ 1002a7cc     wsc.obj
 0001:000297e4       ??_C@_0BJ@LPBEEFAF@?$DM?9?9?9?9?9?5WscSendMessageM1?6?$AA@ 1002a7e4     wsc.obj
 0001:00029800       ??_C@_0BJ@NOHBEIK@?9?9?9?9?9?$DO?5WscSendMessageM1?6?$AA@ 1002a800     wsc.obj
 0001:0002981c       ??_C@_0BJ@LNFCPLFM@?$DM?9?9?9?9?9?5WscSendMessageM2?6?$AA@ 1002a81c     wsc.obj
 0001:00029838       ??_C@_0O@GBPMJKNP@HmacData?5?9?9?$DO?5?$AA@ 1002a838     wsc.obj
 0001:00029848       ??_C@_0O@KMOMECFM@HmacLen?5?$DN?5?$CFd?6?$AA@ 1002a848     wsc.obj
 0001:00029858       ??_C@_0BJ@PKBKKND@?9?9?9?9?9?$DO?5WscSendMessageM2?6?$AA@ 1002a858     wsc.obj
 0001:00029874       ??_C@_0BJ@LMJAJBGL@?$DM?9?9?9?9?9?5WscSendMessageM3?6?$AA@ 1002a874     wsc.obj
 0001:00029890       ??_C@_0BJ@OGDMAOE@?9?9?9?9?9?$DO?5WscSendMessageM3?6?$AA@ 1002a890     wsc.obj
 0001:000298ac       ??_C@_0BJ@LJNPIHOO@?$DM?9?9?9?9?9?5WscSendMessageM4?6?$AA@ 1002a8ac     wsc.obj
 0001:000298c8       ??_C@_0BF@OPGHNADP@Plain?5text?5Hmac?5?9?9?$DO?5?$AA@ 1002a8c8     wsc.obj
 0001:000298e0       ??_C@_0BA@FKINPEKN@Plain?5text?5?9?9?$DO?5?$AA@ 1002a8e0     wsc.obj
 0001:000298f0       ??_C@_0BJ@LCMNGGB@?9?9?9?9?9?$DO?5WscSendMessageM4?6?$AA@ 1002a8f0     wsc.obj
 0001:0002990c       ??_C@_0BJ@LIBNONNJ@?$DM?9?9?9?9?9?5WscSendMessageM5?6?$AA@ 1002a90c     wsc.obj
 0001:00029928       ??_C@_0N@MKFKLBOH@AuthKey?5?9?9?$DO?5?$AA@ 1002a928     wsc.obj
 0001:00029938       ??_C@_0BJ@KOOLMFG@?9?9?9?9?9?$DO?5WscSendMessageM5?6?$AA@ 1002a938     wsc.obj
 0001:00029954       ??_C@_0BJ@LKFLFDIA@?$DM?9?9?9?9?9?5WscSendMessageM6?6?$AA@ 1002a954     wsc.obj
 0001:00029970       ??_C@_0BJ@IKIACAP@?9?9?9?9?9?$DO?5WscSendMessageM6?6?$AA@ 1002a970     wsc.obj
 0001:0002998c       ??_C@_0BJ@LLJJDJLH@?$DM?9?9?9?9?9?5WscSendMessageM7?6?$AA@ 1002a98c     wsc.obj
 0001:000299a8       ??_C@_0BJ@JGKGIDI@?9?9?9?9?9?$DO?5WscSendMessageM7?6?$AA@ 1002a9a8     wsc.obj
 0001:000299c4       ??_C@_0BJ@LAMFHOIK@?$DM?9?9?9?9?9?5WscSendMessageM8?6?$AA@ 1002a9c4     wsc.obj
 0001:000299e0       ??_C@_0BP@OIGCEEEN@WscSendMessageM8?3?5EncrType?$DN?$CFd?6?$AA@ 1002a9e0     wsc.obj
 0001:00029a00       ??_C@_0BP@OCBAKHEA@WscSendMessageM8?3?5AuthType?$DN?$CFd?6?$AA@ 1002aa00     wsc.obj
 0001:00029a20       ??_C@_0BJ@CDGCPAF@?9?9?9?9?9?$DO?5WscSendMessageM8?6?$AA@ 1002aa20     wsc.obj
 0001:00029a3c       ??_C@_0BJ@PLHIBPFM@?$DM?9?9?9?9?9?5WscSendEapRspAck?6?$AA@ 1002aa3c     wsc.obj
 0001:00029a58       ??_C@_0BJ@EJILEOND@?9?9?9?9?9?$DO?5WscSendEapRspAck?6?$AA@ 1002aa58     wsc.obj
 0001:00029a74       ??_C@_0BK@JPPOOFAH@?$DM?9?9?9?9?9?5WscSendEapRspNack?6?$AA@ 1002aa74     wsc.obj
 0001:00029a90       ??_C@_0BK@OCELIIOH@?9?9?9?9?9?$DO?5WscSendEapRspNack?6?$AA@ 1002aa90     wsc.obj
 0001:00029aac       ??_C@_0BK@HJKBINNH@?$DM?9?9?9?9?9?5WscSendEapRspDone?6?$AA@ 1002aaac     wsc.obj
 0001:00029ac8       ??_C@_0BK@EBEOADH@?9?9?9?9?9?$DO?5WscSendEapRspDone?6?$AA@ 1002aac8     wsc.obj
 0001:00029ae4       ??_C@_0BJ@KBOAINPA@?$DM?9?9?9?9?9?5WscRecvMessageM1?6?$AA@ 1002aae4     wsc.obj
 0001:00029b00       ??_C@_0CI@OOIOIFMJ@WscRecvMessageM1?5?9?9?$DO?5Unknown?5IE?5@ 1002ab00     wsc.obj
 0001:00029b28       ??_C@_0CJ@NNNCNNEP@WscRecvMessageM1?5?9?9?$DO?5ConfigError@ 1002ab28     wsc.obj
 0001:00029b54       ??_C@_0DH@GDFEDEJ@WscRecvMessageM1?5?9?9?$DO?5Device?5Pass@ 1002ab54     wsc.obj
 0001:00029b8c       ??_C@_0DL@DFMKPKKN@?5?$CB?$CB?$CB?$CB?$CB?5The?5peer?5is?5a?5configured?5@ 1002ab8c     wsc.obj
 0001:00029bc8       ??_C@_0CL@DDNFLIGJ@WscRecvMessageM1?5?9?9?$DO?5M1?5is?5too?5l@ 1002abc8     wsc.obj
 0001:00029bf4       ??_C@_0BJ@BDBDNMHP@?9?9?9?9?9?$DO?5WscRecvMessageM1?6?$AA@ 1002abf4     wsc.obj
 0001:00029c10       ??_C@_0BJ@KDKGDDKJ@?$DM?9?9?9?9?9?5WscRecvMessageM2?6?$AA@ 1002ac10     wsc.obj
 0001:00029c2c       ??_C@_0BM@PDFJBOMM@calculated?5?9?9?$DO?50x?$CF08x?9?$CF08x?6?$AA@ 1002ac2c     wsc.obj
 0001:00029c48       ??_C@_0BE@NJJONEJH@MD?5?9?9?$DO?50x?$CF08x?9?$CF08x?6?$AA@ 1002ac48     wsc.obj
 0001:00029c5c       ??_C@_0CF@GOIFPIGF@WscRecvMessageM2?5?9?9?$DO?5HMAC?5not?5ma@ 1002ac5c     wsc.obj
 0001:00029c84       ??_C@_0CI@NLGDDDJK@WscRecvMessageM2?5?9?9?$DO?5Unknown?5IE?5@ 1002ac84     wsc.obj
 0001:00029cac       ??_C@_0DH@CMIJPDMB@WscRecvMessageM2?5?9?9?$DO?5Device?5Pass@ 1002acac     wsc.obj
 0001:00029ce4       ??_C@_0CJ@CPIFDALH@WscRecvMessageM2?5?9?9?$DO?5ConfigError@ 1002ace4     wsc.obj
 0001:00029d10       ??_C@_0CK@DPGPDHHC@Rx?5M2?5Compare?5enrollee?5nonce?5mis@ 1002ad10     wsc.obj
 0001:00029d3c       ??_C@_0CL@EKBFDNKN@WscRecvMessageM2?5?9?9?$DO?5M2?5is?5too?5l@ 1002ad3c     wsc.obj
 0001:00029d68       ??_C@_0BJ@BBFFGCCG@?9?9?9?9?9?$DO?5WscRecvMessageM2?6?$AA@ 1002ad68     wsc.obj
 0001:00029d84       ??_C@_0BK@CPECPFDP@?$DM?9?9?9?9?9?5WscRecvMessageM2D?6?$AA@ 1002ad84     wsc.obj
 0001:00029da0       ??_C@_0CJ@FFECGKNB@WscRecvMessageM2D?5?9?9?$DO?5Unknown?5IE@ 1002ada0     wsc.obj
 0001:00029dcc       ??_C@_0CN@JAIFPBFM@Rx?5M2D?3?5It?8s?5not?5our?5own?5Enrolle@ 1002adcc     wsc.obj
 0001:00029dfc       ??_C@_0BK@FCPHJINP@?9?9?9?9?9?$DO?5WscRecvMessageM2D?6?$AA@ 1002adfc     wsc.obj
 0001:00029e18       ??_C@_0BJ@KCGEFJJO@?$DM?9?9?9?9?9?5WscRecvMessageM3?6?$AA@ 1002ae18     wsc.obj
 0001:00029e34       ??_C@_0CF@HJKNJMKF@WscRecvMessageM3?5?9?9?$DO?5HMAC?5not?5ma@ 1002ae34     wsc.obj
 0001:00029e5c       ??_C@_0CI@HOOIKDJE@WscRecvMessageM3?5?9?9?$DO?5Unknown?5IE?5@ 1002ae5c     wsc.obj
 0001:00029e84       ??_C@_0CL@NAJNEBAN@Rx?5M3?5Compare?5registrar?5nonce?5mi@ 1002ae84     wsc.obj
 0001:00029eb0       ??_C@_0CL@NEHKEDCO@WscRecvMessageM3?5?9?9?$DO?5M3?5is?5too?5l@ 1002aeb0     wsc.obj
 0001:00029edc       ??_C@_0BJ@BAJHAIBB@?9?9?9?9?9?$DO?5WscRecvMessageM3?6?$AA@ 1002aedc     wsc.obj
 0001:00029ef8       ??_C@_0BJ@KHCLEPBL@?$DM?9?9?9?9?9?5WscRecvMessageM4?6?$AA@ 1002aef8     wsc.obj
 0001:00029f14       ??_C@_0CF@BMHEKCOF@WscRecvMessageM4?5?9?9?$DO?5HMAC?5not?5ma@ 1002af14     wsc.obj
 0001:00029f3c       ??_C@_0CJ@KMJHNFKL@WscRecvMessageM4?5?9?9?$DO?5RHash1?5not?5@ 1002af3c     wsc.obj
 0001:00029f68       ??_C@_0CI@LALIFPDM@WscRecvMessageM4?5?9?9?$DO?5Unknown?5IE?5@ 1002af68     wsc.obj
 0001:00029f90       ??_C@_0CD@KNPKGBAD@ApEncrSettings?5len?5?$DN?5?$CFd?0?5data?5?9?9@ 1002af90     wsc.obj
 0001:00029fb4       ??_C@_0DJ@JNFPHBKB@EncrSetting?5length?5is?5out?5of?5ran@ 1002afb4     wsc.obj
 0001:00029ff0       ??_C@_0CK@KELPDHLM@Rx?5M4?5Compare?5enrollee?5nonce?5mis@ 1002aff0     wsc.obj
 0001:0002a01c       ??_C@_0CL@LJJEDGCF@WscRecvMessageM4?5?9?9?$DO?5M4?5is?5too?5l@ 1002b01c     wsc.obj
 0001:0002a048       ??_C@_0BJ@BFNIBOJE@?9?9?9?9?9?$DO?5WscRecvMessageM4?6?$AA@ 1002b048     wsc.obj
 0001:0002a064       ??_C@_0BJ@KGOJCFCM@?$DM?9?9?9?9?9?5WscRecvMessageM5?6?$AA@ 1002b064     wsc.obj
 0001:0002a080       ??_C@_0CF@LFMMGCF@WscRecvMessageM5?5?9?9?$DO?5HMAC?5not?5ma@ 1002b080     wsc.obj
 0001:0002a0a8       ??_C@_0CJ@EKAIHOIK@WscRecvMessageM5?5?9?9?$DO?5EHash1?5not?5@ 1002b0a8     wsc.obj
 0001:0002a0d4       ??_C@_0CI@BFDDMPDC@WscRecvMessageM5?5?9?9?$DO?5Unknown?5IE?5@ 1002b0d4     wsc.obj
 0001:0002a0fc       ??_C@_0CB@NHKEAHF@EncrSettings?5len?5?$DN?5?$CFd?0?5data?5?9?9?$DO?5@ 1002b0fc     wsc.obj
 0001:0002a120       ??_C@_0CL@KMNKHOLK@Rx?5M5?5Compare?5registrar?5nonce?5mi@ 1002b120     wsc.obj
 0001:0002a14c       ??_C@_0CL@CHPLEIKG@WscRecvMessageM5?5?9?9?$DO?5M5?5is?5too?5l@ 1002b14c     wsc.obj
 0001:0002a178       ??_C@_0BJ@BEBKHEKD@?9?9?9?9?9?$DO?5WscRecvMessageM5?6?$AA@ 1002b178     wsc.obj
 0001:0002a194       ??_C@_0BJ@KEKPJLHF@?$DM?9?9?9?9?9?5WscRecvMessageM6?6?$AA@ 1002b194     wsc.obj
 0001:0002a1b0       ??_C@_0CF@DCCEGLGF@WscRecvMessageM6?5?9?9?$DO?5HMAC?5not?5ma@ 1002b1b0     wsc.obj
 0001:0002a1d8       ??_C@_0CJ@KIKAPELN@WscRecvMessageM6?5?9?9?$DO?5RHash2?5not?5@ 1002b1d8     wsc.obj
 0001:0002a204       ??_C@_0CI@CANOHJGB@WscRecvMessageM6?5?9?9?$DO?5Unknown?5IE?5@ 1002b204     wsc.obj
 0001:0002a22c       ??_C@_0CK@GENPMKDJ@Rx?5M6?5Compare?5enrollee?5nonce?5mis@ 1002b22c     wsc.obj
 0001:0002a258       ??_C@_0CL@FODLMNGC@WscRecvMessageM6?5?9?9?$DO?5M6?5is?5too?5l@ 1002b258     wsc.obj
 0001:0002a284       ??_C@_0BJ@BGFMMKPK@?9?9?9?9?9?$DO?5WscRecvMessageM6?6?$AA@ 1002b284     wsc.obj
 0001:0002a2a0       ??_C@_0BJ@KFGNPBEC@?$DM?9?9?9?9?9?5WscRecvMessageM7?6?$AA@ 1002b2a0     wsc.obj
 0001:0002a2bc       ??_C@_0CF@CFAMAPKF@WscRecvMessageM7?5?9?9?$DO?5HMAC?5not?5ma@ 1002b2bc     wsc.obj
 0001:0002a2e4       ??_C@_0CJ@EODPFPJM@WscRecvMessageM7?5?9?9?$DO?5EHash2?5not?5@ 1002b2e4     wsc.obj
 0001:0002a310       ??_C@_0CI@IFFFOJGP@WscRecvMessageM7?5?9?9?$DO?5Unknown?5IE?5@ 1002b310     wsc.obj
 0001:0002a338       ??_C@_0CL@DBMIGJOI@Rx?5M7?5Compare?5registrar?5nonce?5mi@ 1002b338     wsc.obj
 0001:0002a364       ??_C@_0CL@MAFELDOB@WscRecvMessageM7?5?9?9?$DO?5M7?5is?5too?5l@ 1002b364     wsc.obj
 0001:0002a390       ??_C@_0BJ@BHJOKAMN@?9?9?9?9?9?$DO?5WscRecvMessageM7?6?$AA@ 1002b390     wsc.obj
 0001:0002a3ac       ??_C@_0BJ@KODBLGHP@?$DM?9?9?9?9?9?5WscRecvMessageM8?6?$AA@ 1002b3ac     wsc.obj
 0001:0002a3c8       ??_C@_0CF@PJJGBHOF@WscRecvMessageM8?5?9?9?$DO?5HMAC?5not?5ma@ 1002b3c8     wsc.obj
 0001:0002a3f0       ??_C@_0CI@GHAOIGHA@WscRecvMessageM8?5?9?9?$DO?5Unknown?5IE?5@ 1002b3f0     wsc.obj
 0001:0002a418       ??_C@_0CK@EIGODAGB@Rx?5M8?5Compare?5enrollee?5nonce?5mis@ 1002b418     wsc.obj
 0001:0002a444       ??_C@_0CL@IFOHCHHE@WscRecvMessageM8?5?9?9?$DO?5M8?5is?5too?5l@ 1002b444     wsc.obj
 0001:0002a470       ??_C@_0BJ@BMMCOHPA@?9?9?9?9?9?$DO?5WscRecvMessageM8?6?$AA@ 1002b470     wsc.obj
 0001:0002a48c       ??_C@_0BK@HABFLNLH@?$DM?9?9?9?9?9?5WscReceiveEapFail?6?$AA@ 1002b48c     wsc.obj
 0001:0002a4a8       ??_C@_0BK@NKANAFH@?9?9?9?9?9?$DO?5WscReceiveEapFail?6?$AA@ 1002b4a8     wsc.obj
 0001:0002a4c4       ??_C@_0BK@PGLEMJDL@?$DM?9?9?9?9?9?5WscReceiveEapNack?6?$AA@ 1002b4c4     wsc.obj
 0001:0002a4e0       ??_C@_0CJ@NIMMNHEG@WscReceiveEapNack?5?9?9?$DO?5Unknown?5IE@ 1002b4e0     wsc.obj
 0001:0002a50c       ??_C@_0CK@KAODABKM@WscReceiveEapNack?5?9?9?$DO?5ConfigErro@ 1002b50c     wsc.obj
 0001:0002a538       ??_C@_0CN@KMOBJFLJ@Rx?5Nack?5Compare?5registrar?5nonce?5@ 1002b538     wsc.obj
 0001:0002a568       ??_C@_0CM@BCNMMJFO@Rx?5Nack?5Compare?5enrollee?5nonce?5m@ 1002b568     wsc.obj
 0001:0002a594       ??_C@_0BK@ILABKENL@?9?9?9?9?9?$DO?5WscReceiveEapNack?6?$AA@ 1002b594     wsc.obj
 0001:0002a5b0       ??_C@_0BK@BAOLKBOL@?$DM?9?9?9?9?9?5WscReceiveEapDone?6?$AA@ 1002b5b0     wsc.obj
 0001:0002a5cc       ??_C@_0CJ@HHKDKMDN@WscReceiveEapDone?5?9?9?$DO?5Unknown?5IE@ 1002b5cc     wsc.obj
 0001:0002a5f8       ??_C@_0CN@GMMIGDMB@Rx?5Done?5Compare?5registrar?5nonce?5@ 1002b5f8     wsc.obj
 0001:0002a628       ??_C@_0BK@GNFOMMAL@?9?9?9?9?9?$DO?5WscReceiveEapDone?6?$AA@ 1002b628     wsc.obj
 0001:0002a644       ??_C@_0CJ@MGGDNAMO@WscParseEncrSettings?5?9?9?$DO?5HMAC?5no@ 1002b644     wsc.obj
 0001:0002a670       ??_C@_0CM@BKHKGIFE@WscParseEncrSettings?5?9?9?$DO?5Unknown@ 1002b670     wsc.obj
 0001:0002a69c       ??_C@_0DF@GAHBINDG@WscParseEncrSettings?5?9?9?$DO?5Enrolle@ 1002b69c     wsc.obj
 0001:0002a6d4       ??_C@_0DP@FPFEGPF@WscProcessCredential?5?9?9?$DO?5?$CFd?5prof@ 1002b6d4     wsc.obj
 0001:0002a714       ??_C@_0CM@MIIGLMIC@WscProcessCredential?5?9?9?$DO?5Unknown@ 1002b714     wsc.obj
 0001:0002a740       ??_C@_0CD@FGNAFNLE@WscProcessCredential?3?5EncrType?$DN?$CF@ 1002b740     wsc.obj
 0001:0002a764       ??_C@_0CD@FMKCLOLJ@WscProcessCredential?3?5AuthType?$DN?$CF@ 1002b764     wsc.obj
 0001:0002a788       ??_C@_0BP@OILGNAIG@WscProcessCredential?3?5Ssid?$DN?$CFs?6?$AA@ 1002b788     wsc.obj
 0001:0002a7a8       ??_C@_0BK@MDAIILPG@?$DM?9?9?9?9?9?5WscMakeProbeReqIE?6?$AA@ 1002b7a8     wsc.obj
 0001:0002a7c4       ??_C@_0BK@LOLNOGBG@?9?9?9?9?9?$DO?5WscMakeProbeReqIE?6?$AA@ 1002b7c4     wsc.obj
 0001:0002a7e0       ??_C@_0BD@FOPKHDBA@?$CB?$CB?$CB?5?5WscStop?5?$CB?$CB?$CB?5?6?$AA@ 1002b7e0     wsc.obj
 0001:0002a7f4       ??_C@_0CL@GEHCEPJN@Start?5WscAutoGenProfile?5?$CK?$CK?$CK?$CK?$CK?$CK?$CK?$CK@ 1002b7f4     wsc.obj
 0001:0002a820       ??_C@_0IB@NJPMFJAK@?$CF02X?$CF02X?$CF02X?$CF02X?$CF02X?$CF02X?$CF02X?$CF02X@ 1002b820     wsc.obj
 0001:0002a8a4       ??_C@_0BE@HGMAMNJC@ExRegNW?$CF02X?$CF02X?$CF02X?$AA@ 1002b8a4     wsc.obj
 0001:0002a8b8       ??_C@_0DH@BAIEDKCD@?$CFs?3?5Not?5support?5WPS?5LED?5mode?5?$CITh@ 1002b8b8     wsc.obj
 0001:0002a8f0       ??_C@_0DD@CBDHNFAP@?$CFs?3?5Support?5WPS?5LED?5mode?5?$CIThe?5WP@ 1002b8f0     wsc.obj
 0001:0002a924       ??_C@_0BF@BLHJGKHE@WscSupportWPSLEDMode?$AA@ 1002b924     wsc.obj
 0001:0002a93c       ??_C@_0BH@BMNLJGJJ@WscSupportWPSLEDMode10?$AA@ 1002b93c     wsc.obj
 0001:0002a954       ??_C@_0BO@NCMPDHN@?$CFs?3?5WSC?5Entryption?5Type?5?$DN?5?$CFd?6?$AA@ 1002b954     wsc.obj
 0001:0002a978       ??_C@_1FA@DCMPPJPB@?$AAC?$AA?3?$AA?2?$AAW?$AAi?$AAn?$AAC?$AAE?$AA6?$AA?4?$AA0?$AA?2?$AAN?$AAe?$AAw?$AA?2?$AAR?$AAT?$AA2?$AA8?$AA7?$AA0?$AA_?$AAv?$AA1?$AA?4?$AA4?$AA?4?$AA9?$AA?4?$AA0?$AA?2@ 1002b978     wsc.obj
 0001:0002a9c8       ??_C@_0CF@FFOMGLDA@?$CFs?3?5Incorrect?5encryption?5types?5?$CI@ 1002b9c8     wsc.obj
 0001:0002a9f0       ??_C@_0BI@MNIDNGFH@WscAPHasSecuritySetting?$AA@ 1002b9f0     wsc.obj
 0001:0002ac08       k256                       1002bc08     wsc_crypto.obj
 0001:0002ad08       i256                       1002bd08     wsc_crypto.obj
 0001:0002d550       ??_C@_0CF@GPDDPEFB@WscEncryptData?3?5EncryptFinal?5fai@ 1002e550     wsc_crypto.obj
 0001:0002d578       ??_C@_0CG@BOGEEMDE@WscEncryptData?3?5EncryptUpdate?5fa@ 1002e578     wsc_crypto.obj
 0001:0002d5a0       ??_C@_0CE@GJPGFBCD@WscEncryptData?3?5EncryptInit?5fail@ 1002e5a0     wsc_crypto.obj
 0001:0002d5c4       ??_C@_0CF@NBOLINEN@WscDecryptData?3?5DecryptFinal?5fai@ 1002e5c4     wsc_crypto.obj
 0001:0002d5ec       ??_C@_0CG@KNLMIAC@WscDecryptData?3?5DecryptUpdate?5fa@ 1002e5ec     wsc_crypto.obj
 0001:0002d614       ??_C@_0CE@KGGGPBEJ@WscEncryptData?3?5DecryptInit?5fail@ 1002e614     wsc_crypto.obj
 0001:0002d638       ??_C@_0DN@HPIJHNPI@WscDeriveKey?3?5Key?5derivation?5gen@ 1002e638     wsc_crypto.obj
 0001:0002d678       ??_C@_0CJ@MAHBDKKE@WscDeriveKey?3?5Deriving?5a?5key?5of?5@ 1002e678     wsc_crypto.obj
 0001:0002d8a8       ??_C@_0O@JOFHMEPJ@TPC?3?5?$DM?9?9?9?5?$CFs?6?$AA@ 1002e8a8     tpc.obj
 0001:0002d8b8       ??_C@_0DP@EMNAOFFG@TPC?3?5?$CFs?0?5MaxTxPowerCapability?5?$DN?5@ 1002e8b8     tpc.obj
 0001:0002d8f8       ??_C@_0HP@KOGLMGGF@TPC?3?5?$CFs?0?5pAd?9?$DOStaCfg?4MDCtrl?4dot1@ 1002e8f8     tpc.obj
 0001:0002d978       ??_C@_0O@KAKOOCPO@TPC?3?5?9?9?9?$DO?5?$CFs?6?$AA@ 1002e978     tpc.obj
 0001:0002d988       ??_C@_0N@JJAJFPGP@InitMDSMCtrl?$AA@ 1002e988     tpc.obj
 0001:0002d998       ??_C@_0KA@ELPADLHA@TPC?3?5?$CFs?3?5pAd?9?$DOStaCfg?4MDSMCtrl?4as@ 1002e998     tpc.obj
 0001:0002da38       ??_C@_0GO@FJIFBGEC@TPC?3?5?$CFs?3?5Incorrect?5maximum?5trans@ 1002ea38     tpc.obj
 0001:0002daa8       ??_C@_0BI@BDDLEHLE@MDSMCalculateMaxTxPower?$AA@ 1002eaa8     tpc.obj
 0001:0002dac0       ??_C@_0BM@GLOFFMM@MDSMCreatePowerCapabilityIE?$AA@ 1002eac0     tpc.obj
 0001:0002dae0       ??_C@_0HP@OADIJPE@TPC?3?5?$CFs?3?5RealTxPower?5?$DN?5?$CFd?5dBm?5?$CIp@ 1002eae0     tpc.obj
 0001:0002db60       ??_C@_0BK@ENDACFEG@MDSMCalaculateRealTxPower?$AA@ 1002eb60     tpc.obj
 0001:0002dd80       ??_C@_0DJ@FPJKMOHA@TDLS?5?9?5MlmeTdlsSetupReqAction?$CI?$CJ?5@ 1002ed80     tdls.obj
 0001:0002ddbc       ??_C@_0CP@DAPLNMGJ@TDLS?5?9?5MlmeTdlsSetupReqAction?$CI?$CJ?5@ 1002edbc     tdls.obj
 0001:0002ddf0       ??_C@_0EN@PALFGKHA@TDLS?5?9?5MlmeTdlsSetupReqAction?$CI?$CJ?5@ 1002edf0     tdls.obj
 0001:0002de40       ??_C@_0DK@KAFPOHGE@TDLS?5?9?5MlmeTdlsSetupReqAction?$CI?$CJ?5@ 1002ee40     tdls.obj
 0001:0002de7c       ??_C@_0CC@OJIOACMM@TDLS?5?9?5MlmeTdlsSetupReqAction?$CI?$CJ?5@ 1002ee7c     tdls.obj
 0001:0002dea0       ??_C@_0DL@ICPBJHJG@TDLS?5?9?5PeerTdlsMsgAction?$CI?$CJ?5Actio@ 1002eea0     tdls.obj
 0001:0002dedc       ??_C@_0DN@OJEGBFMP@TDLS?5?9?5PeerTdlsMsgAction?$CI?$CJ?5Actio@ 1002eedc     tdls.obj
 0001:0002df1c       ??_C@_0DM@DLAIODLD@TDLS?5?9?5PeerTdlsMsgAction?$CI?$CJ?5Actio@ 1002ef1c     tdls.obj
 0001:0002df58       ??_C@_0DM@GMBEOGPE@TDLS?5?9?5PeerTdlsMsgAction?$CI?$CJ?5Actio@ 1002ef58     tdls.obj
 0001:0002df98       ??_C@_0EC@BGFECALP@PeerTdlsMsgAction?3?5Received?5a?5me@ 1002ef98     tdls.obj
 0001:0002dfe0       ??_C@_0FD@DACCPNHM@TDLS?5?9?5PeerTdlsSetupReqAction?$CI?$CJ?5@ 1002efe0     tdls.obj
 0001:0002e034       ??_C@_0CD@NBDEOAFN@RT2870Dump?5PeerTdlsSetupReqActio@ 1002f034     tdls.obj
 0001:0002e058       ??_C@_0BI@GMBMKCGI@TDLS?5?9?5Generate?5ANonce?6?$AA@ 1002f058     tdls.obj
 0001:0002e070       ??_C@_0DJ@IOAEGPBG@TDLS?5?9?5PeerTdlsSetupReqAction?$CI?$CJ?5@ 1002f070     tdls.obj
 0001:0002e0ac       ??_C@_0CM@ECODOMCO@TDLS?5?9?5TPKMsg1Process?$CI?$CJ?5Failed?0?5@ 1002f0ac     tdls.obj
 0001:0002e0d8       ??_C@_0FJ@OFKIBDBN@TDLS?5?9?5PeerTdlsSetupReqAction?$CI?$CJ?5@ 1002f0d8     tdls.obj
 0001:0002e134       ??_C@_0DF@GPDICIMF@TDLS?5?9?5PeerTdlsSetupReqAction?$CI?$CJ?5@ 1002f134     tdls.obj
 0001:0002e16c       ??_C@_0DG@HHOHFOIM@TDLS?5?9?5PeerTdlsSetupReqAction?$CI?$CJ?5@ 1002f16c     tdls.obj
 0001:0002e1a8       ??_C@_0FE@EHEMGFLD@TDLS?5?9?5PeerTdlsSetupReqAction?$CI?$CJ?0@ 1002f1a8     tdls.obj
 0001:0002e200       ??_C@_0ED@PGOGIMGE@TDLS?5?9?5PeerTdlsSetupReqAction?$CI?$CJ?0@ 1002f200     tdls.obj
 0001:0002e244       ??_C@_0DM@OBJMJILD@TDLS?5?9?5PeerTdlsSetupReqAction?$CI?$CJ?5@ 1002f244     tdls.obj
 0001:0002e280       ??_C@_0FH@KIDEJAOA@TDLS?5?9?5PeerTdlsSetupReqAction?$CI?$CJ?5@ 1002f280     tdls.obj
 0001:0002e2d8       ??_C@_0CL@MKJICOKH@TDLS?5?3?5Success?0?5delete?5this?5sear@ 1002f2d8     tdls.obj
 0001:0002e304       ??_C@_0DM@CGJHJCJP@TDLS?5?9?5PeerTdlsSetupRspAction?$CI?$CJ?5@ 1002f304     tdls.obj
 0001:0002e340       ??_C@_0IK@HGNNPFHO@TDLS?5?9?5?$CISupRateLen?$CLExtRateLen?$CJ?5?$DN@ 1002f340     tdls.obj
 0001:0002e3d0       ??_C@_0EI@NPJJKFNB@TDLS?5?9?5HT?5cap?5found?0?5mode?5?$CI?$CFd?$CJ?0?5@ 1002f3d0     tdls.obj
 0001:0002e418       ??_C@_0DL@FEAMNMPI@TDLS?5?9?5BA?5BaSizeInUse?5?$DN?5?$CFd?0?5TXBA@ 1002f418     tdls.obj
 0001:0002e454       ??_C@_0DO@KFDNPIOI@TDLS?5?9?5Write?50x?$CFx?5to?5MAC?5registe@ 1002f454     tdls.obj
 0001:0002e494       ??_C@_0CD@JMDLBJBF@TDLS?5?9?5?5OFDM?0?5MinSupportedRate?$DN?$CF@ 1002f494     tdls.obj
 0001:0002e4b8       ??_C@_0CC@NPNKJOGC@TDLS?5?9?5?5CCK?0?5MinSupportedRate?$DN?$CFd@ 1002f4b8     tdls.obj
 0001:0002e4dc       ??_C@_0BF@LENHKELL@TDLS?5?9?5?5WMM?5Capable?6?$AA@ 1002f4dc     tdls.obj
 0001:0002e4f8       ??_C@_0EC@LIJHOBMJ@TDLS?5?9?5Insert?1Update?5MacEntry?5?$CIA@ 1002f4f8     tdls.obj
 0001:0002e540       ??_C@_0EE@KDGDOBNJ@TDLS?5?9?5PeerTdlsSetupRspAction?$CI?$CJ?5@ 1002f540     tdls.obj
 0001:0002e588       ??_C@_0EB@GLFAALPL@?$CK?$CK?$CK?$CK?$CK?$CK?$CK?$CK?$CK?$CK?$CK?$CK?$CK?$CK?$CK?5TDLS?5Setup?5Proce@ 1002f588     tdls.obj
 0001:0002e5d0       ??_C@_0FC@HEKLLLIM@TDLS?5?9?5PeerTdlsSetupRspAction?$CI?$CJ?5@ 1002f5d0     tdls.obj
 0001:0002e624       ??_C@_0DJ@GJBLONHO@TDLS?5?9?5PeerTdlsSetupRspAction?$CI?$CJ?5@ 1002f624     tdls.obj
 0001:0002e660       ??_C@_0CM@FBMLNFFN@TDLS?5?9?5TPKMsg2Process?$CI?$CJ?5Failed?0?5@ 1002f660     tdls.obj
 0001:0002e68c       ??_C@_0DO@IPHNODB@TDLS?5?9?5PeerTdlsSetupRspAction?$CI?$CJ?5@ 1002f68c     tdls.obj
 0001:0002e6d0       ??_C@_0EE@EJPJGLGG@TDLS?5?9?5PeerTdlsSetupRspAction?$CI?$CJ?5@ 1002f6d0     tdls.obj
 0001:0002e714       ??_C@_0CP@EHJAAKOB@TDLS?5?9?5PeerTdlsSetupRspAction?$CI?$CJ?5@ 1002f714     tdls.obj
 0001:0002e748       ??_C@_0GB@HOKNBJJH@TDLS?5?9?5PeerTdlsSetupRspAction?$CI?$CJ?5@ 1002f748     tdls.obj
 0001:0002e7b0       ??_C@_0FN@OANJEPFO@TDLS?5?9?5PeerTdlsSetupRspAction?$CI?$CJ?5@ 1002f7b0     tdls.obj
 0001:0002e810       ??_C@_0GL@MELNHOPM@TDLS?5?9?5PeerTdlsSetupRspAction?$CI?$CJ?5@ 1002f810     tdls.obj
 0001:0002e87c       ??_C@_0DN@EOENPABB@TDLS?5?9?5PeerTdlsSetupConfAction?$CI?$CJ@ 1002f87c     tdls.obj
 0001:0002e8c0       ??_C@_0EF@ODBMCIDI@TDLS?5?9?5PeerTdlsSetupConfAction?$CI?$CJ@ 1002f8c0     tdls.obj
 0001:0002e908       ??_C@_0CM@FPCMDNIM@TDLS?5?9?5TPKMsg3Process?$CI?$CJ?5Failed?0?5@ 1002f908     tdls.obj
 0001:0002e934       ??_C@_0DP@OELADFK@TDLS?5?9?5PeerTdlsSetupConfAction?$CI?$CJ@ 1002f934     tdls.obj
 0001:0002e978       ??_C@_0EC@LDPAMBEF@TDLS?5?9?5PeerTdlsSetupConfAction?$CI?$CJ@ 1002f978     tdls.obj
 0001:0002e9c0       ??_C@_0FL@HAFBDAJL@TDLS?5?9?5PeerTdlsSetupConfAction?$CI?$CJ@ 1002f9c0     tdls.obj
 0001:0002ea20       ??_C@_0GD@OIEINLPE@TDLS?5?9?5PeerTdlsSetupConfAction?$CI?$CJ@ 1002fa20     tdls.obj
 0001:0002ea84       ??_C@_0DA@BAHAMJHO@TDLS?5?9?5PeerTdlsSetupConfAction?$CI?$CJ@ 1002fa84     tdls.obj
 0001:0002eab8       ??_C@_0GL@KJDOLFOP@TDLS?5?9?5PeerTdlsSetupConfAction?$CI?$CJ@ 1002fab8     tdls.obj
 0001:0002eb24       ??_C@_0DJ@GLEIBIGG@TDLS?5?9?5MlmeTdlsTearDownAction?$CI?$CJ?5@ 1002fb24     tdls.obj
 0001:0002eb60       ??_C@_0DF@KEPLBCEF@TDLS?5?9?5MlmeTdlsTearDownAction?$CI?$CJ?5@ 1002fb60     tdls.obj
 0001:0002eb98       ??_C@_0EE@IBEIFPKO@TDLS?5?9?5PeerTdlsTearDownAction?$CI?$CJ?5@ 1002fb98     tdls.obj
 0001:0002ebe0       ??_C@_0EH@FFDMOGCL@TDLS?5?9?5PeerTdlsTearDownAction?$CI?$CJ?5@ 1002fbe0     tdls.obj
 0001:0002ec28       ??_C@_0CP@LHGFHCJH@TDLS?5?9?5PeerTdlsTeardownAction?$CI?$CJ?5@ 1002fc28     tdls.obj
 0001:0002ec58       ??_C@_0FH@JPCCOAHC@TDLS?5?9?5PeerTdlsTearDownAction?$CI?$CJ?5@ 1002fc58     tdls.obj
 0001:0002ecb0       ??_C@_0DF@IHJLFMPC@RTMPSendTDLSTearDownFrame?$CI?$CJ?5allo@ 1002fcb0     tdls.obj
 0001:0002ece8       ??_C@_0BL@IDEMELPC@Send?5TDLS?5TearDown?5Frame?5?6?$AA@ 1002fce8     tdls.obj
 0001:0002ed04       ??_C@_0CE@DCOINAKE@?$DM?$DN?$DN?$DN?$DN?$DN?$DN?$DNTDLSSendPacket?5?5Length?$DN?$CF@ 1002fd04     tdls.obj
 0001:0002ed28       ??_C@_0CE@FCFCDFPC@TDLSSendPacket?$DN?$DN?$DN?$DN?$DN?$DN?$DN?$DO?5?5Length?$DN?$CF@ 1002fd28     tdls.obj
 0001:0002ed4c       ??_C@_0CD@IFKNGNFB@TDLSSendPacket?5return?5?$CIflag?5?$DN?5?$CFx@ 1002fd4c     tdls.obj
 0001:0002ed70       ??_C@_0HC@NBMMGCLO@TdlsTimeout?5?9?5Failed?5to?5wait?5for@ 1002fd70     tdls.obj
 0001:0002ede4       ??_C@_0BP@IMJNOKCB@TDLSSearchLinkId?5?9?5?5not?5found?6?$AA@ 1002fde4     tdls.obj
 0001:0002ee04       ??_C@_0CI@BABBAIGN@TDLSSearchLinkId?5?9?5?5not?5found?5an@ 1002fe04     tdls.obj
 0001:0002ee30       ??_C@_0FG@HCBGPAML@TDLSSearchLinkId?5?9?5Find?5Link?5ID?5@ 1002fe30     tdls.obj
 0001:0002ee88       ??_C@_0CA@CKNNEBLD@TPKMsg2Process?$CI?$CJ?5MIC?5Error?$CB?$CB?$CB?5?6?$AA@ 1002fe88     tdls.obj
 0001:0002eea8       ??_C@_0CA@MNMAOHCE@TPKMsg3Process?$CI?$CJ?5MIC?5Error?$CB?$CB?$CB?5?6?$AA@ 1002fea8     tdls.obj
 0001:0002eec8       ??_C@_09OIPKINFE@TPK?9Name?6?$AA@ 1002fec8     tdls.obj
 0001:0002eed4       ??_C@_0BK@INGKHLNI@RT2870Dump?5TDLSDeriveTPK?6?$AA@ 1002fed4     tdls.obj
 0001:0002eef0       ??_C@_04LJGDOEOA@TPK?6?$AA@ 1002fef0     tdls.obj
 0001:0002eef8       ??_C@_08PDCNPKJD@TDLS?5PMK?$AA@ 1002fef8     tdls.obj
 0001:0002ef04       ??_C@_0DN@LMDMNOIK@?$CFs?5Fail?5to?5alloc?5memory?5for?5pAd?9@ 1002ff04     tdls.obj
 0001:0002ef44       ??_C@_0BC@IECOBAHG@TDLSSearchTabInit?$AA@ 1002ff44     tdls.obj
 0001:0002ef58       ??_C@_0CN@JOIJKDAG@?$CFs?5?3?5pAd?9?$DOStaCfg?4pTdlsSearchEntr@ 1002ff58     tdls.obj
 0001:0002ef88       ??_C@_0BF@DHOKPCPK@TDLSSearchTabDestory?$AA@ 1002ff88     tdls.obj
 0001:0002efa0       ??_C@_0EE@GKCOCLEG@TDLSSearchEntyAlloc?3?5pAd?9?$DOStaCfg@ 1002ffa0     tdls.obj
 0001:0002efe8       ??_C@_0EP@GHLLNGMC@TDLS?5?9?5Add?5?$CF02x?3?$CF02x?3?$CF02x?3?$CF02x?3?$CF@ 1002ffe8     tdls.obj
 0001:0002f038       ??_C@_0FG@KEMPADNJ@TDLS?5?9?5ageout?5?$CF02x?3?$CF02x?3?$CF02x?3?$CF02@ 10030038     tdls.obj
 0001:0002f090       ??_C@_0EJ@IDLIHAEN@ageout?5?$CF02x?3?$CF02x?3?$CF02x?3?$CF02x?3?$CF02x?3@ 10030090     tdls.obj
 0001:0002f0dc       ??_C@_0DM@LOEANFAM@?$DM?$DN?$DN?$DN?$DN?5TDLSDiscoveryPacketLearnAn@ 100300dc     tdls.obj
 0001:0002f118       ??_C@_0CI@PPNHLEGN@?$DN?$DN?$DN?$DN?$DO?5TDLSDiscoveryPacketLearnAn@ 10030118     tdls.obj
 0001:0002f140       ??_C@_0CB@GICFOGCD@TDLSDiscoveryPacketLearnAndCheck@ 10030140     tdls.obj
 0001:0002f168       ??_C@_1EA@DLNKEDK@?$AA?$CK?$AA?$CK?$AA?$CK?$AA?5?$AAA?$AAb?$AAo?$AAr?$AAt?$AAT?$AAr?$AAa?$AAn?$AAs?$AAf?$AAe?$AAr?$AA?5?$AAE?$AAR?$AAR?$AAO?$AAR?$AA?3?$AA?$CF?$AAd?$AA?5?$AA?$CK?$AA?$CK?$AA?$CK?$AA?6?$AA?$AA@ 10030168     usbclient:usbclient.obj
 0001:0002f1a8       ??_C@_1EA@OEBLAPPP@?$AA?$CK?$AA?$CK?$AA?$CK?$AA?5?$AAC?$AAl?$AAo?$AAs?$AAe?$AAT?$AAr?$AAa?$AAn?$AAs?$AAf?$AAe?$AAr?$AA?5?$AAE?$AAR?$AAR?$AAO?$AAR?$AA?3?$AA?$CF?$AAd?$AA?5?$AA?$CK?$AA?$CK?$AA?$CK?$AA?6?$AA?$AA@ 100301a8     usbclient:usbclient.obj
 0001:0002f1e8       ??_C@_1GK@NFJEKGG@?$AA?$CK?$AA?$CK?$AA?$CK?$AA?5?$AAC?$AAl?$AAe?$AAa?$AAr?$AAO?$AAr?$AAS?$AAe?$AAt?$AAF?$AAe?$AAa?$AAt?$AAu?$AAr?$AAe?$AA?5?$AAo?$AAn?$AA?5?$AAe?$AAn?$AAd?$AAp?$AAo?$AAi?$AAn@ 100301e8     usbclient:usbclient.obj
 0001:0002f258       ??_C@_1EC@JIGPENPP@?$AA?$CK?$AA?$CK?$AA?$CK?$AA?5?$AAU?$AAn?$AAh?$AAa?$AAn?$AAd?$AAl?$AAe?$AAd?$AA?5?$AAW?$AAa?$AAi?$AAt?$AAR?$AAe?$AAa?$AAs?$AAo?$AAn?$AA?3?$AA?$CF?$AAd?$AA?5?$AA?$CK?$AA?$CK?$AA?$CK?$AA?6@ 10030258     usbclient:usbclient.obj
 0001:0002f2a0       ??_C@_1FO@EGDNIMLN@?$AAC?$AAl?$AAe?$AAa?$AAr?$AAO?$AAr?$AAS?$AAe?$AAt?$AAF?$AAe?$AAa?$AAt?$AAu?$AAr?$AAe?$AA?3?$AAW?$AAA?$AAI?$AAT?$AA_?$AAT?$AAI?$AAM?$AAE?$AAO?$AAU?$AAT?$AA?5?$AAo@ 100302a0     usbclient:usbclient.obj
 0001:0002f300       ??_C@_1DK@IDLOABHP@?$AA?$CK?$AA?$CK?$AA?$CK?$AA?5?$AAR?$AAe?$AAs?$AAe?$AAt?$AAE?$AAv?$AAe?$AAn?$AAt?$AA?5?$AAE?$AAR?$AAR?$AAO?$AAR?$AA?3?$AA?$CF?$AAd?$AA?5?$AA?$CK?$AA?$CK?$AA?$CK?$AA?6?$AA?$AA@ 10030300     usbclient:usbclient.obj
 0001:0002f340       ??_C@_1FE@GJFHKKL@?$AA?$CK?$AA?$CK?$AA?$CK?$AA?5?$AAD?$AAe?$AAf?$AAa?$AAu?$AAl?$AAt?$AAT?$AAr?$AAa?$AAn?$AAs?$AAf?$AAe?$AAr?$AAC?$AAo?$AAm?$AAp?$AAl?$AAe?$AAt?$AAe?$AA?5?$AAE?$AAR?$AAR?$AAO@ 10030340     usbclient:usbclient.obj
 0001:0002f394       ??_C@_1DG@KGMCLKFK@?$AA?$CK?$AA?$CK?$AA?$CK?$AA?5?$AAS?$AAe?$AAt?$AAE?$AAv?$AAe?$AAn?$AAt?$AA?5?$AAE?$AAR?$AAR?$AAO?$AAR?$AA?3?$AA?$CF?$AAd?$AA?5?$AA?$CK?$AA?$CK?$AA?$CK?$AA?6?$AA?$AA@ 10030394     usbclient:usbclient.obj
 0001:0002f3d0       ??_C@_1HC@OIDPFNDL@?$AA?$CK?$AA?$CK?$AA?$CK?$AA?5?$AAG?$AAe?$AAt?$AAS?$AAt?$AAa?$AAt?$AAu?$AAs?$AA?5?$AAo?$AAn?$AA?5?$AAe?$AAn?$AAd?$AAp?$AAo?$AAi?$AAn?$AAt?$AA?3?$AA0?$AAx?$AA?$CF?$AAx?$AA?5?$AAf@ 100303d0     usbclient:usbclient.obj
 0001:0002f448       ??_C@_1EO@LLIJNJID@?$AAG?$AAe?$AAt?$AAS?$AAt?$AAa?$AAt?$AAu?$AAs?$AA?3?$AAW?$AAA?$AAI?$AAT?$AA_?$AAT?$AAI?$AAM?$AAE?$AAO?$AAU?$AAT?$AA?5?$AAo?$AAn?$AA?5?$AAb?$AAI?$AAn?$AAd?$AAe?$AAx@ 10030448     usbclient:usbclient.obj
 0001:0002f498       ??_C@_1EI@EFFJOCFO@?$AA?$CK?$AA?$CK?$AA?$CK?$AA?5?$AAG?$AAe?$AAt?$AAT?$AAr?$AAa?$AAn?$AAs?$AAf?$AAe?$AAr?$AAS?$AAt?$AAa?$AAt?$AAu?$AAs?$AA?5?$AAE?$AAR?$AAR?$AAO?$AAR?$AA?3?$AA?$CF?$AAd?$AA?5?$AA?$CK@ 10030498     usbclient:usbclient.obj
 0001:0002f4e0       ??_C@_1HA@BBDFJFG@?$AAG?$AAe?$AAt?$AAT?$AAr?$AAa?$AAn?$AAs?$AAf?$AAe?$AAr?$AAS?$AAt?$AAa?$AAt?$AAu?$AAs?$AA?5?$AA?$CI?$AAB?$AAy?$AAt?$AAe?$AAs?$AAT?$AAr?$AAa?$AAn?$AAs?$AAf?$AAe?$AAr@ 100304e0     usbclient:usbclient.obj
 0001:0002f550       ??_C@_1JK@HKJHGPDC@?$AAI?$AAs?$AAs?$AAu?$AAe?$AAB?$AAu?$AAl?$AAk?$AAT?$AAr?$AAa?$AAn?$AAs?$AAf?$AAe?$AAr?$AA?5?$AAE?$AAR?$AAR?$AAO?$AAR?$AA?$CI?$AA5?$AA?0?$AA?5?$AAB?$AAy?$AAt?$AAe?$AAs@ 10030550     usbclient:usbclient.obj
 0001:0002f5f0       ??_C@_1FA@COJHPOOL@?$AA?$CK?$AA?$CK?$AA?$CK?$AA?5?$AAI?$AAs?$AAs?$AAu?$AAe?$AAB?$AAu?$AAl?$AAk?$AAT?$AAr?$AAa?$AAn?$AAs?$AAf?$AAe?$AAr?$AA?5?$AAE?$AAR?$AAR?$AAO?$AAR?$AA?$CI?$AA3?$AA?0?$AA?5?$AA?$CF@ 100305f0     usbclient:usbclient.obj
 0001:0002f640       ??_C@_1DI@EENFKOKJ@?$AA?$CF?$AAs?$AA?3?$AAW?$AAA?$AAI?$AAT?$AA_?$AAT?$AAI?$AAM?$AAE?$AAO?$AAU?$AAT?$AA?5?$AAo?$AAn?$AA?5?$AAh?$AAT?$AA?3?$AA0?$AAx?$AA?$CF?$AAx?$AA?6?$AA?$AA@ 10030640     usbclient:usbclient.obj
 0001:0002f678       ??_C@_17HCEMPBGG@?$AAO?$AAU?$AAT?$AA?$AA@ 10030678     usbclient:usbclient.obj
 0001:0002f680       ??_C@_15BNKBCKPG@?$AAI?$AAN?$AA?$AA@ 10030680     usbclient:usbclient.obj
 0001:0002f688       ??_C@_1KE@HEHDFMIE@?$AAI?$AAs?$AAs?$AAu?$AAe?$AAI?$AAn?$AAt?$AAe?$AAr?$AAr?$AAu?$AAp?$AAt?$AAT?$AAr?$AAa?$AAn?$AAs?$AAf?$AAe?$AAr?$AA?5?$AAE?$AAR?$AAR?$AAO?$AAR?$AA?$CI?$AA5?$AA?0?$AA?5@ 10030688     usbclient:usbclient.obj
 0001:0002f730       ??_C@_1FK@KGMBLFKM@?$AA?$CK?$AA?$CK?$AA?$CK?$AA?5?$AAI?$AAs?$AAs?$AAu?$AAe?$AAI?$AAn?$AAt?$AAe?$AAr?$AAr?$AAu?$AAp?$AAt?$AAT?$AAr?$AAa?$AAn?$AAs?$AAf?$AAe?$AAr?$AA?5?$AAE?$AAR?$AAR?$AAO?$AAR@ 10030730     usbclient:usbclient.obj
 0001:0002f790       ??_C@_1JO@FNJJOIFN@?$AAI?$AAs?$AAs?$AAu?$AAe?$AAV?$AAe?$AAn?$AAd?$AAo?$AAr?$AAT?$AAr?$AAa?$AAn?$AAs?$AAf?$AAe?$AAr?$AA?5?$AAE?$AAR?$AAR?$AAO?$AAR?$AA?$CI?$AA5?$AA?0?$AA?5?$AAB?$AAy?$AAt@ 10030790     usbclient:usbclient.obj
 0001:0002f830       ??_C@_1FI@ILPCPOCG@?$AA?$CK?$AA?$CK?$AA?$CK?$AA?5?$AAI?$AAs?$AAs?$AAu?$AAe?$AAV?$AAe?$AAn?$AAd?$AAo?$AAr?$AAT?$AAr?$AAa?$AAn?$AAs?$AAf?$AAe?$AAr?$AA?5?$AAE?$AAR?$AAR?$AAO?$AAR?$AA?$CI?$AA3?$AA?0@ 10030830     usbclient:usbclient.obj
 0001:0002f888       ??_C@_1EM@GADAJNPB@?$AA?$CK?$AA?$CK?$AA?$CK?$AA?5?$AAI?$AAs?$AAD?$AAe?$AAf?$AAa?$AAu?$AAl?$AAt?$AAP?$AAi?$AAp?$AAe?$AAH?$AAa?$AAl?$AAt?$AAe?$AAd?$AA?5?$AAE?$AAR?$AAR?$AAO?$AAR?$AA?3?$AA?$CF?$AAd@ 10030888     usbclient:usbclient.obj
 0001:0002f8d8       ??_C@_1EE@FGLFADDK@?$AA?$CK?$AA?$CK?$AA?$CK?$AA?5?$AAR?$AAe?$AAs?$AAe?$AAt?$AAD?$AAe?$AAf?$AAa?$AAu?$AAl?$AAt?$AAP?$AAi?$AAp?$AAe?$AA?5?$AAf?$AAa?$AAi?$AAl?$AAu?$AAr?$AAe?$AA?5?$AA?$CK?$AA?$CK?$AA?$CK@ 100308d8     usbclient:usbclient.obj
 0001:0002f91c       ??_C@_1DI@MOPNAAFE@?$AA?$CK?$AA?$CK?$AA?$CK?$AA?5?$AAR?$AAe?$AAs?$AAe?$AAt?$AAP?$AAi?$AAp?$AAe?$AA?5?$AAE?$AAR?$AAR?$AAO?$AAR?$AA?3?$AA?$CF?$AAd?$AA?5?$AA?$CK?$AA?$CK?$AA?$CK?$AA?6?$AA?$AA@ 1003091c     usbclient:usbclient.obj
 0001:0002f978       ActionStateMachineInit     10030978 f   action.obj
 0001:0002fad0       MlmeADDBAAction            10030ad0 f   action.obj
 0001:0002feb4       MlmeDELBAAction            10030eb4 f   action.obj
 0001:0003029c       MlmeQOSAction              1003129c f   action.obj
 0001:000302b0       MlmeInvalidAction          100312b0 f   action.obj
 0001:000302dc       PeerAddBAReqAction         100312dc f   action.obj
 0001:00030f38       PeerAddBARspAction         10031f38 f   action.obj
 0001:00031bdc       PeerDelBAAction            10032bdc f   action.obj
 0001:0003222c       PeerSpectrumAction         1003322c f   action.obj
 0001:000323e4       PeerQOSAction              100333e4 f   action.obj
 0001:000323f8       PeerBAAction               100333f8 f   action.obj
 0001:000324d8       PeerPublicAction           100334d8 f   action.obj
 0001:000325c0       StaPeerPublicAction        100335c0 f   action.obj
 0001:0003272c       ApPublicAction             1003372c f   action.obj
 0001:00032774       PeerRMAction               10033774 f   action.obj
 0001:00032790       PeerHTAction               10033790 f   action.obj
 0001:00032cf0       RECBATimerTimeout          10033cf0 f   action.obj
 0001:000337d0       ORIBATimerTimeout          100347d0 f   action.obj
 0001:00034714       ActHeaderInit              10035714 f   action.obj
 0001:00034928       BarHeaderInit              10035928 f   action.obj
 0001:00034c04       QosBADataParse             10035c04 f   action.obj
 0001:00037890       CntlEnqueueForRecv         10038890 f   action.obj
 0001:00038a44       BaAutoManSwitch            10039a44 f   action.obj
 0001:00038cc0       SendPSMPAction             10039cc0 f   action.obj
 0001:00039074       ChannelSwitchSanityCheck   1003a074 f   action.obj
 0001:000391c8       ChannelSwitchAction        1003a1c8 f   action.obj
 0001:00039748       BuildIntolerantChannelRep  1003a748 f   action.obj
 0001:00039b98       Update2040CoexistFrameAndNotify 1003ab98 f   action.obj
 0001:00039c70       Send2040CoexistAction      1003ac70 f   action.obj
 0001:00039e5c       UpdateBssScanParm          1003ae5c f   action.obj
 0001:0003a638       SetEvent                   1003b638 f i action.obj
 0001:0003a670       AcmStateMachineInit        1003b670 f   acm_action.obj
 0001:0003a730       AcmReqCmdAction            1003b730 f   acm_action.obj
 0001:0003af10       ACM_WME_ActionFrameBodyMake 1003bf10 f   acm_action.obj
 0001:0003b0a4       AcmCmdAddTSRequest         1003c0a4 f   acm_action.obj
 0001:0003b2b4       AcmPeerRspHandle           1003c2b4 f   acm_action.obj
 0001:0003b8e8       AcmCmdDelTSSend            1003c8e8 f   acm_action.obj
 0001:0003ba90       AcmCmdTclasReset           1003ca90 f   acm_action.obj
 0001:0003bae4       AironetStateMachineInit    1003cae4 f   aironet.obj
 0001:0003bc10       AironetMsgAction           1003cc10 f   aironet.obj
 0001:0003c760       AironetRequestAction       1003d760 f   aironet.obj
 0001:0003ca78       ChannelLoadRequestAction   1003da78 f   aironet.obj
 0001:0003cce0       NoiseHistRequestAction     1003dce0 f   aironet.obj
 0001:0003cf88       BeaconRequestAction        1003df88 f   aironet.obj
 0001:0003d404       FrameRequestAction         1003e404 f   aironet.obj
 0001:0003d678       PathLossRequestAction      1003e678 f   aironet.obj
 0001:0003dc50       AironetLogRequestAction    1003ec50 f   aironet.obj
 0001:0003e6dc       StatisticsRequestAction    1003f6dc f   aironet.obj
 0001:0003e944       AironetReportAction        1003f944 f   aironet.obj
 0001:0003ed28       AironetFinalReportAction   1003fd28 f   aironet.obj
 0001:0003f298       ChannelLoadReportAction    10040298 f   aironet.obj
 0001:0003f9b8       NoiseHistReportAction      100409b8 f   aironet.obj
 0001:0004069c       BeaconReportAction         1004169c f   aironet.obj
 0001:0004072c       AironetAddBeaconReport     1004172c f   aironet.obj
 0001:000411fc       AironetCreateBeaconReportFromBssTable 100421fc f   aironet.obj
 0001:0004186c       AironetAddFrameTestReport  1004286c f   aironet.obj
 0001:00041cac       FrameTestReportAction      10042cac f   aironet.obj
 0001:0004202c       PathLossReportAction       1004302c f   aironet.obj
 0001:00042478       PathLossTimeOutAction      10043478 f   aironet.obj
 0001:000425c4       PathLossMessageAction      100435c4 f   aironet.obj
 0001:00042d54       StatisticsReportAction     10043d54 f   aironet.obj
 0001:00043730       CCXAironetTimeOutAction    10044730 f   aironet.obj
 0001:000437c0       AironetL2RoamingAction     100447c0 f   aironet.obj
 0001:00043ae4       AironetDirectRoam          10044ae4 f   aironet.obj
 0001:00044058       CCXSearchNBLToSwap         10045058 f   aironet.obj
 0001:00044178       ConvertRssiToSignalQuality 10045178 f   aironet.obj
 0001:00044258       AironetLinkTestAction      10045258 f   aironet.obj
 0001:00044c48       SendAironetReport          10045c48 f   aironet.obj
 0001:00044f44       TxAironetFromSupplicantAction 10045f44 f   aironet.obj
 0001:000451c0       InitCACTspec               100461c0 f   aironet.obj
 0001:00045b18       CacTsMetricsRptTimeoutAction 10046b18 f   aironet.obj
 0001:0004607c       AironetApLogTableInit      1004707c f   aironet.obj
 0001:00046104       AironetApLogEntryUpdate    10047104 f   aironet.obj
 0001:00046284       AironetApLogEntrySet       10047284 f   aironet.obj
 0001:00046354       AironetApLogTableSetNewEntry 10047354 f   aironet.obj
 0001:000466f4       SendEAPOLStart             100476f4 f   aironet.obj
 0001:00046a60       AironetRFRoaming           10047a60 f   aironet.obj
 0001:00046f10       AironetASTScanReq          10047f10 f   aironet.obj
 0001:0004711c       CCXDiagInitMemoryHandler   1004811c f   aironet.obj
 0001:00047344       CCXDiagGetMemory           10048344 f   aironet.obj
 0001:00047580       CCXDiagFreeMemoryHandler   10048580 f   aironet.obj
 0001:000476cc       CCXDiagLogFrame            100486cc f   aironet.obj
 0001:000477bc       TxCCXDiagLogFrames         100487bc f   aironet.obj
 0001:00047c84       RTMPusecDelay              10048c84 f i aironet.obj
 0001:00047d2c       APInitialize               10048d2c f   ap.obj
 0001:00047e28       APStartUp                  10048e28 f   ap.obj
 0001:000496e4       APStop                     1004a6e4 f   ap.obj
 0001:0004989c       APShutdown                 1004a89c f   ap.obj
 0001:000499e0       APCleanupPsQueue           1004a9e0 f   ap.obj
 0001:00049b18       ApLogEvent                 1004ab18 f   ap.obj
 0001:00049d00       APUpdateOperationMode      1004ad00 f   ap.obj
 0001:00049ed0       APUpdateCapabilityAndErpIe 1004aed0 f   ap.obj
 0001:0004a388       ApCheckAccessControlList   1004b388 f   ap.obj
 0001:0004a530       APSsPsInquiry              1004b530 f   ap.obj
 0001:0004a6b0       APPsIndicate               1004b6b0 f   ap.obj
 0001:0004a978       MacTableInitialize         1004b978 f   ap.obj
 0001:0004ab28       MacTableReset              1004bb28 f   ap.obj
 0001:0004b0d4       MacTableInsertWDSEntry     1004c0d4 f   ap.obj
 0001:0004b4e8       MacTableInsertEntry        1004c4e8 f   ap.obj
 0001:0004bad0       MacTableDeleteWDSEntry     1004cad0 f   ap.obj
 0001:0004bbb0       MacTableDeleteEntry        1004cbb0 f   ap.obj
 0001:0004c188       MacTableLookup             1004d188 f   ap.obj
 0001:0004c2f8       MacTableMaintenance        1004d2f8 f   ap.obj
 0001:0004c9e0       WdsTableInsertEntry        1004d9e0 f   ap.obj
 0001:0004ce0c       WdsTableDeleteEntry        1004de0c f   ap.obj
 0001:0004d128       WdsTableLookup             1004e128 f   ap.obj
 0001:0004d270       WdsTableMaintenance        1004e270 f   ap.obj
 0001:0004d43c       ApUpdateAccessControlList  1004e43c f   ap.obj
 0001:0004dc4c       APAssocStateMachineInit    1004ec4c f   ap_assoc.obj
 0001:0004dd00       APPeerAssocReqAction       1004ed00 f   ap_assoc.obj
 0001:0004e858       APPeerReassocReqAction     1004f858 f   ap_assoc.obj
 0001:0004f3a8       APPeerDisassocReqAction    100503a8 f   ap_assoc.obj
 0001:0004f4c8       APMlmeDisassocReqAction    100504c8 f   ap_assoc.obj
 0001:0004f66c       APCls3errAction            1005066c f   ap_assoc.obj
 0001:0004f7f4       APBuildAssociation         100507f4 f   ap_assoc.obj
 0001:000513bc       APAuthStateMachineInit     100523bc f   ap_auth.obj
 0001:00051428       APMlmeDeauthReqAction      10052428 f   ap_auth.obj
 0001:000515c4       APCls2errAction            100525c4 f   ap_auth.obj
 0001:0005174c       APAuthRspStateMachineInit  1005274c f   ap_authrsp.obj
 0001:000517e4       APPeerAuthAtAuthRspIdleAction 100527e4 f   ap_authrsp.obj
 0001:000520b8       APPeerDeauthReqAction      100530b8 f   ap_authrsp.obj
 0001:0005224c       APPeerAuthSimpleRspGenAndSend 1005324c f   ap_authrsp.obj
 0001:00052428       APMakeBssBeacon            10053428 f   ap_connect.obj
 0001:00052dd0       APUpdateBeaconFrame        10053dd0 f   ap_connect.obj
 0001:00053c64       APSendPackets              10054c64 f   ap_data.obj
 0001:00054198       APSendPacket               10055198 f   ap_data.obj
 0001:00054acc       APHardTransmit             10055acc f   ap_data.obj
 0001:000588e8       RTUSBAPHandleRxPacket      100598e8 f   ap_data.obj
 0001:0005c004       APCheckRxError             1005d004 f   ap_data.obj
 0001:0005c060       APCheckClass2Class3Error   1005d060 f   ap_data.obj
 0001:0005c178       APHandleRxPsPoll           1005d178 f   ap_data.obj
 0001:0005c6c0       APBridgeToWdsAndWirelessSta 1005d6c0 f   ap_data.obj
 0001:0005cb30       APCheckNDSClient           1005db30 f   ap_data.obj
 0001:0005cf3c       APQueryInformation         1005df3c f   ap_info.obj
 0001:0005db04       APSetInformation           1005eb04 f   ap_info.obj
 0001:0005fcec       APMlmePeriodicExec         10060cec f   ap_mlme.obj
 0001:0006002c       APMlmeSelectTxRateTable    1006102c f   ap_mlme.obj
 0001:00060bb8       APMlmeSetTxRate            10061bb8 f   ap_mlme.obj
 0001:00060f68       APMlmeDynamicTxRateSwitching 10061f68 f   ap_mlme.obj
 0001:00062604       APQuickResponeForRateUpExec 10063604 f   ap_mlme.obj
 0001:000632b4       APMsgTypeSubst             100642b4 f   ap_mlme.obj
 0001:000636c4       RTMPSetPiggyBack           100646c4 f   ap_mlme.obj
 0001:00063734       APAsicEvaluateRxAnt        10064734 f   ap_mlme.obj
 0001:00063904       APAsicRxAntEvalTimeout     10064904 f   ap_mlme.obj
 0001:00063b60       PeerAssocReqSanity         10064b60 f   ap_sanity.obj
 0001:0006487c       PeerReassocReqSanity       1006587c f   ap_sanity.obj
 0001:00065318       PeerDisassocReqSanity      10066318 f   ap_sanity.obj
 0001:000653e8       PeerDeauthReqSanity        100663e8 f   ap_sanity.obj
 0001:000654b8       APPeerAuthSanity           100664b8 f   ap_sanity.obj
 0001:00065700       APPeerProbeReqSanity       10066700 f   ap_sanity.obj
 0001:00065848       APPeerBeaconAndProbeRspSanity 10066848 f   ap_sanity.obj
 0001:00065ef4       APSyncStateMachineInit     10066ef4 f   ap_sync.obj
 0001:00065f78       APPeerProbeReqAction       10066f78 f   ap_sync.obj
 0001:00066d4c       APPeerBeaconAction         10067d4c f   ap_sync.obj
 0001:00067024       APWapiStateMachineInit     10068024 f   Ap_wapi.obj
 0001:000670b8       APWapiWAI_UnicastReq_Action 100680b8 f   Ap_wapi.obj
 0001:00067284       APWapiWAI_MBcastReq_Action 10068284 f   Ap_wapi.obj
 0001:00067380       APWapiWAIPacketAction      10068380 f   Ap_wapi.obj
 0001:00067660       APWapiWAIPacket_HandleMBcastRsp 10068660 f   Ap_wapi.obj
 0001:00067cd4       APWapiWAIPacket_HandleUnicastRsp 10068cd4 f   Ap_wapi.obj
 0001:000684cc       APWapiSend_MBcastKeyNegotiate_Req 100694cc f   Ap_wapi.obj
 0001:00069064       APWapiSend_UnicastKeyNegotiate_Req 1006a064 f   Ap_wapi.obj
 0001:0006973c       APWapiSend_UnicastKeyNegotiate_Conf 1006a73c f   Ap_wapi.obj
 0001:00069b78       APSTAWapiGen_MIC           1006ab78 f   Ap_wapi.obj
 0001:00069bd4       APSTAWapiGen_MBcastKey     1006abd4 f   Ap_wapi.obj
 0001:00069c30       APSTAWapiGen_BKAndChallengeSeed 1006ac30 f   Ap_wapi.obj
 0001:00069d80       APSTAWapiGen_BKID          1006ad80 f   Ap_wapi.obj
 0001:00069e94       APSTAWapiGen_PairwiseKey   1006ae94 f   Ap_wapi.obj
 0001:00069fac       SMS4Crypt                  1006afac f   Ap_wapi.obj
 0001:0006a728       SMS4KeyExt                 1006b728 f   Ap_wapi.obj
 0001:0006ad50       wpi_encrypt                1006bd50 f   Ap_wapi.obj
 0001:0006af48       wpi_decrypt                1006bf48 f   Ap_wapi.obj
 0001:0006af90       wpi_pmac                   1006bf90 f   Ap_wapi.obj
 0001:0006b0f8       APSTA_IV_ADD               1006c0f8 f   Ap_wapi.obj
 0001:0006b218       APSTA_IV_GREATER_THAN      1006c218 f   Ap_wapi.obj
 0001:0006b2f4       WPAMsgTypeSubst            1006c2f4 f   ap_wpa.obj
 0001:0006b3d4       APWpaStateMachineInit      1006c3d4 f   ap_wpa.obj
 0001:0006b4a0       APWpaEAPPacketAction       1006c4a0 f   ap_wpa.obj
 0001:0006b4b4       APWpaEAPOLASFAlertAction   1006c4b4 f   ap_wpa.obj
 0001:0006b4c8       APWpaEAPOLLogoffAction     1006c4c8 f   ap_wpa.obj
 0001:0006b4dc       PACInquiry                 1006c4dc f   ap_wpa.obj
 0001:0006b544       RTMPCheckWPAframe          1006c544 f   ap_wpa.obj
 0001:0006b79c       RTMPCheckMcast             1006c79c f   ap_wpa.obj
 0001:0006b9b8       RTMPCheckUcast             1006c9b8 f   ap_wpa.obj
 0001:0006bcc0       RTMPCheckAUTH              1006ccc0 f   ap_wpa.obj
 0001:0006bf78       APWpaEAPOLStartAction      1006cf78 f   ap_wpa.obj
 0001:0006c0e0       HandleCounterMeasure       1006d0e0 f   ap_wpa.obj
 0001:0006c31c       APWpaEAPOLKeyAction        1006d31c f   ap_wpa.obj
 0001:0006c984       WPAStart4WayHS             1006d984 f   ap_wpa.obj
 0001:0006cd00       PeerPairMsg2Action         1006dd00 f   ap_wpa.obj
 0001:0006df28       CMTimerExec                1006ef28 f   ap_wpa.obj
 0001:0006e078       WPARetryExec               1006f078 f   ap_wpa.obj
 0001:0006e6a8       Wpa1PeerPairMsg4Action     1006f6a8 f   ap_wpa.obj
 0001:0006eb6c       Wpa2PeerPairMsg4Action     1006fb6c f   ap_wpa.obj
 0001:0006f078       PeerGroupMsg2Action        10070078 f   ap_wpa.obj
 0001:0006f504       WPAHardTransmit            10070504 f   ap_wpa.obj
 0001:00070398       DisAssocAction             10071398 f   ap_wpa.obj
 0001:00070524       GREKEYPeriodicExec         10071524 f   ap_wpa.obj
 0001:00070a3c       WPAMacHeaderInit           10071a3c f   ap_wpa.obj
 0001:00070cd0       CountPTK                   10071cd0 f   ap_wpa.obj
 0001:00070ee0       CountGTK                   10071ee0 f   ap_wpa.obj
 0001:00071040       GetSmall                   10072040 f   ap_wpa.obj
 0001:00071120       GetLarge                   10072120 f   ap_wpa.obj
 0001:00071208       APGenRandom                10072208 f   ap_wpa.obj
 0001:000714a8       AES_GTK_KEY_WRAP           100724a8 f   ap_wpa.obj
 0001:000717a0       RTMPMakeRSNIE              100727a0 f   ap_wpa.obj
 0001:00071e20       APToWirelessSta            10072e20 f   ap_wpa.obj
 0001:0007214c       AssocStateMachineInit      1007314c f   assoc.obj
 0001:00072418       AssocTimeout               10073418 f   assoc.obj
 0001:000724b0       ReassocTimeout             100734b0 f   assoc.obj
 0001:00072548       DisassocTimeout            10073548 f   assoc.obj
 0001:000725e8       MlmeAssocReqAction         100735e8 f   assoc.obj
 0001:000749a8       MlmeReassocReqAction       100759a8 f   assoc.obj
 0001:00076408       MlmeDisassocReqAction      10077408 f   assoc.obj
 0001:00076804       PeerAssocRspAction         10077804 f   assoc.obj
 0001:00076ef4       PeerReassocRspAction       10077ef4 f   assoc.obj
 0001:000776ec       AssocPostProc              100786ec f   assoc.obj
 0001:00077cf4       PeerDisassocAction         10078cf4 f   assoc.obj
 0001:000780f4       AssocTimeoutAction         100790f4 f   assoc.obj
 0001:00078168       ReassocTimeoutAction       10079168 f   assoc.obj
 0001:000781dc       DisassocTimeoutAction      100791dc f   assoc.obj
 0001:00078250       InvalidStateWhenAssoc      10079250 f   assoc.obj
 0001:000782d4       InvalidStateWhenReassoc    100792d4 f   assoc.obj
 0001:00078358       InvalidStateWhenDisassociate 10079358 f   assoc.obj
 0001:000783e4       Cls3errAction              100793e4 f   assoc.obj
 0001:00078628       SwitchBetweenWepAndCkip    10079628 f   assoc.obj
 0001:00078c58       AuthStateMachineInit       10079c58 f   auth.obj
 0001:00078d70       AuthTimeout                10079d70 f   auth.obj
 0001:00078e40       MlmeAuthReqAction          10079e40 f   auth.obj
 0001:00079348       PeerAuthRspAtSeq2Action    1007a348 f   auth.obj
 0001:0007994c       PeerAuthRspAtSeq4Action    1007a94c f   auth.obj
 0001:00079b10       MlmeDeauthReqAction        1007ab10 f   auth.obj
 0001:00079d68       AuthTimeoutAction          1007ad68 f   auth.obj
 0001:00079ddc       InvalidStateWhenAuth       1007addc f   auth.obj
 0001:00079e68       Cls2errAction              1007ae68 f   auth.obj
 0001:0007a01c       AuthRspStateMachineInit    1007b01c f   auth_rsp.obj
 0001:0007a0b0       PeerAuthSimpleRspGenAndSend 1007b0b0 f   auth_rsp.obj
 0001:0007a200       PeerDeauthAction           1007b200 f   auth_rsp.obj
 0001:0007a65c       MlmeCntlInit               1007b65c f   connect.obj
 0001:0007a684       MlmeCntlMachinePerformAction 1007b684 f   connect.obj
 0001:0007ad8c       CntlIdleProc               1007bd8c f   connect.obj
 0001:0007b0d8       CntlOidScanProc            1007c0d8 f   connect.obj
 0001:0007b550       SSIDIsValid                1007c550 f   connect.obj
 0001:0007b608       CntlOidSsidProc            1007c608 f   connect.obj
 0001:0007c340       CntlWscIterate             1007d340 f   connect.obj
 0001:0007c454       CntlOidRTBssidProc         1007d454 f   connect.obj
 0001:0007d2fc       CntlMlmeRoamingProc        1007e2fc f   connect.obj
 0001:0007d500       CntlOidDLSSetupProc        1007e500 f   connect.obj
 0001:0007df84       CntlWaitDisassocProc       1007ef84 f   connect.obj
 0001:0007e124       CntlWaitJoinProc           1007f124 f   connect.obj
 0001:0007e758       CntlWaitStartProc          1007f758 f   connect.obj
 0001:0007e978       CntlWaitAuthProc           1007f978 f   connect.obj
 0001:0007ec34       CntlWaitAuthProc2          1007fc34 f   connect.obj
 0001:0007ef9c       CntlWaitAssocProc          1007ff9c f   connect.obj
 0001:0007f264       CntlWaitReassocProc        10080264 f   connect.obj
 0001:0007f554       CntlOidTDLSRequestProc     10080554 f   connect.obj
 0001:0007faf8       CntlChannelWidth           10080af8 f   connect.obj
 0001:0008016c       LinkUp                     1008116c f   connect.obj
 0001:0008433c       LinkDown                   1008533c f   connect.obj
 0001:000856c0       MlmeCntlConfirm            100866c0 f   connect.obj
 0001:00085700       IterateOnBssTab            10086700 f   connect.obj
 0001:000861a0       IterateOnBssTab2           100871a0 f   connect.obj
 0001:000863ac       JoinParmFill               100873ac f   connect.obj
 0001:000863cc       AssocParmFill              100873cc f   connect.obj
 0001:000864b0       ScanParmFill               100874b0 f   connect.obj
 0001:00086508       DlsParmFill                10087508 f   connect.obj
 0001:00086538       TdlsParmFill               10087538 f   connect.obj
 0001:00086568       DisassocParmFill           10087568 f   connect.obj
 0001:00086614       DeauthParmFill             10087614 f   connect.obj
 0001:000866c0       StartParmFill              100876c0 f   connect.obj
 0001:00086724       AuthParmFill               10087724 f   connect.obj
 0001:000867e0       ComposePsPoll              100877e0 f   connect.obj
 0001:00086b78       ComposeNullFrame           10087b78 f   connect.obj
 0001:00086f68       MakeIbssBeacon             10087f68 f   connect.obj
 0001:00087cc0       DlsStateMachineInit        10088cc0 f   dls.obj
 0001:00087e4c       MlmeDlsReqAction           10088e4c f   dls.obj
 0001:00088248       PeerDlsReqAction           10089248 f   dls.obj
 0001:000890f8       PeerDlsRspAction           1008a0f8 f   dls.obj
 0001:00089d68       MlmeDlsTearDownAction      1008ad68 f   dls.obj
 0001:0008a1d0       PeerDlsTearDownAction      1008b1d0 f   dls.obj
 0001:0008a630       RTMPCheckDLSTimeOut        1008b630 f   dls.obj
 0001:0008acbc       RTMPRcvFrameDLSCheck       1008bcbc f   dls.obj
 0001:0008badc       RTMPCheckDLSFrame          1008cadc f   dls.obj
 0001:0008bd1c       RTMPSendDLSTearDownFrame   1008cd1c f   dls.obj
 0001:0008becc       RTMPSendSTAKeyRequest      1008cecc f   dls.obj
 0001:0008c62c       RTMPSendSTAKeyHandShake    1008d62c f   dls.obj
 0001:0008cd78       DlsTimeout                 1008dd78 f   dls.obj
 0001:0008ceb0       DlsTearDown                1008deb0 f   dls.obj
 0001:0008d1fc       DlsDeleteMacTableEntry     1008e1fc f   dls.obj
 0001:0008d254       LeapMacHeaderInit          1008e254 f   leap.obj
 0001:0008d518       RogueApTableInit           1008e518 f   leap.obj
 0001:0008d58c       RogueApTableSearch         1008e58c f   leap.obj
 0001:0008d630       RogueApEntrySet            1008e630 f   leap.obj
 0001:0008d6ec       RogueApTableSetEntry       1008e6ec f   leap.obj
 0001:0008d844       RogueApTableDeleteEntry    1008e844 f   leap.obj
 0001:0008d968       LeapSendRogueAPReport      1008e968 f   leap.obj
 0001:0008d9d4       CCXAdjacentAPReport        1008e9d4 f   leap.obj
 0001:0008e1ac       CCXAAPReasonCodeReport     1008f1ac f   leap.obj
 0001:0008e544       MD4Init                    1008f544 f   md4.obj
 0001:0008e5c4       MD4Update                  1008f5c4 f   md4.obj
 0001:0008e74c       MD4Final                   1008f74c f   md4.obj
 0001:0008e820       MD4Transform               1008f820 f   md4.obj
 0001:0008f858       Encode                     10090858 f   md4.obj
 0001:0008f988       Decode                     10090988 f   md4.obj
 0001:0008fa60       MD4_memcpy                 10090a60 f   md4.obj
 0001:0008fac8       MD4_memset                 10090ac8 f   md4.obj
 0001:0008fb34       md5_mac                    10090b34 f   md5.obj
 0001:0008fbb4       hmac_md5                   10090bb4 f   md5.obj
 0001:0008fd48       MD5Init                    10090d48 f   md5.obj
 0001:0008fdc8       MD5Update                  10090dc8 f   md5.obj
 0001:0008ff68       MD5Final                   10090f68 f   md5.obj
 0001:0009008c       MD5Transform               1009108c f   md5.obj
 0001:00091b90       SHAInit                    10092b90 f   md5.obj
 0001:00091c84       SHAUpdate                  10092c84 f   md5.obj
 0001:00092420       SHAFinal                   10093420 f   md5.obj
 0001:00092650       SHA256_Init                10093650 f   md5.obj
 0001:000926c8       SHA256_Hash                100936c8 f   md5.obj
 0001:00092cc4       SHA256_Append              10093cc4 f   md5.obj
 0001:00092e40       SHA256_End                 10093e40 f   md5.obj
 0001:000930e8       SHA256                     100940e8 f   md5.obj
 0001:00093150       aes_set_key                10094150 f   md5.obj
 0001:00093fc8       aes_encrypt                10094fc8 f   md5.obj
 0001:00096984       aes_decrypt                10097984 f   md5.obj
 0001:00099344       leftshift_onebit           1009a344 f   md5.obj
 0001:00099420       do_padding                 1009a420 f   md5.obj
 0001:000994dc       generate_subkey            1009a4dc f   md5.obj
 0001:000996dc       AES_128_CMAC               1009a6dc f   md5.obj
 0001:00099a38       MlmeInit                   1009aa38 f   mlme.obj
 0001:0009a000       MlmeHandler                1009b000 f   mlme.obj
 0001:0009a510       MlmeHalt                   1009b510 f   mlme.obj
 0001:0009a898       MlmeSuspend                1009b898 f   mlme.obj
 0001:0009ac0c       MlmeResume                 1009bc0c f   mlme.obj
 0001:0009ad8c       MlmePeriodicExec           1009bd8c f   mlme.obj
 0001:0009b5bc       STAMlmePeriodicExec        1009c5bc f   mlme.obj
 0001:0009f144       LinkDownExec               100a0144 f   mlme.obj
 0001:0009f1cc       LinkUpExec                 100a01cc f   mlme.obj
 0001:0009f254       MlmeAutoScan               100a0254 f   mlme.obj
 0001:0009f2e8       MlmeAutoReconnectLastSSID  100a02e8 f   mlme.obj
 0001:0009f47c       MlmeValidateSSID           100a047c f   mlme.obj
 0001:0009f510       MlmeIsVisibleSSID          100a0510 f   mlme.obj
 0001:0009f5bc       MlmeValidateSetSSID        100a05bc f   mlme.obj
 0001:0009f678       MlmeCheckForRoaming        100a0678 f   mlme.obj
 0001:0009f68c       MlmeCheckForFastRoaming    100a068c f   mlme.obj
 0001:000a0400       MlmeCalculateChannelQuality 100a1400 f   mlme.obj
 0001:000a089c       MlmeSetTxRate              100a189c f   mlme.obj
 0001:000a1bc4       MlmeUpdateLimitTxRateTable 100a2bc4 f   mlme.obj
 0001:000a1f10       MlmeSelectTxRateTable      100a2f10 f   mlme.obj
 0001:000a3a4c       MlmeDynamicTxRateSwitching 100a4a4c f   mlme.obj
 0001:000a6524       StaQuickResponeForRateUpExec 100a7524 f   mlme.obj
 0001:000a71f4       MlmeCheckPsmChange         100a81f4 f   mlme.obj
 0001:000a734c       MlmeSetPsm                 100a834c f   mlme.obj
 0001:000a740c       MlmeSetTxPreamble          100a840c f   mlme.obj
 0001:000a7504       MlmeUpdateTxRates          100a8504 f   mlme.obj
 0001:000a9138       MlmeUpdateHtTxRates        100aa138 f   mlme.obj
 0001:000a9f08       AsicUpdateAutoFallBackTable 100aaf08 f   mlme.obj
 0001:000aa7b8       AsicUpdateProtect          100ab7b8 f   mlme.obj
 0001:000aaf38       MlmeRadioOff               100abf38 f   mlme.obj
 0001:000ab510       MlmeRadioOn                100ac510 f   mlme.obj
 0001:000ab848       BssTableInit               100ac848 f   mlme.obj
 0001:000ab8e4       BATableInit                100ac8e4 f   mlme.obj
 0001:000ab9b8       BssTableSearch             100ac9b8 f   mlme.obj
 0001:000abfc4       BssSsidTableSearch         100acfc4 f   mlme.obj
 0001:000ac154       BssTableSearchWithSSID     100ad154 f   mlme.obj
 0001:000ac364       BssTableDeleteEntry        100ad364 f   mlme.obj
 0001:000ac52c       BssTableDeleteEntryByBssid 100ad52c f   mlme.obj
 0001:000ac5f4       BssTableDeleteEntryByChannel 100ad5f4 f   mlme.obj
 0001:000ac948       BATableDeleteORIEntry      100ad948 f   mlme.obj
 0001:000acb88       BATableDeleteRECEntry      100adb88 f   mlme.obj
 0001:000ad0c0       BATableTearRECEntry        100ae0c0 f   mlme.obj
 0001:000ad408       BATableTearORIEntry        100ae408 f   mlme.obj
 0001:000ad828       BssEntrySet                100ae828 f   mlme.obj
 0001:000ae264       BssTableSetEntry           100af264 f   mlme.obj
 0001:000ae818       BATableInsertEntry         100af818 f   mlme.obj
 0001:000af3fc       TriEventInit               100b03fc f   mlme.obj
 0001:000af498       TriEventTableSetEntry      100b0498 f   mlme.obj
 0001:000af70c       BssTableSsidSort           100b070c f   mlme.obj
 0001:000b034c       BssTableSortByRssi         100b134c f   mlme.obj
 0001:000b08cc       BssCipherParse             100b18cc f   mlme.obj
 0001:000b1b48       MacAddrRandomBssid         100b2b48 f   mlme.obj
 0001:000b1bc8       MgtMacHeaderInit           100b2bc8 f   mlme.obj
 0001:000b1e18       MakeOutgoingFrame          100b2e18 f   mlme.obj
 0001:000b1edc       MlmeQueueInit              100b2edc f   mlme.obj
 0001:000b1fd4       MlmeEnqueue                100b2fd4 f   mlme.obj
 0001:000b224c       MlmeEnqueueForRecv         100b324c f   mlme.obj
 0001:000b268c       MlmeDequeue                100b368c f   mlme.obj
 0001:000b2798       MlmeRestartStateMachine    100b3798 f   mlme.obj
 0001:000b2cd0       MlmePostRestartStateMachine 100b3cd0 f   mlme.obj
 0001:000b2df8       MlmeQueueEmpty             100b3df8 f   mlme.obj
 0001:000b2e68       MlmeQueueFull              100b3e68 f   mlme.obj
 0001:000b2f0c       MlmeQueueClean             100b3f0c f   mlme.obj
 0001:000b3038       MlmeQueueDestroy           100b4038 f   mlme.obj
 0001:000b309c       MsgTypeSubst               100b409c f   mlme.obj
 0001:000b395c       StateMachineInit           100b495c f   mlme.obj
 0001:000b3a50       StateMachineSetAction      100b4a50 f   mlme.obj
 0001:000b3aec       StateMachinePerformAction  100b4aec f   mlme.obj
 0001:000b3b68       Drop                       100b4b68 f   mlme.obj
 0001:000b3b7c       LfsrInit                   100b4b7c f   mlme.obj
 0001:000b3bc8       RandomByte                 100b4bc8 f   mlme.obj
 0001:000b3cbc       AsicSwitchChannel          100b4cbc f   mlme.obj
 0001:000b5edc       AsicLockChannel            100b6edc f   mlme.obj
 0001:000b5ef0       AsicAntennaSelect          100b6ef0 f   mlme.obj
 0001:000b5f04       AsicAntennaSetting         100b6f04 f   mlme.obj
 0001:000b5f20       AsicAdjustTxPower          100b6f20 f   mlme.obj
 0001:000b81f8       AsicSleepThenAutoWakeup    100b91f8 f   mlme.obj
 0001:000b8300       AsicForceSleep             100b9300 f   mlme.obj
 0001:000b8374       AsicForceWakeup            100b9374 f   mlme.obj
 0001:000b8410       AsicSetBssid               100b9410 f   mlme.obj
 0001:000b85a0       AsicSetMcastWC             100b95a0 f   mlme.obj
 0001:000b862c       AsicSetBssidWC             100b962c f   mlme.obj
 0001:000b8640       AsicDelWcidTab             100b9640 f   mlme.obj
 0001:000b86e4       AsicSetCarrierDetectAction 100b96e4 f   mlme.obj
 0001:000b87d4       AsicDisableSync            100b97d4 f   mlme.obj
 0001:000b8880       AsicEnableRDG              100b9880 f   mlme.obj
 0001:000b892c       AsicDisableRDG             100b992c f   mlme.obj
 0001:000b89f4       AsicEnablePiggyB           100b99f4 f   mlme.obj
 0001:000b8a64       AsicDisablePiggyB          100b9a64 f   mlme.obj
 0001:000b8ad8       AsicEnableBssSync          100b9ad8 f   mlme.obj
 0001:000b8c4c       AsicEnableIbssSync         100b9c4c f   mlme.obj
 0001:000b8f6c       AsicSetEdcaParm            100b9f6c f   mlme.obj
 0001:000b9bc4       AsicSetSlotTime            100babc4 f   mlme.obj
 0001:000b9d84       AsicBbpTuning              100bad84 f   mlme.obj
 0001:000babc4       AsicUpdateWCIDAttribute    100bbbc4 f   mlme.obj
 0001:000bac80       AsicUpdateWCIDIVEIV        100bbc80 f   mlme.obj
 0001:000bace8       AsicUpdateRxWCIDTable      100bbce8 f   mlme.obj
 0001:000badcc       AsicAddKeyEntry            100bbdcc f   mlme.obj
 0001:000bb2c8       AsicAddWcidCipherEntry     100bc2c8 f   mlme.obj
 0001:000bb398       AsicAddSharedKeyEntry      100bc398 f   mlme.obj
 0001:000bb9e0       AsicRemoveSharedKeyMode    100bc9e0 f   mlme.obj
 0001:000bbc1c       AsicRemoveKeyEntry         100bcc1c f   mlme.obj
 0001:000bbc9c       AsicRemoveSharedKeyEntry   100bcc9c f   mlme.obj
 0001:000bbf24       AsicAddPairwiseKeyEntry    100bcf24 f   mlme.obj
 0001:000bbf38       AsicRemovePairwiseKeyEntry 100bcf38 f   mlme.obj
 0001:000bbf4c       AsicSendCommanToMcu        100bcf4c f   mlme.obj
 0001:000bc128       RTMPCheckRates             100bd128 f   mlme.obj
 0001:000bc2e4       RTMPCheckChannel           100bd2e4 f   mlme.obj
 0001:000bc510       RTMPCheckHt                100bd510 f   mlme.obj
 0001:000bd858       RTMPCheckAddHtInfoIe       100be858 f   mlme.obj
 0001:000bd920       AsicSetRxAnt               100be920 f   mlme.obj
 0001:000bdac8       AsicEvaluateRxAnt          100beac8 f   mlme.obj
 0001:000bde84       AsicRxAntEvalTimeout       100bee84 f   mlme.obj
 0001:000bdec0       AsicRxAntEvalAction        100beec0 f   mlme.obj
 0001:000be39c       RadarDetectionStart        100bf39c f   mlme.obj
 0001:000be3d0       RadarDetectionStop         100bf3d0 f   mlme.obj
 0001:000be400       RadarChannelCheck          100bf400 f   mlme.obj
 0001:000be538       MlmeThread                 100bf538 f   mlme.obj
 0001:000be690       MlmeFreeMemory             100bf690 f   mlme.obj
 0001:000bee44       MlmeAllocateMemory         100bfe44 f   mlme.obj
 0001:000bf254       MlmeInitMemoryHandler      100c0254 f   mlme.obj
 0001:000bf608       MlmeFreeMemoryHandler      100c0608 f   mlme.obj
 0001:000bf74c       RTMPUpdateMlmeRate         100c074c f   mlme.obj
 0001:000bfc2c       RTMPMaxRssi                100c0c2c f   mlme.obj
 0001:000bfd24       RTMPSetAGCInitValue        100c0d24 f   mlme.obj
 0001:000c041c       CarrierDetectTimeout       100c141c f   mlme.obj
 0001:000c0458       CarrierDetectTimeoutAction 100c1458 f   mlme.obj
 0001:000c08cc       AsicSendBA                 100c18cc f   mlme.obj
 0001:000c0fc0       AsicSendNullFrame          100c1fc0 f   mlme.obj
 0001:000c17b0       RTUSBFilterCalibration     100c27b0 f   mlme.obj
 0001:000c1df0       SSIDLUpdateBssEntry        100c2df0 f   mlme.obj
 0001:000c2998       AsicCheckCommandOk         100c3998 f   mlme.obj
 0001:000c2be4       InitDesiredTSSITable       100c3be4 f   mlme.obj
 0001:000c3a34       GetDesiredTSSI             100c4a34 f   mlme.obj
 0001:000c3d5c       RRMInitNHMCtrl             100c4d5c f   mlme.obj
 0001:000c3eb8       RRMGetIPIDensities         100c4eb8 f   mlme.obj
 0001:000c43e8       CKIP_key_permute           100c53e8 f   rtmp_ckipmic.obj
 0001:000c475c       mix_column_DWORD32         100c575c f   rtmp_ckipmic.obj
 0001:000c4874       RTMPCkipMicInit            100c5874 f   rtmp_ckipmic.obj
 0001:000c48dc       RTMPCkipInsertCMIC         100c58dc f   rtmp_ckipmic.obj
 0001:000c4d1c       RTMPCkipCalCMIC            100c5d1c f   rtmp_ckipmic.obj
 0001:000c5088       RTMPCkipDecrypt            100c6088 f   rtmp_ckipmic.obj
 0001:000c53c0       RTMGetPCkipPK              100c63c0 f   rtmp_ckipmic.obj
 0001:000c5548       RTMPMicUpdate              100c6548 f i rtmp_ckipmic.obj
 0001:000c574c       RTMPMicGetCoefficient      100c674c f i rtmp_ckipmic.obj
 0001:000c58b4       RTMPAesEncrypt             100c68b4 f i rtmp_ckipmic.obj
 0001:000c5b18       next_key@8                 100c6b18 f i rtmp_ckipmic.obj
 0001:000c5c98       byte_sub_shift_row@8       100c6c98 f i rtmp_ckipmic.obj
 0001:000c5f28       RTMPMicFinal               100c6f28 f i rtmp_ckipmic.obj
 0001:000c61a8       BtCheckWifiThroughputOverLimit 100c71a8 f   rtmp_cobt.obj
 0001:000c6424       BtCheckBusy                100c7424 f   rtmp_cobt.obj
 0001:000c6ad0       InitBTCoexistence          100c7ad0 f   rtmp_cobt.obj
 0001:000c6ffc       BtCoexistDetectExecAtCmdThread 100c7ffc f   rtmp_cobt.obj
 0001:000c7d9c       BtCoexistDetectExecAtTimer 100c8d9c f   rtmp_cobt.obj
 0001:000c7f7c       RTMPQueryInformation       100c8f7c f   rtmp_info.obj
 0001:000ccce4       RTMPSetInformation         100cdce4 f   rtmp_info.obj
 0001:000cf24c       STAQueryInformation        100d024c f   rtmp_info.obj
 0001:000d3868       STASetInformation          100d4868 f   rtmp_info.obj
 0001:000dd13c       RTMPWPAAddKeyProc          100de13c f   rtmp_info.obj
 0001:000decc0       RTMPWPARemoveKeyProc       100dfcc0 f   rtmp_info.obj
 0001:000defb8       RTMPWPARemoveAllKeys       100dffb8 f   rtmp_info.obj
 0001:000df10c       RTMPIndicateWPA2Status     100e010c f   rtmp_info.obj
 0001:000df5bc       RTMPSetPhyMode             100e05bc f   rtmp_info.obj
 0001:000e0170       RTMPOPModeSwitching        100e1170 f   rtmp_info.obj
 0001:000e03cc       RTMPAddBSSIDCipher         100e13cc f   rtmp_info.obj
 0001:000e100c       RTMPSetHT                  100e200c f   rtmp_info.obj
 0001:000e3040       RTMPUpdateHTIE             100e4040 f   rtmp_info.obj
 0001:000e35e4       LEDConnectionStart         100e45e4 f   rtmp_info.obj
 0001:000e3700       LEDConnectionCompletion    100e4700 f   rtmp_info.obj
 0001:000e3888       RTMPMantainAdhocList       100e4888 f   rtmp_info.obj
 0001:000e3a54       BitReverse                 100e4a54 f   rtmp_init.obj
 0001:000e3aec       RTMPAllocAdapterBlock      100e4aec f   rtmp_init.obj
 0001:000e3c10       NICInitTransmit            100e4c10 f   rtmp_init.obj
 0001:000e4690       CreateThreads              100e5690 f   rtmp_init.obj
 0001:000e4900       NICInitRecv                100e5900 f   rtmp_init.obj
 0001:000e4c64       RTUSBBulkReceiveDPC        100e5c64 f   rtmp_init.obj
 0001:000e4d80       RTUSBRxPacketDPC           100e5d80 f   rtmp_init.obj
 0001:000e4e90       RTUSBKickbulkoutDPC        100e5e90 f   rtmp_init.obj
 0001:000e4fdc       FreeNICRecv                100e5fdc f   rtmp_init.obj
 0001:000e51a4       FreeNICTransmit            100e61a4 f   rtmp_init.obj
 0001:000e5610       DisallocateAllSpinLock     100e6610 f   rtmp_init.obj
 0001:000e5894       RTMPInitAdapterBlock       100e6894 f   rtmp_init.obj
 0001:000e6090       ReleaseAdapter             100e7090 f   rtmp_init.obj
 0001:000e6114       RTMPReadTxPwrPerRate       100e7114 f   rtmp_init.obj
 0001:000e6bec       RTMPReadChannelPwr         100e7bec f   rtmp_init.obj
 0001:000e8040       IsRalinkEncStr             100e9040 f   rtmp_init.obj
 0001:000e8198       DecryptWepRegistry         100e9198 f   rtmp_init.obj
 0001:000e834c       NICReadRegParameters       100e934c f   rtmp_init.obj
 0001:000e9dac       RTUSBWriteHWMACAddress     100eadac f   rtmp_init.obj
 0001:000e9ff0       NICReadEEPROMParameters    100eaff0 f   rtmp_init.obj
 0001:000eb374       RT30xxInitAsic             100ec374 f   rtmp_init.obj
 0001:000ec30c       NICInitAsicFromEEPROM      100ed30c f   rtmp_init.obj
 0001:000ed578       PostBBPInitialization      100ee578 f   rtmp_init.obj
 0001:000ed804       PostRFInitialization       100ee804 f   rtmp_init.obj
 0001:000ed950       NICWaitMACReady            100ee950 f   rtmp_init.obj
 0001:000ed9bc       NICInitializeAsic          100ee9bc f   rtmp_init.obj
 0001:000ee600       NICIssueReset              100ef600 f   rtmp_init.obj
 0001:000ee614       NICCheckForHang            100ef614 f   rtmp_init.obj
 0001:000ee63c       NICUpdateRawCounters       100ef63c f   rtmp_init.obj
 0001:000ee9c0       NICResetFromError          100ef9c0 f   rtmp_init.obj
 0001:000ee9fc       NICLoadFirmware            100ef9fc f   rtmp_init.obj
 0001:000ef2bc       LoadExternalEEPROMImage    100f02bc f   rtmp_init.obj
 0001:000ef4d0       RTMPEqualMemory            100f04d0 f   rtmp_init.obj
 0001:000ef58c       RTMPCompareMemory          100f058c f   rtmp_init.obj
 0001:000ef66c       RTMPZeroMemory             100f066c f   rtmp_init.obj
 0001:000ef6d8       RTMPFillMemory             100f06d8 f   rtmp_init.obj
 0001:000ef744       RTMPMoveMemory             100f0744 f   rtmp_init.obj
 0001:000ef81c       UserCfgInit                100f081c f   rtmp_init.obj
 0001:000f0fa0       EnableTwoPhasesScanOperation 100f1fa0 f   rtmp_init.obj
 0001:000f1030       BtoH                       100f2030 f   rtmp_init.obj
 0001:000f10e4       AtoH                       100f20e4 f   rtmp_init.obj
 0001:000f11b4       RTMPPatchMacBbpBug         100f21b4 f   rtmp_init.obj
 0001:000f11c8       RTMPInitTimer              100f21c8 f   rtmp_init.obj
 0001:000f1224       RTMPSetTimer               100f2224 f   rtmp_init.obj
 0001:000f12d8       RTMPCancelTimer            100f22d8 f   rtmp_init.obj
 0001:000f135c       RTMPSetLED                 100f235c f   rtmp_init.obj
 0001:000f1e50       RTMPSetSignalLED           100f2e50 f   rtmp_init.obj
 0001:000f1f7c       RTMPEnableRxTx             100f2f7c f   rtmp_init.obj
 0001:000f226c       RTMPReadSafelyRemoveFlag   100f326c f   rtmp_init.obj
 0001:000f2394       RTMPPrepareCTSFrame        100f3394 f   rtmp_init.obj
 0001:000f26f4       RTMPSetMessageEvent        100f36f4 f   rtmp_init.obj
 0001:000f2a0c       AsicRadioOff               100f3a0c f   rtmp_init.obj
 0001:000f2e5c       AsicRFOn                   100f3e5c f   rtmp_init.obj
 0001:000f3244       AsicRadioOn                100f4244 f   rtmp_init.obj
 0001:000f3434       DriverEntry                100f4434 f   rtmp_main.obj
 0001:000f36e0       RTMPInitialize             100f46e0 f   rtmp_main.obj
 0001:000f4134       RTMPCheckForHang           100f5134 f   rtmp_main.obj
 0001:000f42c8       RTMPHalt                   100f52c8 f   rtmp_main.obj
 0001:000f4af4       RTMPReset                  100f5af4 f   rtmp_main.obj
 0001:000f4b74       RTMPTransferData           100f5b74 f   rtmp_main.obj
 0001:000f4e1c       RTMPPnPEventNotify         100f5e1c f   rtmp_main.obj
 0001:000f5190       RTMPShutdown               100f6190 f   rtmp_main.obj
 0001:000f5260       JunkThread                 100f6260 f   rtmp_main.obj
 0001:000f5578       RTMPTkipGetUInt32          100f6578 f   rtmp_tkip.obj
 0001:000f5604       RTMPTkipPutUInt32          100f6604 f   rtmp_tkip.obj
 0001:000f5674       RTMPTkipSetMICKey          100f6674 f   rtmp_tkip.obj
 0001:000f5718       RTMPTkipAppendByte         100f6718 f   rtmp_tkip.obj
 0001:000f5984       RTMPTkipAppend             100f6984 f   rtmp_tkip.obj
 0001:000f59e0       RTMPTkipGetMIC             100f69e0 f   rtmp_tkip.obj
 0001:000f5a80       RTMPInitTkipEngine         100f6a80 f   rtmp_tkip.obj
 0001:000f5b58       RTMPInitMICEngine          100f6b58 f   rtmp_tkip.obj
 0001:000f5be4       RTMPTkipCompareMICValue    100f6be4 f   rtmp_tkip.obj
 0001:000f5e64       RTMPTkipCompareMICValueWithLLC 100f6e64 f   rtmp_tkip.obj
 0001:000f60f8       RTMPCalculateMICValue      100f70f8 f   rtmp_tkip.obj
 0001:000f62fc       tkip_sbox                  100f72fc f   rtmp_tkip.obj
 0001:000f63f4       rotr1                      100f73f4 f   rtmp_tkip.obj
 0001:000f6470       RTMPTkipMixKey             100f7470 f   rtmp_tkip.obj
 0001:000f6fec       construct_mic_header1      100f7fec f   rtmp_tkip.obj
 0001:000f71c0       construct_mic_header2      100f81c0 f   rtmp_tkip.obj
 0001:000f743c       construct_mic_iv           100f843c f   rtmp_tkip.obj
 0001:000f75fc       bitwise_xor                100f85fc f   rtmp_tkip.obj
 0001:000f7684       aes128k128d                100f8684 f   rtmp_tkip.obj
 0001:000f7908       construct_ctr_preload      100f8908 f   rtmp_tkip.obj
 0001:000f7af8       GetMacHdrLength            100f8af8 f   rtmp_tkip.obj
 0001:000f7ca8       RTMPSoftEncryptTKIP        100f8ca8 f   rtmp_tkip.obj
 0001:000f8488       RTMPSoftDecryptTKIP        100f9488 f   rtmp_tkip.obj
 0001:000f8b48       RTMPSoftEncryptAES         100f9b48 f   rtmp_tkip.obj
 0001:000f9364       RTMPSoftDecryptAES         100fa364 f   rtmp_tkip.obj
 0001:000f9a40       ccmp128_init               100faa40 f   rtmp_tkip.obj
 0001:000fa3d8       ccmp128_encrypt            100fb3d8 f   rtmp_tkip.obj
 0001:000facf4       ccmp128_decrypt            100fbcf4 f   rtmp_tkip.obj
 0001:000fb698       ccmp128_finalize           100fc698 f   rtmp_tkip.obj
 0001:000fb8e0       RTMPSoftEncryptMgmtAES     100fc8e0 f   rtmp_tkip.obj
 0001:000fbfc0       RTMPSoftDecryptMgmtAES     100fcfc0 f   rtmp_tkip.obj
 0001:000fc588       byte_sub                   100fd588 f i rtmp_tkip.obj
 0001:000fc818       shift_row                  100fd818 f i rtmp_tkip.obj
 0001:000fc9a4       mix_column                 100fd9a4 f i rtmp_tkip.obj
 0001:000fcbd0       RTMPInitWepEngine          100fdbd0 f   rtmp_wep.obj
 0001:000fcd28       RTMPEncryptData            100fdd28 f   rtmp_wep.obj
 0001:000fcd9c       RTMPDecryptData            100fdd9c f   rtmp_wep.obj
 0001:000fd08c       ARCFOUR_INIT               100fe08c f   rtmp_wep.obj
 0001:000fd1c8       ARCFOUR_BYTE               100fe1c8 f   rtmp_wep.obj
 0001:000fd2c8       ARCFOUR_DECRYPT            100fe2c8 f   rtmp_wep.obj
 0001:000fd34c       ARCFOUR_ENCRYPT            100fe34c f   rtmp_wep.obj
 0001:000fd3d0       WPAARCFOUR_ENCRYPT         100fe3d0 f   rtmp_wep.obj
 0001:000fd484       RTMP_CALC_FCS32            100fe484 f   rtmp_wep.obj
 0001:000fd514       RTMPSetICV                 100fe514 f   rtmp_wep.obj
 0001:000fd57c       RTUSBInitTxDesc            100fe57c f   rtusb_bulk.obj
 0001:000fd590       RTUSBInitHTTxDesc          100fe590 f   rtusb_bulk.obj
 0001:000fd5a4       RTUSBInitRxDesc            100fe5a4 f   rtusb_bulk.obj
 0001:000fd5b8       RTUSBUpdateTxD             100fe5b8 f   rtusb_bulk.obj
 0001:000fd5cc       RTUSBComposeUnit           100fe5cc f   rtusb_bulk.obj
 0001:000fe95c       RTUSBBulkOutDataPacket     100ff95c f   rtusb_bulk.obj
 0001:000ffa84       RTUSBBulkOutDataPacketComplete 10100a84 f   rtusb_bulk.obj
 0001:000ffed4       RTUSBBulkOutNullFrame      10100ed4 f   rtusb_bulk.obj
 0001:00100190       RTUSBBulkOutNullFrameComplete 10101190 f   rtusb_bulk.obj
 0001:001003fc       RTUSBBulkOutRTSFrame       101013fc f   rtusb_bulk.obj
 0001:001007b4       RTUSBBulkOutRTSFrameComplete 101017b4 f   rtusb_bulk.obj
 0001:00100a70       RTUSBBulkOutMLMEPacket     10101a70 f   rtusb_bulk.obj
 0001:00100dc8       RTUSBBulkOutMLMEPacketComplete 10101dc8 f   rtusb_bulk.obj
 0001:00101280       RTUSBBulkOutPsPoll         10102280 f   rtusb_bulk.obj
 0001:001014e0       RTUSBBulkOutPsPollComplete 101024e0 f   rtusb_bulk.obj
 0001:0010174c       RTUSBBulkReceive           1010274c f   rtusb_bulk.obj
 0001:00101b94       RTUSBBulkRxComplete        10102b94 f   rtusb_bulk.obj
 0001:00102020       RTUSBKickBulkOut           10103020 f   rtusb_bulk.obj
 0001:001024f0       RTUSBCleanUpDataBulkOutQueue 101034f0 f   rtusb_bulk.obj
 0001:00102660       RTUSBCleanUpMLMEBulkOutQueue 10103660 f   rtusb_bulk.obj
 0001:001027ac       RTUSBCancelPendingIRPs     101037ac f   rtusb_bulk.obj
 0001:001027d0       RTUSBCancelPendingBulkInIRP 101037d0 f   rtusb_bulk.obj
 0001:0010284c       RTUSBCancelPendingBulkOutIRP 1010384c f   rtusb_bulk.obj
 0001:00102c60       Sniff2BytesFromNdisBuffer  10103c60 f   rtusb_data.obj
 0001:00102e44       RTMPSendPackets            10103e44 f   rtusb_data.obj
 0001:001032dc       RTMPSendPacket             101042dc f   rtusb_data.obj
 0001:00103f78       RTMPDeQueuePacket          10104f78 f   rtusb_data.obj
 0001:00104660       RTUSBFreeDescriptorRequest 10105660 f   rtusb_data.obj
 0001:00104b50       RTUSBRejectPendingPackets  10105b50 f   rtusb_data.obj
 0001:00104f88       RTUSBSuspendMsduTransmission 10105f88 f   rtusb_data.obj
 0001:001050a4       RTUSBResumeMsduTransmission 101060a4 f   rtusb_data.obj
 0001:001053b4       RTUSBCalcDuration          101063b4 f   rtusb_data.obj
 0001:00105590       RTMPWriteTxWI              10106590 f   rtusb_data.obj
 0001:00105e50       RTMPWriteTxInfo            10106e50 f   rtusb_data.obj
 0001:00105f90       TxFrameIsAggregatible      10106f90 f   rtusb_data.obj
 0001:0010606c       RTMPFreeNdisPacket         1010706c f   rtusb_data.obj
 0001:00106140       RTMPDecideSegmentEnd       10107140 f   rtusb_data.obj
 0001:00106204       RTUSBHardTransmit          10107204 f   rtusb_data.obj
 0001:0010cc3c       RTUSBRxPacket              1010dc3c f   rtusb_data.obj
 0001:001128a8       RTUSBDequeueMLMEPacket     101138a8 f   rtusb_data.obj
 0001:00112bb8       RTUSBCleanUpMLMEWaitQueue  10113bb8 f   rtusb_data.obj
 0001:00112d50       MiniportMMRequest          10113d50 f   rtusb_data.obj
 0001:001131f0       RTMPApplyPacketFilter      101141f0 f   rtusb_data.obj
 0001:001135cc       RTMPCheckRxWI              101145cc f   rtusb_data.obj
 0001:00114034       RTMPReportMicError         10115034 f   rtusb_data.obj
 0001:00114230       RTUSBMlmeHardTransmit      10115230 f   rtusb_data.obj
 0001:00114efc       RTMPSendNullFrame          10115efc f   rtusb_data.obj
 0001:001158e4       RTMPSendNullFrameForDirect 101168e4 f   rtusb_data.obj
 0001:001161f4       RTMPSendRTSCTSFrame        101171f4 f   rtusb_data.obj
 0001:00116208       RTMPCalcDuration           10117208 f   rtusb_data.obj
 0001:001163fc       RTMPCheckDHCPFrame         101173fc f   rtusb_data.obj
 0001:001166b0       RTMPCheckTxSIPPacket       101176b0 f   rtusb_data.obj
 0001:00116b5c       RTMPCheckRxSIPPacket       10117b5c f   rtusb_data.obj
 0001:00116e18       MailBoxTOExec              10117e18 f   rtusb_data.obj
 0001:00116ee4       RTMPSearchTupleCache       10117ee4 f   rtusb_data.obj
 0001:00117034       RTMPUpdateTupleCache       10118034 f   rtusb_data.obj
 0001:001175ec       MulticastRate_NRateToOFDMRate 101185ec f   rtusb_data.obj
 0001:00117754       RTMPSendBAR                10118754 f   rtusb_data.obj
 0001:001185a0       RTMPSendTxWaitQueue        101195a0 f   rtusb_data.obj
 0001:00118a80       MCSToPhyRateIn500kps       10119a80 f   rtusb_data.obj
 0001:00118e6c       RTUSBFirmwareRun           10119e6c f   rtusb_io.obj
 0001:00118ed4       InitEFuseConfig            10119ed4 f   rtusb_io.obj
 0001:00118ff0       FlashInstallationWith8KBFirmware 10119ff0 f   rtusb_io.obj
 0001:001190f4       RTUSBFirmwareOpmode        1011a0f4 f   rtusb_io.obj
 0001:0011915c       RTUSBVenderReset           1011a15c f   rtusb_io.obj
 0001:00119200       RTUSBSingleWrite           1011a200 f   rtusb_io.obj
 0001:00119268       RTUSBMultiRead             1011a268 f   rtusb_io.obj
 0001:001192d0       RTUSBMultiWrite2           1011a2d0 f   rtusb_io.obj
 0001:00119338       RTUSBMultiWrite            1011a338 f   rtusb_io.obj
 0001:0011945c       RTUSBReadMACRegister       1011a45c f   rtusb_io.obj
 0001:001194c4       RTUSBWriteMACRegister      1011a4c4 f   rtusb_io.obj
 0001:0011959c       RTUSBReadBBPRegister       1011a59c f   rtusb_io.obj
 0001:00119780       RTUSBWriteBBPRegister      1011a780 f   rtusb_io.obj
 0001:0011991c       RTUSBWriteRFRegister       1011a91c f   rtusb_io.obj
 0001:00119a08       RT30xxWriteRFRegister      1011aa08 f   rtusb_io.obj
 0001:00119b40       RT3572WriteBBPR66          1011ab40 f   rtusb_io.obj
 0001:00119c48       RT30xxReadRFRegister       1011ac48 f   rtusb_io.obj
 0001:00119dec       eFusePhysicalReadRegisters 1011adec f   rtusb_io.obj
 0001:00119f74       eFuseReadRegisters         1011af74 f   rtusb_io.obj
 0001:0011a174       eFuseRead                  1011b174 f   rtusb_io.obj
 0001:0011a238       eFuseReadPhysical          1011b238 f   rtusb_io.obj
 0001:0011a300       eFusePhysicalWriteRegisters 1011b300 f   rtusb_io.obj
 0001:0011a6d4       eFuseWritePhysical         1011b6d4 f   rtusb_io.obj
 0001:0011a7a8       eFuseWriteRegisters        1011b7a8 f   rtusb_io.obj
 0001:0011b310       eFuseWrite                 1011c310 f   rtusb_io.obj
 0001:0011b3c8       RTUSBReadEEPROM            1011c3c8 f   rtusb_io.obj
 0001:0011b4ec       RTUSBWriteEEPROM           1011c4ec f   rtusb_io.obj
 0001:0011b55c       RTUSBPutToSleep            1011c55c f   rtusb_io.obj
 0001:0011b5d0       RTUSBWakeUp                1011c5d0 f   rtusb_io.obj
 0001:0011b638       RTUSBInitializeCmdQ        1011c638 f   rtusb_io.obj
 0001:0011b678       RTUSBEnqueueCmdFromNdis    1011c678 f   rtusb_io.obj
 0001:0011bacc       RTUSBEnqueueInternalCmd    1011cacc f   rtusb_io.obj
 0001:0011be5c       RTUSBDequeueCmd            1011ce5c f   rtusb_io.obj
 0001:0011bee8       RTUSB_VendorRequest        1011cee8 f   rtusb_io.obj
 0001:0011c438       RTUSB_InterfaceStop        1011d438 f   rtusb_io.obj
 0001:0011c49c       RTUSB_ResetPipe            1011d49c f   rtusb_io.obj
 0001:0011c70c       RTUSB_ResetDevice          1011d70c f   rtusb_io.obj
 0001:0011c850       RTUSB_AbortPipe            1011d850 f   rtusb_io.obj
 0001:0011c9e4       RTUSB_ReadVersion          1011d9e4 f   rtusb_io.obj
 0001:0011cac0       RTUSB_HandleBulkInFail     1011dac0 f   rtusb_io.obj
 0001:0011cb9c       RTUSB_GetPortStatus        1011db9c f   rtusb_io.obj
 0001:0011cc1c       RTUSB_EndpointUsage        1011dc1c f   rtusb_io.obj
 0001:0011ce64       RTUSB_ReBulkOut            1011de64 f   rtusb_io.obj
 0001:0011d3a8       RTUSBCmdThread             1011e3a8 f   rtusb_io.obj
 0001:001246e0       RTUSBQueryHardWareRegister 101256e0 f   rtusb_io.obj
 0001:00124c54       RTUSBSetHardWareRegister   10125c54 f   rtusb_io.obj
 0001:001279d4       MlmeScanReqSanity          101289d4 f   sanity.obj
 0001:00127b58       MlmeStartReqSanity         10128b58 f   sanity.obj
 0001:00127bf0       MlmeAssocReqSanity         10128bf0 f   sanity.obj
 0001:00127ce4       MlmeAuthReqSanity          10128ce4 f   sanity.obj
 0001:00127e34       PeerAssocRspSanity         10128e34 f   sanity.obj
 0001:00128900       PeerDisassocSanity         10129900 f   sanity.obj
 0001:00128af0       PeerDeauthSanity           10129af0 f   sanity.obj
 0001:00128ce0       PeerAuthSanity             10129ce0 f   sanity.obj
 0001:00128f20       PeerProbeReqSanity         10129f20 f   sanity.obj
 0001:0012915c       PeerBeaconAndProbeRspSanity 1012a15c f   sanity.obj
 0001:0012b678       PeerBeaconAndProbeRspSanity2 1012c678 f   sanity.obj
 0001:0012b8a8       PeerAddBAReqActionSanity   1012c8a8 f   sanity.obj
 0001:0012bb70       PeerAddBARspActionSanity   1012cb70 f   sanity.obj
 0001:0012bd10       PeerDelBAActionSanity      1012cd10 f   sanity.obj
 0001:0012bdc4       GetTimBit                  1012cdc4 f   sanity.obj
 0001:0012bfd0       ChannelSanity              1012cfd0 f   sanity.obj
 0001:0012c078       NetworkTypeInUseSanity     1012d078 f   sanity.obj
 0001:0012c144       PeerTxTypeInUseSanity      1012d144 f   sanity.obj
 0001:0012c2f0       RTMPWPAWepKeySanity        1012d2f0 f   sanity.obj
 0001:0012c5e4       RTMPRemoveKeySanity        1012d5e4 f   sanity.obj
 0001:0012c990       MlmeAddBAReqSanity         1012d990 f   sanity.obj
 0001:0012cacc       MlmeDelBAReqSanity         1012dacc f   sanity.obj
 0001:0012cba8       MlmeDlsReqSanity           1012dba8 f   sanity.obj
 0001:0012cbfc       PeerDlsReqSanity           1012dbfc f   sanity.obj
 0001:0012ce34       PeerDlsRspSanity           1012de34 f   sanity.obj
 0001:0012d060       PeerDlsTearDownSanity      1012e060 f   sanity.obj
 0001:0012d108       PeerAcmRspSanity           1012e108 f   sanity.obj
 0001:0012d188       MlmeTdlsReqSanity          1012e188 f   sanity.obj
 0001:0012d1dc       PeerTdlsSetupReqSanity     1012e1dc f   sanity.obj
 0001:0012d878       PeerTdlsSetupRspSanity     1012e878 f   sanity.obj
 0001:0012df9c       PeerTdlsSetupConfSanity    1012ef9c f   sanity.obj
 0001:0012e6d8       PeerTdlsTearDownSanity     1012f6d8 f   sanity.obj
 0001:0012ea3c       STAWapiStateMachineInit    1012fa3c f   Sta_wapi.obj
 0001:0012eaa0       STAWapiWAIPacketAction     1012faa0 f   Sta_wapi.obj
 0001:0012eec8       STAWapiWAIPacket_HandleMBcastReq 1012fec8 f   Sta_wapi.obj
 0001:0012ffc0       STAWapiWAIPacket_HandleUnicastReq 10130fc0 f   Sta_wapi.obj
 0001:00130710       STAWapiWAIPacket_HandleUnicastConf 10131710 f   Sta_wapi.obj
 0001:00130ea4       STAWapiSend_MBcastKeyNegotiate_Rsp 10131ea4 f   Sta_wapi.obj
 0001:001312b8       STAWapiSend_UnicastKeyNegotiate_Rsp 101322b8 f   Sta_wapi.obj
 0001:00131680       STAWapi_RxSMS4Decrypt      10132680 f   Sta_wapi.obj
 0001:001323c0       SyncStateMachineInit       101333c0 f   sync.obj
 0001:00132614       BeaconTimeout              10133614 f   sync.obj
 0001:001326ac       ScanTimeout                101336ac f   sync.obj
 0001:00132744       InvalidStateNullFunction   10133744 f   sync.obj
 0001:001327a0       MlmeScanReqAction          101337a0 f   sync.obj
 0001:00133050       MlmeJoinReqAction          10134050 f   sync.obj
 0001:00133afc       MlmeStartReqAction         10134afc f   sync.obj
 0001:001344ac       PeerBeaconAtScanAction     101354ac f   sync.obj
 0001:001354d4       PeerBeaconAtJoinAction     101364d4 f   sync.obj
 0001:00136920       PeerBeacon                 10137920 f   sync.obj
 0001:00139d08       PeerProbeReqAction         1013ad08 f   sync.obj
 0001:0013a7ec       BeaconTimeoutAtJoinAction  1013b7ec f   sync.obj
 0001:0013a9d4       ScanTimeoutAction          1013b9d4 f   sync.obj
 0001:0013b0ec       HasHiddenAPAtThisChannel   1013c0ec f   sync.obj
 0001:0013b26c       ScanNextChannel            1013c26c f   sync.obj
 0001:0013ccb8       InvalidStateWhenScan       1013dcb8 f   sync.obj
 0001:0013d198       InvalidStateWhenJoin       1013e198 f   sync.obj
 0001:0013d8b8       InvalidStateWhenStart      1013e8b8 f   sync.obj
 0001:0013d980       EnqueuePsPoll              1013e980 f   sync.obj
 0001:0013da30       EnqueueBeaconFrame         1013ea30 f   sync.obj
 0001:0013db4c       EnqueueProbeRequest        1013eb4c f   sync.obj
 0001:0013dcd0       BuildChannelList           1013ecd0 f   sync.obj
 0001:0013ebbc       FirstChannel               1013fbbc f   sync.obj
 0001:0013ec08       NextChannel                1013fc08 f   sync.obj
 0001:0013ed74       ChangeToCellPowerLimit     1013fd74 f   sync.obj
 0001:0013eea8       ConvertToRssi              1013fea8 f   sync.obj
 0001:0013f0ec       BuildEffectedChannelList   101400ec f   sync.obj
 0001:0013f614       DeleteEffectedChannelList  10140614 f   sync.obj
 0001:0013f6ac       AddToRepositList           101406ac f   sync.obj
 0001:001404c0       IsValidChannel             101414c0 f   sync.obj
 0001:00140590       RTMPCheckBWOffset          10141590 f   sync.obj
 0001:00140a9c       StaAdhocUpdateMacTableEntry 10141a9c f   sync.obj
 0001:00141e00       MlmeProbeInactiveStation   10142e00 f   sync.obj
 0001:00141fc4       DllEntry                   10142fc4 f   wince.obj
 0001:00142084       RTUSBCE_ClosePipe          10143084 f   wince.obj
 0001:00142164       RTUSBCE_RemoveDeviceContext 10143164 f   wince.obj
 0001:00142314       RTUSBCE_DeviceNotify       10143314 f   wince.obj
 0001:0014286c       RTUSBCE_ConfigureDevice    1014386c f   wince.obj
 0001:001433a0       RTUSBCE_InterfaceStart     101443a0 f   wince.obj
 0001:001436e4       USBDeviceAttach            101446e4 f   wince.obj
 0001:00143a94       USBInstallDriver           10144a94 f   wince.obj
 0001:00143c98       USBUnInstallDriver         10144c98 f   wince.obj
 0001:00143e04       LoadVIDFromRegistry        10144e04 f   wince.obj
 0001:00144198       ParseUsbDescriptors        10145198 f   wince.obj
 0001:00145200       RTMPCopyUnicodeString      10146200 f   wince.obj
 0001:00145388       DBGDUMP_HEX                10146388 f   wince.obj
 0001:00145798       TestMoveMemory             10146798 f   wince.obj
 0001:00145c34       DumpSystemInfo             10146c34 f   wince.obj
 0001:00145d0c       WpaMsgTypeSubst            10146d0c f   wpa.obj
 0001:00145dec       WpaPskStateMachineInit     10146dec f   wpa.obj
 0001:00145e58       WpaEAPOLKeyAction          10146e58 f   wpa.obj
 0001:001466ec       WpaPairMsg1Action          101476ec f   wpa.obj
 0001:00146d00       WpaPairMsg3Action          10147d00 f   wpa.obj
 0001:00147490       WpaGroupMsg1Action         10148490 f   wpa.obj
 0001:00147d14       WpaMacHeaderInit           10148d14 f   wpa.obj
 0001:00147fc0       WpaHardTransmit            10148fc0 f   wpa.obj
 0001:001486e0       HMAC_SHA1                  101496e0 f   wpa.obj
 0001:00148874       PRF                        10149874 f   wpa.obj
 0001:001489e4       CCKMPRF                    101499e4 f   wpa.obj
 0001:00148b18       WpaCountPTK                10149b18 f   wpa.obj
 0001:00148e98       GenRandom                  10149e98 f   wpa.obj
 0001:00149118       AES_GTK_KEY_UNWRAP         1014a118 f   wpa.obj
 0001:00149300       HMAC_SHA256                1014a300 f   wpa.obj
 0001:001494d4       FT_KDF                     1014a4d4 f   wpa.obj
 0001:00149688       WscStateMachineInit        1014a688 f   wsc.obj
 0001:001498a0       WscEAPAction               1014a8a0 f   wsc.obj
 0001:001499c8       WscEAPEnrolleeAction       1014a9c8 f   wsc.obj
 0001:0014a498       WscEAPRegistrarAction      1014b498 f   wsc.obj
 0001:0014afd8       WscRxMsgType               1014bfd8 f   wsc.obj
 0001:0014b548       WscMsgTypeSubst            1014c548 f   wsc.obj
 0001:0014b638       WscConnectTimeout          1014c638 f   wsc.obj
 0001:0014ba18       WscScanTimeout             1014ca18 f   wsc.obj
 0001:0014baf4       WscPBCTimeout              1014caf4 f   wsc.obj
 0001:0014bb74       WscPINTimeout              1014cb74 f   wsc.obj
 0001:0014bbe4       WscEAPRxTimeout            1014cbe4 f   wsc.obj
 0001:0014bdfc       WscM8WaitEapFailTimeout    1014cdfc f   wsc.obj
 0001:0014bea4       WscEapM2Timeout            1014cea4 f   wsc.obj
 0001:0014bf50       WscLEDTimer                1014cf50 f   wsc.obj
 0001:0014c238       WscSkipTurnOffLEDTimer     1014d238 f   wsc.obj
 0001:0014c29c       WscPushPBCAction           1014d29c f   wsc.obj
 0001:0014c4d4       WscScanExec                1014d4d4 f   wsc.obj
 0001:0014c638       WscPBCExec                 1014d638 f   wsc.obj
 0001:0014c918       WscPINExec                 1014d918 f   wsc.obj
 0001:0014c934       WscPBCBssTableSort         1014d934 f   wsc.obj
 0001:0014d874       WscPBCModeAPSearch         1014e874 f   wsc.obj
 0001:0014e4bc       WscPINModeAPSearch         1014f4bc f   wsc.obj
 0001:0014f0d4       WscCheckWPSAP              101500d4 f   wsc.obj
 0001:0014f8c4       WscMacHeaderInit           101508c4 f   wsc.obj
 0001:0014fb38       WscStartAction             10150b38 f   wsc.obj
 0001:0014fe94       WscInitRegistrarPair       10150e94 f   wsc.obj
 0001:001507cc       MakeWSCEAPFrame            101517cc f   wsc.obj
 0001:00150b9c       WscSendEapRspId            10151b9c f   wsc.obj
 0001:00150eec       WscSendMessageM1           10151eec f   wsc.obj
 0001:001518b4       WscSendMessageM2           101528b4 f   wsc.obj
 0001:00152594       WscSendMessageM3           10153594 f   wsc.obj
 0001:00152c5c       WscSendMessageM4           10153c5c f   wsc.obj
 0001:00153688       WscSendMessageM5           10154688 f   wsc.obj
 0001:00153e8c       WscSendMessageM6           10154e8c f   wsc.obj
 0001:001546ac       WscSendMessageM7           101556ac f   wsc.obj
 0001:00154eb0       WscSendMessageM8           10155eb0 f   wsc.obj
 0001:00155c80       WscSendEapRspAck           10156c80 f   wsc.obj
 0001:00155f14       WscSendEapRspNack          10156f14 f   wsc.obj
 0001:001561d4       WscSendEapRspDone          101571d4 f   wsc.obj
 0001:00156400       WscRecvMessageM1           10157400 f   wsc.obj
 0001:00156c60       WscRecvMessageM2           10157c60 f   wsc.obj
 0001:0015786c       WscRecvMessageM2D          1015886c f   wsc.obj
 0001:00157cf4       WscRecvMessageM3           10158cf4 f   wsc.obj
 0001:00158428       WscRecvMessageM4           10159428 f   wsc.obj
 0001:00158de8       WscRecvMessageM5           10159de8 f   wsc.obj
 0001:0015974c       WscRecvMessageM6           1015a74c f   wsc.obj
 0001:0015a0b4       WscRecvMessageM7           1015b0b4 f   wsc.obj
 0001:0015aa2c       WscRecvMessageM8           1015ba2c f   wsc.obj
 0001:0015b25c       WscReceiveEapFail          1015c25c f   wsc.obj
 0001:0015b2ac       WscReceiveEapNack          1015c2ac f   wsc.obj
 0001:0015b83c       WscReceiveEapDone          1015c83c f   wsc.obj
 0001:0015bbd8       WscParseEncrSettings       1015cbd8 f   wsc.obj
 0001:0015c43c       WscProcessCredential       1015d43c f   wsc.obj
 0001:0015cb4c       WscMakeProbeReqIE          1015db4c f   wsc.obj
 0001:0015d0a4       WscStop                    1015e0a4 f   wsc.obj
 0001:0015d204       WscAutoGenProfile          1015e204 f   wsc.obj
 0001:0015d4f8       WscSupportWPSLEDMode       1015e4f8 f   wsc.obj
 0001:0015d62c       WscSupportWPSLEDMode10     1015e62c f   wsc.obj
 0001:0015d700       WscAPHasSecuritySetting    1015e700 f   wsc.obj
 0001:0015d838       sha256_compile             1015e838 f   wsc_crypto.obj
 0001:0015fd68       sha256_hash                10160d68 f   wsc_crypto.obj
 0001:0015ff58       sha256_begin               10160f58 f   wsc_crypto.obj
 0001:0015ffa0       sha256_end                 10160fa0 f   wsc_crypto.obj
 0001:001602e8       sha256                     101612e8 f   wsc_crypto.obj
 0001:0016032c       sha2_begin                 1016132c f   wsc_crypto.obj
 0001:001603c8       sha2_hash                  101613c8 f   wsc_crypto.obj
 0001:00160404       sha2_end                   10161404 f   wsc_crypto.obj
 0001:00160440       sha2                       10161440 f   wsc_crypto.obj
 0001:001604b0       hmac_sha_begin             101614b0 f   wsc_crypto.obj
 0001:001604d4       hmac_sha_key               101614d4 f   wsc_crypto.obj
 0001:001605cc       hmac_sha_data              101615cc f   wsc_crypto.obj
 0001:00160718       hmac_sha_end               10161718 f   wsc_crypto.obj
 0001:0016087c       hmac_sha                   1016187c f   wsc_crypto.obj
 0001:001608e8       KD_hmac_sha256             101618e8 f   wsc_crypto.obj
 0001:001609e4       AES_encrypt                101619e4 f   wsc_crypto.obj
 0001:0016147c       AES_decrypt                1016247c f   wsc_crypto.obj
 0001:00161f14       AES_set_encrypt_key        10162f14 f   wsc_crypto.obj
 0001:00162964       AES_cbc_encrypt            10163964 f   wsc_crypto.obj
 0001:00162e60       AES_set_decrypt_key        10163e60 f   wsc_crypto.obj
 0001:00163564       EVP_aes_128_cbc            10164564 f   wsc_crypto.obj
 0001:0016357c       EVP_EncryptInit            1016457c f   wsc_crypto.obj
 0001:00163628       EVP_EncryptUpdate          10164628 f   wsc_crypto.obj
 0001:0016379c       EVP_EncryptFinal           1016479c f   wsc_crypto.obj
 0001:00163858       EVP_DecryptInit            10164858 f   wsc_crypto.obj
 0001:00163904       EVP_DecryptUpdate          10164904 f   wsc_crypto.obj
 0001:00163a54       EVP_DecryptFinal           10164a54 f   wsc_crypto.obj
 0001:00163b2c       WscEncryptData             10164b2c f   wsc_crypto.obj
 0001:00163d3c       WscDecryptData             10164d3c f   wsc_crypto.obj
 0001:00163f4c       WscDeriveKey               10164f4c f   wsc_crypto.obj
 0001:001641fc       GenerateDHPublicKey        101651fc f   wsc_crypto.obj
 0001:001642d4       GenerateDHSecreteKey       101652d4 f   wsc_crypto.obj
 0001:001643a8       NN_Decode                  101653a8 f   wsc_crypto.obj
 0001:001644d0       NN_Encode                  101654d0 f   wsc_crypto.obj
 0001:001645e0       NN_Assign                  101655e0 f   wsc_crypto.obj
 0001:00164658       NN_AssignZero              10165658 f   wsc_crypto.obj
 0001:001646bc       NN_Sub                     101656bc f   wsc_crypto.obj
 0001:001647fc       NN_Mult                    101657fc f   wsc_crypto.obj
 0001:0016494c       NN_LShift                  1016594c f   wsc_crypto.obj
 0001:00164a44       NN_RShift                  10165a44 f   wsc_crypto.obj
 0001:00164b3c       NN_Div                     10165b3c f   wsc_crypto.obj
 0001:00164e90       NN_Mod                     10165e90 f   wsc_crypto.obj
 0001:00164ee0       NN_ModMult                 10165ee0 f   wsc_crypto.obj
 0001:00164f44       NN_ModExp                  10165f44 f   wsc_crypto.obj
 0001:00165154       NN_Cmp                     10166154 f   wsc_crypto.obj
 0001:00165540       NN_Digits                  10166540 f   wsc_crypto.obj
 0001:00165628       NN_DigitMult               10166628 f   wsc_crypto.obj
 0001:001657a4       NN_DigitDiv                101667a4 f   wsc_crypto.obj
 0001:00165b20       InitMDSMCtrl               10166b20 f   tpc.obj
 0001:00165cf8       MDSMCalculateMaxTxPower    10166cf8 f   tpc.obj
 0001:00165e50       MDSMCreatePowerCapabilityIE 10166e50 f   tpc.obj
 0001:00165f14       MDSMCalaculateRealTxPower  10166f14 f   tpc.obj
 0001:00165ff0       TdlsStateMachineInit       10166ff0 f   tdls.obj
 0001:00166140       MlmeTdlsSetupReqAction     10167140 f   tdls.obj
 0001:00166c6c       PeerTdlsMsgAction          10167c6c f   tdls.obj
 0001:00166dbc       PeerTdlsSetupReqAction     10167dbc f   tdls.obj
 0001:00168564       PeerTdlsSetupRspAction     10169564 f   tdls.obj
 0001:0016b150       PeerTdlsSetupConfAction    1016c150 f   tdls.obj
 0001:0016cef8       MlmeTdlsTearDownAction     1016def8 f   tdls.obj
 0001:0016d534       PeerTdlsTearDownAction     1016e534 f   tdls.obj
 0001:0016dae4       RTMPCheckTDLSFrame         1016eae4 f   tdls.obj
 0001:0016dbe4       RTMPSendTDLSTearDownFrame  1016ebe4 f   tdls.obj
 0001:0016e184       TDLSSendPacket             1016f184 f   tdls.obj
 0001:0016e54c       TdlsTimeout                1016f54c f   tdls.obj
 0001:0016e700       TdlsTearDown               1016f700 f   tdls.obj
 0001:0016ecf0       TdlsDeleteMacTableEntry    1016fcf0 f   tdls.obj
 0001:0016ed48       TDLSSearchLinkId           1016fd48 f   tdls.obj
 0001:0016ef3c       TPKMsg1Process             1016ff3c f   tdls.obj
 0001:0016f250       TPKMsg2Process             10170250 f   tdls.obj
 0001:0016f7e8       TPKMsg3Process             101707e8 f   tdls.obj
 0001:0016fd70       TDLSDeriveTPK              10170d70 f   tdls.obj
 0001:00170214       TDLSTableInit              10171214 f   tdls.obj
 0001:001702e0       TDLSSearchTabInit          101712e0 f   tdls.obj
 0001:001705c4       TDLSSearchTabDestory       101715c4 f   tdls.obj
 0001:001706f0       TDLSSearchEntyAlloc        101716f0 f   tdls.obj
 0001:00170834       TDLSSearchEntyFree         10171834 f   tdls.obj
 0001:00170954       TLDSSearchEntryLookup      10171954 f   tdls.obj
 0001:00170a70       TDLSSearchEntryUpdate      10171a70 f   tdls.obj
 0001:00170dd0       TDLSSearchEntryDelete      10171dd0 f   tdls.obj
 0001:00171158       TDLSSearchTabMaintain      10172158 f   tdls.obj
 0001:00171510       TDLSLinkMaintenance        10172510 f   tdls.obj
 0001:00171784       TDLSDiscoveryPacketLearnAndCheck 10172784 f   tdls.obj
 0001:001719e4       EventModify                101729e4 f   Coredll:COREDLL.dll
 0001:001719f4       NKDbgPrintfW               101729f4 f   Coredll:COREDLL.dll
 0001:00171a04       ExitThread                 10172a04 f   Coredll:COREDLL.dll
 0001:00171a14       WaitForSingleObject        10172a14 f   Coredll:COREDLL.dll
 0001:00171a24       CeGetThreadPriority        10172a24 f   Coredll:COREDLL.dll
 0001:00171a34       CeSetThreadPriority        10172a34 f   Coredll:COREDLL.dll
 0001:00171a44       GetLastError               10172a44 f   Coredll:COREDLL.dll
 0001:00171a54       CreateThread               10172a54 f   Coredll:COREDLL.dll
 0001:00171a64       CreateEventW               10172a64 f   Coredll:COREDLL.dll
 0001:00171a74       InterlockedExchange        10172a74 f   Coredll:COREDLL.dll
 0001:00171a84       InterlockedDecrement       10172a84 f   Coredll:COREDLL.dll
 0001:00171a94       InterlockedIncrement       10172a94 f   Coredll:COREDLL.dll
 0001:00171aa4       Sleep                      10172aa4 f   Coredll:COREDLL.dll
 0001:00171ab4       SetLastError               10172ab4 f   Coredll:COREDLL.dll
 0001:00171ac4       DisableThreadLibraryCalls  10172ac4 f   Coredll:COREDLL.dll
 0001:00171ad4       RegisterDbgZones           10172ad4 f   Coredll:COREDLL.dll
 0001:00171ae4       TerminateThread            10172ae4 f   Coredll:COREDLL.dll
 0001:00171af4       GetExitCodeThread          10172af4 f   Coredll:COREDLL.dll
 0001:00171b04       RegCloseKey                10172b04 f   Coredll:COREDLL.dll
 0001:00171b14       RegQueryValueExW           10172b14 f   Coredll:COREDLL.dll
 0001:00171b24       RegOpenKeyExW              10172b24 f   Coredll:COREDLL.dll
 0001:00171b34       GetSystemInfo              10172b34 f   Coredll:COREDLL.dll
 0001:00171b44       StringCbPrintfA            10172b44 f   Coredll:COREDLL.dll
 0001:00171b54       DbgPrint                   10172b54 f   ndis:NDIS.dll
 0001:00171b64       NdisReleaseSpinLock        10172b64 f   ndis:NDIS.dll
 0001:00171b74       NdisAcquireSpinLock        10172b74 f   ndis:NDIS.dll
 0001:00171b84       NdisMSleep                 10172b84 f   ndis:NDIS.dll
 0001:00171b94       NdisGetSystemUpTime        10172b94 f   ndis:NDIS.dll
 0001:00171ba4       NdisStallExecution         10172ba4 f   ndis:NDIS.dll
 0001:00171bb4       NdisFreeMemory             10172bb4 f   ndis:NDIS.dll
 0001:00171bc4       NdisAllocateBuffer         10172bc4 f   ndis:NDIS.dll
 0001:00171bd4       NdisFreePacket             10172bd4 f   ndis:NDIS.dll
 0001:00171be4       NdisAllocateMemoryWithTag  10172be4 f   ndis:NDIS.dll
 0001:00171bf4       NdisAllocatePacket         10172bf4 f   ndis:NDIS.dll
 0001:00171c04       NdisAllocateSpinLock       10172c04 f   ndis:NDIS.dll
 0001:00171c14       NdisFreeSpinLock           10172c14 f   ndis:NDIS.dll
 0001:00171c24       NdisInterlockedDecrement   10172c24 f   ndis:NDIS.dll
 0001:00171c34       NdisGetCurrentSystemTime   10172c34 f   ndis:NDIS.dll
 0001:00171c44       NdisQueryPacket            10172c44 f   ndis:NDIS.dll
 0001:00171c54       NdisAllocateBufferPool     10172c54 f   ndis:NDIS.dll
 0001:00171c64       NdisAllocatePacketPool     10172c64 f   ndis:NDIS.dll
 0001:00171c74       NdisInitializeNPagedLookasideList 10172c74 f   ndis:NDIS.dll
 0001:00171c84       NdisDeleteNPagedLookasideList 10172c84 f   ndis:NDIS.dll
 0001:00171c94       NdisFreeBufferPool         10172c94 f   ndis:NDIS.dll
 0001:00171ca4       NdisFreePacketPool         10172ca4 f   ndis:NDIS.dll
 0001:00171cb4       NdisCloseConfiguration     10172cb4 f   ndis:NDIS.dll
 0001:00171cc4       NdisUnicodeStringToAnsiString 10172cc4 f   ndis:NDIS.dll
 0001:00171cd4       NdisReadConfiguration      10172cd4 f   ndis:NDIS.dll
 0001:00171ce4       NdisOpenConfiguration      10172ce4 f   ndis:NDIS.dll
 0001:00171cf4       NdisCloseFile              10172cf4 f   ndis:NDIS.dll
 0001:00171d04       NdisUnmapFile              10172d04 f   ndis:NDIS.dll
 0001:00171d14       NdisMapFile                10172d14 f   ndis:NDIS.dll
 0001:00171d24       NdisOpenFile               10172d24 f   ndis:NDIS.dll
 0001:00171d34       NdisInitializeString       10172d34 f   ndis:NDIS.dll
 0001:00171d44       NdisMInitializeTimer       10172d44 f   ndis:NDIS.dll
 0001:00171d54       NdisSetTimer               10172d54 f   ndis:NDIS.dll
 0001:00171d64       NdisMSetPeriodicTimer      10172d64 f   ndis:NDIS.dll
 0001:00171d74       NdisMCancelTimer           10172d74 f   ndis:NDIS.dll
 0001:00171d84       NdisTerminateWrapper       10172d84 f   ndis:NDIS.dll
 0001:00171d94       NdisMRegisterMiniport      10172d94 f   ndis:NDIS.dll
 0001:00171da4       NdisInitializeWrapper      10172da4 f   ndis:NDIS.dll
 0001:00171db4       NdisMGetDeviceProperty     10172db4 f   ndis:NDIS.dll
 0001:00171dc4       NdisMSetAttributesEx       10172dc4 f   ndis:NDIS.dll
 0001:00171dd4       NdisInterlockedIncrement   10172dd4 f   ndis:NDIS.dll
 0001:00171de4       NdisFreeBuffer             10172de4 f   ndis:NDIS.dll
 0001:00171df4       NdisUnchainBufferAtFront   10172df4 f   ndis:NDIS.dll
 0001:00171e04       NdisFreeToNPagedLookasideList 10172e04 f   ndis:NDIS.dll
 0001:00171e14       NdisAllocateFromNPagedLookasideList 10172e14 f   ndis:NDIS.dll
 0001:00171e24       NdisDeregisterAdapter      10172e24 f   ndis:NDIS.dll
 0001:00171e34       NdisRegisterAdapter        10172e34 f   ndis:NDIS.dll
 0001:00171e44       RegisterClientSettings     10172e44 f   usbd:USBD.dll
 0001:00171e54       RegisterClientDriverID     10172e54 f   usbd:USBD.dll
 0001:00171e64       UnRegisterClientDriverID   10172e64 f   usbd:USBD.dll
 0001:00171e74       UnRegisterClientSettings   10172e74 f   usbd:USBD.dll
 0001:00171e84       AbortTransfer              10172e84 f   usbclient:usbclient.obj
 0001:00171f28       CloseTransferHandle        10172f28 f   usbclient:usbclient.obj
 0001:00171fc8       ClearOrSetFeature          10172fc8 f   usbclient:usbclient.obj
 0001:00172284       DefaultTransferComplete    10173284 f   usbclient:usbclient.obj
 0001:00172370       GetStatus                  10173370 f   usbclient:usbclient.obj
 0001:001725e8       GetTransferStatus          101735e8 f   usbclient:usbclient.obj
 0001:00172734       IssueBulkTransfer          10173734 f   usbclient:usbclient.obj
 0001:00172ae4       IssueInterruptTransfer     10173ae4 f   usbclient:usbclient.obj
 0001:00172e8c       IssueVendorTransfer        10173e8c f   usbclient:usbclient.obj
 0001:0017322c       ResetDefaultEndpoint       1017422c f   usbclient:usbclient.obj
 0001:00173378       ResetBulkEndpoint          10174378 f   usbclient:usbclient.obj
 0001:00173478       ResetPipe                  10174478 f   usbclient:usbclient.obj
 0001:00173550       _ResetEvent                10174550 f i usbclient:usbclient.obj
 0001:001735ec       ResetEvent                 101745ec f i usbclient:usbclient.obj
 0001:00173624       __security_init_cookie     10174624 f   corelib0:seccinit.obj
 0001:001736ec       __GSHandlerCheck           101746ec f   corelib0:gshandler.obj
 0001:00173734       __GSHandlerCheckCommon     10174734 f   corelib0:gshandler.obj
 0001:001737dc       __security_check_cookie    101747dc f   corelib0:armsecgs.obj
 0001:001737f0       __gsfailure                101747f0 f   corelib0:armsecgs.obj
 0001:00173834       memcpy                     10174834 f   corelib1:COREDLL.dll
 0001:00173844       memset                     10174844 f   corelib1:COREDLL.dll
 0001:00173854       __rt_sdiv                  10174854 f   corelib1:COREDLL.dll
 0001:00173864       __rt_udiv                  10174864 f   corelib1:COREDLL.dll
 0001:00173874       strlen                     10174874 f   corelib1:COREDLL.dll
 0001:00173884       strcpy                     10174884 f   corelib1:COREDLL.dll
 0001:00173894       memmove                    10174894 f   corelib1:COREDLL.dll
 0001:001738a4       __rt_udiv64by64            101748a4 f   corelib1:COREDLL.dll
 0001:001738b4       sprintf                    101748b4 f   corelib1:COREDLL.dll
 0001:001738c4       __security_gen_cookie2     101748c4 f   corelib1:COREDLL.dll
 0001:001738d4       __report_gsfailure         101748d4 f   corelib1:COREDLL.dll
 0001:00173ca8       __IMPORT_DESCRIPTOR_COREDLL 10174ca8     Coredll:COREDLL.dll
 0001:00173cbc       __IMPORT_DESCRIPTOR_NDIS   10174cbc     ndis:NDIS.dll
 0001:00173cd0       __IMPORT_DESCRIPTOR_USBD   10174cd0     usbd:USBD.dll
 0001:00173ce4       __NULL_IMPORT_DESCRIPTOR   10174ce4     Coredll:COREDLL.dll
 0002:00000000       __imp_EventModify          10176000     Coredll:COREDLL.dll
 0002:00000004       __imp_NKDbgPrintfW         10176004     Coredll:COREDLL.dll
 0002:00000008       __imp_ExitThread           10176008     Coredll:COREDLL.dll
 0002:0000000c       __imp_WaitForSingleObject  1017600c     Coredll:COREDLL.dll
 0002:00000010       __imp_CeGetThreadPriority  10176010     Coredll:COREDLL.dll
 0002:00000014       __imp_CeSetThreadPriority  10176014     Coredll:COREDLL.dll
 0002:00000018       __imp_GetLastError         10176018     Coredll:COREDLL.dll
 0002:0000001c       __imp_CreateThread         1017601c     Coredll:COREDLL.dll
 0002:00000020       __imp_CreateEventW         10176020     Coredll:COREDLL.dll
 0002:00000024       __imp_InterlockedExchange  10176024     Coredll:COREDLL.dll
 0002:00000028       __imp_InterlockedDecrement 10176028     Coredll:COREDLL.dll
 0002:0000002c       __imp_InterlockedIncrement 1017602c     Coredll:COREDLL.dll
 0002:00000030       __imp_Sleep                10176030     Coredll:COREDLL.dll
 0002:00000034       __imp_SetLastError         10176034     Coredll:COREDLL.dll
 0002:00000038       __imp_DisableThreadLibraryCalls 10176038     Coredll:COREDLL.dll
 0002:0000003c       __imp_RegisterDbgZones     1017603c     Coredll:COREDLL.dll
 0002:00000040       __imp_TerminateThread      10176040     Coredll:COREDLL.dll
 0002:00000044       __imp_GetExitCodeThread    10176044     Coredll:COREDLL.dll
 0002:00000048       __imp_RegCloseKey          10176048     Coredll:COREDLL.dll
 0002:0000004c       __imp_RegQueryValueExW     1017604c     Coredll:COREDLL.dll
 0002:00000050       __imp_RegOpenKeyExW        10176050     Coredll:COREDLL.dll
 0002:00000054       __imp_GetSystemInfo        10176054     Coredll:COREDLL.dll
 0002:00000058       __imp_StringCbPrintfA      10176058     Coredll:COREDLL.dll
 0002:0000005c       __imp___security_gen_cookie2 1017605c     corelib1:COREDLL.dll
 0002:00000060       __imp_sprintf              10176060     corelib1:COREDLL.dll
 0002:00000064       __imp___rt_udiv64by64      10176064     corelib1:COREDLL.dll
 0002:00000068       __imp_memmove              10176068     corelib1:COREDLL.dll
 0002:0000006c       __imp_strcpy               1017606c     corelib1:COREDLL.dll
 0002:00000070       __imp_strlen               10176070     corelib1:COREDLL.dll
 0002:00000074       __imp___rt_udiv            10176074     corelib1:COREDLL.dll
 0002:00000078       __imp___rt_sdiv            10176078     corelib1:COREDLL.dll
 0002:0000007c       __imp_memset               1017607c     corelib1:COREDLL.dll
 0002:00000080       __imp_memcpy               10176080     corelib1:COREDLL.dll
 0002:00000084       __imp___report_gsfailure   10176084     corelib1:COREDLL.dll
 0002:00000088       \177COREDLL_NULL_THUNK_DATA 10176088     Coredll:COREDLL.dll
 0002:0000008c       __imp_NdisAllocateSpinLock 1017608c     ndis:NDIS.dll
 0002:00000090       __imp_NdisFreeSpinLock     10176090     ndis:NDIS.dll
 0002:00000094       __imp_NdisInterlockedDecrement 10176094     ndis:NDIS.dll
 0002:00000098       __imp_NdisGetCurrentSystemTime 10176098     ndis:NDIS.dll
 0002:0000009c       __imp_NdisQueryPacket      1017609c     ndis:NDIS.dll
 0002:000000a0       __imp_NdisAllocateBufferPool 101760a0     ndis:NDIS.dll
 0002:000000a4       __imp_NdisAllocatePacketPool 101760a4     ndis:NDIS.dll
 0002:000000a8       __imp_NdisInitializeNPagedLookasideList 101760a8     ndis:NDIS.dll
 0002:000000ac       __imp_NdisDeleteNPagedLookasideList 101760ac     ndis:NDIS.dll
 0002:000000b0       __imp_NdisAllocatePacket   101760b0     ndis:NDIS.dll
 0002:000000b4       __imp_NdisFreePacketPool   101760b4     ndis:NDIS.dll
 0002:000000b8       __imp_NdisCloseConfiguration 101760b8     ndis:NDIS.dll
 0002:000000bc       __imp_NdisUnicodeStringToAnsiString 101760bc     ndis:NDIS.dll
 0002:000000c0       __imp_NdisReadConfiguration 101760c0     ndis:NDIS.dll
 0002:000000c4       __imp_NdisOpenConfiguration 101760c4     ndis:NDIS.dll
 0002:000000c8       __imp_NdisCloseFile        101760c8     ndis:NDIS.dll
 0002:000000cc       __imp_NdisUnmapFile        101760cc     ndis:NDIS.dll
 0002:000000d0       __imp_NdisMapFile          101760d0     ndis:NDIS.dll
 0002:000000d4       __imp_NdisOpenFile         101760d4     ndis:NDIS.dll
 0002:000000d8       __imp_NdisInitializeString 101760d8     ndis:NDIS.dll
 0002:000000dc       __imp_NdisMInitializeTimer 101760dc     ndis:NDIS.dll
 0002:000000e0       __imp_NdisSetTimer         101760e0     ndis:NDIS.dll
 0002:000000e4       __imp_NdisMSetPeriodicTimer 101760e4     ndis:NDIS.dll
 0002:000000e8       __imp_NdisMCancelTimer     101760e8     ndis:NDIS.dll
 0002:000000ec       __imp_NdisTerminateWrapper 101760ec     ndis:NDIS.dll
 0002:000000f0       __imp_NdisMRegisterMiniport 101760f0     ndis:NDIS.dll
 0002:000000f4       __imp_NdisInitializeWrapper 101760f4     ndis:NDIS.dll
 0002:000000f8       __imp_NdisMGetDeviceProperty 101760f8     ndis:NDIS.dll
 0002:000000fc       __imp_NdisMSetAttributesEx 101760fc     ndis:NDIS.dll
 0002:00000100       __imp_NdisInterlockedIncrement 10176100     ndis:NDIS.dll
 0002:00000104       __imp_NdisFreeBuffer       10176104     ndis:NDIS.dll
 0002:00000108       __imp_NdisUnchainBufferAtFront 10176108     ndis:NDIS.dll
 0002:0000010c       __imp_NdisFreeToNPagedLookasideList 1017610c     ndis:NDIS.dll
 0002:00000110       __imp_NdisAllocateFromNPagedLookasideList 10176110     ndis:NDIS.dll
 0002:00000114       __imp_NdisDeregisterAdapter 10176114     ndis:NDIS.dll
 0002:00000118       __imp_NdisRegisterAdapter  10176118     ndis:NDIS.dll
 0002:0000011c       __imp_DbgPrint             1017611c     ndis:NDIS.dll
 0002:00000120       __imp_NdisReleaseSpinLock  10176120     ndis:NDIS.dll
 0002:00000124       __imp_NdisAcquireSpinLock  10176124     ndis:NDIS.dll
 0002:00000128       __imp_NdisMSleep           10176128     ndis:NDIS.dll
 0002:0000012c       __imp_NdisGetSystemUpTime  1017612c     ndis:NDIS.dll
 0002:00000130       __imp_NdisAllocateMemoryWithTag 10176130     ndis:NDIS.dll
 0002:00000134       __imp_NdisFreePacket       10176134     ndis:NDIS.dll
 0002:00000138       __imp_NdisAllocateBuffer   10176138     ndis:NDIS.dll
 0002:0000013c       __imp_NdisFreeMemory       1017613c     ndis:NDIS.dll
 0002:00000140       __imp_NdisStallExecution   10176140     ndis:NDIS.dll
 0002:00000144       __imp_NdisFreeBufferPool   10176144     ndis:NDIS.dll
 0002:00000148       \177NDIS_NULL_THUNK_DATA   10176148     ndis:NDIS.dll
 0002:0000014c       __imp_UnRegisterClientDriverID 1017614c     usbd:USBD.dll
 0002:00000150       __imp_RegisterClientDriverID 10176150     usbd:USBD.dll
 0002:00000154       __imp_RegisterClientSettings 10176154     usbd:USBD.dll
 0002:00000158       __imp_UnRegisterClientSettings 10176158     usbd:USBD.dll
 0002:0000015c       \177USBD_NULL_THUNK_DATA   1017615c     usbd:USBD.dll
 0002:0000048c       CISCO_OUI                  1017648c     aironet.obj
 0002:0000059c       pEventText                 1017659c     ap.obj
 0002:00000c14       CipherSuiteWPAPSKTKIPLen   10176c14     ap_info.obj
 0002:00000c18       APSupportedOids            10176c18     ap_info.obj
 0002:00000e00       CipherSuiteWPAPSKTKIP      10176e00     ap_info.obj
 0002:00001254       CipherSuiteWAPIPsk         10177254     Ap_wapi.obj
 0002:0000126a       CipherSuiteWAPIPskLen      1017726a     Ap_wapi.obj
 0002:0000126b       CipherSuiteWAPICertLen     1017726b     Ap_wapi.obj
 0002:0000126c       CipherSuiteWAPICert        1017726c     Ap_wapi.obj
 0002:00001284       WAPI_PROTOTYPE             10177284     Ap_wapi.obj
 0002:00001288       WAPI_INIT_PN               10177288     Ap_wapi.obj
 0002:0000141c       OUI_WPA_WEP40              1017741c     ap_wpa.obj
 0002:00001420       OUI_WPA_TKIP               10177420     ap_wpa.obj
 0002:00001424       OUI_WPA_CCMP               10177424     ap_wpa.obj
 0002:00001428       OUI_WPA2_WEP40             10177428     ap_wpa.obj
 0002:0000142c       OUI_WPA2_TKIP              1017742c     ap_wpa.obj
 0002:00001430       OUI_WPA2_CCMP              10177430     ap_wpa.obj
 0002:00001544       CipherWpaTemplate          10177544     assoc.obj
 0002:0000155c       CipherWpaTemplateLen       1017755c     assoc.obj
 0002:0000155d       CipherWpa2TemplateLen      1017755d     assoc.obj
 0002:00001560       CipherWpa2Template         10177560     assoc.obj
 0002:00001578       CcxVerIE                   10177578     assoc.obj
 0002:000018ac       CipherSuiteWpaNoneTkip     101778ac     connect.obj
 0002:000018c2       CipherSuiteWpaNoneTkipLen  101778c2     connect.obj
 0002:000018c3       CipherSuiteWpaNoneAesLen   101778c3     connect.obj
 0002:000018c4       CipherSuiteWpaNoneAes      101778c4     connect.obj
 0002:00001afc       SNAP_LEAP_ROGUEAP_HDR      10177afc     leap.obj
 0002:00001c18       PADDING                    10177c18     md4.obj
 0002:0000469c       RateSwitchTable11B         1017a69c     mlme.obj
 0002:000046b5       SupRateIe                  1017a6b5     mlme.obj
 0002:000046b6       ExtRateIe                  1017a6b6     mlme.obj
 0002:000046b7       HtCapIe                    1017a6b7     mlme.obj
 0002:000046b8       RateSwitchTable            1017a6b8     mlme.obj
 0002:0000475d       AddHtInfoIe                1017a75d     mlme.obj
 0002:0000475e       NewExtChanIe               1017a75e     mlme.obj
 0002:0000475f       ExtHtCapIe                 1017a75f     mlme.obj
 0002:00004760       RateSwitchTable11BG        1017a760     mlme.obj
 0002:00004797       ErpIe                      1017a797     mlme.obj
 0002:00004798       RateSwitchTable11G         1017a798     mlme.obj
 0002:000047c5       DsIe                       1017a7c5     mlme.obj
 0002:000047c6       TimIe                      1017a7c6     mlme.obj
 0002:000047c7       WpaIe                      1017a7c7     mlme.obj
 0002:000047c8       RateSwitchTable11N1S       1017a7c8     mlme.obj
 0002:00004809       Wpa2Ie                     1017a809     mlme.obj
 0002:0000480a       IbssIe                     1017a80a     mlme.obj
 0002:0000480b       CcxIe                      1017a80b     mlme.obj
 0002:0000480c       RateSwitchTable11N2SForABand 1017a80c     mlme.obj
 0002:00004848       RateSwitchTable11N2S       1017a848     mlme.obj
 0002:00004893       BssIntRepIe                1017a893     mlme.obj
 0002:00004894       RateSwitchTable11BGN2SForABand 1017a894     mlme.obj
 0002:000048d0       RateSwitchTable11BGN1S     1017a8d0     mlme.obj
 0002:00004911       BssCoexistIe               1017a911     mlme.obj
 0002:00004918       RateSwitchTable11BGN2S     1017a918     mlme.obj
 0002:00004968       ReasonString               1017a968     mlme.obj
 0002:000049b0       BasicRateMask              1017a9b0     mlme.obj
 0002:000049e0       MULTICAST_ADDR             1017a9e0     mlme.obj
 0002:000049e8       BROADCAST_ADDR             1017a9e8     mlme.obj
 0002:000049f0       RssiSafeLevelForTxRate     1017a9f0     mlme.obj
 0002:00004a00       Phy11BNextRateDownward     1017aa00     mlme.obj
 0002:00004a04       Phy11BNextRateUpward       1017aa04     mlme.obj
 0002:00004a08       Phy11BGNextRateDownward    1017aa08     mlme.obj
 0002:00004a14       Phy11BGNextRateUpward      1017aa14     mlme.obj
 0002:00004a20       Phy11ANextRateDownward     1017aa20     mlme.obj
 0002:00004a2c       Phy11ANextRateUpward       1017aa2c     mlme.obj
 0002:00004a38       RateUpPER                  1017aa38     mlme.obj
 0002:00004a50       RateDownPER                1017aa50     mlme.obj
 0002:00004a68       RateIdToMbps               1017aa68     mlme.obj
 0002:00004a78       RateIdTo500Kbps            1017aa78     mlme.obj
 0002:00004a94       SES_OUI                    1017aa94     mlme.obj
 0002:00004a98       RateOFDMToCCK              1017aa98     mlme.obj
 0002:00004aa0       RF2850RegTable             1017aaa0     mlme.obj
 0002:00004f50       FreqItems3020              1017af50     mlme.obj
 0002:00004f88       FreqItems3572              1017af88     mlme.obj
 0002:0000505c       AntStr                     1017b05c     mlme.obj
 0002:0000506c       NIC_VENDOR_DESC            1017b06c     oem.obj
 0002:00005088       NIC_VENDOR_DESC_LEN        1017b088     oem.obj
 0002:0000508c       NIC_WPS_DESC               1017b08c     oem.obj
 0002:0000509c       NIC_WPS_DESC_LEN           1017b09c     oem.obj
 0002:000050a0       NIC_VENDOR_DRIVER_VERSION  1017b0a0     oem.obj
 0002:000050a4       LINKNAME_STRING            1017b0a4     oem.obj
 0002:000050cc       NTDEVICE_STRING            1017b0cc     oem.obj
 0002:00005420       Wpa2AuthEncryptPairs       1017b420     rtmp_info.obj
 0002:00005490       ralinkrate                 1017b490     rtmp_info.obj
 0002:00005690       STASupportedOids           1017b690     rtmp_info.obj
 0002:00005aec       BIT8                       1017baec     rtmp_init.obj
 0002:00005af8       BIT32                      1017baf8     rtmp_init.obj
 0002:00005b78       CipherName                 1017bb78     rtmp_init.obj
 0002:00005b98       NICRegTable                1017bb98     rtmp_init.obj
 0002:00006768       BBPRegTable                1017c768     rtmp_init.obj
 0002:00006788       RFRegTable                 1017c788     rtmp_init.obj
 0002:000067b0       RF3572RegTable             1017c7b0     rtmp_init.obj
 0002:000067f0       RF3320RegTable             1017c7f0     rtmp_init.obj
 0002:00006830       TxPowerTuningTable         1017c830     rtmp_init.obj
 0002:000068c8       MACRegTable                1017c8c8     rtmp_init.obj
 0002:000069b8       FirmwareImage              1017c9b8     rtmp_init.obj
 0002:000074e8       FirmwareV2Image            1017d4e8     rtmp_init.obj
 0002:00008124       RTDebugLevel               1017e124     rtmp_main.obj
 0002:00008238       Tkip_Sbox_Lower            1017e238     rtmp_tkip.obj
 0002:00008638       Tkip_Sbox_Upper            1017e638     rtmp_tkip.obj
 0002:00009164       EpToQueue                  1017f164     rtusb_bulk.obj
 0002:0000916c       AMSDUPadShift              1017f16c     rtusb_bulk.obj
 0002:0000928c       SNAP_802_1H                1017f28c     rtusb_data.obj
 0002:00009294       SNAP_BRIDGE_TUNNEL         1017f294     rtusb_data.obj
 0002:0000929c       SNAP_AIRONET               1017f29c     rtusb_data.obj
 0002:000092a4       CKIP_LLC_SNAP              1017f2a4     rtusb_data.obj
 0002:000092ac       AIRONET_PROTOCOL           1017f2ac     rtusb_data.obj
 0002:000092b0       EAPOL_LLC_SNAP             1017f2b0     rtusb_data.obj
 0002:000092b8       WAI_LLC_SNAP               1017f2b8     rtusb_data.obj
 0002:000092c0       EAPOL                      1017f2c0     rtusb_data.obj
 0002:000092c4       IPX                        1017f2c4     rtusb_data.obj
 0002:000092c8       APPLE_TALK                 1017f2c8     rtusb_data.obj
 0002:000092cc       RateIdToPlcpSignal         1017f2cc     rtusb_data.obj
 0002:000092d8       OfdmSignalToRateId         1017f2d8     rtusb_data.obj
 0002:000092e8       OfdmRateToRxwiMCS          1017f2e8     rtusb_data.obj
 0002:000092f4       RxwiMCSToOfdmRate          1017f2f4     rtusb_data.obj
 0002:00009300       MCSToMbps                  1017f300     rtusb_data.obj
 0002:00009320       default_cwmin              1017f320     rtusb_data.obj
 0002:00009324       default_cwmax              1017f324     rtusb_data.obj
 0002:00009328       default_sta_aifsn          1017f328     rtusb_data.obj
 0002:0000932c       MapUserPriorityToAccessCategory 1017f32c     rtusb_data.obj
 0002:00009554       WPA_OUI                    1017f554     sanity.obj
 0002:00009558       RSN_OUI                    1017f558     sanity.obj
 0002:0000955c       WPS_OUI                    1017f55c     sanity.obj
 0002:00009560       WME_INFO_ELEM              1017f560     sanity.obj
 0002:00009568       WME_PARM_ELEM              1017f568     sanity.obj
 0002:00009570       RALINK_OUI                 1017f570     sanity.obj
 0002:00009574       PRE_N_HT_OUI               1017f574     sanity.obj
 0002:00009578       SSIDL_OUI                  1017f578     sanity.obj
 0002:0000968c       WAIHEAD                    1017f68c     Sta_wapi.obj
 0002:00009694       WAPI_INIT_SEQ              1017f694     Sta_wapi.obj
 0002:000097a4       A_BAND_REGION_0_CHANNEL_LIST 1017f7a4     sync.obj
 0002:000097b4       A_BAND_REGION_1_CHANNEL_LIST 1017f7b4     sync.obj
 0002:000097c8       A_BAND_REGION_2_CHANNEL_LIST 1017f7c8     sync.obj
 0002:000097d0       A_BAND_REGION_3_CHANNEL_LIST 1017f7d0     sync.obj
 0002:000097d8       A_BAND_REGION_4_CHANNEL_LIST 1017f7d8     sync.obj
 0002:000097e0       A_BAND_REGION_5_CHANNEL_LIST 1017f7e0     sync.obj
 0002:000097e4       A_BAND_REGION_6_CHANNEL_LIST 1017f7e4     sync.obj
 0002:000097e8       A_BAND_REGION_7_CHANNEL_LIST 1017f7e8     sync.obj
 0002:00009800       A_BAND_REGION_8_CHANNEL_LIST 1017f800     sync.obj
 0002:00009804       A_BAND_REGION_9_CHANNEL_LIST 1017f804     sync.obj
 0002:0000981c       A_BAND_REGION_10_CHANNEL_LIST 1017f81c     sync.obj
 0002:00009828       A_BAND_REGION_11_CHANNEL_LIST 1017f828     sync.obj
 0002:0000983c       A_BAND_REGION_12_CHANNEL_LIST 1017f83c     sync.obj
 0002:00009850       A_BAND_REGION_13_CHANNEL_LIST 1017f850     sync.obj
 0002:00009864       A_BAND_REGION_14_CHANNEL_LIST 1017f864     sync.obj
 0002:00009878       A_BAND_REGION_15_CHANNEL_LIST 1017f878     sync.obj
 0002:00009880       A_BAND_REGION_16_CHANNEL_LIST 1017f880     sync.obj
 0002:0000989c       BaSizeArray                1017f89c     sync.obj
 0002:000099b0       SupportedDev               1017f9b0     wince.obj
 0002:00009c50       dpCurSettings              1017fc50     wince.obj
 0002:0000a1a4       CipherWpaPskTkip           101801a4     wpa.obj
 0002:0000a1bc       CipherWpaPskTkipLen        101801bc     wpa.obj
 0002:0000a1bd       CipherWpaPskAesLen         101801bd     wpa.obj
 0002:0000a1be       CipherSuiteCiscoCCKMLen    101801be     wpa.obj
 0002:0000a1bf       CipherSuiteCiscoCCKMWPALen 101801bf     wpa.obj
 0002:0000a1c0       CipherWpaPskAes            101801c0     wpa.obj
 0002:0000a1d8       CipherSuiteCiscoCCKMCKIP   101801d8     wpa.obj
 0002:0000a1f0       CipherSuiteCiscoCCKMCkipCmic 101801f0     wpa.obj
 0002:0000a208       CipherSuiteCiscoCCKMCmic   10180208     wpa.obj
 0002:0000a220       CipherSuiteCiscoCCKMWep40  10180220     wpa.obj
 0002:0000a238       CipherSuiteCiscoCCKMWep104 10180238     wpa.obj
 0002:0000a250       CipherSuiteCiscoCCKMTkip   10180250     wpa.obj
 0002:0000a268       CipherSuiteCiscoCCKMAES    10180268     wpa.obj
 0002:0000a280       CipherSuiteCiscoCCKMTkip24 10180280     wpa.obj
 0002:0000a29a       CipherSuiteCiscoCCKMTkip24Len 1018029a     wpa.obj
 0002:0000a29b       CipherSuiteCCXTkipLen      1018029b     wpa.obj
 0002:0000a29c       CipherSuiteCCXTkip         1018029c     wpa.obj
 0002:0000a2b4       CipherSuiteCiscoCCKMWPA2Tkip 101802b4     wpa.obj
 0002:0000a2ca       CipherSuiteCiscoCCKMWPA2Len 101802ca     wpa.obj
 0002:0000a2cc       CipherSuiteCiscoCCKMWPA2AES 101802cc     wpa.obj
 0002:0000a3f4       Wsc_Uuid                   101803f4     wsc.obj
 0002:0000a404       Wsc_Manufacture            10180404     wsc.obj
 0002:0000a420       Wsc_Model_Name             10180420     wsc.obj
 0002:0000a438       Wsc_Model_Number           10180438     wsc.obj
 0002:0000a440       Wsc_Model_Serial           10180440     wsc.obj
 0002:0000a44c       Wsc_Pri_Dev_Type           1018044c     wsc.obj
 0002:0000a454       Wsc_Dev_Name_R             10180454     wsc.obj
 0002:0000a468       Wsc_Personal_String        10180468     wsc.obj
 0002:0000a490       EnrolleeMsg                10180490     wsc.obj
 0002:0000a4b0       RegistrarMsg               101804b0     wsc.obj
 0002:0000a4d0       THOME_303V_MODEL_NAME      101804d0     wsc.obj
 0002:0000a4dc       THOME_303V_MODEL_NUMBER_000 101804dc     wsc.obj
 0002:0000a4e8       THOME_303V_MODEL_NUMBER_001 101804e8     wsc.obj
 0002:0000a7d4       dot11dhCountry             101807d4     tpc.obj
 0002:0000a7d5       dot11dhHoppingPatternParameters 101807d5     tpc.obj
 0002:0000a7d6       dot11dhHoppingPatternTable 101807d6     tpc.obj
 0002:0000a7d7       dot11dhRequest             101807d7     tpc.obj
 0002:0000a7d8       dot11dhPowerConstraint     101807d8     tpc.obj
 0002:0000a7d9       dot11dhPowerCapability     101807d9     tpc.obj
 0002:0000a7da       dot11dhTPCRequest          101807da     tpc.obj
 0002:0000a7db       dot11dhTPCReport           101807db     tpc.obj
 0002:0000a7dc       dot11dhSupportedChannel    101807dc     tpc.obj
 0002:0000a7dd       dot11dhChannelSwitchAnnouncement 101807dd     tpc.obj
 0002:0000a7de       dot11dhMeasurementRequest  101807de     tpc.obj
 0002:0000a7df       dot11dhMeasurementReport   101807df     tpc.obj
 0002:0000a7e0       dot11dhQuiet               101807e0     tpc.obj
 0002:0000a7e1       dot11dhIbssDFS             101807e1     tpc.obj
 0002:0000a8f4       TDLS_LLC_SNAP              101808f4     tdls.obj
 0002:0000a8fc       TDLS_LLC_SNAP_WITH_CATEGORY 101808fc     tdls.obj
 0002:0000a906       LinkIdIe                   10180906     tdls.obj
 0002:0000a907       QosCapIe                   10180907     tdls.obj
 0002:0000a908       TDLS_ETHERTYPE             10180908     tdls.obj
 0002:0000a90a       FastTransIe                1018090a     tdls.obj
 0002:0000a90b       TimeoutIntIe               1018090b     tdls.obj
 0002:0000a90c       CipherSuiteTDLSWpa2PskTkip 1018090c     tdls.obj
 0002:0000a922       CipherSuiteTDLSLen         10180922     tdls.obj
 0002:0000a924       CipherSuiteTDLSWpa2PskAes  10180924     tdls.obj
 0002:0000a93c       __security_cookie          1018093c     corelib0:seccinit.obj
 0002:0000a940       __security_cookie_complement 10180940     corelib0:seccinit.obj
 0002:0000b968       desiredTSSIOverCCK         10181968     mlme.obj
 0002:0000b96c       desiredTSSIOverOFDM        1018196c     mlme.obj
 0002:0000b974       desiredTSSIOverHT          10181974     mlme.obj
 0002:0000b97c       desiredTSSIOverHTUsingSTBC 1018197c     mlme.obj
 0002:0000b984       ZERO_MAC_ADDR              10181984     mlme.obj
 0002:0000b98a       SsidIe                     1018198a     mlme.obj
 0002:0000b98c       ZeroSsid                   1018198c     mlme.obj
 0002:0000b9e0       PlainText                  101819e0     <common>
 0002:0000bfc0       CipherText                 10181fc0     <common>
 0002:0000c5a0       HmacData                   101825a0     <common>
 0002:0000d5a0       OutMsgBuf                  101835a0     <common>
 0002:0000e158       GUsbFuncs                  10184158     <common>
 0002:0000e15c       GhDevice                   1018415c     <common>
 0002:0000e160       GUsbInterface              10184160     <common>
 0002:0000e180       LocalStrings               10184180     <common>
 0002:0000e840       PPURB_BULK_OR_INTERRUPT_TRANSFER 10184840     <common>
 0002:0000e844       PURB_BULK_OR_INTERRUPT_TRANSFER 10184844     <common>

 entry point at        0001:00141fc4

 Static symbols

 0001:00091e88       SHAHashBlock               10092e88 f   md5.obj
 0001:0015ffc4       sha_end1                   10160fc4 f   wsc_crypto.obj
 0001:00165230       NN_AddDigitMult            10166230 f   wsc_crypto.obj
 0001:001653b0       NN_SubDigitMult            101663b0 f   wsc_crypto.obj
 0001:001655bc       NN_DigitBits               101665bc f   wsc_crypto.obj
